 config_plugin_instances

 Timestamp is 614c8045 (Thu Sep 23 13:25:25 2021)

 Preferred load address is 10000000

 Start         Length     Name                   Class
 0001:00000000 00000129H .text$di                CODE
 0001:00000130 0000d84cH .text$mn                CODE
 0001:0000d97c 00002429H .text$x                 CODE
 0001:0000fda5 00000063H .text$yd                CODE
 0002:00000000 00000d48H .idata$5                DATA
 0002:00000d48 00000004H .CRT$XCA                DATA
 0002:00000d4c 00000024H .CRT$XCU                DATA
 0002:00000d70 00000004H .CRT$XCZ                DATA
 0002:00000d74 00000004H .CRT$XIA                DATA
 0002:00000d78 00000004H .CRT$XIAA               DATA
 0002:00000d7c 00000004H .CRT$XIC                DATA
 0002:00000d80 00000004H .CRT$XIZ                DATA
 0002:00000d88 00004038H .rdata                  DATA
 0002:00004dc0 00001210H .rdata$r                DATA
 0002:00005fd0 00000110H .rdata$sxdata           DATA
 0002:000060e0 00000004H .rtc$IAA                DATA
 0002:000060e4 00000004H .rtc$IZZ                DATA
 0002:000060e8 00000004H .rtc$TAA                DATA
 0002:000060ec 00000004H .rtc$TZZ                DATA
 0002:000060f0 00002164H .xdata$x                DATA
 0002:00008260 00000575H .edata                  DATA
 0002:000087d8 00000050H .idata$2                DATA
 0002:00008828 00000014H .idata$3                DATA
 0002:0000883c 00000d48H .idata$4                DATA
 0002:00009584 0000875cH .idata$6                DATA
 0003:00000000 000001f4H .data                   DATA
 0003:000001f4 00000630H .data$r                 DATA
 0003:00000828 0000055cH .bss                    DATA
 0004:00000000 000000e8H .rsrc$01                DATA
 0004:000000f0 00000b20H .rsrc$02                DATA

  Address         Publics by Value              Rva+Base       Lib:Object

 0000:00000000       ___guard_fids_table        00000000     <absolute>
 0000:00000000       ___guard_fids_count        00000000     <absolute>
 0000:00000000       ___guard_flags             00000000     <absolute>
 0000:00000044       ___safe_se_handler_count   00000044     <absolute>
 0000:00000000       ___ImageBase               10000000     <linker-defined>
 0001:00000130       ??0?$QGuardedPtr@VQPopupMenu@@@@QAE@XZ 10001130 f i config_plugin_instances.obj
 0001:00000130       ??0?$QGuardedPtr@VQDockWindow@@@@QAE@XZ 10001130 f i config_plugin_instances.obj
 0001:00000171       ??0config_plugin_base@@QAE@ABVQString@@00@Z 10001171 f i config_plugin_instances.obj
 0001:000001fe       ??0config_plugin_instances@@QAE@ABVQString@@00@Z 100011fe f   config_plugin_instances.obj
 0001:0000087c       ??1?$QDict@VQAction@@@@UAE@XZ 1000187c f i config_plugin_instances.obj
 0001:000008af       ??1?$QGuardedPtr@VQPopupMenu@@@@QAE@XZ 100018af f i config_plugin_instances.obj
 0001:000008af       ??1?$QGuardedPtr@VQDockWindow@@@@QAE@XZ 100018af f i config_plugin_instances.obj
 0001:000008b4       ??1?$QPtrList@VQPopupMenu@@@@UAE@XZ 100018b4 f i config_plugin_instances.obj
 0001:000008e7       ??1QDockWindowList@@UAE@XZ 100018e7 f i config_plugin_instances.obj
 0001:00000930       ??1QPopupMenuList@@UAE@XZ  10001930 f i config_plugin_instances.obj
 0001:00000962       ??1config_plugin_base@@UAE@XZ 10001962 f i config_plugin_instances.obj
 0001:000009bc       ??1config_plugin_instances@@UAE@XZ 100019bc f   config_plugin_instances.obj
 0001:00000a6c       ??4?$QGuardedPtr@VQPopupMenu@@@@QAEAAV0@PAVQPopupMenu@@@Z 10001a6c f i config_plugin_instances.obj
 0001:00000a6c       ??4?$QGuardedPtr@VQDockWindow@@@@QAEAAV0@PAVQDockWindow@@@Z 10001a6c f i config_plugin_instances.obj
 0001:00000aca       ??_EQPopupMenu@@WCI@AEPAXI@Z 10001aca f i config_plugin_instances.obj
 0001:00000ad2       ??_EQPopupMenu@@WIM@AEPAXI@Z 10001ad2 f i config_plugin_instances.obj
 0001:00000add       ??_EQToolBar@@WCI@AEPAXI@Z 10001add f i config_plugin_instances.obj
 0001:00000ae5       ??_Econfig_plugin_base@@WCI@AEPAXI@Z 10001ae5 f i config_plugin_instances.obj
 0001:00000aed       ??_Econfig_plugin_instances@@WCI@AEPAXI@Z 10001aed f i config_plugin_instances.obj
 0001:00000af5       ??_E?$QDict@VQAction@@@@UAEPAXI@Z 10001af5 f i config_plugin_instances.obj
 0001:00000af5       ??_G?$QDict@VQAction@@@@UAEPAXI@Z 10001af5 f i config_plugin_instances.obj
 0001:00000b14       ??_G?$QPtrList@VQPopupMenu@@@@UAEPAXI@Z 10001b14 f i config_plugin_instances.obj
 0001:00000b14       ??_E?$QPtrList@VQPopupMenu@@@@UAEPAXI@Z 10001b14 f i config_plugin_instances.obj
 0001:00000b33       ??_GQAction@@UAEPAXI@Z     10001b33 f i config_plugin_instances.obj
 0001:00000b33       ??_EQAction@@UAEPAXI@Z     10001b33 f i config_plugin_instances.obj
 0001:00000b53       ??_EQDockWindowList@@UAEPAXI@Z 10001b53 f i config_plugin_instances.obj
 0001:00000b53       ??_GQDockWindowList@@UAEPAXI@Z 10001b53 f i config_plugin_instances.obj
 0001:00000b72       ??_GQGuardedPtrPrivate@@UAEPAXI@Z 10001b72 f i config_plugin_instances.obj
 0001:00000b72       ??_EQGuardedPtrPrivate@@UAEPAXI@Z 10001b72 f i config_plugin_instances.obj
 0001:00000b92       ??_EQPopupMenu@@UAEPAXI@Z  10001b92 f i config_plugin_instances.obj
 0001:00000b92       ??_GQPopupMenu@@UAEPAXI@Z  10001b92 f i config_plugin_instances.obj
 0001:00000bb2       ??_EQPopupMenuList@@UAEPAXI@Z 10001bb2 f i config_plugin_instances.obj
 0001:00000bb2       ??_GQPopupMenuList@@UAEPAXI@Z 10001bb2 f i config_plugin_instances.obj
 0001:00000bd1       ??_EQToolBar@@UAEPAXI@Z    10001bd1 f i config_plugin_instances.obj
 0001:00000bd1       ??_GQToolBar@@UAEPAXI@Z    10001bd1 f i config_plugin_instances.obj
 0001:00000bf1       ??_Gconfig_plugin_base@@UAEPAXI@Z 10001bf1 f i config_plugin_instances.obj
 0001:00000bf1       ??_Econfig_plugin_base@@UAEPAXI@Z 10001bf1 f i config_plugin_instances.obj
 0001:00000c10       ??_Econfig_plugin_instances@@UAEPAXI@Z 10001c10 f i config_plugin_instances.obj
 0001:00000c10       ??_Gconfig_plugin_instances@@UAEPAXI@Z 10001c10 f i config_plugin_instances.obj
 0001:00000c2f       ?about@config_plugin_base@@UAE?AVQString@@XZ 10001c2f f i config_plugin_instances.obj
 0001:00000c85       ?about@config_plugin_instances@@UAE?AVQString@@XZ 10001c85 f   config_plugin_instances.obj
 0001:00000d2d       ?activate@config_plugin_instances@@UAEX_N@Z 10001d2d f   config_plugin_instances.obj
 0001:00000f6e       ?dummy@config_plugin_instancesDlg@@QAEXXZ 10001f6e f i config_plugin_instancesdlgimpl.obj
 0001:00000f6e       ?apply@config_plugin_base@@UAEXXZ 10001f6e f i config_plugin_instances.obj
 0001:00000f6f       ?apply@config_plugin_instances@@UAEXXZ 10001f6f f   config_plugin_instances.obj
 0001:00001006       ?clear@?$QDict@VQAction@@@@UAEXXZ 10002006 f i config_plugin_instances.obj
 0001:0000100c       ?closeEvent@config_plugin_base@@UAEXPAVQCloseEvent@@@Z 1000200c f i config_plugin_instances.obj
 0001:0000101a       ?closeEvent@config_plugin_instances@@UAEXPAVQCloseEvent@@@Z 1000201a f   config_plugin_instances.obj
 0001:00001076       ?count@?$QDict@VQAction@@@@UBEIXZ 10002076 f i config_plugin_instances.obj
 0001:0000107a       ?db@@YAXABVQString@@@Z     1000207a f   config_plugin_instances.obj
 0001:000010c2       ?deleteItem@?$QDict@VQAction@@@@EAEXPAX@Z 100020c2 f i config_plugin_instances.obj
 0001:000010c2       ?deleteItem@?$QPtrList@VQPopupMenu@@@@EAEXPAX@Z 100020c2 f i config_plugin_instances.obj
 0001:000010dd       ?deref@?$QGuardedPtr@VQDockWindow@@@@AAEXXZ 100020dd f i config_plugin_instances.obj
 0001:000010dd       ?deref@?$QGuardedPtr@VQPopupMenu@@@@AAEXXZ 100020dd f i config_plugin_instances.obj
 0001:000010f2       ?deviceContextMenu@config_plugin_instances@@QAEXHHABVQPoint@@@Z 100020f2 f   config_plugin_instances.obj
 0001:0000110a       ?isDirty@config_plugin_base@@UAE_NXZ 1000210a f i config_plugin_instances.obj
 0001:0000110a       ?validate@config_plugin_base@@UAE_NXZ 1000210a f i config_plugin_instances.obj
 0001:0000110a       ?qt_static_property@cfg_Table@@SA_NPAVQObject@@HHPAVQVariant@@@Z 1000210a f i cfg_widgets001:moc_cfg_Table.obj
 0001:0000110d       ?isDirty@config_plugin_instances@@UAE_NXZ 1000210d f   config_plugin_instances.obj
 0001:0000111a       ?menus@config_plugin_base@@UAE?AVQPopupMenuList@@XZ 1000211a f i config_plugin_instances.obj
 0001:0000113d       ?menus@config_plugin_instances@@UAE?AVQPopupMenuList@@XZ 1000213d f   config_plugin_instances.obj
 0001:00001187       ?metaObject@config_plugin_instances@@UBEPAVQMetaObject@@XZ 10002187 f i config_plugin_instances.obj
 0001:0000118c       ?navigate@config_plugin_base@@UAEXABVQString@@0@Z 1000218c f i config_plugin_instances.obj
 0001:0000118f       ?navigate@config_plugin_instances@@UAEXABVQString@@0@Z 1000218f f   config_plugin_instances.obj
 0001:0000120b       ?setReadOnly@config_plugin_instancesDlg@@QAEX_N@Z 1000220b f i config_plugin_instancesdlgimpl.obj
 0001:0000120b       ?activate@config_plugin_base@@UAEX_N@Z 1000220b f i config_plugin_instances.obj
 0001:0000120b       ?reply@config_plugin_base@@UAEXPAVresponse@@@Z 1000220b f i config_plugin_instances.obj
 0001:0000120e       ?reply@config_plugin_instances@@UAEXPAVresponse@@@Z 1000220e f   config_plugin_instances.obj
 0001:0000161d       ?resizeEvent@config_plugin_instances@@UAEXPAVQResizeEvent@@@Z 1000261d f   config_plugin_instances.obj
 0001:00001652       ?textStatus@response@@QAE?AVQString@@W4status@1@@Z 10002652 f i config_plugin_instances.obj
 0001:000016a1       ?toolbars@config_plugin_base@@UAE?AVQDockWindowList@@XZ 100026a1 f i config_plugin_instances.obj
 0001:000016c4       ?toolbars@config_plugin_instances@@UAE?AVQDockWindowList@@XZ 100026c4 f   config_plugin_instances.obj
 0001:0000171c       ??0config_plugin_instancesDlg@@QAE@ABVQString@@PAVQWidget@@PBDI@Z 1000271c f   config_plugin_instancesdlgimpl.obj
 0001:00001dc4       ??1?$QPtrList@VdeviceRow@@@@UAE@XZ 10002dc4 f i config_plugin_instancesdlgimpl.obj
 0001:00001df7       ??1?$QPtrList@VgroupRow@@@@UAE@XZ 10002df7 f i config_plugin_instancesdlgimpl.obj
 0001:00001e2a       ??1?$QPtrList@VviewRow@@@@UAE@XZ 10002e2a f i config_plugin_instancesdlgimpl.obj
 0001:00001e5d       ??1config_plugin_instancesDlg@@UAE@XZ 10002e5d f   config_plugin_instancesdlgimpl.obj
 0001:00001f1f       ??_Econfig_plugin_instancesDlg@@WCI@AEPAXI@Z 10002f1f f i config_plugin_instancesdlgimpl.obj
 0001:00001f27       ??_G?$QPtrList@VdeviceRow@@@@UAEPAXI@Z 10002f27 f i config_plugin_instancesdlgimpl.obj
 0001:00001f27       ??_E?$QPtrList@VdeviceRow@@@@UAEPAXI@Z 10002f27 f i config_plugin_instancesdlgimpl.obj
 0001:00001f46       ??_G?$QPtrList@VgroupRow@@@@UAEPAXI@Z 10002f46 f i config_plugin_instancesdlgimpl.obj
 0001:00001f46       ??_E?$QPtrList@VgroupRow@@@@UAEPAXI@Z 10002f46 f i config_plugin_instancesdlgimpl.obj
 0001:00001f65       ??_G?$QPtrList@VviewRow@@@@UAEPAXI@Z 10002f65 f i config_plugin_instancesdlgimpl.obj
 0001:00001f65       ??_E?$QPtrList@VviewRow@@@@UAEPAXI@Z 10002f65 f i config_plugin_instancesdlgimpl.obj
 0001:00001f84       ??_EQDomDocument@@UAEPAXI@Z 10002f84 f i config_plugin_instancesdlgimpl.obj
 0001:00001f84       ??_GQDomDocument@@UAEPAXI@Z 10002f84 f i config_plugin_instancesdlgimpl.obj
 0001:00001fa4       ??_EQDomElement@@UAEPAXI@Z 10002fa4 f i config_plugin_instancesdlgimpl.obj
 0001:00001fa4       ??_GQDomElement@@UAEPAXI@Z 10002fa4 f i config_plugin_instancesdlgimpl.obj
 0001:00001fc4       ??_Econfig_plugin_instancesDlg@@UAEPAXI@Z 10002fc4 f i config_plugin_instancesdlgimpl.obj
 0001:00001fc4       ??_Gconfig_plugin_instancesDlg@@UAEPAXI@Z 10002fc4 f i config_plugin_instancesdlgimpl.obj
 0001:00001fe3       ?addDeviceNodeFromRow@config_plugin_instancesDlg@@QAE_NH@Z 10002fe3 f   config_plugin_instancesdlgimpl.obj
 0001:00002445       ?addGroupToInstanceNodeFromRow@config_plugin_instancesDlg@@QAE_NHVQString@@@Z 10003445 f   config_plugin_instancesdlgimpl.obj
 0001:000026e0       ?addViewNodeFromRow@config_plugin_instancesDlg@@QAE_NH@Z 100036e0 f   config_plugin_instancesdlgimpl.obj
 0001:00002920       ?clear@?$QPtrList@VviewRow@@@@UAEXXZ 10003920 f i config_plugin_instancesdlgimpl.obj
 0001:00002920       ?clear@?$QPtrList@VgroupRow@@@@UAEXXZ 10003920 f i config_plugin_instancesdlgimpl.obj
 0001:00002920       ?clear@?$QPtrList@VdeviceRow@@@@UAEXXZ 10003920 f i config_plugin_instancesdlgimpl.obj
 0001:00002920       ?clear@?$QPtrList@VQPopupMenu@@@@UAEXXZ 10003920 f i config_plugin_instances.obj
 0001:00002926       ?clipboardDataChange@config_plugin_instancesDlg@@QAEXXZ 10003926 f   config_plugin_instancesdlgimpl.obj
 0001:00002b13       ?copySelectedToClipboard@config_plugin_instancesDlg@@QAEXXZ 10003b13 f   config_plugin_instancesdlgimpl.obj
 0001:00002e3f       ?count@?$QPtrList@VgroupRow@@@@UBEIXZ 10003e3f f i config_plugin_instancesdlgimpl.obj
 0001:00002e3f       ?count@?$QPtrList@VviewRow@@@@UBEIXZ 10003e3f f i config_plugin_instancesdlgimpl.obj
 0001:00002e3f       ?count@?$QPtrList@VdeviceRow@@@@UBEIXZ 10003e3f f i config_plugin_instancesdlgimpl.obj
 0001:00002e3f       ?count@?$QPtrList@VQPopupMenu@@@@UBEIXZ 10003e3f f i config_plugin_instances.obj
 0001:00002e43       ?deleteItem@?$QPtrList@VgroupRow@@@@EAEXPAX@Z 10003e43 f i config_plugin_instancesdlgimpl.obj
 0001:00002e43       ?deleteItem@?$QPtrList@VdeviceRow@@@@EAEXPAX@Z 10003e43 f i config_plugin_instancesdlgimpl.obj
 0001:00002e43       ?deleteItem@?$QPtrList@VviewRow@@@@EAEXPAX@Z 10003e43 f i config_plugin_instancesdlgimpl.obj
 0001:00002e5d       ?deviceInstanceChanged@config_plugin_instancesDlg@@QAEXHH@Z 10003e5d f   config_plugin_instancesdlgimpl.obj
 0001:00002ee1       ?doCreateNewInstance@config_plugin_instancesDlg@@QAEXXZ 10003ee1 f   config_plugin_instancesdlgimpl.obj
 0001:00003321       ?doDeleteInstance@config_plugin_instancesDlg@@QAEXXZ 10004321 f   config_plugin_instancesdlgimpl.obj
 0001:00003cc5       ?doDuplicateInstance@config_plugin_instancesDlg@@QAEXXZ 10004cc5 f   config_plugin_instancesdlgimpl.obj
 0001:0000513a       ?doStartRename@config_plugin_instancesDlg@@QAEXXZ 1000613a f   config_plugin_instancesdlgimpl.obj
 0001:00005147       ?groupNameIsUnique@config_plugin_instancesDlg@@QAE_NVQString@@@Z 10006147 f   config_plugin_instancesdlgimpl.obj
 0001:000051d3       ?instanceNameIsUnique@config_plugin_instancesDlg@@QAE_NVQString@@@Z 100061d3 f   config_plugin_instancesdlgimpl.obj
 0001:0000539c       ?load@config_plugin_instancesDlg@@QAE_NABVQString@@@Z 1000639c f   config_plugin_instancesdlgimpl.obj
 0001:0000631c       ?metaObject@config_plugin_instancesDlg@@UBEPAVQMetaObject@@XZ 1000731c f i config_plugin_instancesdlgimpl.obj
 0001:00006321       ?pasteCompositesXMLFragment@config_plugin_instancesDlg@@QAEXXZ 10007321 f   config_plugin_instancesdlgimpl.obj
 0001:00006a88       ?pasteDeviceData@config_plugin_instancesDlg@@QAEXXZ 10007a88 f   config_plugin_instancesdlgimpl.obj
 0001:00007425       ?pasteGroupData@config_plugin_instancesDlg@@QAEXXZ 10008425 f   config_plugin_instancesdlgimpl.obj
 0001:00007b07       ?pasteOptions@config_plugin_instancesDlg@@QAEXXZ 10008b07 f   config_plugin_instancesdlgimpl.obj
 0001:00007b97       ?save@config_plugin_instancesDlg@@QAE_NABVQString@@@Z 10008b97 f   config_plugin_instancesdlgimpl.obj
 0001:00007c3d       ?selectDevicetypes@config_plugin_instancesDlg@@QAEXHHHABVQPoint@@@Z 10008c3d f   config_plugin_instancesdlgimpl.obj
 0001:00007de2       ?setClean@config_plugin_instancesDlg@@QAEXXZ 10008de2 f   config_plugin_instancesdlgimpl.obj
 0001:00007dea       ?setDirty@config_plugin_instancesDlg@@QAEXXZ 10008dea f   config_plugin_instancesdlgimpl.obj
 0001:00007e33       ?typeIsValid@config_plugin_instancesDlg@@QAE_NVQString@@@Z 10008e33 f   config_plugin_instancesdlgimpl.obj
 0001:00007e6f       ?valueCompositeGroupChanged@config_plugin_instancesDlg@@QAEXHH@Z 10008e6f f   config_plugin_instancesdlgimpl.obj
 0001:000081c6       ?valueCompositeTopChanged@config_plugin_instancesDlg@@QAEXHH@Z 100091c6 f   config_plugin_instancesdlgimpl.obj
 0001:00008454       ?valueDevicesChanged@config_plugin_instancesDlg@@QAEXHH@Z 10009454 f   config_plugin_instancesdlgimpl.obj
 0001:00008a15       ?viewGroupChanged@config_plugin_instancesDlg@@QAEXHH@Z 10009a15 f   config_plugin_instancesdlgimpl.obj
 0001:00008a9d       ?viewInstanceChanged@config_plugin_instancesDlg@@QAEXHH@Z 10009a9d f   config_plugin_instancesdlgimpl.obj
 0001:00008f51       ??0deviceRow@@QAE@ABVQString@@0000000@Z 10009f51 f   deviceRow.obj
 0001:00009027       ??1deviceRow@@UAE@XZ       1000a027 f   deviceRow.obj
 0001:000090af       ??_EdeviceRow@@UAEPAXI@Z   1000a0af f i deviceRow.obj
 0001:000090af       ??_GdeviceRow@@UAEPAXI@Z   1000a0af f i deviceRow.obj
 0001:000090ce       ??0devicetypesBase@@QAE@PAVQWidget@@PBD_NI@Z 1000a0ce f   devicetypes.obj
 0001:000093d9       ??1devicetypesBase@@UAE@XZ 1000a3d9 f   devicetypes.obj
 0001:000093ec       ??_EQHBoxLayout@@WCI@AEPAXI@Z 1000a3ec f i devicetypes.obj
 0001:000093f4       ??_EQLabel@@WCI@AEPAXI@Z   1000a3f4 f i devicetypes.obj
 0001:000093fc       ??_EQListBox@@WCI@AEPAXI@Z 1000a3fc f i devicetypes.obj
 0001:00009404       ??_EQPushButton@@WCI@AEPAXI@Z 1000a404 f i devicetypes.obj
 0001:0000940c       ??_EQVBoxLayout@@WCI@AEPAXI@Z 1000a40c f i devicetypes.obj
 0001:00009414       ??_EdevicetypesBase@@WCI@AEPAXI@Z 1000a414 f i devicetypes.obj
 0001:0000941c       ??_EQHBoxLayout@@UAEPAXI@Z 1000a41c f i devicetypes.obj
 0001:0000941c       ??_GQHBoxLayout@@UAEPAXI@Z 1000a41c f i devicetypes.obj
 0001:0000943c       ??_EQLabel@@UAEPAXI@Z      1000a43c f i devicetypes.obj
 0001:0000943c       ??_GQLabel@@UAEPAXI@Z      1000a43c f i devicetypes.obj
 0001:0000945c       ??_EQListBox@@UAEPAXI@Z    1000a45c f i devicetypes.obj
 0001:0000945c       ??_GQListBox@@UAEPAXI@Z    1000a45c f i devicetypes.obj
 0001:0000947c       ??_EQPushButton@@UAEPAXI@Z 1000a47c f i devicetypes.obj
 0001:0000947c       ??_GQPushButton@@UAEPAXI@Z 1000a47c f i devicetypes.obj
 0001:0000949c       ??_EQSpacerItem@@UAEPAXI@Z 1000a49c f i devicetypes.obj
 0001:0000949c       ??_GQSpacerItem@@UAEPAXI@Z 1000a49c f i devicetypes.obj
 0001:000094bc       ??_EQVBoxLayout@@UAEPAXI@Z 1000a4bc f i devicetypes.obj
 0001:000094bc       ??_GQVBoxLayout@@UAEPAXI@Z 1000a4bc f i devicetypes.obj
 0001:000094dc       ??_EdevicetypesBase@@UAEPAXI@Z 1000a4dc f i devicetypes.obj
 0001:000094dc       ??_GdevicetypesBase@@UAEPAXI@Z 1000a4dc f i devicetypes.obj
 0001:000094fb       ?languageChange@devicetypesBase@@MAEXXZ 1000a4fb f   devicetypes.obj
 0001:00009606       ?metaObject@devicetypesBase@@UBEPAVQMetaObject@@XZ 1000a606 f i devicetypes.obj
 0001:0000960b       ??0devicetypes@@QAE@PAVQWidget@@PBD_NI@Z 1000a60b f   devicetypesimpl.obj
 0001:00009636       ??1devicetypes@@UAE@XZ     1000a636 f   devicetypesimpl.obj
 0001:00009648       ??_Edevicetypes@@WCI@AEPAXI@Z 1000a648 f i devicetypesimpl.obj
 0001:00009650       ??_Gdevicetypes@@UAEPAXI@Z 1000a650 f i devicetypesimpl.obj
 0001:00009650       ??_Edevicetypes@@UAEPAXI@Z 1000a650 f i devicetypesimpl.obj
 0001:0000966f       ?metaObject@devicetypes@@UBEPAVQMetaObject@@XZ 1000a66f f i devicetypesimpl.obj
 0001:00009674       ??0groupRow@@QAE@ABVQString@@0@Z 1000a674 f   groupRow.obj
 0001:000096c5       ??1groupRow@@UAE@XZ        1000a6c5 f   groupRow.obj
 0001:000096fc       ??_EgroupRow@@UAEPAXI@Z    1000a6fc f i groupRow.obj
 0001:000096fc       ??_GgroupRow@@UAEPAXI@Z    1000a6fc f i groupRow.obj
 0001:0000971b       ??0instancesCustomTable@@QAE@PAVQWidget@@PBD@Z 1000a71b f   instancesCustomTable.obj
 0001:00009796       ??1cfg_Table@@UAE@XZ       1000a796 f i instancesCustomTable.obj
 0001:0000979c       ??1instancesCustomTable@@UAE@XZ 1000a79c f   instancesCustomTable.obj
 0001:000097dc       ??_EinstancesCustomTable@@WCI@AEPAXI@Z 1000a7dc f i instancesCustomTable.obj
 0001:000097e4       ??_GinstancesCustomTable@@UAEPAXI@Z 1000a7e4 f i instancesCustomTable.obj
 0001:000097e4       ??_EinstancesCustomTable@@UAEPAXI@Z 1000a7e4 f i instancesCustomTable.obj
 0001:00009803       ?metaObject@instancesCustomTable@@UBEPAVQMetaObject@@XZ 1000a803 f i instancesCustomTable.obj
 0001:00009808       ?sortColumn@instancesCustomTable@@QAEXHHH@Z 1000a808 f   instancesCustomTable.obj
 0001:000098dd       ?className@devicetypesBase@@UBEPBDXZ 1000a8dd f   moc_devicetypes.obj
 0001:000098e3       ?qt_cast@devicetypesBase@@UAEPAXPBD@Z 1000a8e3 f   moc_devicetypes.obj
 0001:00009911       ?qt_emit@devicetypesBase@@UAE_NHPAUQUObject@@@Z 1000a911 f   moc_devicetypes.obj
 0001:0000991b       ?qt_invoke@devicetypesBase@@UAE_NHPAUQUObject@@@Z 1000a91b f   moc_devicetypes.obj
 0001:0000994d       ?qt_property@devicetypesBase@@UAE_NHHPAVQVariant@@@Z 1000a94d f   moc_devicetypes.obj
 0001:00009957       ?staticMetaObject@devicetypesBase@@SAPAVQMetaObject@@XZ 1000a957 f   moc_devicetypes.obj
 0001:000099a1       ?tr@devicetypesBase@@SA?AVQString@@PBD0@Z 1000a9a1 f   moc_devicetypes.obj
 0001:000099e4       ?className@devicetypes@@UBEPBDXZ 1000a9e4 f   moc_devicetypesimpl.obj
 0001:000099ea       ?qt_cast@devicetypes@@UAEPAXPBD@Z 1000a9ea f   moc_devicetypesimpl.obj
 0001:00009a17       ?qt_emit@devicetypes@@UAE_NHPAUQUObject@@@Z 1000aa17 f   moc_devicetypesimpl.obj
 0001:00009a20       ?qt_invoke@devicetypes@@UAE_NHPAUQUObject@@@Z 1000aa20 f   moc_devicetypesimpl.obj
 0001:00009a29       ?qt_property@devicetypes@@UAE_NHHPAVQVariant@@@Z 1000aa29 f   moc_devicetypesimpl.obj
 0001:00009a32       ?staticMetaObject@devicetypes@@SAPAVQMetaObject@@XZ 1000aa32 f   moc_devicetypesimpl.obj
 0001:00009a76       ??_Econfig_plugin_desc_base@@UAEPAXI@Z 1000aa76 f i plugindesc.obj
 0001:00009a76       ??_Gplugindesc@@UAEPAXI@Z  1000aa76 f i plugindesc.obj
 0001:00009a76       ??_Eplugindesc@@UAEPAXI@Z  1000aa76 f i plugindesc.obj
 0001:00009a76       ??_Gconfig_plugin_desc_base@@UAEPAXI@Z 1000aa76 f i plugindesc.obj
 0001:00009a96       ?create@plugindesc@@UAEPAVconfig_plugin_base@@ABVQString@@00@Z 1000aa96 f   plugindesc.obj
 0001:00009ad1       ?keys@plugindesc@@UAE?AVQStringList@@ABVQString@@0@Z 1000aad1 f   plugindesc.obj
 0001:00009b2c       ?pixmap@plugindesc@@UAE?AVQPixmap@@ABVQString@@@Z 1000ab2c f   plugindesc.obj
 0001:00009b4b       _load_bncs_config_plugin_desc 1000ab4b f   plugindesc.obj
 0001:00009b61       ??0viewRow@@QAE@ABVQString@@000@Z 1000ab61 f   viewRow.obj
 0001:00009bde       ??1viewRow@@UAE@XZ         1000abde f   viewRow.obj
 0001:00009c32       ??_EviewRow@@UAEPAXI@Z     1000ac32 f i viewRow.obj
 0001:00009c32       ??_GviewRow@@UAEPAXI@Z     1000ac32 f i viewRow.obj
 0001:00009c51       ??0config_plugin_instancesDlgBase@@QAE@PAVQWidget@@PBDI@Z 1000ac51 f   config_plugin_instancesdlg.obj
 0001:0000a375       ??1config_plugin_instancesDlgBase@@UAE@XZ 1000b375 f   config_plugin_instancesdlg.obj
 0001:0000a3b5       ??_EQTabWidget@@WCI@AEPAXI@Z 1000b3b5 f i config_plugin_instancesdlg.obj
 0001:0000a3bd       ??_EQWidget@@WCI@AEPAXI@Z  1000b3bd f i config_plugin_instancesdlg.obj
 0001:0000a3c5       ??_Econfig_plugin_instancesDlgBase@@WCI@AEPAXI@Z 1000b3c5 f i config_plugin_instancesdlg.obj
 0001:0000a3cd       ??_GQTabWidget@@UAEPAXI@Z  1000b3cd f i config_plugin_instancesdlg.obj
 0001:0000a3cd       ??_EQTabWidget@@UAEPAXI@Z  1000b3cd f i config_plugin_instancesdlg.obj
 0001:0000a3ed       ??_GQWidget@@UAEPAXI@Z     1000b3ed f i config_plugin_instancesdlg.obj
 0001:0000a3ed       ??_EQWidget@@UAEPAXI@Z     1000b3ed f i config_plugin_instancesdlg.obj
 0001:0000a40d       ??_Econfig_plugin_instancesDlgBase@@UAEPAXI@Z 1000b40d f i config_plugin_instancesdlg.obj
 0001:0000a40d       ??_Gconfig_plugin_instancesDlgBase@@UAEPAXI@Z 1000b40d f i config_plugin_instancesdlg.obj
 0001:0000a42c       ?languageChange@config_plugin_instancesDlgBase@@MAEXXZ 1000b42c f   config_plugin_instancesdlg.obj
 0001:0000a5ba       ?metaObject@config_plugin_instancesDlgBase@@UBEPAVQMetaObject@@XZ 1000b5ba f i config_plugin_instancesdlg.obj
 0001:0000a5bf       ?className@config_plugin_instances@@UBEPBDXZ 1000b5bf f   moc_config_plugin_instances.obj
 0001:0000a5c5       ?command@config_plugin_instances@@IAEXVQString@@0@Z 1000b5c5 f   moc_config_plugin_instances.obj
 0001:0000a685       ?qt_cast@config_plugin_instances@@UAEPAXPBD@Z 1000b685 f   moc_config_plugin_instances.obj
 0001:0000a6b3       ?qt_emit@config_plugin_instances@@UAE_NHPAUQUObject@@@Z 1000b6b3 f   moc_config_plugin_instances.obj
 0001:0000a717       ?qt_invoke@config_plugin_instances@@UAE_NHPAUQUObject@@@Z 1000b717 f   moc_config_plugin_instances.obj
 0001:0000a752       ?qt_property@config_plugin_instances@@UAE_NHHPAVQVariant@@@Z 1000b752 f   moc_config_plugin_instances.obj
 0001:0000a752       ?qt_property@config_plugin_instancesDlgBase@@UAE_NHHPAVQVariant@@@Z 1000b752 f   moc_config_plugin_instancesdlg.obj
 0001:0000a75c       ?staticMetaObject@config_plugin_instances@@SAPAVQMetaObject@@XZ 1000b75c f   moc_config_plugin_instances.obj
 0001:0000a85d       ?className@config_plugin_instancesDlgBase@@UBEPBDXZ 1000b85d f   moc_config_plugin_instancesdlg.obj
 0001:0000a863       ?qt_cast@config_plugin_instancesDlgBase@@UAEPAXPBD@Z 1000b863 f   moc_config_plugin_instancesdlg.obj
 0001:0000a891       ?qt_emit@config_plugin_instancesDlgBase@@UAE_NHPAUQUObject@@@Z 1000b891 f   moc_config_plugin_instancesdlg.obj
 0001:0000a89b       ?qt_invoke@config_plugin_instancesDlgBase@@UAE_NHPAUQUObject@@@Z 1000b89b f   moc_config_plugin_instancesdlg.obj
 0001:0000a8cd       ?staticMetaObject@config_plugin_instancesDlgBase@@SAPAVQMetaObject@@XZ 1000b8cd f   moc_config_plugin_instancesdlg.obj
 0001:0000a917       ?tr@config_plugin_instancesDlgBase@@SA?AVQString@@PBD0@Z 1000b917 f   moc_config_plugin_instancesdlg.obj
 0001:0000a95a       ?className@config_plugin_instancesDlg@@UBEPBDXZ 1000b95a f   moc_config_plugin_instancesdlgimpl.obj
 0001:0000a960       ?command@config_plugin_instancesDlg@@IAEXVQString@@0@Z 1000b960 f   moc_config_plugin_instancesdlgimpl.obj
 0001:0000aa20       ?qt_cast@config_plugin_instancesDlg@@UAEPAXPBD@Z 1000ba20 f   moc_config_plugin_instancesdlgimpl.obj
 0001:0000aa4d       ?qt_emit@config_plugin_instancesDlg@@UAE_NHPAUQUObject@@@Z 1000ba4d f   moc_config_plugin_instancesdlgimpl.obj
 0001:0000aab0       ?qt_invoke@config_plugin_instancesDlg@@UAE_NHPAUQUObject@@@Z 1000bab0 f   moc_config_plugin_instancesdlgimpl.obj
 0001:0000ace4       ?qt_property@config_plugin_instancesDlg@@UAE_NHHPAVQVariant@@@Z 1000bce4 f   moc_config_plugin_instancesdlgimpl.obj
 0001:0000aced       ?staticMetaObject@config_plugin_instancesDlg@@SAPAVQMetaObject@@XZ 1000bced f   moc_config_plugin_instancesdlgimpl.obj
 0001:0000b134       ?className@instancesCustomTable@@UBEPBDXZ 1000c134 f   moc_instancesCustomTable.obj
 0001:0000b13a       ?qt_cast@instancesCustomTable@@UAEPAXPBD@Z 1000c13a f   moc_instancesCustomTable.obj
 0001:0000b167       ?qt_emit@instancesCustomTable@@UAE_NHPAUQUObject@@@Z 1000c167 f   moc_instancesCustomTable.obj
 0001:0000b170       ?qt_invoke@instancesCustomTable@@UAE_NHPAUQUObject@@@Z 1000c170 f   moc_instancesCustomTable.obj
 0001:0000b1ce       ?qt_property@instancesCustomTable@@UAE_NHHPAVQVariant@@@Z 1000c1ce f   moc_instancesCustomTable.obj
 0001:0000b1d7       ?staticMetaObject@instancesCustomTable@@SAPAVQMetaObject@@XZ 1000c1d7 f   moc_instancesCustomTable.obj
 0001:0000b2e9       ?staticMetaObject@toolWindowBase@@SAPAVQMetaObject@@XZ 1000c2e9 f   moc_toolwindow.obj
 0001:0000b333       ?staticMetaObject@toolWindow@@SAPAVQMetaObject@@XZ 1000c333 f   moc_toolwindowimpl.obj
 0001:0000b3e0       ?setName@QWidget@@UAEXPBD@Z 1000c3e0 f   qt-mt323:qt-mt323.dll
 0001:0000b3e6       ?closeEvent@QWidget@@MAEXPAVQCloseEvent@@@Z 1000c3e6 f   qt-mt323:qt-mt323.dll
 0001:0000b3ec       ?activateItemAt@QPopupMenu@@UAEXH@Z 1000c3ec f   qt-mt323:qt-mt323.dll
 0001:0000b3f2       ?addTo@QAction@@UAE_NPAVQWidget@@@Z 1000c3f2 f   qt-mt323:qt-mt323.dll
 0001:0000b3f8       ?addedTo@QAction@@MAEXHPAVQPopupMenu@@@Z 1000c3f8 f   qt-mt323:qt-mt323.dll
 0001:0000b3fe       ?addedTo@QAction@@MAEXPAVQWidget@@0@Z 1000c3fe f   qt-mt323:qt-mt323.dll
 0001:0000b404       ?adjustSize@QWidget@@UAEXXZ 1000c404 f   qt-mt323:qt-mt323.dll
 0001:0000b40a       ?checkConnectArgs@QObject@@MAE_NPBDPBV1@0@Z 1000c40a f   qt-mt323:qt-mt323.dll
 0001:0000b410       ?childEvent@QObject@@MAEXPAVQChildEvent@@@Z 1000c410 f   qt-mt323:qt-mt323.dll
 0001:0000b416       ?className@QAction@@UBEPBDXZ 1000c416 f   qt-mt323:qt-mt323.dll
 0001:0000b41c       ?className@QGuardedPtrPrivate@@UBEPBDXZ 1000c41c f   qt-mt323:qt-mt323.dll
 0001:0000b422       ?className@QPopupMenu@@UBEPBDXZ 1000c422 f   qt-mt323:qt-mt323.dll
 0001:0000b428       ?className@QToolBar@@UBEPBDXZ 1000c428 f   qt-mt323:qt-mt323.dll
 0001:0000b42e       ?className@QWidget@@UBEPBDXZ 1000c42e f   qt-mt323:qt-mt323.dll
 0001:0000b434       ?clear@?$QPtrList@VQDockWindow@@@@UAEXXZ 1000c434 f   qt-mt323:qt-mt323.dll
 0001:0000b43a       ?clear@QToolBar@@UAEXXZ    1000c43a f   qt-mt323:qt-mt323.dll
 0001:0000b440       ?close@QWidget@@UAE_N_N@Z  1000c440 f   qt-mt323:qt-mt323.dll
 0001:0000b446       ?closeEvent@QPopupMenu@@MAEXPAVQCloseEvent@@@Z 1000c446 f   qt-mt323:qt-mt323.dll
 0001:0000b44c       ?cmd@QPaintDevice@@MAE_NHPAVQPainter@@PATQPDevCmdParam@@@Z 1000c44c f   qt-mt323:qt-mt323.dll
 0001:0000b452       ?compareItems@QGList@@MAEHPAX0@Z 1000c452 f   qt-mt323:qt-mt323.dll
 0001:0000b458       ?connectNotify@QObject@@MAEXPBD@Z 1000c458 f   qt-mt323:qt-mt323.dll
 0001:0000b45e       ?contextMenuEvent@QDockWindow@@MAEXPAVQContextMenuEvent@@@Z 1000c45e f   qt-mt323:qt-mt323.dll
 0001:0000b464       ?contextMenuEvent@QWidget@@MAEXPAVQContextMenuEvent@@@Z 1000c464 f   qt-mt323:qt-mt323.dll
 0001:0000b46a       ?count@?$QPtrList@VQDockWindow@@@@UBEIXZ 1000c46a f   qt-mt323:qt-mt323.dll
 0001:0000b470       ?create@QWidget@@MAEXPAUHWND__@@_N1@Z 1000c470 f   qt-mt323:qt-mt323.dll
 0001:0000b476       ?customEvent@QObject@@MAEXPAVQCustomEvent@@@Z 1000c476 f   qt-mt323:qt-mt323.dll
 0001:0000b47c       ?customWhatsThis@QPopupMenu@@UBE_NXZ 1000c47c f   qt-mt323:qt-mt323.dll
 0001:0000b482       ?customWhatsThis@QWidget@@UBE_NXZ 1000c482 f   qt-mt323:qt-mt323.dll
 0001:0000b488       ?deleteItem@?$QPtrList@VQDockWindow@@@@EAEXPAX@Z 1000c488 f   qt-mt323:qt-mt323.dll
 0001:0000b48e       ?destroy@QWidget@@MAEX_N0@Z 1000c48e f   qt-mt323:qt-mt323.dll
 0001:0000b494       ?disconnectNotify@QObject@@MAEXPBD@Z 1000c494 f   qt-mt323:qt-mt323.dll
 0001:0000b49a       ?dock@QDockWindow@@UAEXXZ  1000c49a f   qt-mt323:qt-mt323.dll
 0001:0000b4a0       ?dragEnterEvent@QWidget@@MAEXPAVQDragEnterEvent@@@Z 1000c4a0 f   qt-mt323:qt-mt323.dll
 0001:0000b4a6       ?dragLeaveEvent@QWidget@@MAEXPAVQDragLeaveEvent@@@Z 1000c4a6 f   qt-mt323:qt-mt323.dll
 0001:0000b4ac       ?dragMoveEvent@QWidget@@MAEXPAVQDragMoveEvent@@@Z 1000c4ac f   qt-mt323:qt-mt323.dll
 0001:0000b4b2       ?drawContents@QDockWindow@@MAEXPAVQPainter@@@Z 1000c4b2 f   qt-mt323:qt-mt323.dll
 0001:0000b4b8       ?drawContents@QPopupMenu@@MAEXPAVQPainter@@@Z 1000c4b8 f   qt-mt323:qt-mt323.dll
 0001:0000b4be       ?drawFrame@QDockWindow@@MAEXPAVQPainter@@@Z 1000c4be f   qt-mt323:qt-mt323.dll
 0001:0000b4c4       ?drawFrame@QFrame@@MAEXPAVQPainter@@@Z 1000c4c4 f   qt-mt323:qt-mt323.dll
 0001:0000b4ca       ?dropEvent@QWidget@@MAEXPAVQDropEvent@@@Z 1000c4ca f   qt-mt323:qt-mt323.dll
 0001:0000b4d0       ?enabledChange@QPopupMenu@@MAEX_N@Z 1000c4d0 f   qt-mt323:qt-mt323.dll
 0001:0000b4d6       ?enabledChange@QWidget@@MAEX_N@Z 1000c4d6 f   qt-mt323:qt-mt323.dll
 0001:0000b4dc       ?enterEvent@QWidget@@MAEXPAVQEvent@@@Z 1000c4dc f   qt-mt323:qt-mt323.dll
 0001:0000b4e2       ?event@QObject@@UAE_NPAVQEvent@@@Z 1000c4e2 f   qt-mt323:qt-mt323.dll
 0001:0000b4e8       ?event@QToolBar@@UAE_NPAVQEvent@@@Z 1000c4e8 f   qt-mt323:qt-mt323.dll
 0001:0000b4ee       ?event@QWidget@@MAE_NPAVQEvent@@@Z 1000c4ee f   qt-mt323:qt-mt323.dll
 0001:0000b4f4       ?eventFilter@QDockWindow@@UAE_NPAVQObject@@PAVQEvent@@@Z 1000c4f4 f   qt-mt323:qt-mt323.dll
 0001:0000b4fa       ?eventFilter@QObject@@UAE_NPAV1@PAVQEvent@@@Z 1000c4fa f   qt-mt323:qt-mt323.dll
 0001:0000b500       ?focusInEvent@QPopupMenu@@MAEXPAVQFocusEvent@@@Z 1000c500 f   qt-mt323:qt-mt323.dll
 0001:0000b506       ?focusInEvent@QWidget@@MAEXPAVQFocusEvent@@@Z 1000c506 f   qt-mt323:qt-mt323.dll
 0001:0000b50c       ?focusNextPrevChild@QPopupMenu@@MAE_N_N@Z 1000c50c f   qt-mt323:qt-mt323.dll
 0001:0000b512       ?focusNextPrevChild@QWidget@@MAE_N_N@Z 1000c512 f   qt-mt323:qt-mt323.dll
 0001:0000b518       ?focusOutEvent@QPopupMenu@@MAEXPAVQFocusEvent@@@Z 1000c518 f   qt-mt323:qt-mt323.dll
 0001:0000b51e       ?focusOutEvent@QWidget@@MAEXPAVQFocusEvent@@@Z 1000c51e f   qt-mt323:qt-mt323.dll
 0001:0000b524       ?fontChange@QWidget@@MAEXABVQFont@@@Z 1000c524 f   qt-mt323:qt-mt323.dll
 0001:0000b52a       ?fontInf@QPaintDevice@@MBEHPAVQFont@@H@Z 1000c52a f   qt-mt323:qt-mt323.dll
 0001:0000b530       ?fontMet@QPaintDevice@@MBEHPAVQFont@@HPBDH@Z 1000c530 f   qt-mt323:qt-mt323.dll
 0001:0000b536       ?frameChanged@QFrame@@MAEXXZ 1000c536 f   qt-mt323:qt-mt323.dll
 0001:0000b53c       ?frameChanged@QPopupMenu@@EAEXXZ 1000c53c f   qt-mt323:qt-mt323.dll
 0001:0000b542       ?handle@QPaintDevice@@UBEPAUHDC__@@XZ 1000c542 f   qt-mt323:qt-mt323.dll
 0001:0000b548       ?heightForWidth@QWidget@@UBEHH@Z 1000c548 f   qt-mt323:qt-mt323.dll
 0001:0000b54e       ?hide@QPopupMenu@@UAEXXZ   1000c54e f   qt-mt323:qt-mt323.dll
 0001:0000b554       ?hide@QToolBar@@UAEXXZ     1000c554 f   qt-mt323:qt-mt323.dll
 0001:0000b55a       ?hide@QWidget@@UAEXXZ      1000c55a f   qt-mt323:qt-mt323.dll
 0001:0000b560       ?hideEvent@QDockWindow@@MAEXPAVQHideEvent@@@Z 1000c560 f   qt-mt323:qt-mt323.dll
 0001:0000b566       ?hideEvent@QWidget@@MAEXPAVQHideEvent@@@Z 1000c566 f   qt-mt323:qt-mt323.dll
 0001:0000b56c       ?imComposeEvent@QWidget@@MAEXPAVQIMEvent@@@Z 1000c56c f   qt-mt323:qt-mt323.dll
 0001:0000b572       ?imEndEvent@QWidget@@MAEXPAVQIMEvent@@@Z 1000c572 f   qt-mt323:qt-mt323.dll
 0001:0000b578       ?imStartEvent@QWidget@@MAEXPAVQIMEvent@@@Z 1000c578 f   qt-mt323:qt-mt323.dll
 0001:0000b57e       ?insertChild@QObject@@UAEXPAV1@@Z 1000c57e f   qt-mt323:qt-mt323.dll
 0001:0000b584       ?keyPressEvent@QPopupMenu@@MAEXPAVQKeyEvent@@@Z 1000c584 f   qt-mt323:qt-mt323.dll
 0001:0000b58a       ?keyPressEvent@QWidget@@MAEXPAVQKeyEvent@@@Z 1000c58a f   qt-mt323:qt-mt323.dll
 0001:0000b590       ?keyReleaseEvent@QWidget@@MAEXPAVQKeyEvent@@@Z 1000c590 f   qt-mt323:qt-mt323.dll
 0001:0000b596       ?leaveEvent@QPopupMenu@@MAEXPAVQEvent@@@Z 1000c596 f   qt-mt323:qt-mt323.dll
 0001:0000b59c       ?leaveEvent@QWidget@@MAEXPAVQEvent@@@Z 1000c59c f   qt-mt323:qt-mt323.dll
 0001:0000b5a2       ?menuContentsChanged@QPopupMenu@@EAEXXZ 1000c5a2 f   qt-mt323:qt-mt323.dll
 0001:0000b5a8       ?menuDelPopup@QPopupMenu@@EAEXPAV1@@Z 1000c5a8 f   qt-mt323:qt-mt323.dll
 0001:0000b5ae       ?menuInsPopup@QPopupMenu@@EAEXPAV1@@Z 1000c5ae f   qt-mt323:qt-mt323.dll
 0001:0000b5b4       ?menuStateChanged@QPopupMenu@@EAEXXZ 1000c5b4 f   qt-mt323:qt-mt323.dll
 0001:0000b5ba       ?metaObject@QAction@@UBEPAVQMetaObject@@XZ 1000c5ba f   qt-mt323:qt-mt323.dll
 0001:0000b5c0       ?metaObject@QGuardedPtrPrivate@@UBEPAVQMetaObject@@XZ 1000c5c0 f   qt-mt323:qt-mt323.dll
 0001:0000b5c6       ?metaObject@QPopupMenu@@UBEPAVQMetaObject@@XZ 1000c5c6 f   qt-mt323:qt-mt323.dll
 0001:0000b5cc       ?metaObject@QToolBar@@UBEPAVQMetaObject@@XZ 1000c5cc f   qt-mt323:qt-mt323.dll
 0001:0000b5d2       ?metaObject@QWidget@@UBEPAVQMetaObject@@XZ 1000c5d2 f   qt-mt323:qt-mt323.dll
 0001:0000b5d8       ?metric@QWidget@@MBEHH@Z   1000c5d8 f   qt-mt323:qt-mt323.dll
 0001:0000b5de       ?minimumSizeHint@QToolBar@@UBE?AVQSize@@XZ 1000c5de f   qt-mt323:qt-mt323.dll
 0001:0000b5e4       ?minimumSizeHint@QWidget@@UBE?AVQSize@@XZ 1000c5e4 f   qt-mt323:qt-mt323.dll
 0001:0000b5ea       ?mouseDoubleClickEvent@QWidget@@MAEXPAVQMouseEvent@@@Z 1000c5ea f   qt-mt323:qt-mt323.dll
 0001:0000b5f0       ?mouseMoveEvent@QPopupMenu@@MAEXPAVQMouseEvent@@@Z 1000c5f0 f   qt-mt323:qt-mt323.dll
 0001:0000b5f6       ?mouseMoveEvent@QWidget@@MAEXPAVQMouseEvent@@@Z 1000c5f6 f   qt-mt323:qt-mt323.dll
 0001:0000b5fc       ?mousePressEvent@QPopupMenu@@MAEXPAVQMouseEvent@@@Z 1000c5fc f   qt-mt323:qt-mt323.dll
 0001:0000b602       ?mousePressEvent@QWidget@@MAEXPAVQMouseEvent@@@Z 1000c602 f   qt-mt323:qt-mt323.dll
 0001:0000b608       ?mouseReleaseEvent@QPopupMenu@@MAEXPAVQMouseEvent@@@Z 1000c608 f   qt-mt323:qt-mt323.dll
 0001:0000b60e       ?mouseReleaseEvent@QWidget@@MAEXPAVQMouseEvent@@@Z 1000c60e f   qt-mt323:qt-mt323.dll
 0001:0000b614       ?move@QWidget@@UAEXHH@Z    1000c614 f   qt-mt323:qt-mt323.dll
 0001:0000b61a       ?moveEvent@QWidget@@MAEXPAVQMoveEvent@@@Z 1000c61a f   qt-mt323:qt-mt323.dll
 0001:0000b620       ?newItem@QPtrCollection@@MAEPAXPAX@Z 1000c620 f   qt-mt323:qt-mt323.dll
 0001:0000b626       ?paintEvent@QFrame@@MAEXPAVQPaintEvent@@@Z 1000c626 f   qt-mt323:qt-mt323.dll
 0001:0000b62c       ?paintEvent@QPopupMenu@@MAEXPAVQPaintEvent@@@Z 1000c62c f   qt-mt323:qt-mt323.dll
 0001:0000b632       ?paintEvent@QWidget@@MAEXPAVQPaintEvent@@@Z 1000c632 f   qt-mt323:qt-mt323.dll
 0001:0000b638       ?paletteChange@QWidget@@MAEXABVQPalette@@@Z 1000c638 f   qt-mt323:qt-mt323.dll
 0001:0000b63e       ?polish@QWidget@@UAEXXZ    1000c63e f   qt-mt323:qt-mt323.dll
 0001:0000b644       ?property@QObject@@UBE?AVQVariant@@PBD@Z 1000c644 f   qt-mt323:qt-mt323.dll
 0001:0000b64a       ?qt_cast@QAction@@UAEPAXPBD@Z 1000c64a f   qt-mt323:qt-mt323.dll
 0001:0000b650       ?qt_cast@QGuardedPtrPrivate@@UAEPAXPBD@Z 1000c650 f   qt-mt323:qt-mt323.dll
 0001:0000b656       ?qt_cast@QPopupMenu@@UAEPAXPBD@Z 1000c656 f   qt-mt323:qt-mt323.dll
 0001:0000b65c       ?qt_cast@QToolBar@@UAEPAXPBD@Z 1000c65c f   qt-mt323:qt-mt323.dll
 0001:0000b662       ?qt_cast@QWidget@@UAEPAXPBD@Z 1000c662 f   qt-mt323:qt-mt323.dll
 0001:0000b668       ?qt_emit@QAction@@UAE_NHPAUQUObject@@@Z 1000c668 f   qt-mt323:qt-mt323.dll
 0001:0000b66e       ?qt_emit@QGuardedPtrPrivate@@UAE_NHPAUQUObject@@@Z 1000c66e f   qt-mt323:qt-mt323.dll
 0001:0000b674       ?qt_emit@QPopupMenu@@UAE_NHPAUQUObject@@@Z 1000c674 f   qt-mt323:qt-mt323.dll
 0001:0000b67a       ?qt_emit@QToolBar@@UAE_NHPAUQUObject@@@Z 1000c67a f   qt-mt323:qt-mt323.dll
 0001:0000b680       ?qt_emit@QWidget@@UAE_NHPAUQUObject@@@Z 1000c680 f   qt-mt323:qt-mt323.dll
 0001:0000b686       ?qt_invoke@QAction@@UAE_NHPAUQUObject@@@Z 1000c686 f   qt-mt323:qt-mt323.dll
 0001:0000b68c       ?qt_invoke@QGuardedPtrPrivate@@UAE_NHPAUQUObject@@@Z 1000c68c f   qt-mt323:qt-mt323.dll
 0001:0000b692       ?qt_invoke@QPopupMenu@@UAE_NHPAUQUObject@@@Z 1000c692 f   qt-mt323:qt-mt323.dll
 0001:0000b698       ?qt_invoke@QToolBar@@UAE_NHPAUQUObject@@@Z 1000c698 f   qt-mt323:qt-mt323.dll
 0001:0000b69e       ?qt_invoke@QWidget@@UAE_NHPAUQUObject@@@Z 1000c69e f   qt-mt323:qt-mt323.dll
 0001:0000b6a4       ?qt_property@QAction@@UAE_NHHPAVQVariant@@@Z 1000c6a4 f   qt-mt323:qt-mt323.dll
 0001:0000b6aa       ?qt_property@QGuardedPtrPrivate@@UAE_NHHPAVQVariant@@@Z 1000c6aa f   qt-mt323:qt-mt323.dll
 0001:0000b6b0       ?qt_property@QPopupMenu@@UAE_NHHPAVQVariant@@@Z 1000c6b0 f   qt-mt323:qt-mt323.dll
 0001:0000b6b6       ?qt_property@QToolBar@@UAE_NHHPAVQVariant@@@Z 1000c6b6 f   qt-mt323:qt-mt323.dll
 0001:0000b6bc       ?qt_property@QWidget@@UAE_NHHPAVQVariant@@@Z 1000c6bc f   qt-mt323:qt-mt323.dll
 0001:0000b6c2       ?read@QGDict@@MAEAAVQDataStream@@AAV2@AAPAX@Z 1000c6c2 f   qt-mt323:qt-mt323.dll
 0001:0000b6c8       ?read@QGList@@MAEAAVQDataStream@@AAV2@AAPAX@Z 1000c6c8 f   qt-mt323:qt-mt323.dll
 0001:0000b6ce       ?removeChild@QObject@@UAEXPAV1@@Z 1000c6ce f   qt-mt323:qt-mt323.dll
 0001:0000b6d4       ?removeFrom@QAction@@UAE_NPAVQWidget@@@Z 1000c6d4 f   qt-mt323:qt-mt323.dll
 0001:0000b6da       ?reparent@QWidget@@UAEXPAV1@IABVQPoint@@_N@Z 1000c6da f   qt-mt323:qt-mt323.dll
 0001:0000b6e0       ?resize@QWidget@@UAEXHH@Z  1000c6e0 f   qt-mt323:qt-mt323.dll
 0001:0000b6e6       ?resizeEvent@QFrame@@MAEXPAVQResizeEvent@@@Z 1000c6e6 f   qt-mt323:qt-mt323.dll
 0001:0000b6ec       ?resizeEvent@QToolBar@@MAEXPAVQResizeEvent@@@Z 1000c6ec f   qt-mt323:qt-mt323.dll
 0001:0000b6f2       ?resizeEvent@QWidget@@MAEXPAVQResizeEvent@@@Z 1000c6f2 f   qt-mt323:qt-mt323.dll
 0001:0000b6f8       ?resolution@QPaintDevice@@UBEHXZ 1000c6f8 f   qt-mt323:qt-mt323.dll
 0001:0000b6fe       ?setAccel@QAction@@UAEXABVQKeySequence@@@Z 1000c6fe f   qt-mt323:qt-mt323.dll
 0001:0000b704       ?setAcceptDrops@QWidget@@UAEX_N@Z 1000c704 f   qt-mt323:qt-mt323.dll
 0001:0000b70a       ?setActiveItem@QPopupMenu@@UAEXH@Z 1000c70a f   qt-mt323:qt-mt323.dll
 0001:0000b710       ?setActiveWindow@QWidget@@UAEXXZ 1000c710 f   qt-mt323:qt-mt323.dll
 0001:0000b716       ?setAutoMask@QWidget@@UAEX_N@Z 1000c716 f   qt-mt323:qt-mt323.dll
 0001:0000b71c       ?setBackgroundColor@QWidget@@UAEXABVQColor@@@Z 1000c71c f   qt-mt323:qt-mt323.dll
 0001:0000b722       ?setBackgroundMode@QWidget@@UAEXW4BackgroundMode@Qt@@@Z 1000c722 f   qt-mt323:qt-mt323.dll
 0001:0000b728       ?setBackgroundOrigin@QWidget@@UAEXW4BackgroundOrigin@1@@Z 1000c728 f   qt-mt323:qt-mt323.dll
 0001:0000b72e       ?setBackgroundPixmap@QWidget@@UAEXABVQPixmap@@@Z 1000c72e f   qt-mt323:qt-mt323.dll
 0001:0000b734       ?setCaption@QDockWindow@@UAEXABVQString@@@Z 1000c734 f   qt-mt323:qt-mt323.dll
 0001:0000b73a       ?setCaption@QWidget@@UAEXABVQString@@@Z 1000c73a f   qt-mt323:qt-mt323.dll
 0001:0000b740       ?setCheckable@QPopupMenu@@UAEX_N@Z 1000c740 f   qt-mt323:qt-mt323.dll
 0001:0000b746       ?setCloseMode@QDockWindow@@UAEXH@Z 1000c746 f   qt-mt323:qt-mt323.dll
 0001:0000b74c       ?setCursor@QWidget@@UAEXABVQCursor@@@Z 1000c74c f   qt-mt323:qt-mt323.dll
 0001:0000b752       ?setEnabled@QAction@@UAEX_N@Z 1000c752 f   qt-mt323:qt-mt323.dll
 0001:0000b758       ?setEnabled@QWidget@@UAEX_N@Z 1000c758 f   qt-mt323:qt-mt323.dll
 0001:0000b75e       ?setEraseColor@QWidget@@UAEXABVQColor@@@Z 1000c75e f   qt-mt323:qt-mt323.dll
 0001:0000b764       ?setErasePixmap@QWidget@@UAEXABVQPixmap@@@Z 1000c764 f   qt-mt323:qt-mt323.dll
 0001:0000b76a       ?setFirstItemActive@QPopupMenu@@EAEXXZ 1000c76a f   qt-mt323:qt-mt323.dll
 0001:0000b770       ?setFixedExtentHeight@QDockWindow@@UAEXH@Z 1000c770 f   qt-mt323:qt-mt323.dll
 0001:0000b776       ?setFixedExtentWidth@QDockWindow@@UAEXH@Z 1000c776 f   qt-mt323:qt-mt323.dll
 0001:0000b77c       ?setFocus@QWidget@@UAEXXZ  1000c77c f   qt-mt323:qt-mt323.dll
 0001:0000b782       ?setFocusPolicy@QWidget@@UAEXW4FocusPolicy@1@@Z 1000c782 f   qt-mt323:qt-mt323.dll
 0001:0000b788       ?setFocusProxy@QWidget@@UAEXPAV1@@Z 1000c788 f   qt-mt323:qt-mt323.dll
 0001:0000b78e       ?setFont@QPopupMenu@@UAEXABVQFont@@@Z 1000c78e f   qt-mt323:qt-mt323.dll
 0001:0000b794       ?setFont@QWidget@@UAEXABVQFont@@@Z 1000c794 f   qt-mt323:qt-mt323.dll
 0001:0000b79a       ?setFrameRect@QFrame@@UAEXABVQRect@@@Z 1000c79a f   qt-mt323:qt-mt323.dll
 0001:0000b7a0       ?setFrameStyle@QFrame@@UAEXH@Z 1000c7a0 f   qt-mt323:qt-mt323.dll
 0001:0000b7a6       ?setGeometry@QWidget@@UAEXABVQRect@@@Z 1000c7a6 f   qt-mt323:qt-mt323.dll
 0001:0000b7ac       ?setGeometry@QWidget@@UAEXHHHH@Z 1000c7ac f   qt-mt323:qt-mt323.dll
 0001:0000b7b2       ?setHorizontallyStretchable@QDockWindow@@UAEX_N@Z 1000c7b2 f   qt-mt323:qt-mt323.dll
 0001:0000b7b8       ?setIcon@QWidget@@UAEXABVQPixmap@@@Z 1000c7b8 f   qt-mt323:qt-mt323.dll
 0001:0000b7be       ?setIconSet@QAction@@UAEXABVQIconSet@@@Z 1000c7be f   qt-mt323:qt-mt323.dll
 0001:0000b7c4       ?setIconText@QWidget@@UAEXABVQString@@@Z 1000c7c4 f   qt-mt323:qt-mt323.dll
 0001:0000b7ca       ?setId@QMenuData@@UAEXHH@Z 1000c7ca f   qt-mt323:qt-mt323.dll
 0001:0000b7d0       ?setKeyCompression@QWidget@@MAEX_N@Z 1000c7d0 f   qt-mt323:qt-mt323.dll
 0001:0000b7d6       ?setLabel@QToolBar@@UAEXABVQString@@@Z 1000c7d6 f   qt-mt323:qt-mt323.dll
 0001:0000b7dc       ?setLineWidth@QFrame@@UAEXH@Z 1000c7dc f   qt-mt323:qt-mt323.dll
 0001:0000b7e2       ?setMargin@QFrame@@UAEXH@Z 1000c7e2 f   qt-mt323:qt-mt323.dll
 0001:0000b7e8       ?setMask@QWidget@@UAEXABVQBitmap@@@Z 1000c7e8 f   qt-mt323:qt-mt323.dll
 0001:0000b7ee       ?setMask@QWidget@@UAEXABVQRegion@@@Z 1000c7ee f   qt-mt323:qt-mt323.dll
 0001:0000b7f4       ?setMaximumSize@QWidget@@UAEXHH@Z 1000c7f4 f   qt-mt323:qt-mt323.dll
 0001:0000b7fa       ?setMenuText@QAction@@UAEXABVQString@@@Z 1000c7fa f   qt-mt323:qt-mt323.dll
 0001:0000b800       ?setMicroFocusHint@QWidget@@MAEXHHHH_NPAVQFont@@@Z 1000c800 f   qt-mt323:qt-mt323.dll
 0001:0000b806       ?setMidLineWidth@QFrame@@UAEXH@Z 1000c806 f   qt-mt323:qt-mt323.dll
 0001:0000b80c       ?setMinimumSize@QToolBar@@UAEXHH@Z 1000c80c f   qt-mt323:qt-mt323.dll
 0001:0000b812       ?setMinimumSize@QWidget@@UAEXHH@Z 1000c812 f   qt-mt323:qt-mt323.dll
 0001:0000b818       ?setMouseTracking@QWidget@@UAEX_N@Z 1000c818 f   qt-mt323:qt-mt323.dll
 0001:0000b81e       ?setMovingEnabled@QDockWindow@@UAEX_N@Z 1000c81e f   qt-mt323:qt-mt323.dll
 0001:0000b824       ?setName@QObject@@UAEXPBD@Z 1000c824 f   qt-mt323:qt-mt323.dll
 0001:0000b82a       ?setNewLine@QDockWindow@@UAEX_N@Z 1000c82a f   qt-mt323:qt-mt323.dll
 0001:0000b830       ?setOffset@QDockWindow@@UAEXH@Z 1000c830 f   qt-mt323:qt-mt323.dll
 0001:0000b836       ?setOn@QAction@@UAEX_N@Z   1000c836 f   qt-mt323:qt-mt323.dll
 0001:0000b83c       ?setOpaqueMoving@QDockWindow@@UAEX_N@Z 1000c83c f   qt-mt323:qt-mt323.dll
 0001:0000b842       ?setOrientation@QToolBar@@UAEXW4Orientation@Qt@@@Z 1000c842 f   qt-mt323:qt-mt323.dll
 0001:0000b848       ?setPalette@QWidget@@UAEXABVQPalette@@@Z 1000c848 f   qt-mt323:qt-mt323.dll
 0001:0000b84e       ?setPaletteBackgroundColor@QWidget@@UAEXABVQColor@@@Z 1000c84e f   qt-mt323:qt-mt323.dll
 0001:0000b854       ?setPaletteBackgroundPixmap@QWidget@@UAEXABVQPixmap@@@Z 1000c854 f   qt-mt323:qt-mt323.dll
 0001:0000b85a       ?setProperty@QObject@@UAE_NPBDABVQVariant@@@Z 1000c85a f   qt-mt323:qt-mt323.dll
 0001:0000b860       ?setResizeEnabled@QDockWindow@@UAEX_N@Z 1000c860 f   qt-mt323:qt-mt323.dll
 0001:0000b866       ?setResolution@QPaintDevice@@UAEXH@Z 1000c866 f   qt-mt323:qt-mt323.dll
 0001:0000b86c       ?setSizeIncrement@QWidget@@UAEXHH@Z 1000c86c f   qt-mt323:qt-mt323.dll
 0001:0000b872       ?setSizePolicy@QWidget@@UAEXVQSizePolicy@@@Z 1000c872 f   qt-mt323:qt-mt323.dll
 0001:0000b878       ?setStatusTip@QAction@@UAEXABVQString@@@Z 1000c878 f   qt-mt323:qt-mt323.dll
 0001:0000b87e       ?setStretchableWidget@QToolBar@@UAEXPAVQWidget@@@Z 1000c87e f   qt-mt323:qt-mt323.dll
 0001:0000b884       ?setText@QAction@@UAEXABVQString@@@Z 1000c884 f   qt-mt323:qt-mt323.dll
 0001:0000b88a       ?setToggleAction@QAction@@UAEX_N@Z 1000c88a f   qt-mt323:qt-mt323.dll
 0001:0000b890       ?setToolTip@QAction@@UAEXABVQString@@@Z 1000c890 f   qt-mt323:qt-mt323.dll
 0001:0000b896       ?setUpdatesEnabled@QWidget@@UAEX_N@Z 1000c896 f   qt-mt323:qt-mt323.dll
 0001:0000b89c       ?setVerticallyStretchable@QDockWindow@@UAEX_N@Z 1000c89c f   qt-mt323:qt-mt323.dll
 0001:0000b8a2       ?setWFlags@QWidget@@MAEXI@Z 1000c8a2 f   qt-mt323:qt-mt323.dll
 0001:0000b8a8       ?setWState@QWidget@@MAEXI@Z 1000c8a8 f   qt-mt323:qt-mt323.dll
 0001:0000b8ae       ?setWhatsThis@QAction@@UAEXABVQString@@@Z 1000c8ae f   qt-mt323:qt-mt323.dll
 0001:0000b8b4       ?setWidget@QDockWindow@@UAEXPAVQWidget@@@Z 1000c8b4 f   qt-mt323:qt-mt323.dll
 0001:0000b8ba       ?show@QPopupMenu@@UAEXXZ   1000c8ba f   qt-mt323:qt-mt323.dll
 0001:0000b8c0       ?show@QToolBar@@UAEXXZ     1000c8c0 f   qt-mt323:qt-mt323.dll
 0001:0000b8c6       ?show@QWidget@@UAEXXZ      1000c8c6 f   qt-mt323:qt-mt323.dll
 0001:0000b8cc       ?showEvent@QDockWindow@@MAEXPAVQShowEvent@@@Z 1000c8cc f   qt-mt323:qt-mt323.dll
 0001:0000b8d2       ?showEvent@QWidget@@MAEXPAVQShowEvent@@@Z 1000c8d2 f   qt-mt323:qt-mt323.dll
 0001:0000b8d8       ?showMaximized@QWidget@@UAEXXZ 1000c8d8 f   qt-mt323:qt-mt323.dll
 0001:0000b8de       ?showMinimized@QWidget@@UAEXXZ 1000c8de f   qt-mt323:qt-mt323.dll
 0001:0000b8e4       ?showNormal@QWidget@@UAEXXZ 1000c8e4 f   qt-mt323:qt-mt323.dll
 0001:0000b8ea       ?sizeHint@QDockWindow@@UBE?AVQSize@@XZ 1000c8ea f   qt-mt323:qt-mt323.dll
 0001:0000b8f0       ?sizeHint@QPopupMenu@@UBE?AVQSize@@XZ 1000c8f0 f   qt-mt323:qt-mt323.dll
 0001:0000b8f6       ?sizeHint@QWidget@@UBE?AVQSize@@XZ 1000c8f6 f   qt-mt323:qt-mt323.dll
 0001:0000b8fc       ?sizePolicy@QWidget@@UBE?AVQSizePolicy@@XZ 1000c8fc f   qt-mt323:qt-mt323.dll
 0001:0000b902       ?styleChange@QPopupMenu@@MAEXAAVQStyle@@@Z 1000c902 f   qt-mt323:qt-mt323.dll
 0001:0000b908       ?styleChange@QToolBar@@MAEXAAVQStyle@@@Z 1000c908 f   qt-mt323:qt-mt323.dll
 0001:0000b90e       ?styleChange@QWidget@@MAEXAAVQStyle@@@Z 1000c90e f   qt-mt323:qt-mt323.dll
 0001:0000b914       ?tabletEvent@QWidget@@MAEXPAVQTabletEvent@@@Z 1000c914 f   qt-mt323:qt-mt323.dll
 0001:0000b91a       ?timerEvent@QObject@@MAEXPAVQTimerEvent@@@Z 1000c91a f   qt-mt323:qt-mt323.dll
 0001:0000b920       ?timerEvent@QPopupMenu@@MAEXPAVQTimerEvent@@@Z 1000c920 f   qt-mt323:qt-mt323.dll
 0001:0000b926       ?undock@QDockWindow@@UAEXPAVQWidget@@@Z 1000c926 f   qt-mt323:qt-mt323.dll
 0001:0000b92c       ?undock@QDockWindow@@UAEXXZ 1000c92c f   qt-mt323:qt-mt323.dll
 0001:0000b932       ?unsetCursor@QWidget@@UAEXXZ 1000c932 f   qt-mt323:qt-mt323.dll
 0001:0000b938       ?updateItem@QPopupMenu@@UAEXH@Z 1000c938 f   qt-mt323:qt-mt323.dll
 0001:0000b93e       ?updateMask@QWidget@@MAEXXZ 1000c93e f   qt-mt323:qt-mt323.dll
 0001:0000b944       ?wheelEvent@QWidget@@MAEXPAVQWheelEvent@@@Z 1000c944 f   qt-mt323:qt-mt323.dll
 0001:0000b94a       ?winEvent@QWidget@@MAE_NPAUtagMSG@@@Z 1000c94a f   qt-mt323:qt-mt323.dll
 0001:0000b950       ?windowActivationChange@QWidget@@MAEX_N@Z 1000c950 f   qt-mt323:qt-mt323.dll
 0001:0000b956       ?write@QGDict@@MBEAAVQDataStream@@AAV2@PAX@Z 1000c956 f   qt-mt323:qt-mt323.dll
 0001:0000b95c       ?write@QGList@@MBEAAVQDataStream@@AAV2@PAX@Z 1000c95c f   qt-mt323:qt-mt323.dll
 0001:0000b962       ?replaceChild@QDomNode@@UAE?AV1@ABV1@0@Z 1000c962 f   qt-mt323:qt-mt323.dll
 0001:0000b968       ?removeChild@QDomNode@@UAE?AV1@ABV1@@Z 1000c968 f   qt-mt323:qt-mt323.dll
 0001:0000b96e       ?appendChild@QDomNode@@UAE?AV1@ABV1@@Z 1000c96e f   qt-mt323:qt-mt323.dll
 0001:0000b974       ?cloneNode@QDomNode@@UBE?AV1@_N@Z 1000c974 f   qt-mt323:qt-mt323.dll
 0001:0000b97a       ?firstChild@QDomNode@@UBE?AV1@XZ 1000c97a f   qt-mt323:qt-mt323.dll
 0001:0000b980       ?nextSibling@QDomNode@@UBE?AV1@XZ 1000c980 f   qt-mt323:qt-mt323.dll
 0001:0000b986       ?attributes@QDomElement@@UBE?AVQDomNamedNodeMap@@XZ 1000c986 f   qt-mt323:qt-mt323.dll
 0001:0000b98c       ?attributes@QDomNode@@UBE?AVQDomNamedNodeMap@@XZ 1000c98c f   qt-mt323:qt-mt323.dll
 0001:0000b992       ?childNodes@QDomNode@@UBE?AVQDomNodeList@@XZ 1000c992 f   qt-mt323:qt-mt323.dll
 0001:0000b998       ?elementsByTagName@QDomElement@@UBE?AVQDomNodeList@@ABVQString@@@Z 1000c998 f   qt-mt323:qt-mt323.dll
 0001:0000b99e       ?elementsByTagNameNS@QDomElement@@UBE?AVQDomNodeList@@ABVQString@@0@Z 1000c99e f   qt-mt323:qt-mt323.dll
 0001:0000b9a4       ?hasAttributes@QDomNode@@UBE_NXZ 1000c9a4 f   qt-mt323:qt-mt323.dll
 0001:0000b9aa       ?hasChildNodes@QDomNode@@UBE_NXZ 1000c9aa f   qt-mt323:qt-mt323.dll
 0001:0000b9b0       ?insertAfter@QDomNode@@UAE?AV1@ABV1@0@Z 1000c9b0 f   qt-mt323:qt-mt323.dll
 0001:0000b9b6       ?insertBefore@QDomNode@@UAE?AV1@ABV1@0@Z 1000c9b6 f   qt-mt323:qt-mt323.dll
 0001:0000b9bc       ?isAttr@QDomNode@@UBE_NXZ  1000c9bc f   qt-mt323:qt-mt323.dll
 0001:0000b9c2       ?isCDATASection@QDomNode@@UBE_NXZ 1000c9c2 f   qt-mt323:qt-mt323.dll
 0001:0000b9c8       ?isCharacterData@QDomNode@@UBE_NXZ 1000c9c8 f   qt-mt323:qt-mt323.dll
 0001:0000b9ce       ?isComment@QDomNode@@UBE_NXZ 1000c9ce f   qt-mt323:qt-mt323.dll
 0001:0000b9d4       ?isDocument@QDomDocument@@UBE_NXZ 1000c9d4 f   qt-mt323:qt-mt323.dll
 0001:0000b9da       ?isDocument@QDomNode@@UBE_NXZ 1000c9da f   qt-mt323:qt-mt323.dll
 0001:0000b9e0       ?isDocumentFragment@QDomNode@@UBE_NXZ 1000c9e0 f   qt-mt323:qt-mt323.dll
 0001:0000b9e6       ?isDocumentType@QDomNode@@UBE_NXZ 1000c9e6 f   qt-mt323:qt-mt323.dll
 0001:0000b9ec       ?isElement@QDomElement@@UBE_NXZ 1000c9ec f   qt-mt323:qt-mt323.dll
 0001:0000b9f2       ?isElement@QDomNode@@UBE_NXZ 1000c9f2 f   qt-mt323:qt-mt323.dll
 0001:0000b9f8       ?isEntity@QDomNode@@UBE_NXZ 1000c9f8 f   qt-mt323:qt-mt323.dll
 0001:0000b9fe       ?isEntityReference@QDomNode@@UBE_NXZ 1000c9fe f   qt-mt323:qt-mt323.dll
 0001:0000ba04       ?isNotation@QDomNode@@UBE_NXZ 1000ca04 f   qt-mt323:qt-mt323.dll
 0001:0000ba0a       ?isProcessingInstruction@QDomNode@@UBE_NXZ 1000ca0a f   qt-mt323:qt-mt323.dll
 0001:0000ba10       ?isSupported@QDomNode@@UBE_NABVQString@@0@Z 1000ca10 f   qt-mt323:qt-mt323.dll
 0001:0000ba16       ?isText@QDomNode@@UBE_NXZ  1000ca16 f   qt-mt323:qt-mt323.dll
 0001:0000ba1c       ?lastChild@QDomNode@@UBE?AV1@XZ 1000ca1c f   qt-mt323:qt-mt323.dll
 0001:0000ba22       ?localName@QDomNode@@UBE?AVQString@@XZ 1000ca22 f   qt-mt323:qt-mt323.dll
 0001:0000ba28       ?namespaceURI@QDomNode@@UBE?AVQString@@XZ 1000ca28 f   qt-mt323:qt-mt323.dll
 0001:0000ba2e       ?nodeName@QDomNode@@UBE?AVQString@@XZ 1000ca2e f   qt-mt323:qt-mt323.dll
 0001:0000ba34       ?nodeType@QDomDocument@@UBE?AW4NodeType@QDomNode@@XZ 1000ca34 f   qt-mt323:qt-mt323.dll
 0001:0000ba3a       ?nodeType@QDomElement@@UBE?AW4NodeType@QDomNode@@XZ 1000ca3a f   qt-mt323:qt-mt323.dll
 0001:0000ba40       ?nodeValue@QDomNode@@UBE?AVQString@@XZ 1000ca40 f   qt-mt323:qt-mt323.dll
 0001:0000ba46       ?normalize@QDomNode@@UAEXXZ 1000ca46 f   qt-mt323:qt-mt323.dll
 0001:0000ba4c       ?ownerDocument@QDomNode@@UBE?AVQDomDocument@@XZ 1000ca4c f   qt-mt323:qt-mt323.dll
 0001:0000ba52       ?parentNode@QDomNode@@UBE?AV1@XZ 1000ca52 f   qt-mt323:qt-mt323.dll
 0001:0000ba58       ?prefix@QDomNode@@UBE?AVQString@@XZ 1000ca58 f   qt-mt323:qt-mt323.dll
 0001:0000ba5e       ?previousSibling@QDomNode@@UBE?AV1@XZ 1000ca5e f   qt-mt323:qt-mt323.dll
 0001:0000ba64       ?setNodeValue@QDomNode@@UAEXABVQString@@@Z 1000ca64 f   qt-mt323:qt-mt323.dll
 0001:0000ba6a       ?setPrefix@QDomNode@@UAEXABVQString@@@Z 1000ca6a f   qt-mt323:qt-mt323.dll
 0001:0000ba70       ?minimumSizeHint@QDialog@@UBE?AVQSize@@XZ 1000ca70 f   qt-mt323:qt-mt323.dll
 0001:0000ba76       ?accept@QDialog@@MAEXXZ    1000ca76 f   qt-mt323:qt-mt323.dll
 0001:0000ba7c       ?addChild@QScrollView@@UAEXPAVQWidget@@HH@Z 1000ca7c f   qt-mt323:qt-mt323.dll
 0001:0000ba82       ?addItem@QBoxLayout@@UAEXPAVQLayoutItem@@@Z 1000ca82 f   qt-mt323:qt-mt323.dll
 0001:0000ba88       ?childEvent@QLayout@@MAEXPAVQChildEvent@@@Z 1000ca88 f   qt-mt323:qt-mt323.dll
 0001:0000ba8e       ?className@QHBoxLayout@@UBEPBDXZ 1000ca8e f   qt-mt323:qt-mt323.dll
 0001:0000ba94       ?className@QLabel@@UBEPBDXZ 1000ca94 f   qt-mt323:qt-mt323.dll
 0001:0000ba9a       ?className@QListBox@@UBEPBDXZ 1000ca9a f   qt-mt323:qt-mt323.dll
 0001:0000baa0       ?className@QPushButton@@UBEPBDXZ 1000caa0 f   qt-mt323:qt-mt323.dll
 0001:0000baa6       ?className@QVBoxLayout@@UBEPBDXZ 1000caa6 f   qt-mt323:qt-mt323.dll
 0001:0000baac       ?clearSelection@QListBox@@UAEXXZ 1000caac f   qt-mt323:qt-mt323.dll
 0001:0000bab2       ?closeEvent@QDialog@@MAEXPAVQCloseEvent@@@Z 1000cab2 f   qt-mt323:qt-mt323.dll
 0001:0000bab8       ?contentsContextMenuEvent@QListBox@@MAEXPAVQContextMenuEvent@@@Z 1000cab8 f   qt-mt323:qt-mt323.dll
 0001:0000babe       ?contentsDragEnterEvent@QScrollView@@MAEXPAVQDragEnterEvent@@@Z 1000cabe f   qt-mt323:qt-mt323.dll
 0001:0000bac4       ?contentsDragLeaveEvent@QScrollView@@MAEXPAVQDragLeaveEvent@@@Z 1000cac4 f   qt-mt323:qt-mt323.dll
 0001:0000baca       ?contentsDragMoveEvent@QScrollView@@MAEXPAVQDragMoveEvent@@@Z 1000caca f   qt-mt323:qt-mt323.dll
 0001:0000bad0       ?contentsDropEvent@QScrollView@@MAEXPAVQDropEvent@@@Z 1000cad0 f   qt-mt323:qt-mt323.dll
 0001:0000bad6       ?contentsMouseDoubleClickEvent@QScrollView@@MAEXPAVQMouseEvent@@@Z 1000cad6 f   qt-mt323:qt-mt323.dll
 0001:0000badc       ?contentsMouseMoveEvent@QScrollView@@MAEXPAVQMouseEvent@@@Z 1000cadc f   qt-mt323:qt-mt323.dll
 0001:0000bae2       ?contentsMousePressEvent@QScrollView@@MAEXPAVQMouseEvent@@@Z 1000cae2 f   qt-mt323:qt-mt323.dll
 0001:0000bae8       ?contentsMouseReleaseEvent@QScrollView@@MAEXPAVQMouseEvent@@@Z 1000cae8 f   qt-mt323:qt-mt323.dll
 0001:0000baee       ?contentsWheelEvent@QScrollView@@MAEXPAVQWheelEvent@@@Z 1000caee f   qt-mt323:qt-mt323.dll
 0001:0000baf4       ?contextMenuEvent@QDialog@@MAEXPAVQContextMenuEvent@@@Z 1000caf4 f   qt-mt323:qt-mt323.dll
 0001:0000bafa       ?contextMenuEvent@QScrollView@@MAEXPAVQContextMenuEvent@@@Z 1000cafa f   qt-mt323:qt-mt323.dll
 0001:0000bb00       ?done@QDialog@@MAEXH@Z     1000cb00 f   qt-mt323:qt-mt323.dll
 0001:0000bb06       ?drawButton@QPushButton@@MAEXPAVQPainter@@@Z 1000cb06 f   qt-mt323:qt-mt323.dll
 0001:0000bb0c       ?drawButtonLabel@QPushButton@@MAEXPAVQPainter@@@Z 1000cb0c f   qt-mt323:qt-mt323.dll
 0001:0000bb12       ?drawContents@QLabel@@MAEXPAVQPainter@@@Z 1000cb12 f   qt-mt323:qt-mt323.dll
 0001:0000bb18       ?drawContents@QScrollView@@EAEXPAVQPainter@@@Z 1000cb18 f   qt-mt323:qt-mt323.dll
 0001:0000bb1e       ?drawContents@QScrollView@@MAEXPAVQPainter@@HHHH@Z 1000cb1e f   qt-mt323:qt-mt323.dll
 0001:0000bb24       ?drawContentsOffset@QScrollView@@MAEXPAVQPainter@@HHHHHH@Z 1000cb24 f   qt-mt323:qt-mt323.dll
 0001:0000bb2a       ?enabledChange@QButton@@MAEX_N@Z 1000cb2a f   qt-mt323:qt-mt323.dll
 0001:0000bb30       ?ensureCurrentVisible@QListBox@@UAEXXZ 1000cb30 f   qt-mt323:qt-mt323.dll
 0001:0000bb36       ?eventFilter@QDialog@@MAE_NPAVQObject@@PAVQEvent@@@Z 1000cb36 f   qt-mt323:qt-mt323.dll
 0001:0000bb3c       ?eventFilter@QLayout@@MAE_NPAVQObject@@PAVQEvent@@@Z 1000cb3c f   qt-mt323:qt-mt323.dll
 0001:0000bb42       ?eventFilter@QListBox@@MAE_NPAVQObject@@PAVQEvent@@@Z 1000cb42 f   qt-mt323:qt-mt323.dll
 0001:0000bb48       ?expanding@QBoxLayout@@UBE?AW4ExpandData@QSizePolicy@@XZ 1000cb48 f   qt-mt323:qt-mt323.dll
 0001:0000bb4e       ?expanding@QSpacerItem@@UBE?AW4ExpandData@QSizePolicy@@XZ 1000cb4e f   qt-mt323:qt-mt323.dll
 0001:0000bb54       ?focusInEvent@QListBox@@MAEXPAVQFocusEvent@@@Z 1000cb54 f   qt-mt323:qt-mt323.dll
 0001:0000bb5a       ?focusInEvent@QPushButton@@MAEXPAVQFocusEvent@@@Z 1000cb5a f   qt-mt323:qt-mt323.dll
 0001:0000bb60       ?focusNextPrevChild@QScrollView@@MAE_N_N@Z 1000cb60 f   qt-mt323:qt-mt323.dll
 0001:0000bb66       ?focusOutEvent@QListBox@@MAEXPAVQFocusEvent@@@Z 1000cb66 f   qt-mt323:qt-mt323.dll
 0001:0000bb6c       ?focusOutEvent@QPushButton@@MAEXPAVQFocusEvent@@@Z 1000cb6c f   qt-mt323:qt-mt323.dll
 0001:0000bb72       ?fontChange@QLabel@@MAEXABVQFont@@@Z 1000cb72 f   qt-mt323:qt-mt323.dll
 0001:0000bb78       ?fontChange@QScrollView@@MAEXABVQFont@@@Z 1000cb78 f   qt-mt323:qt-mt323.dll
 0001:0000bb7e       ?frameChanged@QScrollView@@MAEXXZ 1000cb7e f   qt-mt323:qt-mt323.dll
 0001:0000bb84       ?geometry@QLayout@@UBE?AVQRect@@XZ 1000cb84 f   qt-mt323:qt-mt323.dll
 0001:0000bb8a       ?geometry@QSpacerItem@@UBE?AVQRect@@XZ 1000cb8a f   qt-mt323:qt-mt323.dll
 0001:0000bb90       ?hasHeightForWidth@QBoxLayout@@UBE_NXZ 1000cb90 f   qt-mt323:qt-mt323.dll
 0001:0000bb96       ?hasHeightForWidth@QLayoutItem@@UBE_NXZ 1000cb96 f   qt-mt323:qt-mt323.dll
 0001:0000bb9c       ?heightForWidth@QBoxLayout@@UBEHH@Z 1000cb9c f   qt-mt323:qt-mt323.dll
 0001:0000bba2       ?heightForWidth@QLabel@@UBEHH@Z 1000cba2 f   qt-mt323:qt-mt323.dll
 0001:0000bba8       ?heightForWidth@QLayoutItem@@UBEHH@Z 1000cba8 f   qt-mt323:qt-mt323.dll
 0001:0000bbae       ?hide@QDialog@@UAEXXZ      1000cbae f   qt-mt323:qt-mt323.dll
 0001:0000bbb4       ?hitButton@QButton@@MBE_NABVQPoint@@@Z 1000cbb4 f   qt-mt323:qt-mt323.dll
 0001:0000bbba       ?invalidate@QBoxLayout@@UAEXXZ 1000cbba f   qt-mt323:qt-mt323.dll
 0001:0000bbc0       ?invalidate@QLayoutItem@@UAEXXZ 1000cbc0 f   qt-mt323:qt-mt323.dll
 0001:0000bbc6       ?invertSelection@QListBox@@UAEXXZ 1000cbc6 f   qt-mt323:qt-mt323.dll
 0001:0000bbcc       ?isEmpty@QLayout@@UBE_NXZ  1000cbcc f   qt-mt323:qt-mt323.dll
 0001:0000bbd2       ?isEmpty@QSpacerItem@@UBE_NXZ 1000cbd2 f   qt-mt323:qt-mt323.dll
 0001:0000bbd8       ?iterator@QBoxLayout@@UAE?AVQLayoutIterator@@XZ 1000cbd8 f   qt-mt323:qt-mt323.dll
 0001:0000bbde       ?iterator@QLayoutItem@@UAE?AVQLayoutIterator@@XZ 1000cbde f   qt-mt323:qt-mt323.dll
 0001:0000bbe4       ?keyPressEvent@QButton@@MAEXPAVQKeyEvent@@@Z 1000cbe4 f   qt-mt323:qt-mt323.dll
 0001:0000bbea       ?keyPressEvent@QDialog@@MAEXPAVQKeyEvent@@@Z 1000cbea f   qt-mt323:qt-mt323.dll
 0001:0000bbf0       ?keyPressEvent@QListBox@@MAEXPAVQKeyEvent@@@Z 1000cbf0 f   qt-mt323:qt-mt323.dll
 0001:0000bbf6       ?keyReleaseEvent@QButton@@MAEXPAVQKeyEvent@@@Z 1000cbf6 f   qt-mt323:qt-mt323.dll
 0001:0000bbfc       ?layout@QLayout@@UAEPAV1@XZ 1000cbfc f   qt-mt323:qt-mt323.dll
 0001:0000bc02       ?layout@QLayoutItem@@UAEPAVQLayout@@XZ 1000cc02 f   qt-mt323:qt-mt323.dll
 0001:0000bc08       ?maximumSize@QBoxLayout@@UBE?AVQSize@@XZ 1000cc08 f   qt-mt323:qt-mt323.dll
 0001:0000bc0e       ?maximumSize@QSpacerItem@@UBE?AVQSize@@XZ 1000cc0e f   qt-mt323:qt-mt323.dll
 0001:0000bc14       ?metaObject@QHBoxLayout@@UBEPAVQMetaObject@@XZ 1000cc14 f   qt-mt323:qt-mt323.dll
 0001:0000bc1a       ?metaObject@QLabel@@UBEPAVQMetaObject@@XZ 1000cc1a f   qt-mt323:qt-mt323.dll
 0001:0000bc20       ?metaObject@QListBox@@UBEPAVQMetaObject@@XZ 1000cc20 f   qt-mt323:qt-mt323.dll
 0001:0000bc26       ?metaObject@QPushButton@@UBEPAVQMetaObject@@XZ 1000cc26 f   qt-mt323:qt-mt323.dll
 0001:0000bc2c       ?metaObject@QVBoxLayout@@UBEPAVQMetaObject@@XZ 1000cc2c f   qt-mt323:qt-mt323.dll
 0001:0000bc32       ?minimumSize@QBoxLayout@@UBE?AVQSize@@XZ 1000cc32 f   qt-mt323:qt-mt323.dll
 0001:0000bc38       ?minimumSize@QSpacerItem@@UBE?AVQSize@@XZ 1000cc38 f   qt-mt323:qt-mt323.dll
 0001:0000bc3e       ?minimumSizeHint@QLabel@@UBE?AVQSize@@XZ 1000cc3e f   qt-mt323:qt-mt323.dll
 0001:0000bc44       ?minimumSizeHint@QListBox@@UBE?AVQSize@@XZ 1000cc44 f   qt-mt323:qt-mt323.dll
 0001:0000bc4a       ?mouseDoubleClickEvent@QListBox@@MAEXPAVQMouseEvent@@@Z 1000cc4a f   qt-mt323:qt-mt323.dll
 0001:0000bc50       ?mouseMoveEvent@QButton@@MAEXPAVQMouseEvent@@@Z 1000cc50 f   qt-mt323:qt-mt323.dll
 0001:0000bc56       ?mouseMoveEvent@QListBox@@MAEXPAVQMouseEvent@@@Z 1000cc56 f   qt-mt323:qt-mt323.dll
 0001:0000bc5c       ?mousePressEvent@QButton@@MAEXPAVQMouseEvent@@@Z 1000cc5c f   qt-mt323:qt-mt323.dll
 0001:0000bc62       ?mousePressEvent@QListBox@@MAEXPAVQMouseEvent@@@Z 1000cc62 f   qt-mt323:qt-mt323.dll
 0001:0000bc68       ?mouseReleaseEvent@QButton@@MAEXPAVQMouseEvent@@@Z 1000cc68 f   qt-mt323:qt-mt323.dll
 0001:0000bc6e       ?mouseReleaseEvent@QListBox@@MAEXPAVQMouseEvent@@@Z 1000cc6e f   qt-mt323:qt-mt323.dll
 0001:0000bc74       ?move@QDialog@@UAEXHH@Z    1000cc74 f   qt-mt323:qt-mt323.dll
 0001:0000bc7a       ?move@QPushButton@@UAEXHH@Z 1000cc7a f   qt-mt323:qt-mt323.dll
 0001:0000bc80       ?moveChild@QScrollView@@UAEXPAVQWidget@@HH@Z 1000cc80 f   qt-mt323:qt-mt323.dll
 0001:0000bc86       ?paintCell@QListBox@@MAEXPAVQPainter@@HH@Z 1000cc86 f   qt-mt323:qt-mt323.dll
 0001:0000bc8c       ?paintEvent@QButton@@MAEXPAVQPaintEvent@@@Z 1000cc8c f   qt-mt323:qt-mt323.dll
 0001:0000bc92       ?qt_cast@QHBoxLayout@@UAEPAXPBD@Z 1000cc92 f   qt-mt323:qt-mt323.dll
 0001:0000bc98       ?qt_cast@QLabel@@UAEPAXPBD@Z 1000cc98 f   qt-mt323:qt-mt323.dll
 0001:0000bc9e       ?qt_cast@QListBox@@UAEPAXPBD@Z 1000cc9e f   qt-mt323:qt-mt323.dll
 0001:0000bca4       ?qt_cast@QPushButton@@UAEPAXPBD@Z 1000cca4 f   qt-mt323:qt-mt323.dll
 0001:0000bcaa       ?qt_cast@QVBoxLayout@@UAEPAXPBD@Z 1000ccaa f   qt-mt323:qt-mt323.dll
 0001:0000bcb0       ?qt_emit@QHBoxLayout@@UAE_NHPAUQUObject@@@Z 1000ccb0 f   qt-mt323:qt-mt323.dll
 0001:0000bcb6       ?qt_emit@QLabel@@UAE_NHPAUQUObject@@@Z 1000ccb6 f   qt-mt323:qt-mt323.dll
 0001:0000bcbc       ?qt_emit@QListBox@@UAE_NHPAUQUObject@@@Z 1000ccbc f   qt-mt323:qt-mt323.dll
 0001:0000bcc2       ?qt_emit@QPushButton@@UAE_NHPAUQUObject@@@Z 1000ccc2 f   qt-mt323:qt-mt323.dll
 0001:0000bcc8       ?qt_emit@QVBoxLayout@@UAE_NHPAUQUObject@@@Z 1000ccc8 f   qt-mt323:qt-mt323.dll
 0001:0000bcce       ?qt_invoke@QHBoxLayout@@UAE_NHPAUQUObject@@@Z 1000ccce f   qt-mt323:qt-mt323.dll
 0001:0000bcd4       ?qt_invoke@QLabel@@UAE_NHPAUQUObject@@@Z 1000ccd4 f   qt-mt323:qt-mt323.dll
 0001:0000bcda       ?qt_invoke@QListBox@@UAE_NHPAUQUObject@@@Z 1000ccda f   qt-mt323:qt-mt323.dll
 0001:0000bce0       ?qt_invoke@QPushButton@@UAE_NHPAUQUObject@@@Z 1000cce0 f   qt-mt323:qt-mt323.dll
 0001:0000bce6       ?qt_invoke@QVBoxLayout@@UAE_NHPAUQUObject@@@Z 1000cce6 f   qt-mt323:qt-mt323.dll
 0001:0000bcec       ?qt_property@QHBoxLayout@@UAE_NHHPAVQVariant@@@Z 1000ccec f   qt-mt323:qt-mt323.dll
 0001:0000bcf2       ?qt_property@QLabel@@UAE_NHHPAVQVariant@@@Z 1000ccf2 f   qt-mt323:qt-mt323.dll
 0001:0000bcf8       ?qt_property@QListBox@@UAE_NHHPAVQVariant@@@Z 1000ccf8 f   qt-mt323:qt-mt323.dll
 0001:0000bcfe       ?qt_property@QPushButton@@UAE_NHHPAVQVariant@@@Z 1000ccfe f   qt-mt323:qt-mt323.dll
 0001:0000bd04       ?qt_property@QVBoxLayout@@UAE_NHHPAVQVariant@@@Z 1000cd04 f   qt-mt323:qt-mt323.dll
 0001:0000bd0a       ?reject@QDialog@@MAEXXZ    1000cd0a f   qt-mt323:qt-mt323.dll
 0001:0000bd10       ?removeChild@QScrollView@@UAEXPAVQObject@@@Z 1000cd10 f   qt-mt323:qt-mt323.dll
 0001:0000bd16       ?resize@QDialog@@UAEXHH@Z  1000cd16 f   qt-mt323:qt-mt323.dll
 0001:0000bd1c       ?resize@QPushButton@@UAEXHH@Z 1000cd1c f   qt-mt323:qt-mt323.dll
 0001:0000bd22       ?resize@QScrollView@@UAEXHH@Z 1000cd22 f   qt-mt323:qt-mt323.dll
 0001:0000bd28       ?resizeContents@QScrollView@@UAEXHH@Z 1000cd28 f   qt-mt323:qt-mt323.dll
 0001:0000bd2e       ?resizeEvent@QDialog@@MAEXPAVQResizeEvent@@@Z 1000cd2e f   qt-mt323:qt-mt323.dll
 0001:0000bd34       ?resizeEvent@QLabel@@MAEXPAVQResizeEvent@@@Z 1000cd34 f   qt-mt323:qt-mt323.dll
 0001:0000bd3a       ?resizeEvent@QListBox@@MAEXPAVQResizeEvent@@@Z 1000cd3a f   qt-mt323:qt-mt323.dll
 0001:0000bd40       ?resizeEvent@QPushButton@@MAEXPAVQResizeEvent@@@Z 1000cd40 f   qt-mt323:qt-mt323.dll
 0001:0000bd46       ?selectAll@QListBox@@UAEX_N@Z 1000cd46 f   qt-mt323:qt-mt323.dll
 0001:0000bd4c       ?setAccel@QButton@@UAEXABVQKeySequence@@@Z 1000cd4c f   qt-mt323:qt-mt323.dll
 0001:0000bd52       ?setAlignment@QLabel@@UAEXH@Z 1000cd52 f   qt-mt323:qt-mt323.dll
 0001:0000bd58       ?setAlignment@QLayoutItem@@UAEXH@Z 1000cd58 f   qt-mt323:qt-mt323.dll
 0001:0000bd5e       ?setAutoAdd@QLayout@@UAEX_N@Z 1000cd5e f   qt-mt323:qt-mt323.dll
 0001:0000bd64       ?setAutoDefault@QPushButton@@UAEX_N@Z 1000cd64 f   qt-mt323:qt-mt323.dll
 0001:0000bd6a       ?setAutoRepeat@QButton@@UAEX_N@Z 1000cd6a f   qt-mt323:qt-mt323.dll
 0001:0000bd70       ?setAutoResize@QLabel@@UAEX_N@Z 1000cd70 f   qt-mt323:qt-mt323.dll
 0001:0000bd76       ?setBottomItem@QListBox@@UAEXH@Z 1000cd76 f   qt-mt323:qt-mt323.dll
 0001:0000bd7c       ?setBuddy@QLabel@@UAEXPAVQWidget@@@Z 1000cd7c f   qt-mt323:qt-mt323.dll
 0001:0000bd82       ?setColumnMode@QListBox@@UAEXH@Z 1000cd82 f   qt-mt323:qt-mt323.dll
 0001:0000bd88       ?setColumnMode@QListBox@@UAEXW4LayoutMode@1@@Z 1000cd88 f   qt-mt323:qt-mt323.dll
 0001:0000bd8e       ?setContentsPos@QScrollView@@UAEXHH@Z 1000cd8e f   qt-mt323:qt-mt323.dll
 0001:0000bd94       ?setCornerWidget@QScrollView@@UAEXPAVQWidget@@@Z 1000cd94 f   qt-mt323:qt-mt323.dll
 0001:0000bd9a       ?setCurrentItem@QListBox@@UAEXH@Z 1000cd9a f   qt-mt323:qt-mt323.dll
 0001:0000bda0       ?setCurrentItem@QListBox@@UAEXPAVQListBoxItem@@@Z 1000cda0 f   qt-mt323:qt-mt323.dll
 0001:0000bda6       ?setDefault@QPushButton@@UAEX_N@Z 1000cda6 f   qt-mt323:qt-mt323.dll
 0001:0000bdac       ?setDown@QButton@@UAEX_N@Z 1000cdac f   qt-mt323:qt-mt323.dll
 0001:0000bdb2       ?setDragAutoScroll@QScrollView@@UAEX_N@Z 1000cdb2 f   qt-mt323:qt-mt323.dll
 0001:0000bdb8       ?setEnabled@QScrollView@@UAEX_N@Z 1000cdb8 f   qt-mt323:qt-mt323.dll
 0001:0000bdbe       ?setFont@QLabel@@UAEXABVQFont@@@Z 1000cdbe f   qt-mt323:qt-mt323.dll
 0001:0000bdc4       ?setFont@QListBox@@UAEXABVQFont@@@Z 1000cdc4 f   qt-mt323:qt-mt323.dll
 0001:0000bdca       ?setGeometry@QBoxLayout@@UAEXABVQRect@@@Z 1000cdca f   qt-mt323:qt-mt323.dll
 0001:0000bdd0       ?setGeometry@QDialog@@UAEXABVQRect@@@Z 1000cdd0 f   qt-mt323:qt-mt323.dll
 0001:0000bdd6       ?setGeometry@QDialog@@UAEXHHHH@Z 1000cdd6 f   qt-mt323:qt-mt323.dll
 0001:0000bddc       ?setGeometry@QPushButton@@UAEXABVQRect@@@Z 1000cddc f   qt-mt323:qt-mt323.dll
 0001:0000bde2       ?setGeometry@QPushButton@@UAEXHHHH@Z 1000cde2 f   qt-mt323:qt-mt323.dll
 0001:0000bde8       ?setGeometry@QSpacerItem@@UAEXABVQRect@@@Z 1000cde8 f   qt-mt323:qt-mt323.dll
 0001:0000bdee       ?setGroup@QButton@@EAEXPAVQButtonGroup@@@Z 1000cdee f   qt-mt323:qt-mt323.dll
 0001:0000bdf4       ?setHBarGeometry@QScrollView@@MAEXAAVQScrollBar@@HHHH@Z 1000cdf4 f   qt-mt323:qt-mt323.dll
 0001:0000bdfa       ?setHScrollBarMode@QScrollView@@UAEXW4ScrollBarMode@1@@Z 1000cdfa f   qt-mt323:qt-mt323.dll
 0001:0000be00       ?setIsMenuButton@QPushButton@@UAEX_N@Z 1000ce00 f   qt-mt323:qt-mt323.dll
 0001:0000be06       ?setMargin@QLayout@@UAEXH@Z 1000ce06 f   qt-mt323:qt-mt323.dll
 0001:0000be0c       ?setMargins@QScrollView@@MAEXHHHH@Z 1000ce0c f   qt-mt323:qt-mt323.dll
 0001:0000be12       ?setMenuBar@QLayout@@UAEXPAVQMenuBar@@@Z 1000ce12 f   qt-mt323:qt-mt323.dll
 0001:0000be18       ?setMovie@QLabel@@UAEXABVQMovie@@@Z 1000ce18 f   qt-mt323:qt-mt323.dll
 0001:0000be1e       ?setNum@QLabel@@UAEXH@Z    1000ce1e f   qt-mt323:qt-mt323.dll
 0001:0000be24       ?setNum@QLabel@@UAEXN@Z    1000ce24 f   qt-mt323:qt-mt323.dll
 0001:0000be2a       ?setOn@QPushButton@@UAEX_N@Z 1000ce2a f   qt-mt323:qt-mt323.dll
 0001:0000be30       ?setPicture@QLabel@@UAEXABVQPicture@@@Z 1000ce30 f   qt-mt323:qt-mt323.dll
 0001:0000be36       ?setPixmap@QButton@@UAEXABVQPixmap@@@Z 1000ce36 f   qt-mt323:qt-mt323.dll
 0001:0000be3c       ?setPixmap@QLabel@@UAEXABVQPixmap@@@Z 1000ce3c f   qt-mt323:qt-mt323.dll
 0001:0000be42       ?setResizePolicy@QScrollView@@UAEXW4ResizePolicy@1@@Z 1000ce42 f   qt-mt323:qt-mt323.dll
 0001:0000be48       ?setRowMode@QListBox@@UAEXH@Z 1000ce48 f   qt-mt323:qt-mt323.dll
 0001:0000be4e       ?setRowMode@QListBox@@UAEXW4LayoutMode@1@@Z 1000ce4e f   qt-mt323:qt-mt323.dll
 0001:0000be54       ?setSelected@QListBox@@UAEXPAVQListBoxItem@@_N@Z 1000ce54 f   qt-mt323:qt-mt323.dll
 0001:0000be5a       ?setSelectionMode@QListBox@@UAEXW4SelectionMode@1@@Z 1000ce5a f   qt-mt323:qt-mt323.dll
 0001:0000be60       ?setSpacing@QLayout@@UAEXH@Z 1000ce60 f   qt-mt323:qt-mt323.dll
 0001:0000be66       ?setState@QButton@@MAEXW4ToggleState@1@@Z 1000ce66 f   qt-mt323:qt-mt323.dll
 0001:0000be6c       ?setText@QButton@@UAEXABVQString@@@Z 1000ce6c f   qt-mt323:qt-mt323.dll
 0001:0000be72       ?setText@QLabel@@UAEXABVQString@@@Z 1000ce72 f   qt-mt323:qt-mt323.dll
 0001:0000be78       ?setToggleType@QButton@@MAEXW4ToggleType@1@@Z 1000ce78 f   qt-mt323:qt-mt323.dll
 0001:0000be7e       ?setTopItem@QListBox@@UAEXH@Z 1000ce7e f   qt-mt323:qt-mt323.dll
 0001:0000be84       ?setVBarGeometry@QScrollView@@MAEXAAVQScrollBar@@HHHH@Z 1000ce84 f   qt-mt323:qt-mt323.dll
 0001:0000be8a       ?setVScrollBarMode@QScrollView@@UAEXW4ScrollBarMode@1@@Z 1000ce8a f   qt-mt323:qt-mt323.dll
 0001:0000be90       ?setVariableHeight@QListBox@@UAEX_N@Z 1000ce90 f   qt-mt323:qt-mt323.dll
 0001:0000be96       ?setVariableWidth@QListBox@@UAEX_N@Z 1000ce96 f   qt-mt323:qt-mt323.dll
 0001:0000be9c       ?show@QDialog@@UAEXXZ      1000ce9c f   qt-mt323:qt-mt323.dll
 0001:0000bea2       ?show@QScrollView@@UAEXXZ  1000cea2 f   qt-mt323:qt-mt323.dll
 0001:0000bea8       ?showEvent@QListBox@@MAEXPAVQShowEvent@@@Z 1000cea8 f   qt-mt323:qt-mt323.dll
 0001:0000beae       ?sizeHint@QBoxLayout@@UBE?AVQSize@@XZ 1000ceae f   qt-mt323:qt-mt323.dll
 0001:0000beb4       ?sizeHint@QDialog@@UBE?AVQSize@@XZ 1000ceb4 f   qt-mt323:qt-mt323.dll
 0001:0000beba       ?sizeHint@QLabel@@UBE?AVQSize@@XZ 1000ceba f   qt-mt323:qt-mt323.dll
 0001:0000bec0       ?sizeHint@QListBox@@UBE?AVQSize@@XZ 1000cec0 f   qt-mt323:qt-mt323.dll
 0001:0000bec6       ?sizeHint@QPushButton@@UBE?AVQSize@@XZ 1000cec6 f   qt-mt323:qt-mt323.dll
 0001:0000becc       ?sizeHint@QSpacerItem@@UBE?AVQSize@@XZ 1000cecc f   qt-mt323:qt-mt323.dll
 0001:0000bed2       ?spacerItem@QLayoutItem@@UAEPAVQSpacerItem@@XZ 1000ced2 f   qt-mt323:qt-mt323.dll
 0001:0000bed8       ?spacerItem@QSpacerItem@@UAEPAV1@XZ 1000ced8 f   qt-mt323:qt-mt323.dll
 0001:0000bede       ?styleChange@QFrame@@MAEXAAVQStyle@@@Z 1000cede f   qt-mt323:qt-mt323.dll
 0001:0000bee4       ?styleChange@QScrollView@@UAEXAAVQStyle@@@Z 1000cee4 f   qt-mt323:qt-mt323.dll
 0001:0000beea       ?updateMask@QPushButton@@MAEXXZ 1000ceea f   qt-mt323:qt-mt323.dll
 0001:0000bef0       ?viewportContextMenuEvent@QScrollView@@MAEXPAVQContextMenuEvent@@@Z 1000cef0 f   qt-mt323:qt-mt323.dll
 0001:0000bef6       ?viewportDragEnterEvent@QScrollView@@MAEXPAVQDragEnterEvent@@@Z 1000cef6 f   qt-mt323:qt-mt323.dll
 0001:0000befc       ?viewportDragLeaveEvent@QScrollView@@MAEXPAVQDragLeaveEvent@@@Z 1000cefc f   qt-mt323:qt-mt323.dll
 0001:0000bf02       ?viewportDragMoveEvent@QScrollView@@MAEXPAVQDragMoveEvent@@@Z 1000cf02 f   qt-mt323:qt-mt323.dll
 0001:0000bf08       ?viewportDropEvent@QScrollView@@MAEXPAVQDropEvent@@@Z 1000cf08 f   qt-mt323:qt-mt323.dll
 0001:0000bf0e       ?viewportMouseDoubleClickEvent@QScrollView@@MAEXPAVQMouseEvent@@@Z 1000cf0e f   qt-mt323:qt-mt323.dll
 0001:0000bf14       ?viewportMouseMoveEvent@QScrollView@@MAEXPAVQMouseEvent@@@Z 1000cf14 f   qt-mt323:qt-mt323.dll
 0001:0000bf1a       ?viewportMousePressEvent@QScrollView@@MAEXPAVQMouseEvent@@@Z 1000cf1a f   qt-mt323:qt-mt323.dll
 0001:0000bf20       ?viewportMouseReleaseEvent@QScrollView@@MAEXPAVQMouseEvent@@@Z 1000cf20 f   qt-mt323:qt-mt323.dll
 0001:0000bf26       ?viewportPaintEvent@QListBox@@UAEXPAVQPaintEvent@@@Z 1000cf26 f   qt-mt323:qt-mt323.dll
 0001:0000bf2c       ?viewportResizeEvent@QScrollView@@MAEXPAVQResizeEvent@@@Z 1000cf2c f   qt-mt323:qt-mt323.dll
 0001:0000bf32       ?viewportWheelEvent@QScrollView@@MAEXPAVQWheelEvent@@@Z 1000cf32 f   qt-mt323:qt-mt323.dll
 0001:0000bf38       ?wheelEvent@QScrollView@@MAEXPAVQWheelEvent@@@Z 1000cf38 f   qt-mt323:qt-mt323.dll
 0001:0000bf3e       ?widget@QLayoutItem@@UAEPAVQWidget@@XZ 1000cf3e f   qt-mt323:qt-mt323.dll
 0001:0000bf44       ?windowActivationChange@QListBox@@MAEX_N@Z 1000cf44 f   qt-mt323:qt-mt323.dll
 0001:0000bf4a       ?sortColumn@QTable@@UAEXH_N0@Z 1000cf4a f   qt-mt323:qt-mt323.dll
 0001:0000bf50       ?setLeftMargin@QTable@@UAEXH@Z 1000cf50 f   qt-mt323:qt-mt323.dll
 0001:0000bf56       ?activateNextCell@QTable@@MAEXXZ 1000cf56 f   qt-mt323:qt-mt323.dll
 0001:0000bf5c       ?addSelection@QTable@@UAEHABVQTableSelection@@@Z 1000cf5c f   qt-mt323:qt-mt323.dll
 0001:0000bf62       ?adjustColumn@QTable@@UAEXH@Z 1000cf62 f   qt-mt323:qt-mt323.dll
 0001:0000bf68       ?adjustRow@QTable@@UAEXH@Z 1000cf68 f   qt-mt323:qt-mt323.dll
 0001:0000bf6e       ?beginEdit@QTable@@MAEPAVQWidget@@HH_N@Z 1000cf6e f   qt-mt323:qt-mt323.dll
 0001:0000bf74       ?cellGeometry@QTable@@UBE?AVQRect@@HH@Z 1000cf74 f   qt-mt323:qt-mt323.dll
 0001:0000bf7a       ?cellRect@QTable@@UBE?AVQRect@@HH@Z 1000cf7a f   qt-mt323:qt-mt323.dll
 0001:0000bf80       ?cellWidget@QTable@@UBEPAVQWidget@@HH@Z 1000cf80 f   qt-mt323:qt-mt323.dll
 0001:0000bf86       ?clearCell@QTable@@UAEXHH@Z 1000cf86 f   qt-mt323:qt-mt323.dll
 0001:0000bf8c       ?clearCellWidget@QTable@@UAEXHH@Z 1000cf8c f   qt-mt323:qt-mt323.dll
 0001:0000bf92       ?columnAt@QTable@@UBEHH@Z  1000cf92 f   qt-mt323:qt-mt323.dll
 0001:0000bf98       ?columnClicked@QTable@@MAEXH@Z 1000cf98 f   qt-mt323:qt-mt323.dll
 0001:0000bf9e       ?columnIndexChanged@QTable@@MAEXHHH@Z 1000cf9e f   qt-mt323:qt-mt323.dll
 0001:0000bfa4       ?columnPos@QTable@@UBEHH@Z 1000cfa4 f   qt-mt323:qt-mt323.dll
 0001:0000bfaa       ?columnWidth@QTable@@UBEHH@Z 1000cfaa f   qt-mt323:qt-mt323.dll
 0001:0000bfb0       ?columnWidthChanged@QTable@@MAEXH@Z 1000cfb0 f   qt-mt323:qt-mt323.dll
 0001:0000bfb6       ?contentsContextMenuEvent@QTable@@MAEXPAVQContextMenuEvent@@@Z 1000cfb6 f   qt-mt323:qt-mt323.dll
 0001:0000bfbc       ?contentsDragEnterEvent@QTable@@MAEXPAVQDragEnterEvent@@@Z 1000cfbc f   qt-mt323:qt-mt323.dll
 0001:0000bfc2       ?contentsDragLeaveEvent@QTable@@MAEXPAVQDragLeaveEvent@@@Z 1000cfc2 f   qt-mt323:qt-mt323.dll
 0001:0000bfc8       ?contentsDragMoveEvent@QTable@@MAEXPAVQDragMoveEvent@@@Z 1000cfc8 f   qt-mt323:qt-mt323.dll
 0001:0000bfce       ?contentsDropEvent@QTable@@MAEXPAVQDropEvent@@@Z 1000cfce f   qt-mt323:qt-mt323.dll
 0001:0000bfd4       ?contentsMouseDoubleClickEvent@QTable@@MAEXPAVQMouseEvent@@@Z 1000cfd4 f   qt-mt323:qt-mt323.dll
 0001:0000bfda       ?contentsMouseMoveEvent@QTable@@MAEXPAVQMouseEvent@@@Z 1000cfda f   qt-mt323:qt-mt323.dll
 0001:0000bfe0       ?contentsMousePressEvent@QTable@@MAEXPAVQMouseEvent@@@Z 1000cfe0 f   qt-mt323:qt-mt323.dll
 0001:0000bfe6       ?contentsMouseReleaseEvent@QTable@@MAEXPAVQMouseEvent@@@Z 1000cfe6 f   qt-mt323:qt-mt323.dll
 0001:0000bfec       ?createEditor@QTable@@MBEPAVQWidget@@HH_N@Z 1000cfec f   qt-mt323:qt-mt323.dll
 0001:0000bff2       ?currentSelection@QTable@@UBEHXZ 1000cff2 f   qt-mt323:qt-mt323.dll
 0001:0000bff8       ?dragObject@QTable@@MAEPAVQDragObject@@XZ 1000cff8 f   qt-mt323:qt-mt323.dll
 0001:0000bffe       ?drawContents@QTable@@EAEXPAVQPainter@@@Z 1000cffe f   qt-mt323:qt-mt323.dll
 0001:0000c004       ?drawContents@QTable@@MAEXPAVQPainter@@HHHH@Z 1000d004 f   qt-mt323:qt-mt323.dll
 0001:0000c00a       ?editCell@QTable@@UAEXHH_N@Z 1000d00a f   qt-mt323:qt-mt323.dll
 0001:0000c010       ?endEdit@QTable@@MAEXHH_N0@Z 1000d010 f   qt-mt323:qt-mt323.dll
 0001:0000c016       ?eventFilter@QTable@@UAE_NPAVQObject@@PAVQEvent@@@Z 1000d016 f   qt-mt323:qt-mt323.dll
 0001:0000c01c       ?focusInEvent@QTable@@MAEXPAVQFocusEvent@@@Z 1000d01c f   qt-mt323:qt-mt323.dll
 0001:0000c022       ?focusOutEvent@QTable@@MAEXPAVQFocusEvent@@@Z 1000d022 f   qt-mt323:qt-mt323.dll
 0001:0000c028       ?hideColumn@QTable@@UAEXH@Z 1000d028 f   qt-mt323:qt-mt323.dll
 0001:0000c02e       ?hideRow@QTable@@UAEXH@Z   1000d02e f   qt-mt323:qt-mt323.dll
 0001:0000c034       ?insertColumns@QTable@@UAEXHH@Z 1000d034 f   qt-mt323:qt-mt323.dll
 0001:0000c03a       ?insertRows@QTable@@UAEXHH@Z 1000d03a f   qt-mt323:qt-mt323.dll
 0001:0000c040       ?insertWidget@QTable@@MAEXHHPAVQWidget@@@Z 1000d040 f   qt-mt323:qt-mt323.dll
 0001:0000c046       ?item@QTable@@UBEPAVQTableItem@@HH@Z 1000d046 f   qt-mt323:qt-mt323.dll
 0001:0000c04c       ?keyPressEvent@QTable@@MAEXPAVQKeyEvent@@@Z 1000d04c f   qt-mt323:qt-mt323.dll
 0001:0000c052       ?minimumSizeHint@QScrollView@@UBE?AVQSize@@XZ 1000d052 f   qt-mt323:qt-mt323.dll
 0001:0000c058       ?mouseDoubleClickEvent@QScrollView@@MAEXPAVQMouseEvent@@@Z 1000d058 f   qt-mt323:qt-mt323.dll
 0001:0000c05e       ?mouseMoveEvent@QScrollView@@MAEXPAVQMouseEvent@@@Z 1000d05e f   qt-mt323:qt-mt323.dll
 0001:0000c064       ?mousePressEvent@QScrollView@@MAEXPAVQMouseEvent@@@Z 1000d064 f   qt-mt323:qt-mt323.dll
 0001:0000c06a       ?mouseReleaseEvent@QScrollView@@MAEXPAVQMouseEvent@@@Z 1000d06a f   qt-mt323:qt-mt323.dll
 0001:0000c070       ?numCols@QTable@@UBEHXZ    1000d070 f   qt-mt323:qt-mt323.dll
 0001:0000c076       ?numRows@QTable@@UBEHXZ    1000d076 f   qt-mt323:qt-mt323.dll
 0001:0000c07c       ?paintCell@QTable@@UAEXPAVQPainter@@HHABVQRect@@_N@Z 1000d07c f   qt-mt323:qt-mt323.dll
 0001:0000c082       ?paintCell@QTable@@UAEXPAVQPainter@@HHABVQRect@@_NABVQColorGroup@@@Z 1000d082 f   qt-mt323:qt-mt323.dll
 0001:0000c088       ?paintEmptyArea@QTable@@MAEXPAVQPainter@@HHHH@Z 1000d088 f   qt-mt323:qt-mt323.dll
 0001:0000c08e       ?paintEvent@QTable@@MAEXPAVQPaintEvent@@@Z 1000d08e f   qt-mt323:qt-mt323.dll
 0001:0000c094       ?paintFocus@QTable@@UAEXPAVQPainter@@ABVQRect@@@Z 1000d094 f   qt-mt323:qt-mt323.dll
 0001:0000c09a       ?pixmap@QTable@@UBE?AVQPixmap@@HH@Z 1000d09a f   qt-mt323:qt-mt323.dll
 0001:0000c0a0       ?removeColumn@QTable@@UAEXH@Z 1000d0a0 f   qt-mt323:qt-mt323.dll
 0001:0000c0a6       ?removeColumns@QTable@@UAEXABV?$QMemArray@H@@@Z 1000d0a6 f   qt-mt323:qt-mt323.dll
 0001:0000c0ac       ?removeRow@QTable@@UAEXH@Z 1000d0ac f   qt-mt323:qt-mt323.dll
 0001:0000c0b2       ?removeRows@QTable@@UAEXABV?$QMemArray@H@@@Z 1000d0b2 f   qt-mt323:qt-mt323.dll
 0001:0000c0b8       ?removeSelection@QTable@@UAEXABVQTableSelection@@@Z 1000d0b8 f   qt-mt323:qt-mt323.dll
 0001:0000c0be       ?removeSelection@QTable@@UAEXH@Z 1000d0be f   qt-mt323:qt-mt323.dll
 0001:0000c0c4       ?resizeData@QTable@@MAEXH@Z 1000d0c4 f   qt-mt323:qt-mt323.dll
 0001:0000c0ca       ?resizeEvent@QScrollView@@MAEXPAVQResizeEvent@@@Z 1000d0ca f   qt-mt323:qt-mt323.dll
 0001:0000c0d0       ?rowAt@QTable@@UBEHH@Z     1000d0d0 f   qt-mt323:qt-mt323.dll
 0001:0000c0d6       ?rowHeight@QTable@@UBEHH@Z 1000d0d6 f   qt-mt323:qt-mt323.dll
 0001:0000c0dc       ?rowHeightChanged@QTable@@MAEXH@Z 1000d0dc f   qt-mt323:qt-mt323.dll
 0001:0000c0e2       ?rowIndexChanged@QTable@@MAEXHHH@Z 1000d0e2 f   qt-mt323:qt-mt323.dll
 0001:0000c0e8       ?rowPos@QTable@@UBEHH@Z    1000d0e8 f   qt-mt323:qt-mt323.dll
 0001:0000c0ee       ?setCellContentFromEditor@QTable@@MAEXHH@Z 1000d0ee f   qt-mt323:qt-mt323.dll
 0001:0000c0f4       ?setCellWidget@QTable@@UAEXHHPAVQWidget@@@Z 1000d0f4 f   qt-mt323:qt-mt323.dll
 0001:0000c0fa       ?setColumnMovingEnabled@QTable@@UAEX_N@Z 1000d0fa f   qt-mt323:qt-mt323.dll
 0001:0000c100       ?setColumnReadOnly@QTable@@UAEXH_N@Z 1000d100 f   qt-mt323:qt-mt323.dll
 0001:0000c106       ?setColumnStretchable@QTable@@UAEXH_N@Z 1000d106 f   qt-mt323:qt-mt323.dll
 0001:0000c10c       ?setColumnWidth@QTable@@UAEXHH@Z 1000d10c f   qt-mt323:qt-mt323.dll
 0001:0000c112       ?setCurrentCell@QTable@@UAEXHH@Z 1000d112 f   qt-mt323:qt-mt323.dll
 0001:0000c118       ?setDragEnabled@QTable@@UAEX_N@Z 1000d118 f   qt-mt323:qt-mt323.dll
 0001:0000c11e       ?setEnabled@QTable@@UAEX_N@Z 1000d11e f   qt-mt323:qt-mt323.dll
 0001:0000c124       ?setFocusStyle@QTable@@UAEXW4FocusStyle@1@@Z 1000d124 f   qt-mt323:qt-mt323.dll
 0001:0000c12a       ?setItem@QTable@@UAEXHHPAVQTableItem@@@Z 1000d12a f   qt-mt323:qt-mt323.dll
 0001:0000c130       ?setNumCols@QTable@@UAEXH@Z 1000d130 f   qt-mt323:qt-mt323.dll
 0001:0000c136       ?setNumRows@QTable@@UAEXH@Z 1000d136 f   qt-mt323:qt-mt323.dll
 0001:0000c13c       ?setPixmap@QTable@@UAEXHHABVQPixmap@@@Z 1000d13c f   qt-mt323:qt-mt323.dll
 0001:0000c142       ?setReadOnly@QTable@@UAEX_N@Z 1000d142 f   qt-mt323:qt-mt323.dll
 0001:0000c148       ?setRowHeight@QTable@@UAEXHH@Z 1000d148 f   qt-mt323:qt-mt323.dll
 0001:0000c14e       ?setRowMovingEnabled@QTable@@UAEX_N@Z 1000d14e f   qt-mt323:qt-mt323.dll
 0001:0000c154       ?setRowReadOnly@QTable@@UAEXH_N@Z 1000d154 f   qt-mt323:qt-mt323.dll
 0001:0000c15a       ?setRowStretchable@QTable@@UAEXH_N@Z 1000d15a f   qt-mt323:qt-mt323.dll
 0001:0000c160       ?setSelectionMode@QTable@@UAEXW4SelectionMode@1@@Z 1000d160 f   qt-mt323:qt-mt323.dll
 0001:0000c166       ?setShowGrid@QTable@@UAEX_N@Z 1000d166 f   qt-mt323:qt-mt323.dll
 0001:0000c16c       ?setSorting@QTable@@UAEX_N@Z 1000d16c f   qt-mt323:qt-mt323.dll
 0001:0000c172       ?setText@QTable@@UAEXHHABVQString@@@Z 1000d172 f   qt-mt323:qt-mt323.dll
 0001:0000c178       ?setTopMargin@QTable@@UAEXH@Z 1000d178 f   qt-mt323:qt-mt323.dll
 0001:0000c17e       ?showColumn@QTable@@UAEXH@Z 1000d17e f   qt-mt323:qt-mt323.dll
 0001:0000c184       ?showEvent@QTable@@MAEXPAVQShowEvent@@@Z 1000d184 f   qt-mt323:qt-mt323.dll
 0001:0000c18a       ?showRow@QTable@@UAEXH@Z   1000d18a f   qt-mt323:qt-mt323.dll
 0001:0000c190       ?sizeHint@QTable@@UBE?AVQSize@@XZ 1000d190 f   qt-mt323:qt-mt323.dll
 0001:0000c196       ?startDrag@QTable@@MAEXXZ  1000d196 f   qt-mt323:qt-mt323.dll
 0001:0000c19c       ?swapCells@QTable@@UAEXHHHH@Z 1000d19c f   qt-mt323:qt-mt323.dll
 0001:0000c1a2       ?swapColumns@QTable@@UAEXHH_N@Z 1000d1a2 f   qt-mt323:qt-mt323.dll
 0001:0000c1a8       ?swapRows@QTable@@UAEXHH_N@Z 1000d1a8 f   qt-mt323:qt-mt323.dll
 0001:0000c1ae       ?takeItem@QTable@@UAEXPAVQTableItem@@@Z 1000d1ae f   qt-mt323:qt-mt323.dll
 0001:0000c1b4       ?text@QTable@@UBE?AVQString@@HH@Z 1000d1b4 f   qt-mt323:qt-mt323.dll
 0001:0000c1ba       ?viewportPaintEvent@QScrollView@@MAEXPAVQPaintEvent@@@Z 1000d1ba f   qt-mt323:qt-mt323.dll
 0001:0000c1c0       ?viewportResizeEvent@QTable@@MAEXPAVQResizeEvent@@@Z 1000d1c0 f   qt-mt323:qt-mt323.dll
 0001:0000c1c6       ?windowActivationChange@QTable@@MAEX_N@Z 1000d1c6 f   qt-mt323:qt-mt323.dll
 0001:0000c1cc       ?addTab@QTabWidget@@UAEXPAVQWidget@@ABVQIconSet@@ABVQString@@@Z 1000d1cc f   qt-mt323:qt-mt323.dll
 0001:0000c1d2       ?addTab@QTabWidget@@UAEXPAVQWidget@@ABVQString@@@Z 1000d1d2 f   qt-mt323:qt-mt323.dll
 0001:0000c1d8       ?addTab@QTabWidget@@UAEXPAVQWidget@@PAVQTab@@@Z 1000d1d8 f   qt-mt323:qt-mt323.dll
 0001:0000c1de       ?className@QTabWidget@@UBEPBDXZ 1000d1de f   qt-mt323:qt-mt323.dll
 0001:0000c1e4       ?eventFilter@QTabWidget@@MAE_NPAVQObject@@PAVQEvent@@@Z 1000d1e4 f   qt-mt323:qt-mt323.dll
 0001:0000c1ea       ?insertTab@QTabWidget@@UAEXPAVQWidget@@ABVQIconSet@@ABVQString@@H@Z 1000d1ea f   qt-mt323:qt-mt323.dll
 0001:0000c1f0       ?insertTab@QTabWidget@@UAEXPAVQWidget@@ABVQString@@H@Z 1000d1f0 f   qt-mt323:qt-mt323.dll
 0001:0000c1f6       ?insertTab@QTabWidget@@UAEXPAVQWidget@@PAVQTab@@H@Z 1000d1f6 f   qt-mt323:qt-mt323.dll
 0001:0000c1fc       ?metaObject@QTabWidget@@UBEPAVQMetaObject@@XZ 1000d1fc f   qt-mt323:qt-mt323.dll
 0001:0000c202       ?minimumSizeHint@QTabWidget@@UBE?AVQSize@@XZ 1000d202 f   qt-mt323:qt-mt323.dll
 0001:0000c208       ?qt_cast@QTabWidget@@UAEPAXPBD@Z 1000d208 f   qt-mt323:qt-mt323.dll
 0001:0000c20e       ?qt_emit@QTabWidget@@UAE_NHPAUQUObject@@@Z 1000d20e f   qt-mt323:qt-mt323.dll
 0001:0000c214       ?qt_invoke@QTabWidget@@UAE_NHPAUQUObject@@@Z 1000d214 f   qt-mt323:qt-mt323.dll
 0001:0000c21a       ?qt_property@QTabWidget@@UAE_NHHPAVQVariant@@@Z 1000d21a f   qt-mt323:qt-mt323.dll
 0001:0000c220       ?removePage@QTabWidget@@UAEXPAVQWidget@@@Z 1000d220 f   qt-mt323:qt-mt323.dll
 0001:0000c226       ?resizeEvent@QTabWidget@@MAEXPAVQResizeEvent@@@Z 1000d226 f   qt-mt323:qt-mt323.dll
 0001:0000c22c       ?showEvent@QTabWidget@@MAEXPAVQShowEvent@@@Z 1000d22c f   qt-mt323:qt-mt323.dll
 0001:0000c232       ?showPage@QTabWidget@@UAEXPAVQWidget@@@Z 1000d232 f   qt-mt323:qt-mt323.dll
 0001:0000c238       ?sizeHint@QTabWidget@@UBE?AVQSize@@XZ 1000d238 f   qt-mt323:qt-mt323.dll
 0001:0000c23e       ?styleChange@QTabWidget@@MAEXAAVQStyle@@@Z 1000d23e f   qt-mt323:qt-mt323.dll
 0001:0000c244       ?updateMask@QTabWidget@@MAEXXZ 1000d244 f   qt-mt323:qt-mt323.dll
 0001:0000c24a       ??0cfg_Table@@QAE@ABV0@@Z  1000d24a f i cfg_widgets001:cfg_Table.obj
 0001:0000c27c       ??0cfg_Table@@QAE@PAVQWidget@@PBD@Z 1000d27c f   cfg_widgets001:cfg_Table.obj
 0001:0000c2d6       ??4cfg_Table@@QAEAAV0@ABV0@@Z 1000d2d6 f i cfg_widgets001:cfg_Table.obj
 0001:0000c2fb       ??_EQStringList@@QAEPAXI@Z 1000d2fb f i cfg_widgets001:cfg_Table.obj
 0001:0000c347       ??_Ecfg_Table@@UAEPAXI@Z   1000d347 f i cfg_widgets001:cfg_Table.obj
 0001:0000c395       ??_Ecfg_Table@@WCI@AEPAXI@Z 1000d395 f i cfg_widgets001:cfg_Table.obj
 0001:0000c39d       ??_Fcfg_Table@@QAEXXZ      1000d39d f i cfg_widgets001:cfg_Table.obj
 0001:0000c3a7       ?clipBoardDataChanged@cfg_Table@@IAEXXZ 1000d3a7 f   cfg_widgets001:cfg_Table.obj
 0001:0000c3fb       ?copyToClipboard@cfg_Table@@QAEXXZ 1000d3fb f   cfg_widgets001:cfg_Table.obj
 0001:0000c50a       ?deleteItems@cfg_Table@@QAEXXZ 1000d50a f   cfg_widgets001:cfg_Table.obj
 0001:0000c596       ?fillUndoBuffer@cfg_Table@@AAEXXZ 1000d596 f   cfg_widgets001:cfg_Table.obj
 0001:0000c70b       ?metaObject@cfg_Table@@UBEPAVQMetaObject@@XZ 1000d70b f i cfg_widgets001:cfg_Table.obj
 0001:0000c710       ?pasteClipboard@cfg_Table@@QAEXXZ 1000d710 f   cfg_widgets001:cfg_Table.obj
 0001:0000cb03       ?qObject@cfg_Table@@QAEPAVQObject@@XZ 1000db03 f i cfg_widgets001:cfg_Table.obj
 0001:0000cb06       ?undoPaste@cfg_Table@@QAEXXZ 1000db06 f   cfg_widgets001:cfg_Table.obj
 0001:0000cc38       ?validateRow@cfg_Table@@MAEHH@Z 1000dc38 f   cfg_widgets001:cfg_Table.obj
 0001:0000cc4a       ?className@cfg_Table@@UBEPBDXZ 1000dc4a f   cfg_widgets001:moc_cfg_Table.obj
 0001:0000cc50       ?clipboardDataValid@cfg_Table@@IAEX_N@Z 1000dc50 f   cfg_widgets001:moc_cfg_Table.obj
 0001:0000cc70       ?dataPasted@cfg_Table@@IAEXXZ 1000dc70 f   cfg_widgets001:moc_cfg_Table.obj
 0001:0000cc85       ?qt_cast@cfg_Table@@UAEPAXPBD@Z 1000dc85 f   cfg_widgets001:moc_cfg_Table.obj
 0001:0000ccb3       ?qt_emit@cfg_Table@@UAE_NHPAUQUObject@@@Z 1000dcb3 f   cfg_widgets001:moc_cfg_Table.obj
 0001:0000ccf7       ?qt_invoke@cfg_Table@@UAE_NHPAUQUObject@@@Z 1000dcf7 f   cfg_widgets001:moc_cfg_Table.obj
 0001:0000cd51       ?qt_property@cfg_Table@@UAE_NHHPAVQVariant@@@Z 1000dd51 f   cfg_widgets001:moc_cfg_Table.obj
 0001:0000cd5b       ?staticMetaObject@cfg_Table@@SAPAVQMetaObject@@XZ 1000dd5b f   cfg_widgets001:moc_cfg_Table.obj
 0001:0000cdda       ?tr@cfg_Table@@SA?AVQString@@PBD0@Z 1000ddda f   cfg_widgets001:moc_cfg_Table.obj
 0001:0000ce1d       ?trUtf8@cfg_Table@@SA?AVQString@@PBD0@Z 1000de1d f   cfg_widgets001:moc_cfg_Table.obj
 0001:0000ce60       ??2@YAPAXI@Z               1000de60 f   MSVCRT:MSVCR120.dll
 0001:0000ce66       ??3@YAXPAX@Z               1000de66 f   MSVCRT:MSVCR120.dll
 0001:0000ce6c       @__security_check_cookie@4 1000de6c f   MSVCRT:secchk.obj
 0001:0000ce7b       __EH_epilog3               1000de7b f   MSVCRT:ehprolg3.obj
 0001:0000ce8f       __EH_epilog3_GS            1000de8f f   MSVCRT:ehprolg3.obj
 0001:0000ce9e       __EH_prolog3               1000de9e f   MSVCRT:ehprolg3.obj
 0001:0000ced1       __EH_prolog3_GS            1000ded1 f   MSVCRT:ehprolg3.obj
 0001:0000cf08       ___CxxFrameHandler3        1000df08 f   MSVCRT:MSVCR120.dll
 0001:0000cf0e       ??_Etype_info@@UAEPAXI@Z   1000df0e f i MSVCRT:ti_inst.obj
 0001:0000cf58       ___atonexitinit            1000df58 f   MSVCRT:atonexit.obj
 0001:0000cf94       __onexit                   1000df94 f   MSVCRT:atonexit.obj
 0001:0000d03d       _atexit                    1000e03d f   MSVCRT:atonexit.obj
 0001:0000d052       __purecall                 1000e052 f   MSVCRT:MSVCR120.dll
 0001:0000d058       ??_L@YGXPAXIHP6EX0@Z1@Z    1000e058 f   MSVCRT:ehvecctr.obj
 0001:0000d0ba       ??_M@YGXPAXIHP6EX0@Z@Z     1000e0ba f   MSVCRT:ehvecdtr.obj
 0001:0000d129       ?__ArrayUnwind@@YGXPAXIHP6EX0@Z@Z 1000e129 f   MSVCRT:ehvecdtr.obj
 0001:0000d1d3       __CRT_INIT@12              1000e1d3 f   MSVCRT:crtdll.obj
 0001:0000d3ca       __DllMainCRTStartup@12     1000e3ca f   MSVCRT:crtdll.obj
 0001:0000d520       ___raise_securityfailure   1000e520 f   MSVCRT:gs_report.obj
 0001:0000d55d       ___report_gsfailure        1000e55d f   MSVCRT:gs_report.obj
 0001:0000d658       ??1type_info@@UAE@XZ       1000e658 f   MSVCRT:MSVCR120.dll
 0001:0000d65e       __lock                     1000e65e f   MSVCRT:MSVCR120.dll
 0001:0000d664       __unlock                   1000e664 f   MSVCRT:MSVCR120.dll
 0001:0000d66a       ___dllonexit               1000e66a f   MSVCRT:MSVCR120.dll
 0001:0000d670       __SEH_prolog4              1000e670 f   MSVCRT:sehprolg4.obj
 0001:0000d6b5       __SEH_epilog4              1000e6b5 f   MSVCRT:sehprolg4.obj
 0001:0000d6c9       __except_handler4          1000e6c9 f   MSVCRT:chandler4gs.obj
 0001:0000d6ec       ?terminate@@YAXXZ          1000e6ec f   MSVCRT:MSVCR120.dll
 0001:0000d6f2       ___CppXcptFilter           1000e6f2 f   MSVCRT:MSVCR120.dll
 0001:0000d6f8       __amsg_exit                1000e6f8 f   MSVCRT:MSVCR120.dll
 0001:0000d700       __FindPESection            1000e700 f   MSVCRT:pesect.obj
 0001:0000d750       __IsNonwritableInCurrentImage 1000e750 f   MSVCRT:pesect.obj
 0001:0000d810       __ValidateImageBase        1000e810 f   MSVCRT:pesect.obj
 0001:0000d841       ___security_init_cookie    1000e841 f   MSVCRT:gs_support.obj
 0001:0000d8dd       _DllMain@12                1000e8dd f   MSVCRT:dllmain.obj
 0001:0000d8ff       __RTC_Initialize           1000e8ff f   MSVCRT:initsect.obj
 0001:0000d91f       __RTC_Terminate            1000e91f f   MSVCRT:initsect.obj
 0001:0000d940       __initterm                 1000e940 f   MSVCRT:MSVCR120.dll
 0001:0000d946       __initterm_e               1000e946 f   MSVCRT:MSVCR120.dll
 0001:0000d94c       ___clean_type_info_names   1000e94c f   MSVCRT:tncleanup.obj
 0001:0000d958       __crt_debugger_hook        1000e958 f   MSVCRT:MSVCR120.dll
 0001:0000d95e       ___crtUnhandledException   1000e95e f   MSVCRT:MSVCR120.dll
 0001:0000d964       ___crtTerminateProcess     1000e964 f   MSVCRT:MSVCR120.dll
 0001:0000d96a       __except_handler4_common   1000e96a f   MSVCRT:MSVCR120.dll
 0001:0000d970       ___clean_type_info_names_internal 1000e970 f   MSVCRT:MSVCR120.dll
 0001:0000d976       _IsProcessorFeaturePresent@4 1000e976 f   kernel32:KERNEL32.dll
 0002:00000000       __imp__DecodePointer@4     10011000     kernel32:KERNEL32.dll
 0002:00000004       __imp__DisableThreadLibraryCalls@4 10011004     kernel32:KERNEL32.dll
 0002:00000008       __imp__GetSystemTimeAsFileTime@4 10011008     kernel32:KERNEL32.dll
 0002:0000000c       __imp__GetCurrentThreadId@0 1001100c     kernel32:KERNEL32.dll
 0002:00000010       __imp__GetCurrentProcessId@0 10011010     kernel32:KERNEL32.dll
 0002:00000014       __imp__QueryPerformanceCounter@4 10011014     kernel32:KERNEL32.dll
 0002:00000018       __imp__IsProcessorFeaturePresent@4 10011018     kernel32:KERNEL32.dll
 0002:0000001c       __imp__IsDebuggerPresent@0 1001101c     kernel32:KERNEL32.dll
 0002:00000020       __imp__EncodePointer@4     10011020     kernel32:KERNEL32.dll
 0002:00000024       \177KERNEL32_NULL_THUNK_DATA 10011024     kernel32:KERNEL32.dll
 0002:00000028       __imp_??3@YAXPAX@Z         10011028     MSVCRT:MSVCR120.dll
 0002:0000002c       __imp____clean_type_info_names_internal 1001102c     MSVCRT:MSVCR120.dll
 0002:00000030       __imp___except_handler4_common 10011030     MSVCRT:MSVCR120.dll
 0002:00000034       __imp____crtTerminateProcess 10011034     MSVCRT:MSVCR120.dll
 0002:00000038       __imp____crtUnhandledException 10011038     MSVCRT:MSVCR120.dll
 0002:0000003c       __imp___crt_debugger_hook  1001103c     MSVCRT:MSVCR120.dll
 0002:00000040       __imp___initterm_e         10011040     MSVCRT:MSVCR120.dll
 0002:00000044       __imp___initterm           10011044     MSVCRT:MSVCR120.dll
 0002:00000048       __imp___malloc_crt         10011048     MSVCRT:MSVCR120.dll
 0002:0000004c       __imp__free                1001104c     MSVCRT:MSVCR120.dll
 0002:00000050       __imp___amsg_exit          10011050     MSVCRT:MSVCR120.dll
 0002:00000054       __imp____CppXcptFilter     10011054     MSVCRT:MSVCR120.dll
 0002:00000058       __imp_?terminate@@YAXXZ    10011058     MSVCRT:MSVCR120.dll
 0002:0000005c       __imp___onexit             1001105c     MSVCRT:MSVCR120.dll
 0002:00000060       __imp____dllonexit         10011060     MSVCRT:MSVCR120.dll
 0002:00000064       __imp___calloc_crt         10011064     MSVCRT:MSVCR120.dll
 0002:00000068       __imp___unlock             10011068     MSVCRT:MSVCR120.dll
 0002:0000006c       __imp___lock               1001106c     MSVCRT:MSVCR120.dll
 0002:00000070       __imp_??1type_info@@UAE@XZ 10011070     MSVCRT:MSVCR120.dll
 0002:00000074       __imp___purecall           10011074     MSVCRT:MSVCR120.dll
 0002:00000078       __imp____CxxFrameHandler3  10011078     MSVCRT:MSVCR120.dll
 0002:0000007c       __imp_??2@YAPAXI@Z         1001107c     MSVCRT:MSVCR120.dll
 0002:00000080       \177MSVCR120_NULL_THUNK_DATA 10011080     MSVCRT:MSVCR120.dll
 0002:00000084       __imp_?fnConfig_icons@@YAPAPBDPBD@Z 10011084     config_icons:config_icons.dll
 0002:00000088       \177config_icons_NULL_THUNK_DATA 10011088     config_icons:config_icons.dll
 0002:0000008c       __imp_??1QAction@@UAE@XZ   1001108c     qt-mt323:qt-mt323.dll
 0002:00000090       __imp_??1?$QPtrList@VQDockWindow@@@@UAE@XZ 10011090     qt-mt323:qt-mt323.dll
 0002:00000094       __imp_??0QToolBar@@QAE@PAVQMainWindow@@PBD@Z 10011094     qt-mt323:qt-mt323.dll
 0002:00000098       __imp_??1QToolBar@@UAE@XZ  10011098     qt-mt323:qt-mt323.dll
 0002:0000009c       __imp_??9QDateTime@@QBE_NABV0@@Z 1001109c     qt-mt323:qt-mt323.dll
 0002:000000a0       __imp_??0QFileInfo@@QAE@ABVQString@@@Z 100110a0     qt-mt323:qt-mt323.dll
 0002:000000a4       __imp_??1QFileInfo@@QAE@XZ 100110a4     qt-mt323:qt-mt323.dll
 0002:000000a8       __imp_?lastModified@QFileInfo@@QBE?AVQDateTime@@XZ 100110a8     qt-mt323:qt-mt323.dll
 0002:000000ac       __imp_??0QGuardedPtrPrivate@@QAE@PAVQObject@@@Z 100110ac     qt-mt323:qt-mt323.dll
 0002:000000b0       __imp_??1QGuardedPtrPrivate@@UAE@XZ 100110b0     qt-mt323:qt-mt323.dll
 0002:000000b4       __imp_?reconnect@QGuardedPtrPrivate@@QAEXPAVQObject@@@Z 100110b4     qt-mt323:qt-mt323.dll
 0002:000000b8       __imp_??0QGDict@@IAE@IW4KeyType@0@_N1@Z 100110b8     qt-mt323:qt-mt323.dll
 0002:000000bc       __imp_??1QGDict@@MAE@XZ    100110bc     qt-mt323:qt-mt323.dll
 0002:000000c0       __imp_?clear@QGDict@@MAEXXZ 100110c0     qt-mt323:qt-mt323.dll
 0002:000000c4       __imp_??0QPopupMenu@@QAE@PAVQWidget@@PBD@Z 100110c4     qt-mt323:qt-mt323.dll
 0002:000000c8       __imp_??1QPopupMenu@@UAE@XZ 100110c8     qt-mt323:qt-mt323.dll
 0002:000000cc       __imp_?exec@QPopupMenu@@QAEHABVQPoint@@H@Z 100110cc     qt-mt323:qt-mt323.dll
 0002:000000d0       __imp_?activateItemAt@QPopupMenu@@UAEXH@Z 100110d0     qt-mt323:qt-mt323.dll
 0002:000000d4       __imp_?addTo@QAction@@UAE_NPAVQWidget@@@Z 100110d4     qt-mt323:qt-mt323.dll
 0002:000000d8       __imp_?addedTo@QAction@@MAEXHPAVQPopupMenu@@@Z 100110d8     qt-mt323:qt-mt323.dll
 0002:000000dc       __imp_?addedTo@QAction@@MAEXPAVQWidget@@0@Z 100110dc     qt-mt323:qt-mt323.dll
 0002:000000e0       __imp_?adjustSize@QWidget@@UAEXXZ 100110e0     qt-mt323:qt-mt323.dll
 0002:000000e4       __imp_?checkConnectArgs@QObject@@MAE_NPBDPBV1@0@Z 100110e4     qt-mt323:qt-mt323.dll
 0002:000000e8       __imp_?childEvent@QObject@@MAEXPAVQChildEvent@@@Z 100110e8     qt-mt323:qt-mt323.dll
 0002:000000ec       __imp_?className@QAction@@UBEPBDXZ 100110ec     qt-mt323:qt-mt323.dll
 0002:000000f0       __imp_?className@QGuardedPtrPrivate@@UBEPBDXZ 100110f0     qt-mt323:qt-mt323.dll
 0002:000000f4       __imp_?className@QPopupMenu@@UBEPBDXZ 100110f4     qt-mt323:qt-mt323.dll
 0002:000000f8       __imp_?className@QToolBar@@UBEPBDXZ 100110f8     qt-mt323:qt-mt323.dll
 0002:000000fc       __imp_?className@QWidget@@UBEPBDXZ 100110fc     qt-mt323:qt-mt323.dll
 0002:00000100       __imp_?clear@?$QPtrList@VQDockWindow@@@@UAEXXZ 10011100     qt-mt323:qt-mt323.dll
 0002:00000104       __imp_?clear@QToolBar@@UAEXXZ 10011104     qt-mt323:qt-mt323.dll
 0002:00000108       __imp_?close@QWidget@@UAE_N_N@Z 10011108     qt-mt323:qt-mt323.dll
 0002:0000010c       __imp_?closeEvent@QPopupMenu@@MAEXPAVQCloseEvent@@@Z 1001110c     qt-mt323:qt-mt323.dll
 0002:00000110       __imp_?cmd@QPaintDevice@@MAE_NHPAVQPainter@@PATQPDevCmdParam@@@Z 10011110     qt-mt323:qt-mt323.dll
 0002:00000114       __imp_?compareItems@QGList@@MAEHPAX0@Z 10011114     qt-mt323:qt-mt323.dll
 0002:00000118       __imp_?connectNotify@QObject@@MAEXPBD@Z 10011118     qt-mt323:qt-mt323.dll
 0002:0000011c       __imp_?contextMenuEvent@QDockWindow@@MAEXPAVQContextMenuEvent@@@Z 1001111c     qt-mt323:qt-mt323.dll
 0002:00000120       __imp_?contextMenuEvent@QWidget@@MAEXPAVQContextMenuEvent@@@Z 10011120     qt-mt323:qt-mt323.dll
 0002:00000124       __imp_?count@?$QPtrList@VQDockWindow@@@@UBEIXZ 10011124     qt-mt323:qt-mt323.dll
 0002:00000128       __imp_?create@QWidget@@MAEXPAUHWND__@@_N1@Z 10011128     qt-mt323:qt-mt323.dll
 0002:0000012c       __imp_?customEvent@QObject@@MAEXPAVQCustomEvent@@@Z 1001112c     qt-mt323:qt-mt323.dll
 0002:00000130       __imp_?customWhatsThis@QPopupMenu@@UBE_NXZ 10011130     qt-mt323:qt-mt323.dll
 0002:00000134       __imp_?customWhatsThis@QWidget@@UBE_NXZ 10011134     qt-mt323:qt-mt323.dll
 0002:00000138       __imp_?deleteItem@?$QPtrList@VQDockWindow@@@@EAEXPAX@Z 10011138     qt-mt323:qt-mt323.dll
 0002:0000013c       __imp_?destroy@QWidget@@MAEX_N0@Z 1001113c     qt-mt323:qt-mt323.dll
 0002:00000140       __imp_?disconnectNotify@QObject@@MAEXPBD@Z 10011140     qt-mt323:qt-mt323.dll
 0002:00000144       __imp_?dock@QDockWindow@@UAEXXZ 10011144     qt-mt323:qt-mt323.dll
 0002:00000148       __imp_?dragEnterEvent@QWidget@@MAEXPAVQDragEnterEvent@@@Z 10011148     qt-mt323:qt-mt323.dll
 0002:0000014c       __imp_?dragLeaveEvent@QWidget@@MAEXPAVQDragLeaveEvent@@@Z 1001114c     qt-mt323:qt-mt323.dll
 0002:00000150       __imp_?dragMoveEvent@QWidget@@MAEXPAVQDragMoveEvent@@@Z 10011150     qt-mt323:qt-mt323.dll
 0002:00000154       __imp_?drawContents@QDockWindow@@MAEXPAVQPainter@@@Z 10011154     qt-mt323:qt-mt323.dll
 0002:00000158       __imp_?drawContents@QPopupMenu@@MAEXPAVQPainter@@@Z 10011158     qt-mt323:qt-mt323.dll
 0002:0000015c       __imp_?drawFrame@QDockWindow@@MAEXPAVQPainter@@@Z 1001115c     qt-mt323:qt-mt323.dll
 0002:00000160       __imp_?drawFrame@QFrame@@MAEXPAVQPainter@@@Z 10011160     qt-mt323:qt-mt323.dll
 0002:00000164       __imp_?dropEvent@QWidget@@MAEXPAVQDropEvent@@@Z 10011164     qt-mt323:qt-mt323.dll
 0002:00000168       __imp_?enabledChange@QPopupMenu@@MAEX_N@Z 10011168     qt-mt323:qt-mt323.dll
 0002:0000016c       __imp_?enabledChange@QWidget@@MAEX_N@Z 1001116c     qt-mt323:qt-mt323.dll
 0002:00000170       __imp_?enterEvent@QWidget@@MAEXPAVQEvent@@@Z 10011170     qt-mt323:qt-mt323.dll
 0002:00000174       __imp_?event@QObject@@UAE_NPAVQEvent@@@Z 10011174     qt-mt323:qt-mt323.dll
 0002:00000178       __imp_?event@QToolBar@@UAE_NPAVQEvent@@@Z 10011178     qt-mt323:qt-mt323.dll
 0002:0000017c       __imp_?event@QWidget@@MAE_NPAVQEvent@@@Z 1001117c     qt-mt323:qt-mt323.dll
 0002:00000180       __imp_?eventFilter@QDockWindow@@UAE_NPAVQObject@@PAVQEvent@@@Z 10011180     qt-mt323:qt-mt323.dll
 0002:00000184       __imp_?eventFilter@QObject@@UAE_NPAV1@PAVQEvent@@@Z 10011184     qt-mt323:qt-mt323.dll
 0002:00000188       __imp_?focusInEvent@QPopupMenu@@MAEXPAVQFocusEvent@@@Z 10011188     qt-mt323:qt-mt323.dll
 0002:0000018c       __imp_?focusInEvent@QWidget@@MAEXPAVQFocusEvent@@@Z 1001118c     qt-mt323:qt-mt323.dll
 0002:00000190       __imp_?focusNextPrevChild@QPopupMenu@@MAE_N_N@Z 10011190     qt-mt323:qt-mt323.dll
 0002:00000194       __imp_?focusNextPrevChild@QWidget@@MAE_N_N@Z 10011194     qt-mt323:qt-mt323.dll
 0002:00000198       __imp_?focusOutEvent@QPopupMenu@@MAEXPAVQFocusEvent@@@Z 10011198     qt-mt323:qt-mt323.dll
 0002:0000019c       __imp_?focusOutEvent@QWidget@@MAEXPAVQFocusEvent@@@Z 1001119c     qt-mt323:qt-mt323.dll
 0002:000001a0       __imp_?fontChange@QWidget@@MAEXABVQFont@@@Z 100111a0     qt-mt323:qt-mt323.dll
 0002:000001a4       __imp_?fontInf@QPaintDevice@@MBEHPAVQFont@@H@Z 100111a4     qt-mt323:qt-mt323.dll
 0002:000001a8       __imp_?fontMet@QPaintDevice@@MBEHPAVQFont@@HPBDH@Z 100111a8     qt-mt323:qt-mt323.dll
 0002:000001ac       __imp_?frameChanged@QFrame@@MAEXXZ 100111ac     qt-mt323:qt-mt323.dll
 0002:000001b0       __imp_?frameChanged@QPopupMenu@@EAEXXZ 100111b0     qt-mt323:qt-mt323.dll
 0002:000001b4       __imp_?handle@QPaintDevice@@UBEPAUHDC__@@XZ 100111b4     qt-mt323:qt-mt323.dll
 0002:000001b8       __imp_?heightForWidth@QWidget@@UBEHH@Z 100111b8     qt-mt323:qt-mt323.dll
 0002:000001bc       __imp_?hide@QPopupMenu@@UAEXXZ 100111bc     qt-mt323:qt-mt323.dll
 0002:000001c0       __imp_?hide@QToolBar@@UAEXXZ 100111c0     qt-mt323:qt-mt323.dll
 0002:000001c4       __imp_?hide@QWidget@@UAEXXZ 100111c4     qt-mt323:qt-mt323.dll
 0002:000001c8       __imp_?hideEvent@QDockWindow@@MAEXPAVQHideEvent@@@Z 100111c8     qt-mt323:qt-mt323.dll
 0002:000001cc       __imp_?hideEvent@QWidget@@MAEXPAVQHideEvent@@@Z 100111cc     qt-mt323:qt-mt323.dll
 0002:000001d0       __imp_?imComposeEvent@QWidget@@MAEXPAVQIMEvent@@@Z 100111d0     qt-mt323:qt-mt323.dll
 0002:000001d4       __imp_?imEndEvent@QWidget@@MAEXPAVQIMEvent@@@Z 100111d4     qt-mt323:qt-mt323.dll
 0002:000001d8       __imp_?imStartEvent@QWidget@@MAEXPAVQIMEvent@@@Z 100111d8     qt-mt323:qt-mt323.dll
 0002:000001dc       __imp_?insertChild@QObject@@UAEXPAV1@@Z 100111dc     qt-mt323:qt-mt323.dll
 0002:000001e0       __imp_?keyPressEvent@QPopupMenu@@MAEXPAVQKeyEvent@@@Z 100111e0     qt-mt323:qt-mt323.dll
 0002:000001e4       __imp_?keyPressEvent@QWidget@@MAEXPAVQKeyEvent@@@Z 100111e4     qt-mt323:qt-mt323.dll
 0002:000001e8       __imp_?keyReleaseEvent@QWidget@@MAEXPAVQKeyEvent@@@Z 100111e8     qt-mt323:qt-mt323.dll
 0002:000001ec       __imp_?leaveEvent@QPopupMenu@@MAEXPAVQEvent@@@Z 100111ec     qt-mt323:qt-mt323.dll
 0002:000001f0       __imp_?leaveEvent@QWidget@@MAEXPAVQEvent@@@Z 100111f0     qt-mt323:qt-mt323.dll
 0002:000001f4       __imp_?menuContentsChanged@QPopupMenu@@EAEXXZ 100111f4     qt-mt323:qt-mt323.dll
 0002:000001f8       __imp_?menuDelPopup@QPopupMenu@@EAEXPAV1@@Z 100111f8     qt-mt323:qt-mt323.dll
 0002:000001fc       __imp_?menuInsPopup@QPopupMenu@@EAEXPAV1@@Z 100111fc     qt-mt323:qt-mt323.dll
 0002:00000200       __imp_?menuStateChanged@QPopupMenu@@EAEXXZ 10011200     qt-mt323:qt-mt323.dll
 0002:00000204       __imp_?metaObject@QAction@@UBEPAVQMetaObject@@XZ 10011204     qt-mt323:qt-mt323.dll
 0002:00000208       __imp_?metaObject@QGuardedPtrPrivate@@UBEPAVQMetaObject@@XZ 10011208     qt-mt323:qt-mt323.dll
 0002:0000020c       __imp_?metaObject@QPopupMenu@@UBEPAVQMetaObject@@XZ 1001120c     qt-mt323:qt-mt323.dll
 0002:00000210       __imp_?metaObject@QToolBar@@UBEPAVQMetaObject@@XZ 10011210     qt-mt323:qt-mt323.dll
 0002:00000214       __imp_?metaObject@QWidget@@UBEPAVQMetaObject@@XZ 10011214     qt-mt323:qt-mt323.dll
 0002:00000218       __imp_?metric@QWidget@@MBEHH@Z 10011218     qt-mt323:qt-mt323.dll
 0002:0000021c       __imp_?minimumSizeHint@QToolBar@@UBE?AVQSize@@XZ 1001121c     qt-mt323:qt-mt323.dll
 0002:00000220       __imp_?minimumSizeHint@QWidget@@UBE?AVQSize@@XZ 10011220     qt-mt323:qt-mt323.dll
 0002:00000224       __imp_?mouseDoubleClickEvent@QWidget@@MAEXPAVQMouseEvent@@@Z 10011224     qt-mt323:qt-mt323.dll
 0002:00000228       __imp_?mouseMoveEvent@QPopupMenu@@MAEXPAVQMouseEvent@@@Z 10011228     qt-mt323:qt-mt323.dll
 0002:0000022c       __imp_?mouseMoveEvent@QWidget@@MAEXPAVQMouseEvent@@@Z 1001122c     qt-mt323:qt-mt323.dll
 0002:00000230       __imp_?mousePressEvent@QPopupMenu@@MAEXPAVQMouseEvent@@@Z 10011230     qt-mt323:qt-mt323.dll
 0002:00000234       __imp_?mousePressEvent@QWidget@@MAEXPAVQMouseEvent@@@Z 10011234     qt-mt323:qt-mt323.dll
 0002:00000238       __imp_?mouseReleaseEvent@QPopupMenu@@MAEXPAVQMouseEvent@@@Z 10011238     qt-mt323:qt-mt323.dll
 0002:0000023c       __imp_?mouseReleaseEvent@QWidget@@MAEXPAVQMouseEvent@@@Z 1001123c     qt-mt323:qt-mt323.dll
 0002:00000240       __imp_?move@QWidget@@UAEXHH@Z 10011240     qt-mt323:qt-mt323.dll
 0002:00000244       __imp_?moveEvent@QWidget@@MAEXPAVQMoveEvent@@@Z 10011244     qt-mt323:qt-mt323.dll
 0002:00000248       __imp_?newItem@QPtrCollection@@MAEPAXPAX@Z 10011248     qt-mt323:qt-mt323.dll
 0002:0000024c       __imp_?paintEvent@QFrame@@MAEXPAVQPaintEvent@@@Z 1001124c     qt-mt323:qt-mt323.dll
 0002:00000250       __imp_?paintEvent@QPopupMenu@@MAEXPAVQPaintEvent@@@Z 10011250     qt-mt323:qt-mt323.dll
 0002:00000254       __imp_?paintEvent@QWidget@@MAEXPAVQPaintEvent@@@Z 10011254     qt-mt323:qt-mt323.dll
 0002:00000258       __imp_?paletteChange@QWidget@@MAEXABVQPalette@@@Z 10011258     qt-mt323:qt-mt323.dll
 0002:0000025c       __imp_?polish@QWidget@@UAEXXZ 1001125c     qt-mt323:qt-mt323.dll
 0002:00000260       __imp_?property@QObject@@UBE?AVQVariant@@PBD@Z 10011260     qt-mt323:qt-mt323.dll
 0002:00000264       __imp_?qt_cast@QAction@@UAEPAXPBD@Z 10011264     qt-mt323:qt-mt323.dll
 0002:00000268       __imp_?qt_cast@QGuardedPtrPrivate@@UAEPAXPBD@Z 10011268     qt-mt323:qt-mt323.dll
 0002:0000026c       __imp_?qt_cast@QPopupMenu@@UAEPAXPBD@Z 1001126c     qt-mt323:qt-mt323.dll
 0002:00000270       __imp_?qt_cast@QToolBar@@UAEPAXPBD@Z 10011270     qt-mt323:qt-mt323.dll
 0002:00000274       __imp_?qt_cast@QWidget@@UAEPAXPBD@Z 10011274     qt-mt323:qt-mt323.dll
 0002:00000278       __imp_?qt_emit@QAction@@UAE_NHPAUQUObject@@@Z 10011278     qt-mt323:qt-mt323.dll
 0002:0000027c       __imp_?qt_emit@QGuardedPtrPrivate@@UAE_NHPAUQUObject@@@Z 1001127c     qt-mt323:qt-mt323.dll
 0002:00000280       __imp_?qt_emit@QPopupMenu@@UAE_NHPAUQUObject@@@Z 10011280     qt-mt323:qt-mt323.dll
 0002:00000284       __imp_?qt_emit@QToolBar@@UAE_NHPAUQUObject@@@Z 10011284     qt-mt323:qt-mt323.dll
 0002:00000288       __imp_?qt_emit@QWidget@@UAE_NHPAUQUObject@@@Z 10011288     qt-mt323:qt-mt323.dll
 0002:0000028c       __imp_?qt_invoke@QAction@@UAE_NHPAUQUObject@@@Z 1001128c     qt-mt323:qt-mt323.dll
 0002:00000290       __imp_?qt_invoke@QGuardedPtrPrivate@@UAE_NHPAUQUObject@@@Z 10011290     qt-mt323:qt-mt323.dll
 0002:00000294       __imp_?qt_invoke@QPopupMenu@@UAE_NHPAUQUObject@@@Z 10011294     qt-mt323:qt-mt323.dll
 0002:00000298       __imp_?qt_invoke@QToolBar@@UAE_NHPAUQUObject@@@Z 10011298     qt-mt323:qt-mt323.dll
 0002:0000029c       __imp_?qt_invoke@QWidget@@UAE_NHPAUQUObject@@@Z 1001129c     qt-mt323:qt-mt323.dll
 0002:000002a0       __imp_?qt_property@QAction@@UAE_NHHPAVQVariant@@@Z 100112a0     qt-mt323:qt-mt323.dll
 0002:000002a4       __imp_?qt_property@QGuardedPtrPrivate@@UAE_NHHPAVQVariant@@@Z 100112a4     qt-mt323:qt-mt323.dll
 0002:000002a8       __imp_?qt_property@QPopupMenu@@UAE_NHHPAVQVariant@@@Z 100112a8     qt-mt323:qt-mt323.dll
 0002:000002ac       __imp_?qt_property@QToolBar@@UAE_NHHPAVQVariant@@@Z 100112ac     qt-mt323:qt-mt323.dll
 0002:000002b0       __imp_?qt_property@QWidget@@UAE_NHHPAVQVariant@@@Z 100112b0     qt-mt323:qt-mt323.dll
 0002:000002b4       __imp_?read@QGDict@@MAEAAVQDataStream@@AAV2@AAPAX@Z 100112b4     qt-mt323:qt-mt323.dll
 0002:000002b8       __imp_?read@QGList@@MAEAAVQDataStream@@AAV2@AAPAX@Z 100112b8     qt-mt323:qt-mt323.dll
 0002:000002bc       __imp_?removeChild@QObject@@UAEXPAV1@@Z 100112bc     qt-mt323:qt-mt323.dll
 0002:000002c0       __imp_?removeFrom@QAction@@UAE_NPAVQWidget@@@Z 100112c0     qt-mt323:qt-mt323.dll
 0002:000002c4       __imp_?reparent@QWidget@@UAEXPAV1@IABVQPoint@@_N@Z 100112c4     qt-mt323:qt-mt323.dll
 0002:000002c8       __imp_?resize@QWidget@@UAEXHH@Z 100112c8     qt-mt323:qt-mt323.dll
 0002:000002cc       __imp_?resizeEvent@QFrame@@MAEXPAVQResizeEvent@@@Z 100112cc     qt-mt323:qt-mt323.dll
 0002:000002d0       __imp_?resizeEvent@QToolBar@@MAEXPAVQResizeEvent@@@Z 100112d0     qt-mt323:qt-mt323.dll
 0002:000002d4       __imp_?resizeEvent@QWidget@@MAEXPAVQResizeEvent@@@Z 100112d4     qt-mt323:qt-mt323.dll
 0002:000002d8       __imp_?resolution@QPaintDevice@@UBEHXZ 100112d8     qt-mt323:qt-mt323.dll
 0002:000002dc       __imp_?setAccel@QAction@@UAEXABVQKeySequence@@@Z 100112dc     qt-mt323:qt-mt323.dll
 0002:000002e0       __imp_?setAcceptDrops@QWidget@@UAEX_N@Z 100112e0     qt-mt323:qt-mt323.dll
 0002:000002e4       __imp_?setActiveItem@QPopupMenu@@UAEXH@Z 100112e4     qt-mt323:qt-mt323.dll
 0002:000002e8       __imp_?setActiveWindow@QWidget@@UAEXXZ 100112e8     qt-mt323:qt-mt323.dll
 0002:000002ec       __imp_?setAutoMask@QWidget@@UAEX_N@Z 100112ec     qt-mt323:qt-mt323.dll
 0002:000002f0       __imp_?setBackgroundColor@QWidget@@UAEXABVQColor@@@Z 100112f0     qt-mt323:qt-mt323.dll
 0002:000002f4       __imp_?setBackgroundMode@QWidget@@UAEXW4BackgroundMode@Qt@@@Z 100112f4     qt-mt323:qt-mt323.dll
 0002:000002f8       __imp_?setBackgroundOrigin@QWidget@@UAEXW4BackgroundOrigin@1@@Z 100112f8     qt-mt323:qt-mt323.dll
 0002:000002fc       __imp_?setBackgroundPixmap@QWidget@@UAEXABVQPixmap@@@Z 100112fc     qt-mt323:qt-mt323.dll
 0002:00000300       __imp_?setCaption@QDockWindow@@UAEXABVQString@@@Z 10011300     qt-mt323:qt-mt323.dll
 0002:00000304       __imp_?setCaption@QWidget@@UAEXABVQString@@@Z 10011304     qt-mt323:qt-mt323.dll
 0002:00000308       __imp_?setCheckable@QPopupMenu@@UAEX_N@Z 10011308     qt-mt323:qt-mt323.dll
 0002:0000030c       __imp_?setCloseMode@QDockWindow@@UAEXH@Z 1001130c     qt-mt323:qt-mt323.dll
 0002:00000310       __imp_?setCursor@QWidget@@UAEXABVQCursor@@@Z 10011310     qt-mt323:qt-mt323.dll
 0002:00000314       __imp_?setEnabled@QAction@@UAEX_N@Z 10011314     qt-mt323:qt-mt323.dll
 0002:00000318       __imp_?setEnabled@QWidget@@UAEX_N@Z 10011318     qt-mt323:qt-mt323.dll
 0002:0000031c       __imp_?setEraseColor@QWidget@@UAEXABVQColor@@@Z 1001131c     qt-mt323:qt-mt323.dll
 0002:00000320       __imp_?setErasePixmap@QWidget@@UAEXABVQPixmap@@@Z 10011320     qt-mt323:qt-mt323.dll
 0002:00000324       __imp_?setFirstItemActive@QPopupMenu@@EAEXXZ 10011324     qt-mt323:qt-mt323.dll
 0002:00000328       __imp_?setFixedExtentHeight@QDockWindow@@UAEXH@Z 10011328     qt-mt323:qt-mt323.dll
 0002:0000032c       __imp_?setFixedExtentWidth@QDockWindow@@UAEXH@Z 1001132c     qt-mt323:qt-mt323.dll
 0002:00000330       __imp_?setFocus@QWidget@@UAEXXZ 10011330     qt-mt323:qt-mt323.dll
 0002:00000334       __imp_?setFocusPolicy@QWidget@@UAEXW4FocusPolicy@1@@Z 10011334     qt-mt323:qt-mt323.dll
 0002:00000338       __imp_?setFocusProxy@QWidget@@UAEXPAV1@@Z 10011338     qt-mt323:qt-mt323.dll
 0002:0000033c       __imp_?setFont@QPopupMenu@@UAEXABVQFont@@@Z 1001133c     qt-mt323:qt-mt323.dll
 0002:00000340       __imp_?setFont@QWidget@@UAEXABVQFont@@@Z 10011340     qt-mt323:qt-mt323.dll
 0002:00000344       __imp_?setFrameRect@QFrame@@UAEXABVQRect@@@Z 10011344     qt-mt323:qt-mt323.dll
 0002:00000348       __imp_?setFrameStyle@QFrame@@UAEXH@Z 10011348     qt-mt323:qt-mt323.dll
 0002:0000034c       __imp_?setGeometry@QWidget@@UAEXABVQRect@@@Z 1001134c     qt-mt323:qt-mt323.dll
 0002:00000350       __imp_?setGeometry@QWidget@@UAEXHHHH@Z 10011350     qt-mt323:qt-mt323.dll
 0002:00000354       __imp_?setHorizontallyStretchable@QDockWindow@@UAEX_N@Z 10011354     qt-mt323:qt-mt323.dll
 0002:00000358       __imp_?setIcon@QWidget@@UAEXABVQPixmap@@@Z 10011358     qt-mt323:qt-mt323.dll
 0002:0000035c       __imp_?setIconSet@QAction@@UAEXABVQIconSet@@@Z 1001135c     qt-mt323:qt-mt323.dll
 0002:00000360       __imp_?setIconText@QWidget@@UAEXABVQString@@@Z 10011360     qt-mt323:qt-mt323.dll
 0002:00000364       __imp_?setId@QMenuData@@UAEXHH@Z 10011364     qt-mt323:qt-mt323.dll
 0002:00000368       __imp_?setKeyCompression@QWidget@@MAEX_N@Z 10011368     qt-mt323:qt-mt323.dll
 0002:0000036c       __imp_?setLabel@QToolBar@@UAEXABVQString@@@Z 1001136c     qt-mt323:qt-mt323.dll
 0002:00000370       __imp_?setLineWidth@QFrame@@UAEXH@Z 10011370     qt-mt323:qt-mt323.dll
 0002:00000374       __imp_?setMargin@QFrame@@UAEXH@Z 10011374     qt-mt323:qt-mt323.dll
 0002:00000378       __imp_?setMask@QWidget@@UAEXABVQBitmap@@@Z 10011378     qt-mt323:qt-mt323.dll
 0002:0000037c       __imp_?setMask@QWidget@@UAEXABVQRegion@@@Z 1001137c     qt-mt323:qt-mt323.dll
 0002:00000380       __imp_?setMaximumSize@QWidget@@UAEXHH@Z 10011380     qt-mt323:qt-mt323.dll
 0002:00000384       __imp_?setMenuText@QAction@@UAEXABVQString@@@Z 10011384     qt-mt323:qt-mt323.dll
 0002:00000388       __imp_?setMicroFocusHint@QWidget@@MAEXHHHH_NPAVQFont@@@Z 10011388     qt-mt323:qt-mt323.dll
 0002:0000038c       __imp_?setMidLineWidth@QFrame@@UAEXH@Z 1001138c     qt-mt323:qt-mt323.dll
 0002:00000390       __imp_?setMinimumSize@QToolBar@@UAEXHH@Z 10011390     qt-mt323:qt-mt323.dll
 0002:00000394       __imp_?setMinimumSize@QWidget@@UAEXHH@Z 10011394     qt-mt323:qt-mt323.dll
 0002:00000398       __imp_?setMouseTracking@QWidget@@UAEX_N@Z 10011398     qt-mt323:qt-mt323.dll
 0002:0000039c       __imp_?setMovingEnabled@QDockWindow@@UAEX_N@Z 1001139c     qt-mt323:qt-mt323.dll
 0002:000003a0       __imp_?setName@QObject@@UAEXPBD@Z 100113a0     qt-mt323:qt-mt323.dll
 0002:000003a4       __imp_?setNewLine@QDockWindow@@UAEX_N@Z 100113a4     qt-mt323:qt-mt323.dll
 0002:000003a8       __imp_?setOffset@QDockWindow@@UAEXH@Z 100113a8     qt-mt323:qt-mt323.dll
 0002:000003ac       __imp_?setOn@QAction@@UAEX_N@Z 100113ac     qt-mt323:qt-mt323.dll
 0002:000003b0       __imp_?setOpaqueMoving@QDockWindow@@UAEX_N@Z 100113b0     qt-mt323:qt-mt323.dll
 0002:000003b4       __imp_?setOrientation@QToolBar@@UAEXW4Orientation@Qt@@@Z 100113b4     qt-mt323:qt-mt323.dll
 0002:000003b8       __imp_?setPalette@QWidget@@UAEXABVQPalette@@@Z 100113b8     qt-mt323:qt-mt323.dll
 0002:000003bc       __imp_?setPaletteBackgroundColor@QWidget@@UAEXABVQColor@@@Z 100113bc     qt-mt323:qt-mt323.dll
 0002:000003c0       __imp_?setPaletteBackgroundPixmap@QWidget@@UAEXABVQPixmap@@@Z 100113c0     qt-mt323:qt-mt323.dll
 0002:000003c4       __imp_?setProperty@QObject@@UAE_NPBDABVQVariant@@@Z 100113c4     qt-mt323:qt-mt323.dll
 0002:000003c8       __imp_?setResizeEnabled@QDockWindow@@UAEX_N@Z 100113c8     qt-mt323:qt-mt323.dll
 0002:000003cc       __imp_?setResolution@QPaintDevice@@UAEXH@Z 100113cc     qt-mt323:qt-mt323.dll
 0002:000003d0       __imp_?setSizeIncrement@QWidget@@UAEXHH@Z 100113d0     qt-mt323:qt-mt323.dll
 0002:000003d4       __imp_?setSizePolicy@QWidget@@UAEXVQSizePolicy@@@Z 100113d4     qt-mt323:qt-mt323.dll
 0002:000003d8       __imp_?setStatusTip@QAction@@UAEXABVQString@@@Z 100113d8     qt-mt323:qt-mt323.dll
 0002:000003dc       __imp_?setStretchableWidget@QToolBar@@UAEXPAVQWidget@@@Z 100113dc     qt-mt323:qt-mt323.dll
 0002:000003e0       __imp_?setText@QAction@@UAEXABVQString@@@Z 100113e0     qt-mt323:qt-mt323.dll
 0002:000003e4       __imp_?setToggleAction@QAction@@UAEX_N@Z 100113e4     qt-mt323:qt-mt323.dll
 0002:000003e8       __imp_?setToolTip@QAction@@UAEXABVQString@@@Z 100113e8     qt-mt323:qt-mt323.dll
 0002:000003ec       __imp_?setUpdatesEnabled@QWidget@@UAEX_N@Z 100113ec     qt-mt323:qt-mt323.dll
 0002:000003f0       __imp_?setVerticallyStretchable@QDockWindow@@UAEX_N@Z 100113f0     qt-mt323:qt-mt323.dll
 0002:000003f4       __imp_?setWFlags@QWidget@@MAEXI@Z 100113f4     qt-mt323:qt-mt323.dll
 0002:000003f8       __imp_?setWState@QWidget@@MAEXI@Z 100113f8     qt-mt323:qt-mt323.dll
 0002:000003fc       __imp_?setWhatsThis@QAction@@UAEXABVQString@@@Z 100113fc     qt-mt323:qt-mt323.dll
 0002:00000400       __imp_?setWidget@QDockWindow@@UAEXPAVQWidget@@@Z 10011400     qt-mt323:qt-mt323.dll
 0002:00000404       __imp_?show@QPopupMenu@@UAEXXZ 10011404     qt-mt323:qt-mt323.dll
 0002:00000408       __imp_?show@QToolBar@@UAEXXZ 10011408     qt-mt323:qt-mt323.dll
 0002:0000040c       __imp_?show@QWidget@@UAEXXZ 1001140c     qt-mt323:qt-mt323.dll
 0002:00000410       __imp_?showEvent@QDockWindow@@MAEXPAVQShowEvent@@@Z 10011410     qt-mt323:qt-mt323.dll
 0002:00000414       __imp_?showEvent@QWidget@@MAEXPAVQShowEvent@@@Z 10011414     qt-mt323:qt-mt323.dll
 0002:00000418       __imp_?showMaximized@QWidget@@UAEXXZ 10011418     qt-mt323:qt-mt323.dll
 0002:0000041c       __imp_?showMinimized@QWidget@@UAEXXZ 1001141c     qt-mt323:qt-mt323.dll
 0002:00000420       __imp_?showNormal@QWidget@@UAEXXZ 10011420     qt-mt323:qt-mt323.dll
 0002:00000424       __imp_?sizeHint@QDockWindow@@UBE?AVQSize@@XZ 10011424     qt-mt323:qt-mt323.dll
 0002:00000428       __imp_?sizeHint@QPopupMenu@@UBE?AVQSize@@XZ 10011428     qt-mt323:qt-mt323.dll
 0002:0000042c       __imp_?sizeHint@QWidget@@UBE?AVQSize@@XZ 1001142c     qt-mt323:qt-mt323.dll
 0002:00000430       __imp_?sizePolicy@QWidget@@UBE?AVQSizePolicy@@XZ 10011430     qt-mt323:qt-mt323.dll
 0002:00000434       __imp_?styleChange@QPopupMenu@@MAEXAAVQStyle@@@Z 10011434     qt-mt323:qt-mt323.dll
 0002:00000438       __imp_?styleChange@QToolBar@@MAEXAAVQStyle@@@Z 10011438     qt-mt323:qt-mt323.dll
 0002:0000043c       __imp_?styleChange@QWidget@@MAEXAAVQStyle@@@Z 1001143c     qt-mt323:qt-mt323.dll
 0002:00000440       __imp_?tabletEvent@QWidget@@MAEXPAVQTabletEvent@@@Z 10011440     qt-mt323:qt-mt323.dll
 0002:00000444       __imp_?timerEvent@QObject@@MAEXPAVQTimerEvent@@@Z 10011444     qt-mt323:qt-mt323.dll
 0002:00000448       __imp_?timerEvent@QPopupMenu@@MAEXPAVQTimerEvent@@@Z 10011448     qt-mt323:qt-mt323.dll
 0002:0000044c       __imp_?undock@QDockWindow@@UAEXPAVQWidget@@@Z 1001144c     qt-mt323:qt-mt323.dll
 0002:00000450       __imp_?undock@QDockWindow@@UAEXXZ 10011450     qt-mt323:qt-mt323.dll
 0002:00000454       __imp_?unsetCursor@QWidget@@UAEXXZ 10011454     qt-mt323:qt-mt323.dll
 0002:00000458       __imp_?updateItem@QPopupMenu@@UAEXH@Z 10011458     qt-mt323:qt-mt323.dll
 0002:0000045c       __imp_?updateMask@QWidget@@MAEXXZ 1001145c     qt-mt323:qt-mt323.dll
 0002:00000460       __imp_?wheelEvent@QWidget@@MAEXPAVQWheelEvent@@@Z 10011460     qt-mt323:qt-mt323.dll
 0002:00000464       __imp_?winEvent@QWidget@@MAE_NPAUtagMSG@@@Z 10011464     qt-mt323:qt-mt323.dll
 0002:00000468       __imp_?windowActivationChange@QWidget@@MAEX_N@Z 10011468     qt-mt323:qt-mt323.dll
 0002:0000046c       __imp_?write@QGDict@@MBEAAVQDataStream@@AAV2@PAX@Z 1001146c     qt-mt323:qt-mt323.dll
 0002:00000470       __imp_?write@QGList@@MBEAAVQDataStream@@AAV2@PAX@Z 10011470     qt-mt323:qt-mt323.dll
 0002:00000474       __imp_?null@QString@@2V1@A 10011474     qt-mt323:qt-mt323.dll
 0002:00000478       __imp_??_7?$QPtrList@VQDockWindow@@@@6B@ 10011478     qt-mt323:qt-mt323.dll
 0002:0000047c       __imp_??0QGArray@@IAE@H@Z  1001147c     qt-mt323:qt-mt323.dll
 0002:00000480       __imp_??1QGArray@@MAE@XZ   10011480     qt-mt323:qt-mt323.dll
 0002:00000484       __imp_?resize@QGArray@@IAE_NI@Z 10011484     qt-mt323:qt-mt323.dll
 0002:00000488       __imp_?sort@QGArray@@IAEXI@Z 10011488     qt-mt323:qt-mt323.dll
 0002:0000048c       __imp_?at@QGArray@@IBEPADI@Z 1001148c     qt-mt323:qt-mt323.dll
 0002:00000490       __imp_??1?$QMemArray@H@@UAE@XZ 10011490     qt-mt323:qt-mt323.dll
 0002:00000494       __imp_?truncate@QString@@QAEXI@Z 10011494     qt-mt323:qt-mt323.dll
 0002:00000498       __imp_?sprintf@QString@@QAAAAV1@PBDZZ 10011498     qt-mt323:qt-mt323.dll
 0002:0000049c       __imp_?find@QString@@QBEHABV1@H_N@Z 1001149c     qt-mt323:qt-mt323.dll
 0002:000004a0       __imp_?contains@QString@@QBEHPBD_N@Z 100114a0     qt-mt323:qt-mt323.dll
 0002:000004a4       __imp_?section@QString@@QBE?AV1@DHHH@Z 100114a4     qt-mt323:qt-mt323.dll
 0002:000004a8       __imp_?upper@QString@@QBE?AV1@XZ 100114a8     qt-mt323:qt-mt323.dll
 0002:000004ac       __imp_?remove@QString@@QAEAAV1@II@Z 100114ac     qt-mt323:qt-mt323.dll
 0002:000004b0       __imp_?remove@QString@@QAEAAV1@D@Z 100114b0     qt-mt323:qt-mt323.dll
 0002:000004b4       __imp_?fromAscii@QString@@SA?AV1@PBDH@Z 100114b4     qt-mt323:qt-mt323.dll
 0002:000004b8       __imp_?latin1@QString@@QBEPBDXZ 100114b8     qt-mt323:qt-mt323.dll
 0002:000004bc       __imp_?startsWith@QString@@QBE_NABV1@@Z 100114bc     qt-mt323:qt-mt323.dll
 0002:000004c0       __imp_??9@YA_NABVQString@@0@Z 100114c0     qt-mt323:qt-mt323.dll
 0002:000004c4       __imp_??8@YA_NABVQString@@0@Z 100114c4     qt-mt323:qt-mt323.dll
 0002:000004c8       __imp_??9@YA_NABVQString@@PBD@Z 100114c8     qt-mt323:qt-mt323.dll
 0002:000004cc       __imp_??0QTextStream@@QAE@PAVQIODevice@@@Z 100114cc     qt-mt323:qt-mt323.dll
 0002:000004d0       __imp_??1QTextStream@@UAE@XZ 100114d0     qt-mt323:qt-mt323.dll
 0002:000004d4       __imp_??6QTextStream@@QAEAAV0@ABVQString@@@Z 100114d4     qt-mt323:qt-mt323.dll
 0002:000004d8       __imp_?begin@?$QValueList@VQString@@@@QAE?AV?$QValueListIterator@VQString@@@@XZ 100114d8     qt-mt323:qt-mt323.dll
 0002:000004dc       __imp_?clear@?$QValueList@VQString@@@@QAEXXZ 100114dc     qt-mt323:qt-mt323.dll
 0002:000004e0       __imp_??6?$QValueList@VQString@@@@QAEAAV0@ABVQString@@@Z 100114e0     qt-mt323:qt-mt323.dll
 0002:000004e4       __imp_?append@?$QValueList@VQString@@@@QAE?AV?$QValueListIterator@VQString@@@@ABVQString@@@Z 100114e4     qt-mt323:qt-mt323.dll
 0002:000004e8       __imp_?first@?$QValueList@VQString@@@@QAEAAVQString@@XZ 100114e8     qt-mt323:qt-mt323.dll
 0002:000004ec       __imp_??A?$QValueList@VQString@@@@QAEAAVQString@@I@Z 100114ec     qt-mt323:qt-mt323.dll
 0002:000004f0       __imp_?contains@?$QValueList@VQString@@@@QBEIABVQString@@@Z 100114f0     qt-mt323:qt-mt323.dll
 0002:000004f4       __imp_?detachInternal@?$QValueList@VQString@@@@AAEXXZ 100114f4     qt-mt323:qt-mt323.dll
 0002:000004f8       __imp_?first@QGList@@IAEPAXXZ 100114f8     qt-mt323:qt-mt323.dll
 0002:000004fc       __imp_?next@QGList@@IAEPAXXZ 100114fc     qt-mt323:qt-mt323.dll
 0002:00000500       __imp_?blockSignals@QObject@@QAEX_N@Z 10011500     qt-mt323:qt-mt323.dll
 0002:00000504       __imp_??0QStringList@@QAE@XZ 10011504     qt-mt323:qt-mt323.dll
 0002:00000508       __imp_?split@QStringList@@SA?AV1@ABVQString@@0_N@Z 10011508     qt-mt323:qt-mt323.dll
 0002:0000050c       __imp_?split@QStringList@@SA?AV1@ABVQChar@@ABVQString@@_N@Z 1001150c     qt-mt323:qt-mt323.dll
 0002:00000510       __imp_??1QStringList@@QAE@XZ 10011510     qt-mt323:qt-mt323.dll
 0002:00000514       __imp_??4QStringList@@QAEAAV0@ABV0@@Z 10011514     qt-mt323:qt-mt323.dll
 0002:00000518       __imp_?hasFocus@QWidget@@QBE_NXZ 10011518     qt-mt323:qt-mt323.dll
 0002:0000051c       __imp_?updateContents@QScrollView@@QAEXXZ 1001151c     qt-mt323:qt-mt323.dll
 0002:00000520       __imp_??0QFile@@QAE@ABVQString@@@Z 10011520     qt-mt323:qt-mt323.dll
 0002:00000524       __imp_??1QFile@@UAE@XZ     10011524     qt-mt323:qt-mt323.dll
 0002:00000528       __imp_?open@QFile@@UAE_NH@Z 10011528     qt-mt323:qt-mt323.dll
 0002:0000052c       __imp_?close@QFile@@UAEXXZ 1001152c     qt-mt323:qt-mt323.dll
 0002:00000530       __imp_??4QDomNode@@QAEAAV0@ABV0@@Z 10011530     qt-mt323:qt-mt323.dll
 0002:00000534       __imp_??1QDomNode@@UAE@XZ  10011534     qt-mt323:qt-mt323.dll
 0002:00000538       __imp_?replaceChild@QDomNode@@UAE?AV1@ABV1@0@Z 10011538     qt-mt323:qt-mt323.dll
 0002:0000053c       __imp_?removeChild@QDomNode@@UAE?AV1@ABV1@@Z 1001153c     qt-mt323:qt-mt323.dll
 0002:00000540       __imp_?appendChild@QDomNode@@UAE?AV1@ABV1@@Z 10011540     qt-mt323:qt-mt323.dll
 0002:00000544       __imp_?cloneNode@QDomNode@@UBE?AV1@_N@Z 10011544     qt-mt323:qt-mt323.dll
 0002:00000548       __imp_?firstChild@QDomNode@@UBE?AV1@XZ 10011548     qt-mt323:qt-mt323.dll
 0002:0000054c       __imp_?nextSibling@QDomNode@@UBE?AV1@XZ 1001154c     qt-mt323:qt-mt323.dll
 0002:00000550       __imp_?isNull@QDomNode@@QBE_NXZ 10011550     qt-mt323:qt-mt323.dll
 0002:00000554       __imp_?toElement@QDomNode@@QAE?AVQDomElement@@XZ 10011554     qt-mt323:qt-mt323.dll
 0002:00000558       __imp_??0QDomDocument@@QAE@XZ 10011558     qt-mt323:qt-mt323.dll
 0002:0000055c       __imp_??0QDomDocument@@QAE@ABVQString@@@Z 1001155c     qt-mt323:qt-mt323.dll
 0002:00000560       __imp_??1QDomDocument@@UAE@XZ 10011560     qt-mt323:qt-mt323.dll
 0002:00000564       __imp_?createElement@QDomDocument@@QAE?AVQDomElement@@ABVQString@@@Z 10011564     qt-mt323:qt-mt323.dll
 0002:00000568       __imp_?documentElement@QDomDocument@@QBE?AVQDomElement@@XZ 10011568     qt-mt323:qt-mt323.dll
 0002:0000056c       __imp_?setContent@QDomDocument@@QAE_NABVQString@@_NPAV2@PAH3@Z 1001156c     qt-mt323:qt-mt323.dll
 0002:00000570       __imp_?setContent@QDomDocument@@QAE_NPAVQIODevice@@PAVQString@@PAH2@Z 10011570     qt-mt323:qt-mt323.dll
 0002:00000574       __imp_?toString@QDomDocument@@QBE?AVQString@@XZ 10011574     qt-mt323:qt-mt323.dll
 0002:00000578       __imp_?toString@QDomDocument@@QBE?AVQString@@H@Z 10011578     qt-mt323:qt-mt323.dll
 0002:0000057c       __imp_??1QDomElement@@UAE@XZ 1001157c     qt-mt323:qt-mt323.dll
 0002:00000580       __imp_?attribute@QDomElement@@QBE?AVQString@@ABV2@0@Z 10011580     qt-mt323:qt-mt323.dll
 0002:00000584       __imp_?setAttribute@QDomElement@@QAEXABVQString@@0@Z 10011584     qt-mt323:qt-mt323.dll
 0002:00000588       __imp_?tagName@QDomElement@@QBE?AVQString@@XZ 10011588     qt-mt323:qt-mt323.dll
 0002:0000058c       __imp_?isRowSelected@QTable@@QBE_NH_N@Z 1001158c     qt-mt323:qt-mt323.dll
 0002:00000590       __imp_?selectCells@QTable@@QAEXHHHH@Z 10011590     qt-mt323:qt-mt323.dll
 0002:00000594       __imp_?setColumnLabels@QTable@@QAEXABVQStringList@@@Z 10011594     qt-mt323:qt-mt323.dll
 0002:00000598       __imp_?currentPageIndex@QTabWidget@@QBEHXZ 10011598     qt-mt323:qt-mt323.dll
 0002:0000059c       __imp_?setOverrideCursor@QApplication@@SAXABVQCursor@@_N@Z 1001159c     qt-mt323:qt-mt323.dll
 0002:000005a0       __imp_?restoreOverrideCursor@QApplication@@SAXXZ 100115a0     qt-mt323:qt-mt323.dll
 0002:000005a4       __imp_?clipboard@QApplication@@SAPAVQClipboard@@XZ 100115a4     qt-mt323:qt-mt323.dll
 0002:000005a8       __imp_?text@QClipboard@@QBE?AVQString@@XZ 100115a8     qt-mt323:qt-mt323.dll
 0002:000005ac       __imp_?setText@QClipboard@@QAEXABVQString@@@Z 100115ac     qt-mt323:qt-mt323.dll
 0002:000005b0       __imp_??0QCursor@@QAE@H@Z  100115b0     qt-mt323:qt-mt323.dll
 0002:000005b4       __imp_??1QCursor@@QAE@XZ   100115b4     qt-mt323:qt-mt323.dll
 0002:000005b8       __imp_?exec@QDialog@@QAEHXZ 100115b8     qt-mt323:qt-mt323.dll
 0002:000005bc       __imp_?insertStringList@QListBox@@QAEXABVQStringList@@H@Z 100115bc     qt-mt323:qt-mt323.dll
 0002:000005c0       __imp_?currentText@QListBox@@QBE?AVQString@@XZ 100115c0     qt-mt323:qt-mt323.dll
 0002:000005c4       __imp_?findItem@QListBox@@QBEPAVQListBoxItem@@ABVQString@@I@Z 100115c4     qt-mt323:qt-mt323.dll
 0002:000005c8       __imp_?attributes@QDomElement@@UBE?AVQDomNamedNodeMap@@XZ 100115c8     qt-mt323:qt-mt323.dll
 0002:000005cc       __imp_?attributes@QDomNode@@UBE?AVQDomNamedNodeMap@@XZ 100115cc     qt-mt323:qt-mt323.dll
 0002:000005d0       __imp_?childNodes@QDomNode@@UBE?AVQDomNodeList@@XZ 100115d0     qt-mt323:qt-mt323.dll
 0002:000005d4       __imp_?elementsByTagName@QDomElement@@UBE?AVQDomNodeList@@ABVQString@@@Z 100115d4     qt-mt323:qt-mt323.dll
 0002:000005d8       __imp_?elementsByTagNameNS@QDomElement@@UBE?AVQDomNodeList@@ABVQString@@0@Z 100115d8     qt-mt323:qt-mt323.dll
 0002:000005dc       __imp_?hasAttributes@QDomNode@@UBE_NXZ 100115dc     qt-mt323:qt-mt323.dll
 0002:000005e0       __imp_?hasChildNodes@QDomNode@@UBE_NXZ 100115e0     qt-mt323:qt-mt323.dll
 0002:000005e4       __imp_?insertAfter@QDomNode@@UAE?AV1@ABV1@0@Z 100115e4     qt-mt323:qt-mt323.dll
 0002:000005e8       __imp_?insertBefore@QDomNode@@UAE?AV1@ABV1@0@Z 100115e8     qt-mt323:qt-mt323.dll
 0002:000005ec       __imp_?isAttr@QDomNode@@UBE_NXZ 100115ec     qt-mt323:qt-mt323.dll
 0002:000005f0       __imp_?isCDATASection@QDomNode@@UBE_NXZ 100115f0     qt-mt323:qt-mt323.dll
 0002:000005f4       __imp_?isCharacterData@QDomNode@@UBE_NXZ 100115f4     qt-mt323:qt-mt323.dll
 0002:000005f8       __imp_?isComment@QDomNode@@UBE_NXZ 100115f8     qt-mt323:qt-mt323.dll
 0002:000005fc       __imp_?isDocument@QDomDocument@@UBE_NXZ 100115fc     qt-mt323:qt-mt323.dll
 0002:00000600       __imp_?isDocument@QDomNode@@UBE_NXZ 10011600     qt-mt323:qt-mt323.dll
 0002:00000604       __imp_?isDocumentFragment@QDomNode@@UBE_NXZ 10011604     qt-mt323:qt-mt323.dll
 0002:00000608       __imp_?isDocumentType@QDomNode@@UBE_NXZ 10011608     qt-mt323:qt-mt323.dll
 0002:0000060c       __imp_?isElement@QDomElement@@UBE_NXZ 1001160c     qt-mt323:qt-mt323.dll
 0002:00000610       __imp_?isElement@QDomNode@@UBE_NXZ 10011610     qt-mt323:qt-mt323.dll
 0002:00000614       __imp_?isEntity@QDomNode@@UBE_NXZ 10011614     qt-mt323:qt-mt323.dll
 0002:00000618       __imp_?isEntityReference@QDomNode@@UBE_NXZ 10011618     qt-mt323:qt-mt323.dll
 0002:0000061c       __imp_?isNotation@QDomNode@@UBE_NXZ 1001161c     qt-mt323:qt-mt323.dll
 0002:00000620       __imp_?isProcessingInstruction@QDomNode@@UBE_NXZ 10011620     qt-mt323:qt-mt323.dll
 0002:00000624       __imp_?isSupported@QDomNode@@UBE_NABVQString@@0@Z 10011624     qt-mt323:qt-mt323.dll
 0002:00000628       __imp_?isText@QDomNode@@UBE_NXZ 10011628     qt-mt323:qt-mt323.dll
 0002:0000062c       __imp_?lastChild@QDomNode@@UBE?AV1@XZ 1001162c     qt-mt323:qt-mt323.dll
 0002:00000630       __imp_?localName@QDomNode@@UBE?AVQString@@XZ 10011630     qt-mt323:qt-mt323.dll
 0002:00000634       __imp_?namespaceURI@QDomNode@@UBE?AVQString@@XZ 10011634     qt-mt323:qt-mt323.dll
 0002:00000638       __imp_?nodeName@QDomNode@@UBE?AVQString@@XZ 10011638     qt-mt323:qt-mt323.dll
 0002:0000063c       __imp_?nodeType@QDomDocument@@UBE?AW4NodeType@QDomNode@@XZ 1001163c     qt-mt323:qt-mt323.dll
 0002:00000640       __imp_?nodeType@QDomElement@@UBE?AW4NodeType@QDomNode@@XZ 10011640     qt-mt323:qt-mt323.dll
 0002:00000644       __imp_?nodeValue@QDomNode@@UBE?AVQString@@XZ 10011644     qt-mt323:qt-mt323.dll
 0002:00000648       __imp_?normalize@QDomNode@@UAEXXZ 10011648     qt-mt323:qt-mt323.dll
 0002:0000064c       __imp_?ownerDocument@QDomNode@@UBE?AVQDomDocument@@XZ 1001164c     qt-mt323:qt-mt323.dll
 0002:00000650       __imp_?parentNode@QDomNode@@UBE?AV1@XZ 10011650     qt-mt323:qt-mt323.dll
 0002:00000654       __imp_?prefix@QDomNode@@UBE?AVQString@@XZ 10011654     qt-mt323:qt-mt323.dll
 0002:00000658       __imp_?previousSibling@QDomNode@@UBE?AV1@XZ 10011658     qt-mt323:qt-mt323.dll
 0002:0000065c       __imp_?setNodeValue@QDomNode@@UAEXABVQString@@@Z 1001165c     qt-mt323:qt-mt323.dll
 0002:00000660       __imp_?setPrefix@QDomNode@@UAEXABVQString@@@Z 10011660     qt-mt323:qt-mt323.dll
 0002:00000664       __imp_??_7?$QMemArray@H@@6B@ 10011664     qt-mt323:qt-mt323.dll
 0002:00000668       __imp_??0QDialog@@QAE@PAVQWidget@@PBD_NI@Z 10011668     qt-mt323:qt-mt323.dll
 0002:0000066c       __imp_??1QDialog@@UAE@XZ   1001166c     qt-mt323:qt-mt323.dll
 0002:00000670       __imp_?resize@QDialog@@QAEXABVQSize@@@Z 10011670     qt-mt323:qt-mt323.dll
 0002:00000674       __imp_?minimumSizeHint@QDialog@@UBE?AVQSize@@XZ 10011674     qt-mt323:qt-mt323.dll
 0002:00000678       __imp_?setSizeGripEnabled@QDialog@@QAEX_N@Z 10011678     qt-mt323:qt-mt323.dll
 0002:0000067c       __imp_??0QLabel@@QAE@PAVQWidget@@PBDI@Z 1001167c     qt-mt323:qt-mt323.dll
 0002:00000680       __imp_??1QLabel@@UAE@XZ    10011680     qt-mt323:qt-mt323.dll
 0002:00000684       __imp_??0QListBox@@QAE@PAVQWidget@@PBDI@Z 10011684     qt-mt323:qt-mt323.dll
 0002:00000688       __imp_??1QListBox@@UAE@XZ  10011688     qt-mt323:qt-mt323.dll
 0002:0000068c       __imp_?insertItem@QListBox@@QAEXABVQString@@H@Z 1001168c     qt-mt323:qt-mt323.dll
 0002:00000690       __imp_?clear@QListBox@@QAEXXZ 10011690     qt-mt323:qt-mt323.dll
 0002:00000694       __imp_??0QPushButton@@QAE@PAVQWidget@@PBD@Z 10011694     qt-mt323:qt-mt323.dll
 0002:00000698       __imp_??1QPushButton@@UAE@XZ 10011698     qt-mt323:qt-mt323.dll
 0002:0000069c       __imp_??1QLayoutItem@@UAE@XZ 1001169c     qt-mt323:qt-mt323.dll
 0002:000006a0       __imp_??0QSpacerItem@@QAE@HHW4SizeType@QSizePolicy@@0@Z 100116a0     qt-mt323:qt-mt323.dll
 0002:000006a4       __imp_?addWidget@QBoxLayout@@QAEXPAVQWidget@@HH@Z 100116a4     qt-mt323:qt-mt323.dll
 0002:000006a8       __imp_?addLayout@QBoxLayout@@QAEXPAVQLayout@@H@Z 100116a8     qt-mt323:qt-mt323.dll
 0002:000006ac       __imp_??0QHBoxLayout@@QAE@PAVQWidget@@HHPBD@Z 100116ac     qt-mt323:qt-mt323.dll
 0002:000006b0       __imp_??1QHBoxLayout@@UAE@XZ 100116b0     qt-mt323:qt-mt323.dll
 0002:000006b4       __imp_??0QVBoxLayout@@QAE@PAVQWidget@@HHPBD@Z 100116b4     qt-mt323:qt-mt323.dll
 0002:000006b8       __imp_??1QVBoxLayout@@UAE@XZ 100116b8     qt-mt323:qt-mt323.dll
 0002:000006bc       __imp_?accept@QDialog@@MAEXXZ 100116bc     qt-mt323:qt-mt323.dll
 0002:000006c0       __imp_?addChild@QScrollView@@UAEXPAVQWidget@@HH@Z 100116c0     qt-mt323:qt-mt323.dll
 0002:000006c4       __imp_?addItem@QBoxLayout@@UAEXPAVQLayoutItem@@@Z 100116c4     qt-mt323:qt-mt323.dll
 0002:000006c8       __imp_?childEvent@QLayout@@MAEXPAVQChildEvent@@@Z 100116c8     qt-mt323:qt-mt323.dll
 0002:000006cc       __imp_?className@QHBoxLayout@@UBEPBDXZ 100116cc     qt-mt323:qt-mt323.dll
 0002:000006d0       __imp_?className@QLabel@@UBEPBDXZ 100116d0     qt-mt323:qt-mt323.dll
 0002:000006d4       __imp_?className@QListBox@@UBEPBDXZ 100116d4     qt-mt323:qt-mt323.dll
 0002:000006d8       __imp_?className@QPushButton@@UBEPBDXZ 100116d8     qt-mt323:qt-mt323.dll
 0002:000006dc       __imp_?className@QVBoxLayout@@UBEPBDXZ 100116dc     qt-mt323:qt-mt323.dll
 0002:000006e0       __imp_?clearSelection@QListBox@@UAEXXZ 100116e0     qt-mt323:qt-mt323.dll
 0002:000006e4       __imp_?closeEvent@QDialog@@MAEXPAVQCloseEvent@@@Z 100116e4     qt-mt323:qt-mt323.dll
 0002:000006e8       __imp_?contentsContextMenuEvent@QListBox@@MAEXPAVQContextMenuEvent@@@Z 100116e8     qt-mt323:qt-mt323.dll
 0002:000006ec       __imp_?contentsDragEnterEvent@QScrollView@@MAEXPAVQDragEnterEvent@@@Z 100116ec     qt-mt323:qt-mt323.dll
 0002:000006f0       __imp_?contentsDragLeaveEvent@QScrollView@@MAEXPAVQDragLeaveEvent@@@Z 100116f0     qt-mt323:qt-mt323.dll
 0002:000006f4       __imp_?contentsDragMoveEvent@QScrollView@@MAEXPAVQDragMoveEvent@@@Z 100116f4     qt-mt323:qt-mt323.dll
 0002:000006f8       __imp_?contentsDropEvent@QScrollView@@MAEXPAVQDropEvent@@@Z 100116f8     qt-mt323:qt-mt323.dll
 0002:000006fc       __imp_?contentsMouseDoubleClickEvent@QScrollView@@MAEXPAVQMouseEvent@@@Z 100116fc     qt-mt323:qt-mt323.dll
 0002:00000700       __imp_?contentsMouseMoveEvent@QScrollView@@MAEXPAVQMouseEvent@@@Z 10011700     qt-mt323:qt-mt323.dll
 0002:00000704       __imp_?contentsMousePressEvent@QScrollView@@MAEXPAVQMouseEvent@@@Z 10011704     qt-mt323:qt-mt323.dll
 0002:00000708       __imp_?contentsMouseReleaseEvent@QScrollView@@MAEXPAVQMouseEvent@@@Z 10011708     qt-mt323:qt-mt323.dll
 0002:0000070c       __imp_?contentsWheelEvent@QScrollView@@MAEXPAVQWheelEvent@@@Z 1001170c     qt-mt323:qt-mt323.dll
 0002:00000710       __imp_?contextMenuEvent@QDialog@@MAEXPAVQContextMenuEvent@@@Z 10011710     qt-mt323:qt-mt323.dll
 0002:00000714       __imp_?contextMenuEvent@QScrollView@@MAEXPAVQContextMenuEvent@@@Z 10011714     qt-mt323:qt-mt323.dll
 0002:00000718       __imp_?done@QDialog@@MAEXH@Z 10011718     qt-mt323:qt-mt323.dll
 0002:0000071c       __imp_?drawButton@QPushButton@@MAEXPAVQPainter@@@Z 1001171c     qt-mt323:qt-mt323.dll
 0002:00000720       __imp_?drawButtonLabel@QPushButton@@MAEXPAVQPainter@@@Z 10011720     qt-mt323:qt-mt323.dll
 0002:00000724       __imp_?drawContents@QLabel@@MAEXPAVQPainter@@@Z 10011724     qt-mt323:qt-mt323.dll
 0002:00000728       __imp_?drawContents@QScrollView@@EAEXPAVQPainter@@@Z 10011728     qt-mt323:qt-mt323.dll
 0002:0000072c       __imp_?drawContents@QScrollView@@MAEXPAVQPainter@@HHHH@Z 1001172c     qt-mt323:qt-mt323.dll
 0002:00000730       __imp_?drawContentsOffset@QScrollView@@MAEXPAVQPainter@@HHHHHH@Z 10011730     qt-mt323:qt-mt323.dll
 0002:00000734       __imp_?enabledChange@QButton@@MAEX_N@Z 10011734     qt-mt323:qt-mt323.dll
 0002:00000738       __imp_?ensureCurrentVisible@QListBox@@UAEXXZ 10011738     qt-mt323:qt-mt323.dll
 0002:0000073c       __imp_?eventFilter@QDialog@@MAE_NPAVQObject@@PAVQEvent@@@Z 1001173c     qt-mt323:qt-mt323.dll
 0002:00000740       __imp_?eventFilter@QLayout@@MAE_NPAVQObject@@PAVQEvent@@@Z 10011740     qt-mt323:qt-mt323.dll
 0002:00000744       __imp_?eventFilter@QListBox@@MAE_NPAVQObject@@PAVQEvent@@@Z 10011744     qt-mt323:qt-mt323.dll
 0002:00000748       __imp_?expanding@QBoxLayout@@UBE?AW4ExpandData@QSizePolicy@@XZ 10011748     qt-mt323:qt-mt323.dll
 0002:0000074c       __imp_?expanding@QSpacerItem@@UBE?AW4ExpandData@QSizePolicy@@XZ 1001174c     qt-mt323:qt-mt323.dll
 0002:00000750       __imp_?focusInEvent@QListBox@@MAEXPAVQFocusEvent@@@Z 10011750     qt-mt323:qt-mt323.dll
 0002:00000754       __imp_?focusInEvent@QPushButton@@MAEXPAVQFocusEvent@@@Z 10011754     qt-mt323:qt-mt323.dll
 0002:00000758       __imp_?focusNextPrevChild@QScrollView@@MAE_N_N@Z 10011758     qt-mt323:qt-mt323.dll
 0002:0000075c       __imp_?focusOutEvent@QListBox@@MAEXPAVQFocusEvent@@@Z 1001175c     qt-mt323:qt-mt323.dll
 0002:00000760       __imp_?focusOutEvent@QPushButton@@MAEXPAVQFocusEvent@@@Z 10011760     qt-mt323:qt-mt323.dll
 0002:00000764       __imp_?fontChange@QLabel@@MAEXABVQFont@@@Z 10011764     qt-mt323:qt-mt323.dll
 0002:00000768       __imp_?fontChange@QScrollView@@MAEXABVQFont@@@Z 10011768     qt-mt323:qt-mt323.dll
 0002:0000076c       __imp_?frameChanged@QScrollView@@MAEXXZ 1001176c     qt-mt323:qt-mt323.dll
 0002:00000770       __imp_?geometry@QLayout@@UBE?AVQRect@@XZ 10011770     qt-mt323:qt-mt323.dll
 0002:00000774       __imp_??0QAction@@QAE@ABVQString@@ABVQIconSet@@0VQKeySequence@@PAVQObject@@PBD_N@Z 10011774     qt-mt323:qt-mt323.dll
 0002:00000778       __imp_?hasHeightForWidth@QBoxLayout@@UBE_NXZ 10011778     qt-mt323:qt-mt323.dll
 0002:0000077c       __imp_?hasHeightForWidth@QLayoutItem@@UBE_NXZ 1001177c     qt-mt323:qt-mt323.dll
 0002:00000780       __imp_?heightForWidth@QBoxLayout@@UBEHH@Z 10011780     qt-mt323:qt-mt323.dll
 0002:00000784       __imp_?heightForWidth@QLabel@@UBEHH@Z 10011784     qt-mt323:qt-mt323.dll
 0002:00000788       __imp_?heightForWidth@QLayoutItem@@UBEHH@Z 10011788     qt-mt323:qt-mt323.dll
 0002:0000078c       __imp_?hide@QDialog@@UAEXXZ 1001178c     qt-mt323:qt-mt323.dll
 0002:00000790       __imp_?hitButton@QButton@@MBE_NABVQPoint@@@Z 10011790     qt-mt323:qt-mt323.dll
 0002:00000794       __imp_?invalidate@QBoxLayout@@UAEXXZ 10011794     qt-mt323:qt-mt323.dll
 0002:00000798       __imp_?invalidate@QLayoutItem@@UAEXXZ 10011798     qt-mt323:qt-mt323.dll
 0002:0000079c       __imp_?invertSelection@QListBox@@UAEXXZ 1001179c     qt-mt323:qt-mt323.dll
 0002:000007a0       __imp_?isEmpty@QLayout@@UBE_NXZ 100117a0     qt-mt323:qt-mt323.dll
 0002:000007a4       __imp_?isEmpty@QSpacerItem@@UBE_NXZ 100117a4     qt-mt323:qt-mt323.dll
 0002:000007a8       __imp_?iterator@QBoxLayout@@UAE?AVQLayoutIterator@@XZ 100117a8     qt-mt323:qt-mt323.dll
 0002:000007ac       __imp_?iterator@QLayoutItem@@UAE?AVQLayoutIterator@@XZ 100117ac     qt-mt323:qt-mt323.dll
 0002:000007b0       __imp_?keyPressEvent@QButton@@MAEXPAVQKeyEvent@@@Z 100117b0     qt-mt323:qt-mt323.dll
 0002:000007b4       __imp_?keyPressEvent@QDialog@@MAEXPAVQKeyEvent@@@Z 100117b4     qt-mt323:qt-mt323.dll
 0002:000007b8       __imp_?keyPressEvent@QListBox@@MAEXPAVQKeyEvent@@@Z 100117b8     qt-mt323:qt-mt323.dll
 0002:000007bc       __imp_?keyReleaseEvent@QButton@@MAEXPAVQKeyEvent@@@Z 100117bc     qt-mt323:qt-mt323.dll
 0002:000007c0       __imp_?layout@QLayout@@UAEPAV1@XZ 100117c0     qt-mt323:qt-mt323.dll
 0002:000007c4       __imp_?layout@QLayoutItem@@UAEPAVQLayout@@XZ 100117c4     qt-mt323:qt-mt323.dll
 0002:000007c8       __imp_?maximumSize@QBoxLayout@@UBE?AVQSize@@XZ 100117c8     qt-mt323:qt-mt323.dll
 0002:000007cc       __imp_?maximumSize@QSpacerItem@@UBE?AVQSize@@XZ 100117cc     qt-mt323:qt-mt323.dll
 0002:000007d0       __imp_?metaObject@QHBoxLayout@@UBEPAVQMetaObject@@XZ 100117d0     qt-mt323:qt-mt323.dll
 0002:000007d4       __imp_?metaObject@QLabel@@UBEPAVQMetaObject@@XZ 100117d4     qt-mt323:qt-mt323.dll
 0002:000007d8       __imp_?metaObject@QListBox@@UBEPAVQMetaObject@@XZ 100117d8     qt-mt323:qt-mt323.dll
 0002:000007dc       __imp_?metaObject@QPushButton@@UBEPAVQMetaObject@@XZ 100117dc     qt-mt323:qt-mt323.dll
 0002:000007e0       __imp_?metaObject@QVBoxLayout@@UBEPAVQMetaObject@@XZ 100117e0     qt-mt323:qt-mt323.dll
 0002:000007e4       __imp_?minimumSize@QBoxLayout@@UBE?AVQSize@@XZ 100117e4     qt-mt323:qt-mt323.dll
 0002:000007e8       __imp_?minimumSize@QSpacerItem@@UBE?AVQSize@@XZ 100117e8     qt-mt323:qt-mt323.dll
 0002:000007ec       __imp_?minimumSizeHint@QLabel@@UBE?AVQSize@@XZ 100117ec     qt-mt323:qt-mt323.dll
 0002:000007f0       __imp_?minimumSizeHint@QListBox@@UBE?AVQSize@@XZ 100117f0     qt-mt323:qt-mt323.dll
 0002:000007f4       __imp_?mouseDoubleClickEvent@QListBox@@MAEXPAVQMouseEvent@@@Z 100117f4     qt-mt323:qt-mt323.dll
 0002:000007f8       __imp_?mouseMoveEvent@QButton@@MAEXPAVQMouseEvent@@@Z 100117f8     qt-mt323:qt-mt323.dll
 0002:000007fc       __imp_?mouseMoveEvent@QListBox@@MAEXPAVQMouseEvent@@@Z 100117fc     qt-mt323:qt-mt323.dll
 0002:00000800       __imp_?mousePressEvent@QButton@@MAEXPAVQMouseEvent@@@Z 10011800     qt-mt323:qt-mt323.dll
 0002:00000804       __imp_?mousePressEvent@QListBox@@MAEXPAVQMouseEvent@@@Z 10011804     qt-mt323:qt-mt323.dll
 0002:00000808       __imp_?mouseReleaseEvent@QButton@@MAEXPAVQMouseEvent@@@Z 10011808     qt-mt323:qt-mt323.dll
 0002:0000080c       __imp_?mouseReleaseEvent@QListBox@@MAEXPAVQMouseEvent@@@Z 1001180c     qt-mt323:qt-mt323.dll
 0002:00000810       __imp_?move@QDialog@@UAEXHH@Z 10011810     qt-mt323:qt-mt323.dll
 0002:00000814       __imp_?move@QPushButton@@UAEXHH@Z 10011814     qt-mt323:qt-mt323.dll
 0002:00000818       __imp_?moveChild@QScrollView@@UAEXPAVQWidget@@HH@Z 10011818     qt-mt323:qt-mt323.dll
 0002:0000081c       __imp_?paintCell@QListBox@@MAEXPAVQPainter@@HH@Z 1001181c     qt-mt323:qt-mt323.dll
 0002:00000820       __imp_?paintEvent@QButton@@MAEXPAVQPaintEvent@@@Z 10011820     qt-mt323:qt-mt323.dll
 0002:00000824       __imp_?qt_cast@QHBoxLayout@@UAEPAXPBD@Z 10011824     qt-mt323:qt-mt323.dll
 0002:00000828       __imp_?qt_cast@QLabel@@UAEPAXPBD@Z 10011828     qt-mt323:qt-mt323.dll
 0002:0000082c       __imp_?qt_cast@QListBox@@UAEPAXPBD@Z 1001182c     qt-mt323:qt-mt323.dll
 0002:00000830       __imp_?qt_cast@QPushButton@@UAEPAXPBD@Z 10011830     qt-mt323:qt-mt323.dll
 0002:00000834       __imp_?qt_cast@QVBoxLayout@@UAEPAXPBD@Z 10011834     qt-mt323:qt-mt323.dll
 0002:00000838       __imp_?qt_emit@QHBoxLayout@@UAE_NHPAUQUObject@@@Z 10011838     qt-mt323:qt-mt323.dll
 0002:0000083c       __imp_?qt_emit@QLabel@@UAE_NHPAUQUObject@@@Z 1001183c     qt-mt323:qt-mt323.dll
 0002:00000840       __imp_?qt_emit@QListBox@@UAE_NHPAUQUObject@@@Z 10011840     qt-mt323:qt-mt323.dll
 0002:00000844       __imp_?qt_emit@QPushButton@@UAE_NHPAUQUObject@@@Z 10011844     qt-mt323:qt-mt323.dll
 0002:00000848       __imp_?qt_emit@QVBoxLayout@@UAE_NHPAUQUObject@@@Z 10011848     qt-mt323:qt-mt323.dll
 0002:0000084c       __imp_?qt_invoke@QHBoxLayout@@UAE_NHPAUQUObject@@@Z 1001184c     qt-mt323:qt-mt323.dll
 0002:00000850       __imp_?qt_invoke@QLabel@@UAE_NHPAUQUObject@@@Z 10011850     qt-mt323:qt-mt323.dll
 0002:00000854       __imp_?qt_invoke@QListBox@@UAE_NHPAUQUObject@@@Z 10011854     qt-mt323:qt-mt323.dll
 0002:00000858       __imp_?qt_invoke@QPushButton@@UAE_NHPAUQUObject@@@Z 10011858     qt-mt323:qt-mt323.dll
 0002:0000085c       __imp_?qt_invoke@QVBoxLayout@@UAE_NHPAUQUObject@@@Z 1001185c     qt-mt323:qt-mt323.dll
 0002:00000860       __imp_?qt_property@QHBoxLayout@@UAE_NHHPAVQVariant@@@Z 10011860     qt-mt323:qt-mt323.dll
 0002:00000864       __imp_?qt_property@QLabel@@UAE_NHHPAVQVariant@@@Z 10011864     qt-mt323:qt-mt323.dll
 0002:00000868       __imp_?qt_property@QListBox@@UAE_NHHPAVQVariant@@@Z 10011868     qt-mt323:qt-mt323.dll
 0002:0000086c       __imp_?qt_property@QPushButton@@UAE_NHHPAVQVariant@@@Z 1001186c     qt-mt323:qt-mt323.dll
 0002:00000870       __imp_?qt_property@QVBoxLayout@@UAE_NHHPAVQVariant@@@Z 10011870     qt-mt323:qt-mt323.dll
 0002:00000874       __imp_?reject@QDialog@@MAEXXZ 10011874     qt-mt323:qt-mt323.dll
 0002:00000878       __imp_?removeChild@QScrollView@@UAEXPAVQObject@@@Z 10011878     qt-mt323:qt-mt323.dll
 0002:0000087c       __imp_?resize@QDialog@@UAEXHH@Z 1001187c     qt-mt323:qt-mt323.dll
 0002:00000880       __imp_?resize@QPushButton@@UAEXHH@Z 10011880     qt-mt323:qt-mt323.dll
 0002:00000884       __imp_?resize@QScrollView@@UAEXHH@Z 10011884     qt-mt323:qt-mt323.dll
 0002:00000888       __imp_?resizeContents@QScrollView@@UAEXHH@Z 10011888     qt-mt323:qt-mt323.dll
 0002:0000088c       __imp_?resizeEvent@QDialog@@MAEXPAVQResizeEvent@@@Z 1001188c     qt-mt323:qt-mt323.dll
 0002:00000890       __imp_?resizeEvent@QLabel@@MAEXPAVQResizeEvent@@@Z 10011890     qt-mt323:qt-mt323.dll
 0002:00000894       __imp_?resizeEvent@QListBox@@MAEXPAVQResizeEvent@@@Z 10011894     qt-mt323:qt-mt323.dll
 0002:00000898       __imp_?resizeEvent@QPushButton@@MAEXPAVQResizeEvent@@@Z 10011898     qt-mt323:qt-mt323.dll
 0002:0000089c       __imp_?selectAll@QListBox@@UAEX_N@Z 1001189c     qt-mt323:qt-mt323.dll
 0002:000008a0       __imp_?setAccel@QButton@@UAEXABVQKeySequence@@@Z 100118a0     qt-mt323:qt-mt323.dll
 0002:000008a4       __imp_?setAlignment@QLabel@@UAEXH@Z 100118a4     qt-mt323:qt-mt323.dll
 0002:000008a8       __imp_?setAlignment@QLayoutItem@@UAEXH@Z 100118a8     qt-mt323:qt-mt323.dll
 0002:000008ac       __imp_?setAutoAdd@QLayout@@UAEX_N@Z 100118ac     qt-mt323:qt-mt323.dll
 0002:000008b0       __imp_?setAutoDefault@QPushButton@@UAEX_N@Z 100118b0     qt-mt323:qt-mt323.dll
 0002:000008b4       __imp_?setAutoRepeat@QButton@@UAEX_N@Z 100118b4     qt-mt323:qt-mt323.dll
 0002:000008b8       __imp_?setAutoResize@QLabel@@UAEX_N@Z 100118b8     qt-mt323:qt-mt323.dll
 0002:000008bc       __imp_?setBottomItem@QListBox@@UAEXH@Z 100118bc     qt-mt323:qt-mt323.dll
 0002:000008c0       __imp_?setBuddy@QLabel@@UAEXPAVQWidget@@@Z 100118c0     qt-mt323:qt-mt323.dll
 0002:000008c4       __imp_?setColumnMode@QListBox@@UAEXH@Z 100118c4     qt-mt323:qt-mt323.dll
 0002:000008c8       __imp_?setColumnMode@QListBox@@UAEXW4LayoutMode@1@@Z 100118c8     qt-mt323:qt-mt323.dll
 0002:000008cc       __imp_?setContentsPos@QScrollView@@UAEXHH@Z 100118cc     qt-mt323:qt-mt323.dll
 0002:000008d0       __imp_?setCornerWidget@QScrollView@@UAEXPAVQWidget@@@Z 100118d0     qt-mt323:qt-mt323.dll
 0002:000008d4       __imp_?setCurrentItem@QListBox@@UAEXH@Z 100118d4     qt-mt323:qt-mt323.dll
 0002:000008d8       __imp_?setCurrentItem@QListBox@@UAEXPAVQListBoxItem@@@Z 100118d8     qt-mt323:qt-mt323.dll
 0002:000008dc       __imp_?setDefault@QPushButton@@UAEX_N@Z 100118dc     qt-mt323:qt-mt323.dll
 0002:000008e0       __imp_?setDown@QButton@@UAEX_N@Z 100118e0     qt-mt323:qt-mt323.dll
 0002:000008e4       __imp_?setDragAutoScroll@QScrollView@@UAEX_N@Z 100118e4     qt-mt323:qt-mt323.dll
 0002:000008e8       __imp_?setEnabled@QScrollView@@UAEX_N@Z 100118e8     qt-mt323:qt-mt323.dll
 0002:000008ec       __imp_?setFont@QLabel@@UAEXABVQFont@@@Z 100118ec     qt-mt323:qt-mt323.dll
 0002:000008f0       __imp_?setFont@QListBox@@UAEXABVQFont@@@Z 100118f0     qt-mt323:qt-mt323.dll
 0002:000008f4       __imp_?setGeometry@QBoxLayout@@UAEXABVQRect@@@Z 100118f4     qt-mt323:qt-mt323.dll
 0002:000008f8       __imp_?setGeometry@QDialog@@UAEXABVQRect@@@Z 100118f8     qt-mt323:qt-mt323.dll
 0002:000008fc       __imp_?setGeometry@QDialog@@UAEXHHHH@Z 100118fc     qt-mt323:qt-mt323.dll
 0002:00000900       __imp_?setGeometry@QPushButton@@UAEXABVQRect@@@Z 10011900     qt-mt323:qt-mt323.dll
 0002:00000904       __imp_?setGeometry@QPushButton@@UAEXHHHH@Z 10011904     qt-mt323:qt-mt323.dll
 0002:00000908       __imp_?setGeometry@QSpacerItem@@UAEXABVQRect@@@Z 10011908     qt-mt323:qt-mt323.dll
 0002:0000090c       __imp_?setGroup@QButton@@EAEXPAVQButtonGroup@@@Z 1001190c     qt-mt323:qt-mt323.dll
 0002:00000910       __imp_?setHBarGeometry@QScrollView@@MAEXAAVQScrollBar@@HHHH@Z 10011910     qt-mt323:qt-mt323.dll
 0002:00000914       __imp_?setHScrollBarMode@QScrollView@@UAEXW4ScrollBarMode@1@@Z 10011914     qt-mt323:qt-mt323.dll
 0002:00000918       __imp_?setIsMenuButton@QPushButton@@UAEX_N@Z 10011918     qt-mt323:qt-mt323.dll
 0002:0000091c       __imp_?setMargin@QLayout@@UAEXH@Z 1001191c     qt-mt323:qt-mt323.dll
 0002:00000920       __imp_?setMargins@QScrollView@@MAEXHHHH@Z 10011920     qt-mt323:qt-mt323.dll
 0002:00000924       __imp_?setMenuBar@QLayout@@UAEXPAVQMenuBar@@@Z 10011924     qt-mt323:qt-mt323.dll
 0002:00000928       __imp_?setMovie@QLabel@@UAEXABVQMovie@@@Z 10011928     qt-mt323:qt-mt323.dll
 0002:0000092c       __imp_?setNum@QLabel@@UAEXH@Z 1001192c     qt-mt323:qt-mt323.dll
 0002:00000930       __imp_?setNum@QLabel@@UAEXN@Z 10011930     qt-mt323:qt-mt323.dll
 0002:00000934       __imp_?setOn@QPushButton@@UAEX_N@Z 10011934     qt-mt323:qt-mt323.dll
 0002:00000938       __imp_?setPicture@QLabel@@UAEXABVQPicture@@@Z 10011938     qt-mt323:qt-mt323.dll
 0002:0000093c       __imp_?setPixmap@QButton@@UAEXABVQPixmap@@@Z 1001193c     qt-mt323:qt-mt323.dll
 0002:00000940       __imp_?setPixmap@QLabel@@UAEXABVQPixmap@@@Z 10011940     qt-mt323:qt-mt323.dll
 0002:00000944       __imp_?setResizePolicy@QScrollView@@UAEXW4ResizePolicy@1@@Z 10011944     qt-mt323:qt-mt323.dll
 0002:00000948       __imp_?setRowMode@QListBox@@UAEXH@Z 10011948     qt-mt323:qt-mt323.dll
 0002:0000094c       __imp_?setRowMode@QListBox@@UAEXW4LayoutMode@1@@Z 1001194c     qt-mt323:qt-mt323.dll
 0002:00000950       __imp_?setSelected@QListBox@@UAEXPAVQListBoxItem@@_N@Z 10011950     qt-mt323:qt-mt323.dll
 0002:00000954       __imp_?setSelectionMode@QListBox@@UAEXW4SelectionMode@1@@Z 10011954     qt-mt323:qt-mt323.dll
 0002:00000958       __imp_?setSpacing@QLayout@@UAEXH@Z 10011958     qt-mt323:qt-mt323.dll
 0002:0000095c       __imp_?setState@QButton@@MAEXW4ToggleState@1@@Z 1001195c     qt-mt323:qt-mt323.dll
 0002:00000960       __imp_?setText@QButton@@UAEXABVQString@@@Z 10011960     qt-mt323:qt-mt323.dll
 0002:00000964       __imp_?setText@QLabel@@UAEXABVQString@@@Z 10011964     qt-mt323:qt-mt323.dll
 0002:00000968       __imp_?setToggleType@QButton@@MAEXW4ToggleType@1@@Z 10011968     qt-mt323:qt-mt323.dll
 0002:0000096c       __imp_?setTopItem@QListBox@@UAEXH@Z 1001196c     qt-mt323:qt-mt323.dll
 0002:00000970       __imp_?setVBarGeometry@QScrollView@@MAEXAAVQScrollBar@@HHHH@Z 10011970     qt-mt323:qt-mt323.dll
 0002:00000974       __imp_?setVScrollBarMode@QScrollView@@UAEXW4ScrollBarMode@1@@Z 10011974     qt-mt323:qt-mt323.dll
 0002:00000978       __imp_?setVariableHeight@QListBox@@UAEX_N@Z 10011978     qt-mt323:qt-mt323.dll
 0002:0000097c       __imp_?setVariableWidth@QListBox@@UAEX_N@Z 1001197c     qt-mt323:qt-mt323.dll
 0002:00000980       __imp_?show@QDialog@@UAEXXZ 10011980     qt-mt323:qt-mt323.dll
 0002:00000984       __imp_?show@QScrollView@@UAEXXZ 10011984     qt-mt323:qt-mt323.dll
 0002:00000988       __imp_?showEvent@QListBox@@MAEXPAVQShowEvent@@@Z 10011988     qt-mt323:qt-mt323.dll
 0002:0000098c       __imp_?sizeHint@QBoxLayout@@UBE?AVQSize@@XZ 1001198c     qt-mt323:qt-mt323.dll
 0002:00000990       __imp_?sizeHint@QDialog@@UBE?AVQSize@@XZ 10011990     qt-mt323:qt-mt323.dll
 0002:00000994       __imp_?sizeHint@QLabel@@UBE?AVQSize@@XZ 10011994     qt-mt323:qt-mt323.dll
 0002:00000998       __imp_?sizeHint@QListBox@@UBE?AVQSize@@XZ 10011998     qt-mt323:qt-mt323.dll
 0002:0000099c       __imp_?sizeHint@QPushButton@@UBE?AVQSize@@XZ 1001199c     qt-mt323:qt-mt323.dll
 0002:000009a0       __imp_?sizeHint@QSpacerItem@@UBE?AVQSize@@XZ 100119a0     qt-mt323:qt-mt323.dll
 0002:000009a4       __imp_?spacerItem@QLayoutItem@@UAEPAVQSpacerItem@@XZ 100119a4     qt-mt323:qt-mt323.dll
 0002:000009a8       __imp_?spacerItem@QSpacerItem@@UAEPAV1@XZ 100119a8     qt-mt323:qt-mt323.dll
 0002:000009ac       __imp_?styleChange@QFrame@@MAEXAAVQStyle@@@Z 100119ac     qt-mt323:qt-mt323.dll
 0002:000009b0       __imp_?styleChange@QScrollView@@UAEXAAVQStyle@@@Z 100119b0     qt-mt323:qt-mt323.dll
 0002:000009b4       __imp_?updateMask@QPushButton@@MAEXXZ 100119b4     qt-mt323:qt-mt323.dll
 0002:000009b8       __imp_?viewportContextMenuEvent@QScrollView@@MAEXPAVQContextMenuEvent@@@Z 100119b8     qt-mt323:qt-mt323.dll
 0002:000009bc       __imp_?viewportDragEnterEvent@QScrollView@@MAEXPAVQDragEnterEvent@@@Z 100119bc     qt-mt323:qt-mt323.dll
 0002:000009c0       __imp_?viewportDragLeaveEvent@QScrollView@@MAEXPAVQDragLeaveEvent@@@Z 100119c0     qt-mt323:qt-mt323.dll
 0002:000009c4       __imp_?viewportDragMoveEvent@QScrollView@@MAEXPAVQDragMoveEvent@@@Z 100119c4     qt-mt323:qt-mt323.dll
 0002:000009c8       __imp_?viewportDropEvent@QScrollView@@MAEXPAVQDropEvent@@@Z 100119c8     qt-mt323:qt-mt323.dll
 0002:000009cc       __imp_?viewportMouseDoubleClickEvent@QScrollView@@MAEXPAVQMouseEvent@@@Z 100119cc     qt-mt323:qt-mt323.dll
 0002:000009d0       __imp_?viewportMouseMoveEvent@QScrollView@@MAEXPAVQMouseEvent@@@Z 100119d0     qt-mt323:qt-mt323.dll
 0002:000009d4       __imp_?viewportMousePressEvent@QScrollView@@MAEXPAVQMouseEvent@@@Z 100119d4     qt-mt323:qt-mt323.dll
 0002:000009d8       __imp_?viewportMouseReleaseEvent@QScrollView@@MAEXPAVQMouseEvent@@@Z 100119d8     qt-mt323:qt-mt323.dll
 0002:000009dc       __imp_?viewportPaintEvent@QListBox@@UAEXPAVQPaintEvent@@@Z 100119dc     qt-mt323:qt-mt323.dll
 0002:000009e0       __imp_?viewportResizeEvent@QScrollView@@MAEXPAVQResizeEvent@@@Z 100119e0     qt-mt323:qt-mt323.dll
 0002:000009e4       __imp_?viewportWheelEvent@QScrollView@@MAEXPAVQWheelEvent@@@Z 100119e4     qt-mt323:qt-mt323.dll
 0002:000009e8       __imp_?wheelEvent@QScrollView@@MAEXPAVQWheelEvent@@@Z 100119e8     qt-mt323:qt-mt323.dll
 0002:000009ec       __imp_?widget@QLayoutItem@@UAEPAVQWidget@@XZ 100119ec     qt-mt323:qt-mt323.dll
 0002:000009f0       __imp_?windowActivationChange@QListBox@@MAEX_N@Z 100119f0     qt-mt323:qt-mt323.dll
 0002:000009f4       __imp_?setSortIndicator@QHeader@@QAEXH_N@Z 100119f4     qt-mt323:qt-mt323.dll
 0002:000009f8       __imp_??1QTable@@UAE@XZ    100119f8     qt-mt323:qt-mt323.dll
 0002:000009fc       __imp_?horizontalHeader@QTable@@QBEPAVQHeader@@XZ 100119fc     qt-mt323:qt-mt323.dll
 0002:00000a00       __imp_?sortColumn@QTable@@UAEXH_N0@Z 10011a00     qt-mt323:qt-mt323.dll
 0002:00000a04       __imp_?setLeftMargin@QTable@@UAEXH@Z 10011a04     qt-mt323:qt-mt323.dll
 0002:00000a08       __imp_?activateNextCell@QTable@@MAEXXZ 10011a08     qt-mt323:qt-mt323.dll
 0002:00000a0c       __imp_?addSelection@QTable@@UAEHABVQTableSelection@@@Z 10011a0c     qt-mt323:qt-mt323.dll
 0002:00000a10       __imp_?adjustColumn@QTable@@UAEXH@Z 10011a10     qt-mt323:qt-mt323.dll
 0002:00000a14       __imp_?adjustRow@QTable@@UAEXH@Z 10011a14     qt-mt323:qt-mt323.dll
 0002:00000a18       __imp_?beginEdit@QTable@@MAEPAVQWidget@@HH_N@Z 10011a18     qt-mt323:qt-mt323.dll
 0002:00000a1c       __imp_?cellGeometry@QTable@@UBE?AVQRect@@HH@Z 10011a1c     qt-mt323:qt-mt323.dll
 0002:00000a20       __imp_?cellRect@QTable@@UBE?AVQRect@@HH@Z 10011a20     qt-mt323:qt-mt323.dll
 0002:00000a24       __imp_?cellWidget@QTable@@UBEPAVQWidget@@HH@Z 10011a24     qt-mt323:qt-mt323.dll
 0002:00000a28       __imp_?clearCell@QTable@@UAEXHH@Z 10011a28     qt-mt323:qt-mt323.dll
 0002:00000a2c       __imp_?clearCellWidget@QTable@@UAEXHH@Z 10011a2c     qt-mt323:qt-mt323.dll
 0002:00000a30       __imp_?columnAt@QTable@@UBEHH@Z 10011a30     qt-mt323:qt-mt323.dll
 0002:00000a34       __imp_?columnClicked@QTable@@MAEXH@Z 10011a34     qt-mt323:qt-mt323.dll
 0002:00000a38       __imp_?columnIndexChanged@QTable@@MAEXHHH@Z 10011a38     qt-mt323:qt-mt323.dll
 0002:00000a3c       __imp_?columnPos@QTable@@UBEHH@Z 10011a3c     qt-mt323:qt-mt323.dll
 0002:00000a40       __imp_?columnWidth@QTable@@UBEHH@Z 10011a40     qt-mt323:qt-mt323.dll
 0002:00000a44       __imp_?columnWidthChanged@QTable@@MAEXH@Z 10011a44     qt-mt323:qt-mt323.dll
 0002:00000a48       __imp_?contentsContextMenuEvent@QTable@@MAEXPAVQContextMenuEvent@@@Z 10011a48     qt-mt323:qt-mt323.dll
 0002:00000a4c       __imp_?contentsDragEnterEvent@QTable@@MAEXPAVQDragEnterEvent@@@Z 10011a4c     qt-mt323:qt-mt323.dll
 0002:00000a50       __imp_?contentsDragLeaveEvent@QTable@@MAEXPAVQDragLeaveEvent@@@Z 10011a50     qt-mt323:qt-mt323.dll
 0002:00000a54       __imp_?contentsDragMoveEvent@QTable@@MAEXPAVQDragMoveEvent@@@Z 10011a54     qt-mt323:qt-mt323.dll
 0002:00000a58       __imp_?contentsDropEvent@QTable@@MAEXPAVQDropEvent@@@Z 10011a58     qt-mt323:qt-mt323.dll
 0002:00000a5c       __imp_?contentsMouseDoubleClickEvent@QTable@@MAEXPAVQMouseEvent@@@Z 10011a5c     qt-mt323:qt-mt323.dll
 0002:00000a60       __imp_?contentsMouseMoveEvent@QTable@@MAEXPAVQMouseEvent@@@Z 10011a60     qt-mt323:qt-mt323.dll
 0002:00000a64       __imp_?contentsMousePressEvent@QTable@@MAEXPAVQMouseEvent@@@Z 10011a64     qt-mt323:qt-mt323.dll
 0002:00000a68       __imp_?contentsMouseReleaseEvent@QTable@@MAEXPAVQMouseEvent@@@Z 10011a68     qt-mt323:qt-mt323.dll
 0002:00000a6c       __imp_?createEditor@QTable@@MBEPAVQWidget@@HH_N@Z 10011a6c     qt-mt323:qt-mt323.dll
 0002:00000a70       __imp_?currentSelection@QTable@@UBEHXZ 10011a70     qt-mt323:qt-mt323.dll
 0002:00000a74       __imp_?dragObject@QTable@@MAEPAVQDragObject@@XZ 10011a74     qt-mt323:qt-mt323.dll
 0002:00000a78       __imp_?drawContents@QTable@@EAEXPAVQPainter@@@Z 10011a78     qt-mt323:qt-mt323.dll
 0002:00000a7c       __imp_?drawContents@QTable@@MAEXPAVQPainter@@HHHH@Z 10011a7c     qt-mt323:qt-mt323.dll
 0002:00000a80       __imp_?editCell@QTable@@UAEXHH_N@Z 10011a80     qt-mt323:qt-mt323.dll
 0002:00000a84       __imp_?endEdit@QTable@@MAEXHH_N0@Z 10011a84     qt-mt323:qt-mt323.dll
 0002:00000a88       __imp_?eventFilter@QTable@@UAE_NPAVQObject@@PAVQEvent@@@Z 10011a88     qt-mt323:qt-mt323.dll
 0002:00000a8c       __imp_?focusInEvent@QTable@@MAEXPAVQFocusEvent@@@Z 10011a8c     qt-mt323:qt-mt323.dll
 0002:00000a90       __imp_?focusOutEvent@QTable@@MAEXPAVQFocusEvent@@@Z 10011a90     qt-mt323:qt-mt323.dll
 0002:00000a94       __imp_?hideColumn@QTable@@UAEXH@Z 10011a94     qt-mt323:qt-mt323.dll
 0002:00000a98       __imp_?hideRow@QTable@@UAEXH@Z 10011a98     qt-mt323:qt-mt323.dll
 0002:00000a9c       __imp_?insertColumns@QTable@@UAEXHH@Z 10011a9c     qt-mt323:qt-mt323.dll
 0002:00000aa0       __imp_?insertRows@QTable@@UAEXHH@Z 10011aa0     qt-mt323:qt-mt323.dll
 0002:00000aa4       __imp_?insertWidget@QTable@@MAEXHHPAVQWidget@@@Z 10011aa4     qt-mt323:qt-mt323.dll
 0002:00000aa8       __imp_?item@QTable@@UBEPAVQTableItem@@HH@Z 10011aa8     qt-mt323:qt-mt323.dll
 0002:00000aac       __imp_?keyPressEvent@QTable@@MAEXPAVQKeyEvent@@@Z 10011aac     qt-mt323:qt-mt323.dll
 0002:00000ab0       __imp_?minimumSizeHint@QScrollView@@UBE?AVQSize@@XZ 10011ab0     qt-mt323:qt-mt323.dll
 0002:00000ab4       __imp_?mouseDoubleClickEvent@QScrollView@@MAEXPAVQMouseEvent@@@Z 10011ab4     qt-mt323:qt-mt323.dll
 0002:00000ab8       __imp_?mouseMoveEvent@QScrollView@@MAEXPAVQMouseEvent@@@Z 10011ab8     qt-mt323:qt-mt323.dll
 0002:00000abc       __imp_?mousePressEvent@QScrollView@@MAEXPAVQMouseEvent@@@Z 10011abc     qt-mt323:qt-mt323.dll
 0002:00000ac0       __imp_?mouseReleaseEvent@QScrollView@@MAEXPAVQMouseEvent@@@Z 10011ac0     qt-mt323:qt-mt323.dll
 0002:00000ac4       __imp_?numCols@QTable@@UBEHXZ 10011ac4     qt-mt323:qt-mt323.dll
 0002:00000ac8       __imp_?numRows@QTable@@UBEHXZ 10011ac8     qt-mt323:qt-mt323.dll
 0002:00000acc       __imp_?paintCell@QTable@@UAEXPAVQPainter@@HHABVQRect@@_N@Z 10011acc     qt-mt323:qt-mt323.dll
 0002:00000ad0       __imp_?paintCell@QTable@@UAEXPAVQPainter@@HHABVQRect@@_NABVQColorGroup@@@Z 10011ad0     qt-mt323:qt-mt323.dll
 0002:00000ad4       __imp_?paintEmptyArea@QTable@@MAEXPAVQPainter@@HHHH@Z 10011ad4     qt-mt323:qt-mt323.dll
 0002:00000ad8       __imp_?paintEvent@QTable@@MAEXPAVQPaintEvent@@@Z 10011ad8     qt-mt323:qt-mt323.dll
 0002:00000adc       __imp_?paintFocus@QTable@@UAEXPAVQPainter@@ABVQRect@@@Z 10011adc     qt-mt323:qt-mt323.dll
 0002:00000ae0       __imp_?pixmap@QTable@@UBE?AVQPixmap@@HH@Z 10011ae0     qt-mt323:qt-mt323.dll
 0002:00000ae4       __imp_?removeColumn@QTable@@UAEXH@Z 10011ae4     qt-mt323:qt-mt323.dll
 0002:00000ae8       __imp_?removeColumns@QTable@@UAEXABV?$QMemArray@H@@@Z 10011ae8     qt-mt323:qt-mt323.dll
 0002:00000aec       __imp_?removeRow@QTable@@UAEXH@Z 10011aec     qt-mt323:qt-mt323.dll
 0002:00000af0       __imp_?removeRows@QTable@@UAEXABV?$QMemArray@H@@@Z 10011af0     qt-mt323:qt-mt323.dll
 0002:00000af4       __imp_?removeSelection@QTable@@UAEXABVQTableSelection@@@Z 10011af4     qt-mt323:qt-mt323.dll
 0002:00000af8       __imp_?removeSelection@QTable@@UAEXH@Z 10011af8     qt-mt323:qt-mt323.dll
 0002:00000afc       __imp_?resizeData@QTable@@MAEXH@Z 10011afc     qt-mt323:qt-mt323.dll
 0002:00000b00       __imp_?resizeEvent@QScrollView@@MAEXPAVQResizeEvent@@@Z 10011b00     qt-mt323:qt-mt323.dll
 0002:00000b04       __imp_?rowAt@QTable@@UBEHH@Z 10011b04     qt-mt323:qt-mt323.dll
 0002:00000b08       __imp_?rowHeight@QTable@@UBEHH@Z 10011b08     qt-mt323:qt-mt323.dll
 0002:00000b0c       __imp_?rowHeightChanged@QTable@@MAEXH@Z 10011b0c     qt-mt323:qt-mt323.dll
 0002:00000b10       __imp_?rowIndexChanged@QTable@@MAEXHHH@Z 10011b10     qt-mt323:qt-mt323.dll
 0002:00000b14       __imp_?rowPos@QTable@@UBEHH@Z 10011b14     qt-mt323:qt-mt323.dll
 0002:00000b18       __imp_?setCellContentFromEditor@QTable@@MAEXHH@Z 10011b18     qt-mt323:qt-mt323.dll
 0002:00000b1c       __imp_?setCellWidget@QTable@@UAEXHHPAVQWidget@@@Z 10011b1c     qt-mt323:qt-mt323.dll
 0002:00000b20       __imp_?setColumnMovingEnabled@QTable@@UAEX_N@Z 10011b20     qt-mt323:qt-mt323.dll
 0002:00000b24       __imp_?setColumnReadOnly@QTable@@UAEXH_N@Z 10011b24     qt-mt323:qt-mt323.dll
 0002:00000b28       __imp_?setColumnStretchable@QTable@@UAEXH_N@Z 10011b28     qt-mt323:qt-mt323.dll
 0002:00000b2c       __imp_?setColumnWidth@QTable@@UAEXHH@Z 10011b2c     qt-mt323:qt-mt323.dll
 0002:00000b30       __imp_?setCurrentCell@QTable@@UAEXHH@Z 10011b30     qt-mt323:qt-mt323.dll
 0002:00000b34       __imp_?setDragEnabled@QTable@@UAEX_N@Z 10011b34     qt-mt323:qt-mt323.dll
 0002:00000b38       __imp_?setEnabled@QTable@@UAEX_N@Z 10011b38     qt-mt323:qt-mt323.dll
 0002:00000b3c       __imp_?setFocusStyle@QTable@@UAEXW4FocusStyle@1@@Z 10011b3c     qt-mt323:qt-mt323.dll
 0002:00000b40       __imp_?setItem@QTable@@UAEXHHPAVQTableItem@@@Z 10011b40     qt-mt323:qt-mt323.dll
 0002:00000b44       __imp_?setNumCols@QTable@@UAEXH@Z 10011b44     qt-mt323:qt-mt323.dll
 0002:00000b48       __imp_?setNumRows@QTable@@UAEXH@Z 10011b48     qt-mt323:qt-mt323.dll
 0002:00000b4c       __imp_?setPixmap@QTable@@UAEXHHABVQPixmap@@@Z 10011b4c     qt-mt323:qt-mt323.dll
 0002:00000b50       __imp_?setReadOnly@QTable@@UAEX_N@Z 10011b50     qt-mt323:qt-mt323.dll
 0002:00000b54       __imp_?setRowHeight@QTable@@UAEXHH@Z 10011b54     qt-mt323:qt-mt323.dll
 0002:00000b58       __imp_?setRowMovingEnabled@QTable@@UAEX_N@Z 10011b58     qt-mt323:qt-mt323.dll
 0002:00000b5c       __imp_?setRowReadOnly@QTable@@UAEXH_N@Z 10011b5c     qt-mt323:qt-mt323.dll
 0002:00000b60       __imp_?setRowStretchable@QTable@@UAEXH_N@Z 10011b60     qt-mt323:qt-mt323.dll
 0002:00000b64       __imp_?setSelectionMode@QTable@@UAEXW4SelectionMode@1@@Z 10011b64     qt-mt323:qt-mt323.dll
 0002:00000b68       __imp_?setShowGrid@QTable@@UAEX_N@Z 10011b68     qt-mt323:qt-mt323.dll
 0002:00000b6c       __imp_?setSorting@QTable@@UAEX_N@Z 10011b6c     qt-mt323:qt-mt323.dll
 0002:00000b70       __imp_?setText@QTable@@UAEXHHABVQString@@@Z 10011b70     qt-mt323:qt-mt323.dll
 0002:00000b74       __imp_?setTopMargin@QTable@@UAEXH@Z 10011b74     qt-mt323:qt-mt323.dll
 0002:00000b78       __imp_?showColumn@QTable@@UAEXH@Z 10011b78     qt-mt323:qt-mt323.dll
 0002:00000b7c       __imp_?showEvent@QTable@@MAEXPAVQShowEvent@@@Z 10011b7c     qt-mt323:qt-mt323.dll
 0002:00000b80       __imp_?showRow@QTable@@UAEXH@Z 10011b80     qt-mt323:qt-mt323.dll
 0002:00000b84       __imp_?sizeHint@QTable@@UBE?AVQSize@@XZ 10011b84     qt-mt323:qt-mt323.dll
 0002:00000b88       __imp_?startDrag@QTable@@MAEXXZ 10011b88     qt-mt323:qt-mt323.dll
 0002:00000b8c       __imp_?swapCells@QTable@@UAEXHHHH@Z 10011b8c     qt-mt323:qt-mt323.dll
 0002:00000b90       __imp_?swapColumns@QTable@@UAEXHH_N@Z 10011b90     qt-mt323:qt-mt323.dll
 0002:00000b94       __imp_?swapRows@QTable@@UAEXHH_N@Z 10011b94     qt-mt323:qt-mt323.dll
 0002:00000b98       __imp_?takeItem@QTable@@UAEXPAVQTableItem@@@Z 10011b98     qt-mt323:qt-mt323.dll
 0002:00000b9c       __imp_?text@QTable@@UBE?AVQString@@HH@Z 10011b9c     qt-mt323:qt-mt323.dll
 0002:00000ba0       __imp_?viewportPaintEvent@QScrollView@@MAEXPAVQPaintEvent@@@Z 10011ba0     qt-mt323:qt-mt323.dll
 0002:00000ba4       __imp_?viewportResizeEvent@QTable@@MAEXPAVQResizeEvent@@@Z 10011ba4     qt-mt323:qt-mt323.dll
 0002:00000ba8       __imp_?windowActivationChange@QTable@@MAEX_N@Z 10011ba8     qt-mt323:qt-mt323.dll
 0002:00000bac       __imp_?qstrcmp@@YAHPBD0@Z  10011bac     qt-mt323:qt-mt323.dll
 0002:00000bb0       __imp_?fromLatin1@QString@@SA?AV1@PBDH@Z 10011bb0     qt-mt323:qt-mt323.dll
 0002:00000bb4       __imp_?fromUtf8@QString@@SA?AV1@PBDH@Z 10011bb4     qt-mt323:qt-mt323.dll
 0002:00000bb8       __imp_?qt_cast@QDialog@@UAEPAXPBD@Z 10011bb8     qt-mt323:qt-mt323.dll
 0002:00000bbc       __imp_?qt_invoke@QDialog@@UAE_NHPAUQUObject@@@Z 10011bbc     qt-mt323:qt-mt323.dll
 0002:00000bc0       __imp_?qt_emit@QDialog@@UAE_NHPAUQUObject@@@Z 10011bc0     qt-mt323:qt-mt323.dll
 0002:00000bc4       __imp_?qt_property@QDialog@@UAE_NHHPAVQVariant@@@Z 10011bc4     qt-mt323:qt-mt323.dll
 0002:00000bc8       __imp_?staticMetaObject@QDialog@@SAPAVQMetaObject@@XZ 10011bc8     qt-mt323:qt-mt323.dll
 0002:00000bcc       __imp_?new_metaobject@QMetaObject@@SAPAV1@PBDPAV1@QBUQMetaData@@H2HQBVQMetaProperty@@HQBUQMetaEnum@@HQBUQClassInfo@@H@Z 10011bcc     qt-mt323:qt-mt323.dll
 0002:00000bd0       __imp_??0QMetaObjectCleanUp@@QAE@PBDP6APAVQMetaObject@@XZ@Z 10011bd0     qt-mt323:qt-mt323.dll
 0002:00000bd4       __imp_??1QMetaObjectCleanUp@@QAE@XZ 10011bd4     qt-mt323:qt-mt323.dll
 0002:00000bd8       __imp_?setMetaObject@QMetaObjectCleanUp@@QAEXAAPAVQMetaObject@@@Z 10011bd8     qt-mt323:qt-mt323.dll
 0002:00000bdc       __imp_?translate@QApplication@@QBE?AVQString@@PBD00W4Encoding@1@@Z 10011bdc     qt-mt323:qt-mt323.dll
 0002:00000be0       __imp_?qApp@@3PAVQApplication@@A 10011be0     qt-mt323:qt-mt323.dll
 0002:00000be4       __imp_??0QPixmap@@QAE@XZ   10011be4     qt-mt323:qt-mt323.dll
 0002:00000be8       __imp_?setMaximumSize@QWidget@@QAEXABVQSize@@@Z 10011be8     qt-mt323:qt-mt323.dll
 0002:00000bec       __imp_?resize@QWidget@@QAEXABVQSize@@@Z 10011bec     qt-mt323:qt-mt323.dll
 0002:00000bf0       __imp_?setFrameShape@QFrame@@QAEXW4Shape@1@@Z 10011bf0     qt-mt323:qt-mt323.dll
 0002:00000bf4       __imp_?setFrameShadow@QFrame@@QAEXW4Shadow@1@@Z 10011bf4     qt-mt323:qt-mt323.dll
 0002:00000bf8       __imp_??0QTabWidget@@QAE@PAVQWidget@@PBDI@Z 10011bf8     qt-mt323:qt-mt323.dll
 0002:00000bfc       __imp_??1QTabWidget@@UAE@XZ 10011bfc     qt-mt323:qt-mt323.dll
 0002:00000c00       __imp_?changeTab@QTabWidget@@QAEXPAVQWidget@@ABVQString@@@Z 10011c00     qt-mt323:qt-mt323.dll
 0002:00000c04       __imp_?addTab@QTabWidget@@UAEXPAVQWidget@@ABVQIconSet@@ABVQString@@@Z 10011c04     qt-mt323:qt-mt323.dll
 0002:00000c08       __imp_?addTab@QTabWidget@@UAEXPAVQWidget@@ABVQString@@@Z 10011c08     qt-mt323:qt-mt323.dll
 0002:00000c0c       __imp_?addTab@QTabWidget@@UAEXPAVQWidget@@PAVQTab@@@Z 10011c0c     qt-mt323:qt-mt323.dll
 0002:00000c10       __imp_?className@QTabWidget@@UBEPBDXZ 10011c10     qt-mt323:qt-mt323.dll
 0002:00000c14       __imp_?eventFilter@QTabWidget@@MAE_NPAVQObject@@PAVQEvent@@@Z 10011c14     qt-mt323:qt-mt323.dll
 0002:00000c18       __imp_?insertTab@QTabWidget@@UAEXPAVQWidget@@ABVQIconSet@@ABVQString@@H@Z 10011c18     qt-mt323:qt-mt323.dll
 0002:00000c1c       __imp_?insertTab@QTabWidget@@UAEXPAVQWidget@@ABVQString@@H@Z 10011c1c     qt-mt323:qt-mt323.dll
 0002:00000c20       __imp_?insertTab@QTabWidget@@UAEXPAVQWidget@@PAVQTab@@H@Z 10011c20     qt-mt323:qt-mt323.dll
 0002:00000c24       __imp_?metaObject@QTabWidget@@UBEPAVQMetaObject@@XZ 10011c24     qt-mt323:qt-mt323.dll
 0002:00000c28       __imp_?minimumSizeHint@QTabWidget@@UBE?AVQSize@@XZ 10011c28     qt-mt323:qt-mt323.dll
 0002:00000c2c       __imp_?qt_cast@QTabWidget@@UAEPAXPBD@Z 10011c2c     qt-mt323:qt-mt323.dll
 0002:00000c30       __imp_?qt_emit@QTabWidget@@UAE_NHPAUQUObject@@@Z 10011c30     qt-mt323:qt-mt323.dll
 0002:00000c34       __imp_?qt_invoke@QTabWidget@@UAE_NHPAUQUObject@@@Z 10011c34     qt-mt323:qt-mt323.dll
 0002:00000c38       __imp_?qt_property@QTabWidget@@UAE_NHHPAVQVariant@@@Z 10011c38     qt-mt323:qt-mt323.dll
 0002:00000c3c       __imp_?removePage@QTabWidget@@UAEXPAVQWidget@@@Z 10011c3c     qt-mt323:qt-mt323.dll
 0002:00000c40       __imp_?resizeEvent@QTabWidget@@MAEXPAVQResizeEvent@@@Z 10011c40     qt-mt323:qt-mt323.dll
 0002:00000c44       __imp_?showEvent@QTabWidget@@MAEXPAVQShowEvent@@@Z 10011c44     qt-mt323:qt-mt323.dll
 0002:00000c48       __imp_?showPage@QTabWidget@@UAEXPAVQWidget@@@Z 10011c48     qt-mt323:qt-mt323.dll
 0002:00000c4c       __imp_?sizeHint@QTabWidget@@UBE?AVQSize@@XZ 10011c4c     qt-mt323:qt-mt323.dll
 0002:00000c50       __imp_?styleChange@QTabWidget@@MAEXAAVQStyle@@@Z 10011c50     qt-mt323:qt-mt323.dll
 0002:00000c54       __imp_?updateMask@QTabWidget@@MAEXXZ 10011c54     qt-mt323:qt-mt323.dll
 0002:00000c58       __imp_?receivers@QObject@@IBEPAVQConnectionList@@H@Z 10011c58     qt-mt323:qt-mt323.dll
 0002:00000c5c       __imp_?activate_signal@QObject@@IAEXPAVQConnectionList@@PAUQUObject@@@Z 10011c5c     qt-mt323:qt-mt323.dll
 0002:00000c60       __imp_?staticMetaObject@QWidget@@SAPAVQMetaObject@@XZ 10011c60     qt-mt323:qt-mt323.dll
 0002:00000c64       __imp_??0QUObject@@QAE@XZ  10011c64     qt-mt323:qt-mt323.dll
 0002:00000c68       __imp_??1QUObject@@QAE@XZ  10011c68     qt-mt323:qt-mt323.dll
 0002:00000c6c       __imp_?set@QUType_QString@@QAEXPAUQUObject@@ABVQString@@@Z 10011c6c     qt-mt323:qt-mt323.dll
 0002:00000c70       __imp_?static_QUType_int@@3UQUType_int@@A 10011c70     qt-mt323:qt-mt323.dll
 0002:00000c74       __imp_?static_QUType_QString@@3UQUType_QString@@A 10011c74     qt-mt323:qt-mt323.dll
 0002:00000c78       __imp_?static_QUType_varptr@@3UQUType_varptr@@A 10011c78     qt-mt323:qt-mt323.dll
 0002:00000c7c       __imp_?set@QUType_bool@@QAEXPAUQUObject@@_N@Z 10011c7c     qt-mt323:qt-mt323.dll
 0002:00000c80       __imp_?static_QUType_bool@@3UQUType_bool@@A 10011c80     qt-mt323:qt-mt323.dll
 0002:00000c84       __imp_?static_QUType_ptr@@3UQUType_ptr@@A 10011c84     qt-mt323:qt-mt323.dll
 0002:00000c88       __imp_??1QIconSet@@UAE@XZ  10011c88     qt-mt323:qt-mt323.dll
 0002:00000c8c       __imp_??0QIconSet@@QAE@ABVQPixmap@@W4Size@0@@Z 10011c8c     qt-mt323:qt-mt323.dll
 0002:00000c90       __imp_??1QPixmap@@UAE@XZ   10011c90     qt-mt323:qt-mt323.dll
 0002:00000c94       __imp_??0QPixmap@@QAE@QAPBD@Z 10011c94     qt-mt323:qt-mt323.dll
 0002:00000c98       __imp_??0QKeySequence@@QAE@H@Z 10011c98     qt-mt323:qt-mt323.dll
 0002:00000c9c       __imp_?information@QMessageBox@@SAHPAVQWidget@@ABVQString@@1111HH@Z 10011c9c     qt-mt323:qt-mt323.dll
 0002:00000ca0       __imp_?closeEvent@QWidget@@MAEXPAVQCloseEvent@@@Z 10011ca0     qt-mt323:qt-mt323.dll
 0002:00000ca4       __imp_?rect@QWidget@@QBE?AVQRect@@XZ 10011ca4     qt-mt323:qt-mt323.dll
 0002:00000ca8       __imp_?setName@QWidget@@UAEXPBD@Z 10011ca8     qt-mt323:qt-mt323.dll
 0002:00000cac       __imp_??1QWidget@@UAE@XZ   10011cac     qt-mt323:qt-mt323.dll
 0002:00000cb0       __imp_??0QWidget@@QAE@PAV0@PBDI@Z 10011cb0     qt-mt323:qt-mt323.dll
 0002:00000cb4       __imp_?connect@QObject@@SA_NPBV1@PBD01@Z 10011cb4     qt-mt323:qt-mt323.dll
 0002:00000cb8       __imp_?clear@QGList@@MAEXXZ 10011cb8     qt-mt323:qt-mt323.dll
 0002:00000cbc       __imp_?append@QGList@@IAEXPAX@Z 10011cbc     qt-mt323:qt-mt323.dll
 0002:00000cc0       __imp_??1QGList@@MAE@XZ    10011cc0     qt-mt323:qt-mt323.dll
 0002:00000cc4       __imp_??0QGList@@IAE@XZ    10011cc4     qt-mt323:qt-mt323.dll
 0002:00000cc8       __imp_??H@YA?BVQString@@PBDABV0@@Z 10011cc8     qt-mt323:qt-mt323.dll
 0002:00000ccc       __imp_??H@YA?BVQString@@ABV0@PBD@Z 10011ccc     qt-mt323:qt-mt323.dll
 0002:00000cd0       __imp_??H@YA?BVQString@@ABV0@0@Z 10011cd0     qt-mt323:qt-mt323.dll
 0002:00000cd4       __imp_??8@YA_NABVQString@@PBD@Z 10011cd4     qt-mt323:qt-mt323.dll
 0002:00000cd8       __imp_?endsWith@QString@@QBE_NABV1@@Z 10011cd8     qt-mt323:qt-mt323.dll
 0002:00000cdc       __imp_?ascii@QString@@QBEPBDXZ 10011cdc     qt-mt323:qt-mt323.dll
 0002:00000ce0       __imp_??YQString@@QAEAAV0@ABV0@@Z 10011ce0     qt-mt323:qt-mt323.dll
 0002:00000ce4       __imp_??YQString@@QAEAAV0@PBD@Z 10011ce4     qt-mt323:qt-mt323.dll
 0002:00000ce8       __imp_??0QTable@@QAE@PAVQWidget@@PBD@Z 10011ce8     qt-mt323:qt-mt323.dll
 0002:00000cec       __imp_?numSelections@QTable@@QBEHXZ 10011cec     qt-mt323:qt-mt323.dll
 0002:00000cf0       __imp_?selection@QTable@@QBE?AVQTableSelection@@H@Z 10011cf0     qt-mt323:qt-mt323.dll
 0002:00000cf4       __imp_??0QTable@@QAE@ABV0@@Z 10011cf4     qt-mt323:qt-mt323.dll
 0002:00000cf8       __imp_??4QTable@@QAEAAV0@ABV0@@Z 10011cf8     qt-mt323:qt-mt323.dll
 0002:00000cfc       __imp_?warning@QMessageBox@@SAHPAVQWidget@@ABVQString@@1111HH@Z 10011cfc     qt-mt323:qt-mt323.dll
 0002:00000d00       __imp_?activate_signal@QObject@@IAEXH@Z 10011d00     qt-mt323:qt-mt323.dll
 0002:00000d04       __imp_?activate_signal_bool@QObject@@IAEXH_N@Z 10011d04     qt-mt323:qt-mt323.dll
 0002:00000d08       __imp_?qt_cast@QTable@@UAEPAXPBD@Z 10011d08     qt-mt323:qt-mt323.dll
 0002:00000d0c       __imp_?qt_invoke@QTable@@UAE_NHPAUQUObject@@@Z 10011d0c     qt-mt323:qt-mt323.dll
 0002:00000d10       __imp_?qt_emit@QTable@@UAE_NHPAUQUObject@@@Z 10011d10     qt-mt323:qt-mt323.dll
 0002:00000d14       __imp_?qt_property@QTable@@UAE_NHHPAVQVariant@@@Z 10011d14     qt-mt323:qt-mt323.dll
 0002:00000d18       __imp_?staticMetaObject@QTable@@SAPAVQMetaObject@@XZ 10011d18     qt-mt323:qt-mt323.dll
 0002:00000d1c       __imp_?lower@QString@@QBE?AV1@XZ 10011d1c     qt-mt323:qt-mt323.dll
 0002:00000d20       __imp_?arg@QString@@QBE?AV1@ABV1@H@Z 10011d20     qt-mt323:qt-mt323.dll
 0002:00000d24       __imp_??4QString@@QAEAAV0@PBD@Z 10011d24     qt-mt323:qt-mt323.dll
 0002:00000d28       __imp_??4QString@@QAEAAV0@ABV0@@Z 10011d28     qt-mt323:qt-mt323.dll
 0002:00000d2c       __imp_??1QString@@QAE@XZ   10011d2c     qt-mt323:qt-mt323.dll
 0002:00000d30       __imp_??0QString@@QAE@PBD@Z 10011d30     qt-mt323:qt-mt323.dll
 0002:00000d34       __imp_??0QString@@QAE@ABV0@@Z 10011d34     qt-mt323:qt-mt323.dll
 0002:00000d38       __imp_??0QString@@QAE@XZ   10011d38     qt-mt323:qt-mt323.dll
 0002:00000d3c       __imp_?qDebug@@YAXPBDZZ    10011d3c     qt-mt323:qt-mt323.dll
 0002:00000d40       __imp_?geometry@QSpacerItem@@UBE?AVQRect@@XZ 10011d40     qt-mt323:qt-mt323.dll
 0002:00000d44       \177qt-mt323_NULL_THUNK_DATA 10011d44     qt-mt323:qt-mt323.dll
 0002:00000d48       ___xc_a                    10011d48     MSVCRT:cinitexe.obj
 0002:00000d70       ___xc_z                    10011d70     MSVCRT:cinitexe.obj
 0002:00000d74       ___xi_a                    10011d74     MSVCRT:cinitexe.obj
 0002:00000d80       ___xi_z                    10011d80     MSVCRT:cinitexe.obj
 0002:00000d88       ??_C@_02GIPFHKNO@OK?$AA@   10011d88     config_plugin_instances.obj
 0002:00000d94       ??_SQAction@@6B@           10011d94     config_plugin_instances.obj
 0002:00000e24       ??_SQToolBar@@6BQObject@@@ 10011e24     config_plugin_instances.obj
 0002:00001040       ??_SQToolBar@@6BQPaintDevice@@@ 10012040     config_plugin_instances.obj
 0002:00001064       ??_SQGuardedPtrPrivate@@6B@ 10012064     config_plugin_instances.obj
 0002:000010b8       ??_7QDockWindowList@@6B@   100120b8     config_plugin_instances.obj
 0002:000010dc       ??_SQPopupMenu@@6BQObject@@@ 100120dc     config_plugin_instances.obj
 0002:000012bc       ??_SQPopupMenu@@6BQPaintDevice@@@ 100122bc     config_plugin_instances.obj
 0002:000012e0       ??_SQPopupMenu@@6B@        100122e0     config_plugin_instances.obj
 0002:00001304       ??_7?$QPtrList@VQPopupMenu@@@@6B@ 10012304     config_plugin_instances.obj
 0002:00001328       ??_7QPopupMenuList@@6B@    10012328     config_plugin_instances.obj
 0002:00001348       ??_C@_04OOEBCMBF@FAIL?$AA@ 10012348     config_plugin_instances.obj
 0002:00001350       ??_C@_08OBALAKLA@READONLY?$AA@ 10012350     config_plugin_instances.obj
 0002:0000135c       ??_C@_04KANDKFIK@DONE?$AA@ 1001235c     config_plugin_instances.obj
 0002:00001364       ??_C@_07NFANNNEC@UNKNOWN?$AA@ 10012364     config_plugin_instances.obj
 0002:00001370       ??_7config_plugin_base@@6BQObject@@@ 10012370     config_plugin_instances.obj
 0002:00001548       ??_7config_plugin_base@@6BQPaintDevice@@@ 10012548     config_plugin_instances.obj
 0002:00001568       ??_C@_0EB@GNDACMDJ@?$CC?5?9?5the?5author?5should?5have?5defin@ 10012568     config_plugin_instances.obj
 0002:000015ac       ??_C@_0CH@BDPDPLDP@This?5is?5the?5default?5?$CCAbout?$CC?5text@ 100125ac     config_plugin_instances.obj
 0002:000015d8       ??_7?$QDict@VQAction@@@@6B@ 100125d8     config_plugin_instances.obj
 0002:000015f8       ??_7config_plugin_instances@@6BQObject@@@ 100125f8     config_plugin_instances.obj
 0002:000017d0       ??_7config_plugin_instances@@6BQPaintDevice@@@ 100127d0     config_plugin_instances.obj
 0002:000017f0       ??_C@_0BK@EPFHJJOO@config_plugin_instances?3?5?$AA@ 100127f0     config_plugin_instances.obj
 0002:0000180c       ??_C@_0BN@CEGLABJP@2command?$CI?5QString?0?5QString?5?$CJ?$AA@ 1001280c     config_plugin_instances.obj
 0002:0000182c       ??_C@_0BI@DJGPDCG@Template?5Plugin?5Toolbar?$AA@ 1001282c     config_plugin_instances.obj
 0002:00001844       ??_C@_05LHMKEDEH@?$CGEdit?$AA@ 10012844     config_plugin_instances.obj
 0002:0000184c       ??_C@_03CLCAEGCJ@new?$AA@  1001284c     config_plugin_instances.obj
 0002:00001850       ??_C@_04CCPFBLLC@?$CGNew?$AA@ 10012850     config_plugin_instances.obj
 0002:00001858       ??_C@_07EJAINBEK@filenew?$AA@ 10012858     config_plugin_instances.obj
 0002:00001860       ??_C@_0N@EIIGMNDM@New?5Instance?$AA@ 10012860     config_plugin_instances.obj
 0002:00001870       ??_C@_0BH@MKDOHOFP@1doCreateNewInstance?$CI?$CJ?$AA@ 10012870     config_plugin_instances.obj
 0002:00001888       ??_C@_0N@KCMOKDBB@2activated?$CI?$CJ?$AA@ 10012888     config_plugin_instances.obj
 0002:00001898       ??_C@_06FOBLBEIN@delete?$AA@ 10012898     config_plugin_instances.obj
 0002:000018a0       ??_C@_07FGPBEGNH@?$CGDelete?$AA@ 100128a0     config_plugin_instances.obj
 0002:000018a8       ??_C@_0L@BPDPNFLB@filedelete?$AA@ 100128a8     config_plugin_instances.obj
 0002:000018b4       ??_C@_0BA@LDAHLHDF@Delete?5Instance?$AA@ 100128b4     config_plugin_instances.obj
 0002:000018c4       ??_C@_0BE@GICKJFKI@1doDeleteInstance?$CI?$CJ?$AA@ 100128c4     config_plugin_instances.obj
 0002:000018d8       ??_C@_09KHIKJOBP@duplicate?$AA@ 100128d8     config_plugin_instances.obj
 0002:000018e4       ??_C@_0L@OPDABMB@?$CGDuplicate?$AA@ 100128e4     config_plugin_instances.obj
 0002:000018f0       ??_C@_0BD@NPAGHMKP@Duplicate?5Instance?$AA@ 100128f0     config_plugin_instances.obj
 0002:00001904       ??_C@_0BH@GGHGKFEN@1doDuplicateInstance?$CI?$CJ?$AA@ 10012904     config_plugin_instances.obj
 0002:0000191c       ??_C@_0CO@GJAHOADB@1deviceContextMenu?$CIint?5?0?5int?0?5co@ 1001291c     config_plugin_instances.obj
 0002:0000194c       ??_C@_0DA@BPDJLODM@2contextMenuRequested?$CIint?0?5int?0?5@ 1001294c     config_plugin_instances.obj
 0002:0000197c       ??_C@_06BNCCALCL@unlock?$AA@ 1001297c     config_plugin_instances.obj
 0002:00001984       ??_C@_09JLEOPMAJ@?5?9?5error?$DN?$AA@ 10012984     config_plugin_instances.obj
 0002:00001990       ??_C@_09LBCHCBIC@?5?9?5value?$DN?$AA@ 10012990     config_plugin_instances.obj
 0002:0000199c       ??_C@_0P@ELNNACEA@?5?9?5textStatus?$DN?$AA@ 1001299c     config_plugin_instances.obj
 0002:000019ac       ??_C@_0L@LEAPMKGP@Reply?3?5op?$DN?$AA@ 100129ac     config_plugin_instances.obj
 0002:000019b8       ??_C@_08HNIAHLMM@download?$AA@ 100129b8     config_plugin_instances.obj
 0002:000019c4       ??_C@_0BF@NLODMMOO@config?1instances?4xml?$AA@ 100129c4     config_plugin_instances.obj
 0002:000019dc       ??_C@_01KMDKNFGN@?1?$AA@   100129dc     config_plugin_instances.obj
 0002:000019e0       ??_C@_0BH@FJKOLNHB@config?1devicetypes?4xml?$AA@ 100129e0     config_plugin_instances.obj
 0002:000019f8       ??_C@_0BI@JFAMKGKG@?1config?1devicetypes?4xml?$AA@ 100129f8     config_plugin_instances.obj
 0002:00001a10       ??_C@_06KAOCKAGB@upload?$AA@ 10012a10     config_plugin_instances.obj
 0002:00001a17       ??_C@_00CNPNBAHC@?$AA@     10012a17     config_plugin_instances.obj
 0002:00001a18       ??_C@_05CCAMFJOL@clean?$AA@ 10012a18     config_plugin_instances.obj
 0002:00001a20       ??_C@_0M@EBFEGAAI@Information?$AA@ 10012a20     config_plugin_instances.obj
 0002:00001a2c       ??_C@_0CO@GKAEALGF@Being?5asked?5to?5navigate?5to?5?$CF1?5wi@ 10012a2c     config_plugin_instances.obj
 0002:00001a5c       ??_C@_0N@LJNCPLAD@downloadFile?$AA@ 10012a5c     config_plugin_instances.obj
 0002:00001a6c       ??_C@_0N@EHHLDFOB@checkoutFile?$AA@ 10012a6c     config_plugin_instances.obj
 0002:00001a7c       ??_C@_0L@CIKGEHEG@uploadFile?$AA@ 10012a7c     config_plugin_instances.obj
 0002:00001a88       ??_C@_0HN@FFCELLM@?$DMh3?$DOTemplate?5Configuration?5Plugi@ 10012a88     config_plugin_instances.obj
 0002:00001b08       ??_C@_08HJLKCOJL@13?325?321?$AA@ 10012b08     config_plugin_instances.obj
 0002:00001b14       ??_C@_0M@JEDEHNP@Sep?523?52021?$AA@ 10012b14     config_plugin_instances.obj
 0002:00001b20       ??_C@_09DJMEPPMA@15?515?52?51?$AA@ 10012b20     config_plugin_instancesdlgimpl.obj
 0002:00001b2c       ??_C@_0M@PNMKLMIE@?$CD?5c?5?$CD00ff00?$AA@ 10012b2c     config_plugin_instancesdlgimpl.obj
 0002:00001b38       ??_C@_0M@HNGHCCNN@?4?5c?5?$CDffffff?$AA@ 10012b38     config_plugin_instancesdlgimpl.obj
 0002:00001b44       ??_C@_0BA@HBKNFNPB@?4?4?4?4?4?4?4?4?4?4?4?4?4?$CD?4?$AA@ 10012b44     config_plugin_instancesdlgimpl.obj
 0002:00001b54       ??_C@_0BA@IDMHIFCM@?4?4?4?4?4?4?4?4?4?4?4?4?$CD?$CD?4?$AA@ 10012b54     config_plugin_instancesdlgimpl.obj
 0002:00001b64       ??_C@_0BA@HDIPNCMO@?4?4?4?4?4?4?4?4?4?4?4?$CD?$CD?4?4?$AA@ 10012b64     config_plugin_instancesdlgimpl.obj
 0002:00001b74       ??_C@_0BA@DNHLBJMN@?4?4?4?4?4?4?4?4?4?4?$CD?$CD?4?4?4?$AA@ 10012b74     config_plugin_instancesdlgimpl.obj
 0002:00001b84       ??_C@_0BA@FMKMHIAN@?4?4?4?4?4?4?4?4?4?$CD?$CD?$CD?4?4?4?$AA@ 10012b84     config_plugin_instancesdlgimpl.obj
 0002:00001b94       ??_C@_0BA@KEDMLMLM@?4?4?4?4?4?4?4?4?4?$CD?$CD?4?4?4?4?$AA@ 10012b94     config_plugin_instancesdlgimpl.obj
 0002:00001ba4       ??_C@_0BA@IDKHLKLD@?4?4?4?4?4?4?4?4?$CD?$CD?4?4?4?4?4?$AA@ 10012ba4     config_plugin_instancesdlgimpl.obj
 0002:00001bb4       ??_C@_0BA@BDDPDMCE@?4?4?4?4?4?4?4?$CD?$CD?4?4?4?4?4?4?$AA@ 10012bb4     config_plugin_instancesdlgimpl.obj
 0002:00001bc4       ??_C@_0BA@OPILPFMN@?$CD?4?4?4?4?4?$CD?$CD?$CD?4?4?4?4?4?4?$AA@ 10012bc4     config_plugin_instancesdlgimpl.obj
 0002:00001bd4       ??_C@_0BA@IIIAJCBA@?$CD?$CD?4?4?4?4?$CD?$CD?4?4?4?4?4?4?4?$AA@ 10012bd4     config_plugin_instancesdlgimpl.obj
 0002:00001be4       ??_C@_0BA@PNKEONBF@?4?$CD?$CD?4?4?$CD?$CD?$CD?4?4?4?4?4?4?4?$AA@ 10012be4     config_plugin_instancesdlgimpl.obj
 0002:00001bf4       ??_C@_0BA@CJGGBJNO@?4?4?$CD?$CD?$CD?$CD?$CD?4?4?4?4?4?4?4?4?$AA@ 10012bf4     config_plugin_instancesdlgimpl.obj
 0002:00001c04       ??_C@_0BA@GLGCOCDF@?4?4?4?$CD?$CD?$CD?4?4?4?4?4?4?4?4?4?$AA@ 10012c04     config_plugin_instancesdlgimpl.obj
 0002:00001c14       ??_C@_0BA@OHNKMPEM@?4?4?4?4?$CD?4?4?4?4?4?4?4?4?4?4?$AA@ 10012c14     config_plugin_instancesdlgimpl.obj
 0002:00001c24       ??_C@_09OFODDICG@14?514?52?51?$AA@ 10012c24     config_plugin_instancesdlgimpl.obj
 0002:00001c30       ??_C@_0M@DOCNOBPG@?$CD?5c?5?$CDff0000?$AA@ 10012c30     config_plugin_instancesdlgimpl.obj
 0002:00001c3c       ??_C@_0P@HFKAALMG@?4?4?4?4?4?4?4?4?4?4?4?4?4?4?$AA@ 10012c3c     config_plugin_instancesdlgimpl.obj
 0002:00001c4c       ??_C@_0P@LODEEGMB@?4?4?4?4?$CD?4?4?4?4?4?4?4?4?4?$AA@ 10012c4c     config_plugin_instancesdlgimpl.obj
 0002:00001c5c       ??_C@_0P@NIALIDJO@?4?4?4?$CD?$CD?4?4?4?4?4?$CD?4?4?4?$AA@ 10012c5c     config_plugin_instancesdlgimpl.obj
 0002:00001c6c       ??_C@_0P@CNGKCON@?4?4?4?$CD?$CD?$CD?4?4?$CD?$CD?$CD?$CD?4?4?$AA@ 10012c6c     config_plugin_instancesdlgimpl.obj
 0002:00001c7c       ??_C@_0P@GAEEMDDI@?4?4?4?$CD?$CD?$CD?$CD?$CD?$CD?$CD?$CD?$CD?$CD?4?$AA@ 10012c7c     config_plugin_instancesdlgimpl.obj
 0002:00001c8c       ??_C@_0P@JKPGIILG@?4?4?4?$CD?$CD?$CD?$CD?$CD?$CD?$CD?$CD?4?4?4?$AA@ 10012c8c     config_plugin_instancesdlgimpl.obj
 0002:00001c9c       ??_C@_0P@PMMJENOJ@?4?4?4?4?$CD?$CD?$CD?$CD?$CD?$CD?4?4?4?4?$AA@ 10012c9c     config_plugin_instancesdlgimpl.obj
 0002:00001cac       ??_C@_0P@ILMDBDDA@?4?4?4?4?4?$CD?$CD?$CD?$CD?4?4?4?4?4?$AA@ 10012cac     config_plugin_instancesdlgimpl.obj
 0002:00001cbc       ??_C@_0P@LJHMGMM@?4?$CD?$CD?$CD?$CD?$CD?$CD?4?$CD?$CD?$CD?$CD?$CD?4?$AA@ 10012cbc     config_plugin_instancesdlgimpl.obj
 0002:00001ccc       ??_C@_0P@CECNKDFD@?4?4?$CD?$CD?$CD?$CD?4?4?4?$CD?$CD?$CD?4?4?$AA@ 10012ccc     config_plugin_instancesdlgimpl.obj
 0002:00001cdc       ??_C@_0P@OLAPAKCI@?4?4?4?$CD?4?4?4?4?4?4?4?4?4?4?$AA@ 10012cdc     config_plugin_instancesdlgimpl.obj
 0002:00001cf4       ??_SQDomDocument@@6B@      10012cf4     config_plugin_instancesdlgimpl.obj
 0002:00001d9c       ??_SQDomElement@@6B@       10012d9c     config_plugin_instancesdlgimpl.obj
 0002:00001e48       ??_7config_plugin_instancesDlg@@6BQObject@@@ 10012e48     config_plugin_instancesdlgimpl.obj
 0002:00002000       ??_7config_plugin_instancesDlg@@6BQPaintDevice@@@ 10013000     config_plugin_instancesdlgimpl.obj
 0002:00002020       ??_C@_02EGCJHIOB@id?$AA@   10013020     config_plugin_instancesdlgimpl.obj
 0002:00002024       ??_C@_06OJMPKPAG@alt_id?$AA@ 10013024     config_plugin_instancesdlgimpl.obj
 0002:0000202c       ??_C@_04GPMDFGEJ@type?$AA@ 1001302c     config_plugin_instancesdlgimpl.obj
 0002:00002034       ??_C@_04DMDAAMFM@ref1?$AA@ 10013034     config_plugin_instancesdlgimpl.obj
 0002:0000203c       ??_C@_04BHBNFPJP@ref2?$AA@ 1001303c     config_plugin_instancesdlgimpl.obj
 0002:00002044       ??_C@_04OAGGONO@ref3?$AA@  10013044     config_plugin_instancesdlgimpl.obj
 0002:0000204c       ??_C@_04EBEHPIBJ@ref4?$AA@ 1001304c     config_plugin_instancesdlgimpl.obj
 0002:00002054       ??_C@_08CBBFJFMD@location?$AA@ 10013054     config_plugin_instancesdlgimpl.obj
 0002:00002060       ??_C@_09EIHFMDLJ@composite?$AA@ 10013060     config_plugin_instancesdlgimpl.obj
 0002:0000206c       ??_C@_08EMNENPBA@instance?$AA@ 1001306c     config_plugin_instancesdlgimpl.obj
 0002:00002078       ??_C@_06NKJDBPMM@alt?5id?$AA@ 10013078     config_plugin_instancesdlgimpl.obj
 0002:00002080       ??_C@_06CHPEJBOD@device?$AA@ 10013080     config_plugin_instancesdlgimpl.obj
 0002:00002088       ??_C@_06KLHHMIGM@offset?$AA@ 10013088     config_plugin_instancesdlgimpl.obj
 0002:00002090       ??_C@_07CMPFPFAH@complex?$AA@ 10013090     config_plugin_instancesdlgimpl.obj
 0002:00002098       ??_C@_08LBOGKGFB@Ref?9misc?$AA@ 10013098     config_plugin_instancesdlgimpl.obj
 0002:000020a4       ??_C@_0CA@DAHFGBBD@1deviceInstanceChanged?$CIint?0int?$CJ?$AA@ 100130a4     config_plugin_instancesdlgimpl.obj
 0002:000020c4       ??_C@_0BJ@MBLPBKLC@2currentChanged?$CIint?0int?$CJ?$AA@ 100130c4     config_plugin_instancesdlgimpl.obj
 0002:000020e0       ??_C@_0BO@FGKODAMG@1viewInstanceChanged?$CIint?0int?$CJ?$AA@ 100130e0     config_plugin_instancesdlgimpl.obj
 0002:00002100       ??_C@_0BL@EIAGBBPN@1viewGroupChanged?$CIint?0int?$CJ?$AA@ 10013100     config_plugin_instancesdlgimpl.obj
 0002:0000211c       ??_C@_0BO@JMHFBODC@1valueDevicesChanged?$CIint?0int?$CJ?$AA@ 1001311c     config_plugin_instancesdlgimpl.obj
 0002:0000213c       ??_C@_0BH@DNELPHML@2valueChanged?$CIint?0int?$CJ?$AA@ 1001313c     config_plugin_instancesdlgimpl.obj
 0002:00002154       ??_C@_0CD@OHHECADN@1valueCompositeTopChanged?$CIint?0in@ 10013154     config_plugin_instancesdlgimpl.obj
 0002:00002178       ??_C@_0CF@FLNEAFFI@1valueCompositeGroupChanged?$CIint?0@ 10013178     config_plugin_instancesdlgimpl.obj
 0002:000021a0       ??_C@_0BC@DLEJKFKG@1setEnabled?$CIbool?$CJ?$AA@ 100131a0     config_plugin_instancesdlgimpl.obj
 0002:000021b4       ??_C@_0BK@CGPDLMEB@2clipboardDataValid?$CIbool?$CJ?$AA@ 100131b4     config_plugin_instancesdlgimpl.obj
 0002:000021d0       ??_C@_0BH@HOHNNCNI@1clipboardDataChange?$CI?$CJ?$AA@ 100131d0     config_plugin_instancesdlgimpl.obj
 0002:000021e8       ??_C@_0P@GLIODLHI@2dataChanged?$CI?$CJ?$AA@ 100131e8     config_plugin_instancesdlgimpl.obj
 0002:000021f8       ??_C@_0BL@DBKGCNGD@1copySelectedToClipboard?$CI?$CJ?$AA@ 100131f8     config_plugin_instancesdlgimpl.obj
 0002:00002214       ??_C@_0L@OELOHDKG@2clicked?$CI?$CJ?$AA@ 10013214     config_plugin_instancesdlgimpl.obj
 0002:00002220       ??_C@_0BA@CHFPLOFG@1pasteOptions?$CI?$CJ?$AA@ 10013220     config_plugin_instancesdlgimpl.obj
 0002:00002230       ??_C@_0CP@BDADDEDB@1selectDevicetypes?$CIint?0int?0int?0c@ 10013230     config_plugin_instancesdlgimpl.obj
 0002:00002260       ??_C@_0CL@KICEKPHE@2doubleClicked?$CIint?0int?0int?0const@ 10013260     config_plugin_instancesdlgimpl.obj
 0002:0000228c       ??_C@_0O@BMBALJAJ@instances?4xml?$AA@ 1001328c     config_plugin_instancesdlgimpl.obj
 0002:0000229c       ??_C@_09BJOJOOIO@instances?$AA@ 1001329c     config_plugin_instancesdlgimpl.obj
 0002:000022a8       ??_C@_03ICICOMAL@yes?$AA@  100132a8     config_plugin_instancesdlgimpl.obj
 0002:000022ac       ??_C@_03GCDGINBO@ref?$AA@  100132ac     config_plugin_instancesdlgimpl.obj
 0002:000022b0       ??_C@_07FDMMAPON@device?$DN?$AA@ 100132b0     config_plugin_instancesdlgimpl.obj
 0002:000022b8       ??_C@_07COEHBCAF@offset?$DN?$AA@ 100132b8     config_plugin_instancesdlgimpl.obj
 0002:000022c0       ??_C@_01IHBHIGKO@?0?$AA@   100132c0     config_plugin_instancesdlgimpl.obj
 0002:000022c4       ??_C@_08PEKACIOI@complex?$DN?$AA@ 100132c4     config_plugin_instancesdlgimpl.obj
 0002:000022d0       ??_C@_02KAJCLHKP@no?$AA@   100132d0     config_plugin_instancesdlgimpl.obj
 0002:000022d4       ??_C@_0BA@GIPOJKBK@devicetypes?4xml?$AA@ 100132d4     config_plugin_instancesdlgimpl.obj
 0002:000022e4       ??_C@_0M@EHMABMKM@devicetypes?$AA@ 100132e4     config_plugin_instancesdlgimpl.obj
 0002:000022f0       ??_C@_05CFEJGMAI@dirty?$AA@ 100132f0     config_plugin_instancesdlgimpl.obj
 0002:000022f8       ??_C@_05MGJOOGAJ@group?$AA@ 100132f8     config_plugin_instancesdlgimpl.obj
 0002:00002300       ??_C@_08MJKJKIHF@?0offset?$DN?$AA@ 10013300     config_plugin_instancesdlgimpl.obj
 0002:0000230c       ??_C@_09KEECLHGO@?0complex?$DN?$AA@ 1001330c     config_plugin_instancesdlgimpl.obj
 0002:00002318       ??_C@_0N@EPMEBDCJ@New_Instance?$AA@ 10013318     config_plugin_instancesdlgimpl.obj
 0002:00002328       ??_C@_04LOHLNGLF@New_?$AA@ 10013328     config_plugin_instancesdlgimpl.obj
 0002:00002330       ??_C@_05NMBEKKJO@?$CFd_?$CFs?$AA@ 10013330     config_plugin_instancesdlgimpl.obj
 0002:00002338       ??_C@_09HGPFNIMF@New_Group?$AA@ 10013338     config_plugin_instancesdlgimpl.obj
 0002:00002348       ??_7?$QPtrList@VdeviceRow@@@@6B@ 10013348     config_plugin_instancesdlgimpl.obj
 0002:0000236c       ??_7?$QPtrList@VviewRow@@@@6B@ 1001336c     config_plugin_instancesdlgimpl.obj
 0002:00002390       ??_7?$QPtrList@VgroupRow@@@@6B@ 10013390     config_plugin_instancesdlgimpl.obj
 0002:000023b0       ??_C@_05NGADHBOM@copy_?$AA@ 100133b0     config_plugin_instancesdlgimpl.obj
 0002:000023b8       ??_C@_04JBKCEBKE@_of_?$AA@ 100133b8     config_plugin_instancesdlgimpl.obj
 0002:000023c0       ??_C@_0O@BBDBGNLN@copy_?$CFd_of_?$CFs?$AA@ 100133c0     config_plugin_instancesdlgimpl.obj
 0002:000023d0       ??_C@_0O@EOKMMDDH@doStartRename?$AA@ 100133d0     config_plugin_instancesdlgimpl.obj
 0002:000023e0       ??_C@_01EEMJAFIK@?6?$AA@   100133e0     config_plugin_instancesdlgimpl.obj
 0002:000023e4       ??_C@_01GPOEFGEJ@?7?$AA@   100133e4     config_plugin_instancesdlgimpl.obj
 0002:000023e8       ??_C@_0O@HAENHLF@view_fragment?$AA@ 100133e8     config_plugin_instancesdlgimpl.obj
 0002:000023f8       ??_C@_0BH@OCONPEPH@ITS?5the?5wrong?5XML?5type?$AA@ 100133f8     config_plugin_instancesdlgimpl.obj
 0002:00002414       ??_7deviceRow@@6B@         10013414     deviceRow.obj
 0002:0000241c       ??_7devicetypesBase@@6BQObject@@@ 1001341c     devicetypes.obj
 0002:000025e0       ??_7devicetypesBase@@6BQPaintDevice@@@ 100135e0     devicetypes.obj
 0002:00002604       ??_SQLabel@@6BQObject@@@   10013604     devicetypes.obj
 0002:000027fc       ??_SQLabel@@6BQPaintDevice@@@ 100137fc     devicetypes.obj
 0002:00002824       ??_SQListBox@@6BQObject@@@ 10013824     devicetypes.obj
 0002:00002acc       ??_SQListBox@@6BQPaintDevice@@@ 10013acc     devicetypes.obj
 0002:00002af4       ??_SQPushButton@@6BQObject@@@ 10013af4     devicetypes.obj
 0002:00002ce4       ??_SQPushButton@@6BQPaintDevice@@@ 10013ce4     devicetypes.obj
 0002:00002d0c       ??_SQSpacerItem@@6B@       10013d0c     devicetypes.obj
 0002:00002d54       ??_SQHBoxLayout@@6BQObject@@@ 10013d54     devicetypes.obj
 0002:00002dbc       ??_SQHBoxLayout@@6BQLayoutItem@@@ 10013dbc     devicetypes.obj
 0002:00002e04       ??_SQVBoxLayout@@6BQObject@@@ 10013e04     devicetypes.obj
 0002:00002e6c       ??_SQVBoxLayout@@6BQLayoutItem@@@ 10013e6c     devicetypes.obj
 0002:00002eac       ??_C@_0BA@NOFHCNHA@devicetypesBase?$AA@ 10013eac     devicetypes.obj
 0002:00002ebc       ??_C@_0BG@CNFDHJAF@devicetypesBaseLayout?$AA@ 10013ebc     devicetypes.obj
 0002:00002ed4       ??_C@_0L@KGLFILOJ@textLabel1?$AA@ 10013ed4     devicetypes.obj
 0002:00002ee0       ??_C@_0L@MKCJMJGP@lbDevtypes?$AA@ 10013ee0     devicetypes.obj
 0002:00002eec       ??_C@_07DHCFJLGA@Layout1?$AA@ 10013eec     devicetypes.obj
 0002:00002ef4       ??_C@_08DKBDHOFF@buttonOk?$AA@ 10013ef4     devicetypes.obj
 0002:00002f00       ??_C@_0N@OLKBNHFJ@buttonCancel?$AA@ 10013f00     devicetypes.obj
 0002:00002f10       ??_C@_09DMINLBG@1accept?$CI?$CJ?$AA@ 10013f10     devicetypes.obj
 0002:00002f1c       ??_C@_09OCDCAEKE@1reject?$CI?$CJ?$AA@ 10013f1c     devicetypes.obj
 0002:00002f28       ??_C@_0BN@CAOABEN@Select?5Device?5Type?5from?5list?$AA@ 10013f28     devicetypes.obj
 0002:00002f48       ??_C@_03DDKJIMDC@?$CGOK?$AA@ 10013f48     devicetypes.obj
 0002:00002f4c       ??_C@_07JLEKEEPN@?$CGCancel?$AA@ 10013f4c     devicetypes.obj
 0002:00002f58       ??_7devicetypes@@6BQObject@@@ 10013f58     devicetypesimpl.obj
 0002:0000311c       ??_7devicetypes@@6BQPaintDevice@@@ 1001411c     devicetypesimpl.obj
 0002:00003140       ??_7groupRow@@6B@          10014140     groupRow.obj
 0002:00003148       ??_7instancesCustomTable@@6BQObject@@@ 10014148     instancesCustomTable.obj
 0002:000034ec       ??_7instancesCustomTable@@6BQPaintDevice@@@ 100144ec     instancesCustomTable.obj
 0002:0000350c       ??_C@_0BD@PHPDBBBM@1sortColumn?$CI?5int?5?$CJ?$AA@ 1001450c     instancesCustomTable.obj
 0002:00003520       ??_C@_0BA@HHAILMBL@2clicked?$CI?5int?5?$CJ?$AA@ 10014520     instancesCustomTable.obj
 0002:00003530       ??_C@_0CC@EMCONOHJ@Sorting?5?$CFs?5on?5column?5?$CFd?5asc?5is?5?$CF@ 10014530     instancesCustomTable.obj
 0002:00003560       ??_C@_0P@DMEOIADN@languageChange?$AA@ 10014560     moc_devicetypes.obj
 0002:0000357c       ??_C@_0BB@PFEIHPGD@languageChange?$CI?$CJ?$AA@ 1001457c     moc_devicetypes.obj
 0002:00003590       ??_C@_0M@CNMHJBPM@?$CD?5c?5?$CD07cc02?$AA@ 10014590     plugindesc.obj
 0002:0000359c       ??_C@_08IMFNEMJ@?4?5c?5none?$AA@ 1001459c     plugindesc.obj
 0002:000035a8       ??_C@_0P@DBKONMKJ@?4?4?4?4?4?4?4?4?4?$CD?$CD?4?4?4?$AA@ 100145a8     plugindesc.obj
 0002:000035b8       ??_C@_0P@HPFKBHKK@?4?4?4?4?4?4?4?4?4?4?$CD?$CD?4?4?$AA@ 100145b8     plugindesc.obj
 0002:000035c8       ??_C@_0P@JAJCNDBN@?4?$CD?$CD?$CD?$CD?$CD?$CD?$CD?$CD?$CD?$CD?$CD?$CD?4?$AA@ 100145c8     plugindesc.obj
 0002:000035dc       ??_7config_plugin_desc_base@@6B@ 100145dc     plugindesc.obj
 0002:000035f0       ??_7plugindesc@@6B@        100145f0     plugindesc.obj
 0002:00003600       ??_C@_0BN@EIMOABEO@Home?1System?1Instances?5Editor?$AA@ 10014600     plugindesc.obj
 0002:00003624       ??_7viewRow@@6B@           10014624     viewRow.obj
 0002:0000362c       ??_SQWidget@@6BQObject@@@  1001462c     config_plugin_instancesdlg.obj
 0002:000037e0       ??_SQWidget@@6BQPaintDevice@@@ 100147e0     config_plugin_instancesdlg.obj
 0002:00003804       ??_7config_plugin_instancesDlgBase@@6BQObject@@@ 10014804     config_plugin_instancesdlg.obj
 0002:000039bc       ??_7config_plugin_instancesDlgBase@@6BQPaintDevice@@@ 100149bc     config_plugin_instancesdlg.obj
 0002:000039e4       ??_SQTabWidget@@6BQObject@@@ 100149e4     config_plugin_instancesdlg.obj
 0002:00003bb8       ??_SQTabWidget@@6BQPaintDevice@@@ 10014bb8     config_plugin_instancesdlg.obj
 0002:00003bd8       ??_C@_0BP@IJKKMNIG@config_plugin_instancesDlgBase?$AA@ 10014bd8     config_plugin_instancesdlg.obj
 0002:00003bf8       ??_C@_0CF@NLLDLCJB@config_plugin_instancesDlgBaseLa@ 10014bf8     config_plugin_instancesdlg.obj
 0002:00003c20       ??_C@_07KKDPDMDC@layout5?$AA@ 10014c20     config_plugin_instancesdlg.obj
 0002:00003c28       ??_C@_0N@CJBMCOMC@textLabel1_4?$AA@ 10014c28     config_plugin_instancesdlg.obj
 0002:00003c38       ??_C@_07LDCEANHD@layout4?$AA@ 10014c38     config_plugin_instancesdlg.obj
 0002:00003c40       ??_C@_0L@NNPJCPDK@tabWidget2?$AA@ 10014c40     config_plugin_instancesdlg.obj
 0002:00003c4c       ??_C@_03CEDILPBK@tab?$AA@  10014c4c     config_plugin_instancesdlg.obj
 0002:00003c50       ??_C@_09PEOMDABK@tabLayout?$AA@ 10014c50     config_plugin_instancesdlg.obj
 0002:00003c5c       ??_C@_0N@LCDLKPEC@tableDevices?$AA@ 10014c5c     config_plugin_instancesdlg.obj
 0002:00003c6c       ??_C@_05GBGDENAC@tab_2?$AA@ 10014c6c     config_plugin_instancesdlg.obj
 0002:00003c74       ??_C@_0M@BMGEADGH@tabLayout_2?$AA@ 10014c74     config_plugin_instancesdlg.obj
 0002:00003c80       ??_C@_0N@FKNBLMLL@tableViewTop?$AA@ 10014c80     config_plugin_instancesdlg.obj
 0002:00003c90       ??_C@_0O@EIKBNLHM@labelViewName?$AA@ 10014c90     config_plugin_instancesdlg.obj
 0002:00003ca0       ??_C@_0BA@PGKELDFF@tableViewBottom?$AA@ 10014ca0     config_plugin_instancesdlg.obj
 0002:00003cb0       ??_C@_07PMGFJLLE@layout3?$AA@ 10014cb0     config_plugin_instancesdlg.obj
 0002:00003cb8       ??_C@_0P@OLNHCPGE@pushButtonCopy?$AA@ 10014cb8     config_plugin_instancesdlg.obj
 0002:00003cc8       ??_C@_0BA@HCKBBPGF@pushButtonPaste?$AA@ 10014cc8     config_plugin_instancesdlg.obj
 0002:00003cd8       ??_C@_0BL@JPCBMGIN@config_plugin_instancesDlg?$AA@ 10014cd8     config_plugin_instancesdlg.obj
 0002:00003cf4       ??_C@_0BK@IINAKGOC@?$DMh1?$DOInstances?5Editor?$DM?1h1?$DO?$AA@ 10014cf4     config_plugin_instancesdlg.obj
 0002:00003d10       ??_C@_07MEEAAPDA@Devices?$AA@ 10014d10     config_plugin_instancesdlg.obj
 0002:00003d18       ??_C@_0BK@CLOBKKJE@Details?5for?5selected?5view?$AA@ 10014d18     config_plugin_instancesdlg.obj
 0002:00003d34       ??_C@_05FJJMPDFL@Views?$AA@ 10014d34     config_plugin_instancesdlg.obj
 0002:00003d3c       ??_C@_0BC@NOIFPMEL@Copy?5to?5Clipboard?$AA@ 10014d3c     config_plugin_instancesdlg.obj
 0002:00003d50       ??_C@_0BF@NHKAGICB@Paste?5from?5Clipboard?$AA@ 10014d50     config_plugin_instancesdlg.obj
 0002:00003d68       ??_C@_0BI@KFOKJMEK@config_plugin_instances?$AA@ 10014d68     moc_config_plugin_instances.obj
 0002:00003d80       ??_C@_03DMHICLNI@row?$AA@  10014d80     moc_config_plugin_instances.obj
 0002:00003d84       ??_C@_03HNOLNALI@col?$AA@  10014d84     moc_config_plugin_instances.obj
 0002:00003d88       ??_C@_03PCBNCGFH@pos?$AA@  10014d88     moc_config_plugin_instances.obj
 0002:00003d8c       ??_C@_01CAKFMAIO@?$AO?$AA@ 10014d8c     moc_config_plugin_instances.obj
 0002:00003d9c       ??_C@_0BC@CFACPBFI@deviceContextMenu?$AA@ 10014d9c     moc_config_plugin_instances.obj
 0002:00003dbc       ??_C@_0CJ@LDMFJDPB@deviceContextMenu?$CIint?0int?0const?5@ 10014dbc     moc_config_plugin_instances.obj
 0002:00003df4       ??_C@_07KMMNMMFF@command?$AA@ 10014df4     moc_config_plugin_instances.obj
 0002:00003e08       ??_C@_0BJ@FEFNJDLM@command?$CIQString?0QString?$CJ?$AA@ 10014e08     moc_config_plugin_instances.obj
 0002:00003e48       ??_C@_05JLNEMJLN@dummy?$AA@ 10014e48     moc_config_plugin_instancesdlgimpl.obj
 0002:00003e50       ??_C@_04OPAOLJNL@iRow?$AA@ 10014e50     moc_config_plugin_instancesdlgimpl.obj
 0002:00003e58       ??_C@_04KOJNECLL@iCol?$AA@ 10014e58     moc_config_plugin_instancesdlgimpl.obj
 0002:00003e60       ??_C@_01OJONOECF@b?$AA@    10014e60     moc_config_plugin_instancesdlgimpl.obj
 0002:00003e64       ??_C@_01JBBJJEPG@p?$AA@    10014e64     moc_config_plugin_instancesdlgimpl.obj
 0002:00003e74       ??_C@_0BC@ICLBCFBJ@selectDevicetypes?$AA@ 10014e74     moc_config_plugin_instancesdlgimpl.obj
 0002:00003ea0       ??_C@_0BL@PNMGJKFK@pasteCompositesXMLFragment?$AA@ 10014ea0     moc_config_plugin_instancesdlgimpl.obj
 0002:00003ec8       ??_C@_0P@CBCOJLAF@pasteGroupData?$AA@ 10014ec8     moc_config_plugin_instancesdlgimpl.obj
 0002:00003ed8       ??_C@_09NGNIBPPA@sInstance?$AA@ 10014ed8     moc_config_plugin_instancesdlgimpl.obj
 0002:00003ef0       ??_C@_0BO@ODDJEHBL@addGroupToInstanceNodeFromRow?$AA@ 10014ef0     moc_config_plugin_instancesdlgimpl.obj
 0002:00003f1c       ??_C@_0BD@IPBIONBI@addViewNodeFromRow?$AA@ 10014f1c     moc_config_plugin_instancesdlgimpl.obj
 0002:00003f3c       ??_C@_0BF@FGMCMMJM@addDeviceNodeFromRow?$AA@ 10014f3c     moc_config_plugin_instancesdlgimpl.obj
 0002:00003f60       ??_C@_0BA@JFIHJKKO@pasteDeviceData?$AA@ 10014f60     moc_config_plugin_instancesdlgimpl.obj
 0002:00003f7c       ??_C@_0N@EKEEEBKO@pasteOptions?$AA@ 10014f7c     moc_config_plugin_instancesdlgimpl.obj
 0002:00003f98       ??_C@_0BI@EGNELLPC@copySelectedToClipboard?$AA@ 10014f98     moc_config_plugin_instancesdlgimpl.obj
 0002:00003fbc       ??_C@_0BE@JKIANKML@clipboardDataChange?$AA@ 10014fbc     moc_config_plugin_instancesdlgimpl.obj
 0002:00003fd0       ??_C@_05PPFHJAOM@sName?$AA@ 10014fd0     moc_config_plugin_instancesdlgimpl.obj
 0002:00003fe4       ??_C@_0BC@GIFEBD@groupNameIsUnique?$AA@ 10014fe4     moc_config_plugin_instancesdlgimpl.obj
 0002:00004004       ??_C@_0M@GEAEBOMO@typeIsValid?$AA@ 10015004     moc_config_plugin_instancesdlgimpl.obj
 0002:00004010       ??_C@_04MEMAJGDJ@name?$AA@ 10015010     moc_config_plugin_instancesdlgimpl.obj
 0002:00004024       ??_C@_0BF@LIBNOLFP@instanceNameIsUnique?$AA@ 10015024     moc_config_plugin_instancesdlgimpl.obj
 0002:00004048       ??_C@_0BL@PJJFMCJB@valueCompositeGroupChanged?$AA@ 10015048     moc_config_plugin_instancesdlgimpl.obj
 0002:00004070       ??_C@_0BB@NHEMMLGP@viewGroupChanged?$AA@ 10015070     moc_config_plugin_instancesdlgimpl.obj
 0002:00004090       ??_C@_0BJ@LPCBJNAP@valueCompositeTopChanged?$AA@ 10015090     moc_config_plugin_instancesdlgimpl.obj
 0002:000040b8       ??_C@_0BE@MMOBBHHK@doDuplicateInstance?$AA@ 100150b8     moc_config_plugin_instancesdlgimpl.obj
 0002:000040d8       ??_C@_0BB@EDPBELHO@doDeleteInstance?$AA@ 100150d8     moc_config_plugin_instancesdlgimpl.obj
 0002:000040f8       ??_C@_0BE@DKAGGNGM@doCreateNewInstance?$AA@ 100150f8     moc_config_plugin_instancesdlgimpl.obj
 0002:00004118       ??_C@_0BE@OMMNALMF@valueDevicesChanged?$AA@ 10015118     moc_config_plugin_instancesdlgimpl.obj
 0002:00004138       ??_C@_0BE@HHPEMHID@viewInstanceChanged?$AA@ 10015138     moc_config_plugin_instancesdlgimpl.obj
 0002:0000414c       ??_C@_06JKDNBPMO@column?$AA@ 1001514c     moc_config_plugin_instancesdlgimpl.obj
 0002:00004160       ??_C@_0BG@ONGDJFNJ@deviceInstanceChanged?$AA@ 10015160     moc_config_plugin_instancesdlgimpl.obj
 0002:00004298       ??_C@_07MBMLLJIG@dummy?$CI?$CJ?$AA@ 10015298     moc_config_plugin_instancesdlgimpl.obj
 0002:000042a0       ??_C@_0CN@HMKKHNMI@selectDevicetypes?$CIint?0int?0int?0co@ 100152a0     moc_config_plugin_instancesdlgimpl.obj
 0002:000042d0       ??_C@_0BA@OAHCPFCB@doStartRename?$CI?$CJ?$AA@ 100152d0     moc_config_plugin_instancesdlgimpl.obj
 0002:000042e0       ??_C@_0BN@CCJGLKPB@pasteCompositesXMLFragment?$CI?$CJ?$AA@ 100152e0     moc_config_plugin_instancesdlgimpl.obj
 0002:00004300       ??_C@_0BB@GILCBHBE@pasteGroupData?$CI?$CJ?$AA@ 10015300     moc_config_plugin_instancesdlgimpl.obj
 0002:00004314       ??_C@_0CL@JDCNGBCM@addGroupToInstanceNodeFromRow?$CIin@ 10015314     moc_config_plugin_instancesdlgimpl.obj
 0002:00004340       ??_C@_0BI@GJDBHONK@addViewNodeFromRow?$CIint?$CJ?$AA@ 10015340     moc_config_plugin_instancesdlgimpl.obj
 0002:00004358       ??_C@_0BK@OFDNGOGD@addDeviceNodeFromRow?$CIint?$CJ?$AA@ 10015358     moc_config_plugin_instancesdlgimpl.obj
 0002:00004374       ??_C@_0BC@FCEGPGAJ@pasteDeviceData?$CI?$CJ?$AA@ 10015374     moc_config_plugin_instancesdlgimpl.obj
 0002:00004388       ??_C@_0P@EDEHCCJG@pasteOptions?$CI?$CJ?$AA@ 10015388     moc_config_plugin_instancesdlgimpl.obj
 0002:00004398       ??_C@_0BK@ICBCHFM@copySelectedToClipboard?$CI?$CJ?$AA@ 10015398     moc_config_plugin_instancesdlgimpl.obj
 0002:000043b4       ??_C@_0BG@DMBACHHM@clipboardDataChange?$CI?$CJ?$AA@ 100153b4     moc_config_plugin_instancesdlgimpl.obj
 0002:000043cc       ??_C@_0BL@GLKOMIO@groupNameIsUnique?$CIQString?$CJ?$AA@ 100153cc     moc_config_plugin_instancesdlgimpl.obj
 0002:000043e8       ??_C@_0BF@IENMPPBI@typeIsValid?$CIQString?$CJ?$AA@ 100153e8     moc_config_plugin_instancesdlgimpl.obj
 0002:00004400       ??_C@_0BO@HJADLGAC@instanceNameIsUnique?$CIQString?$CJ?$AA@ 10015400     moc_config_plugin_instancesdlgimpl.obj
 0002:00004420       ??_C@_0CE@DDAHDKDB@valueCompositeGroupChanged?$CIint?0i@ 10015420     moc_config_plugin_instancesdlgimpl.obj
 0002:00004444       ??_C@_0BK@HBIBBLMC@viewGroupChanged?$CIint?0int?$CJ?$AA@ 10015444     moc_config_plugin_instancesdlgimpl.obj
 0002:00004460       ??_C@_0CC@LAGNMADF@valueCompositeTopChanged?$CIint?0int@ 10015460     moc_config_plugin_instancesdlgimpl.obj
 0002:00004484       ??_C@_0BG@CEBLFAOJ@doDuplicateInstance?$CI?$CJ?$AA@ 10015484     moc_config_plugin_instancesdlgimpl.obj
 0002:0000449c       ??_C@_0BD@CCKKAHCC@doDeleteInstance?$CI?$CJ?$AA@ 1001549c     moc_config_plugin_instancesdlgimpl.obj
 0002:000044b0       ??_C@_0BG@IIFDILPL@doCreateNewInstance?$CI?$CJ?$AA@ 100154b0     moc_config_plugin_instancesdlgimpl.obj
 0002:000044c8       ??_C@_0BN@DKHBECKP@valueDevicesChanged?$CIint?0int?$CJ?$AA@ 100154c8     moc_config_plugin_instancesdlgimpl.obj
 0002:000044e8       ??_C@_0BN@PAKKGMFL@viewInstanceChanged?$CIint?0int?$CJ?$AA@ 100154e8     moc_config_plugin_instancesdlgimpl.obj
 0002:00004508       ??_C@_0BP@JGEHCOJP@deviceInstanceChanged?$CIint?0int?$CJ?$AA@ 10015508     moc_config_plugin_instancesdlgimpl.obj
 0002:00004540       ??_C@_0BF@JJOLBABI@instancesCustomTable?$AA@ 10015540     moc_instancesCustomTable.obj
 0002:00004564       ??_C@_0L@BCAIFHPG@sortColumn?$AA@ 10015564     moc_instancesCustomTable.obj
 0002:00004570       ??_C@_03EFEGFOOI@asc?$AA@  10015570     moc_instancesCustomTable.obj
 0002:00004580       ??_C@_04BHGNNCDJ@swap?$AA@ 10015580     moc_instancesCustomTable.obj
 0002:000045b8       ??_C@_0BA@FENDPOLN@sortColumn?$CIint?$CJ?$AA@ 100155b8     moc_instancesCustomTable.obj
 0002:000045c8       ??_C@_0BE@JOPJJAHE@sortColumn?$CIint?0int?$CJ?$AA@ 100155c8     moc_instancesCustomTable.obj
 0002:000045dc       ??_C@_0BI@MDCPDAFE@sortColumn?$CIint?0int?0int?$CJ?$AA@ 100155dc     moc_instancesCustomTable.obj
 0002:000045f4       ??_C@_0P@ECKEJGFB@toolWindowBase?$AA@ 100155f4     moc_toolwindow.obj
 0002:0000461c       ??_C@_0L@IGMLIIOB@toolWindow?$AA@ 1001561c     moc_toolwindowimpl.obj
 0002:00004628       ??_C@_0O@NDCCBDNA@QIconViewItem?$AA@ 10015628     moc_toolwindowimpl.obj
 0002:00004644       ??_C@_0BB@FFKPNNIH@selectionChanged?$AA@ 10015644     moc_toolwindowimpl.obj
 0002:00004664       ??_C@_0CB@DONPBGFK@selectionChanged?$CIQIconViewItem?$CK?$CJ@ 10015664     moc_toolwindowimpl.obj
 0002:00004694       ??_C@_0N@DENPNHIG@fileSelected?$AA@ 10015694     moc_toolwindowimpl.obj
 0002:000046b0       ??_C@_0BN@NHBBIGHD@fileSelected?$CIconst?5QString?$CG?$CJ?$AA@ 100156b0     moc_toolwindowimpl.obj
 0002:000046d4       ??_7cfg_Table@@6BQObject@@@ 100156d4     cfg_widgets001:cfg_Table.obj
 0002:00004a78       ??_7cfg_Table@@6BQPaintDevice@@@ 10015a78     cfg_widgets001:cfg_Table.obj
 0002:00004a98       ??_C@_0BI@DKLEEDHJ@1clipBoardDataChanged?$CI?$CJ?$AA@ 10015a98     cfg_widgets001:cfg_Table.obj
 0002:00004ab0       ??_C@_0BA@NOIFKKAG@2dataChanged?5?$CI?$CJ?$AA@ 10015ab0     cfg_widgets001:cfg_Table.obj
 0002:00004ac0       ??_C@_03MDIDAHKD@?$CGNo?$AA@ 10015ac0     cfg_widgets001:cfg_Table.obj
 0002:00004ac4       ??_C@_04ILFHLBJA@?$CGYes?$AA@ 10015ac4     cfg_widgets001:cfg_Table.obj
 0002:00004ad0       ??_C@_0EG@JCAEPHHD@Selected?5Area?5does?5not?5match?4?6Do@ 10015ad0     cfg_widgets001:cfg_Table.obj
 0002:00004b18       ??_C@_0BB@LNOIOJNO@Database?5Edtitor?$AA@ 10015b18     cfg_widgets001:cfg_Table.obj
 0002:00004b2c       ??_C@_0DO@OOICEDKL@int?5cfg_Table?3?3validateRow?$CIiRow?$CJ@ 10015b2c     cfg_widgets001:cfg_Table.obj
 0002:00004b70       ??_C@_0EE@IEHIFONC@int?5cfg_Table?3?3validateRow?$CIint?5i@ 10015b70     cfg_widgets001:cfg_Table.obj
 0002:00004bb4       ??_C@_09PNEKGGBK@cfg_Table?$AA@ 10015bb4     cfg_widgets001:moc_cfg_Table.obj
 0002:00004bcc       ??_C@_0M@MOKGOAHM@deleteItems?$AA@ 10015bcc     cfg_widgets001:moc_cfg_Table.obj
 0002:00004be4       ??_C@_0BA@FJBCKEJL@copyToClipboard?$AA@ 10015be4     cfg_widgets001:moc_cfg_Table.obj
 0002:00004c00       ??_C@_09CLMPBHDI@undoPaste?$AA@ 10015c00     cfg_widgets001:moc_cfg_Table.obj
 0002:00004c18       ??_C@_0P@FJGFLBMO@pasteClipboard?$AA@ 10015c18     cfg_widgets001:moc_cfg_Table.obj
 0002:00004c34       ??_C@_0BF@CDBOAHLL@clipBoardDataChanged?$AA@ 10015c34     cfg_widgets001:moc_cfg_Table.obj
 0002:00004c88       ??_C@_0O@FBJIJCJH@deleteItems?$CI?$CJ?$AA@ 10015c88     cfg_widgets001:moc_cfg_Table.obj
 0002:00004c98       ??_C@_0BC@DBBGOFIB@copyToClipboard?$CI?$CJ?$AA@ 10015c98     cfg_widgets001:moc_cfg_Table.obj
 0002:00004cac       ??_C@_0M@OGFEJKEA@undoPaste?$CI?$CJ?$AA@ 10015cac     cfg_widgets001:moc_cfg_Table.obj
 0002:00004cb8       ??_C@_0BB@JLAHKIAM@pasteClipboard?$CI?$CJ?$AA@ 10015cb8     cfg_widgets001:moc_cfg_Table.obj
 0002:00004ccc       ??_C@_0BH@OLENEJHN@clipBoardDataChanged?$CI?$CJ?$AA@ 10015ccc     cfg_widgets001:moc_cfg_Table.obj
 0002:00004cf0       ??_C@_0L@OIBMJOP@dataPasted?$AA@ 10015cf0     cfg_widgets001:moc_cfg_Table.obj
 0002:00004d08       ??_C@_0BD@IALCIEJE@clipboardDataValid?$AA@ 10015d08     cfg_widgets001:moc_cfg_Table.obj
 0002:00004d34       ??_C@_0N@EJEGBDAF@dataPasted?$CI?$CJ?$AA@ 10015d34     cfg_widgets001:moc_cfg_Table.obj
 0002:00004d44       ??_C@_0BJ@FABNKMFK@clipboardDataValid?$CIbool?$CJ?$AA@ 10015d44     cfg_widgets001:moc_cfg_Table.obj
 0002:00004d64       ??_7type_info@@6B@         10015d64     MSVCRT:ti_inst.obj
 0002:00004d68       __pRawDllMain              10015d68     MSVCRT:crtdll.obj
 0002:00004d68       __pDefaultRawDllMain       10015d68     MSVCRT:crtdll.obj
 0002:00004d78       __load_config_used         10015d78     MSVCRT:loadcfg.obj
 0002:00004dc0       ??_R3QShared@@8            10015dc0     config_plugin_instances.obj
 0002:00004dd0       ??_R2QShared@@8            10015dd0     config_plugin_instances.obj
 0002:00004dd8       ??_R1A@?0A@EA@QShared@@8   10015dd8     config_plugin_instances.obj
 0002:00004df4       ??_R1A@?0A@EA@QGList@@8    10015df4     config_plugin_instances.obj
 0002:00004e10       ??_R3QGList@@8             10015e10     config_plugin_instances.obj
 0002:00004e20       ??_R2QGList@@8             10015e20     config_plugin_instances.obj
 0002:00004e2c       ??_R1A@?0A@EA@QPtrCollection@@8 10015e2c     config_plugin_instances.obj
 0002:00004e48       ??_R3QPtrCollection@@8     10015e48     config_plugin_instances.obj
 0002:00004e58       ??_R2QPtrCollection@@8     10015e58     config_plugin_instances.obj
 0002:00004e60       ??_R4QToolBar@@6BQObject@@@ 10015e60     config_plugin_instances.obj
 0002:00004e74       ??_R3QToolBar@@8           10015e74     config_plugin_instances.obj
 0002:00004e84       ??_R2QToolBar@@8           10015e84     config_plugin_instances.obj
 0002:00004ea4       ??_R1A@?0A@EA@QToolBar@@8  10015ea4     config_plugin_instances.obj
 0002:00004ec0       ??_R1A@?0A@EA@QDockWindow@@8 10015ec0     config_plugin_instances.obj
 0002:00004edc       ??_R3QDockWindow@@8        10015edc     config_plugin_instances.obj
 0002:00004eec       ??_R2QDockWindow@@8        10015eec     config_plugin_instances.obj
 0002:00004f08       ??_R1A@?0A@EA@QFrame@@8    10015f08     config_plugin_instances.obj
 0002:00004f24       ??_R3QFrame@@8             10015f24     config_plugin_instances.obj
 0002:00004f34       ??_R2QFrame@@8             10015f34     config_plugin_instances.obj
 0002:00004f4c       ??_R1A@?0A@EA@QWidget@@8   10015f4c     config_plugin_instances.obj
 0002:00004f68       ??_R3QWidget@@8            10015f68     config_plugin_instances.obj
 0002:00004f78       ??_R2QWidget@@8            10015f78     config_plugin_instances.obj
 0002:00004f8c       ??_R1A@?0A@EA@QObject@@8   10015f8c     config_plugin_instances.obj
 0002:00004fa8       ??_R3QObject@@8            10015fa8     config_plugin_instances.obj
 0002:00004fb8       ??_R2QObject@@8            10015fb8     config_plugin_instances.obj
 0002:00004fc4       ??_R13?0A@EA@Qt@@8         10015fc4     config_plugin_instances.obj
 0002:00004fe0       ??_R3Qt@@8                 10015fe0     config_plugin_instances.obj
 0002:00004ff0       ??_R2Qt@@8                 10015ff0     config_plugin_instances.obj
 0002:00004ff8       ??_R1A@?0A@EA@Qt@@8        10015ff8     config_plugin_instances.obj
 0002:00005014       ??_R1CI@?0A@EA@QPaintDevice@@8 10016014     config_plugin_instances.obj
 0002:00005030       ??_R3QPaintDevice@@8       10016030     config_plugin_instances.obj
 0002:00005040       ??_R2QPaintDevice@@8       10016040     config_plugin_instances.obj
 0002:00005048       ??_R1A@?0A@EA@QPaintDevice@@8 10016048     config_plugin_instances.obj
 0002:00005064       ??_R4QToolBar@@6BQPaintDevice@@@ 10016064     config_plugin_instances.obj
 0002:00005078       ??_R4QPopupMenu@@6BQObject@@@ 10016078     config_plugin_instances.obj
 0002:0000508c       ??_R3QPopupMenu@@8         1001608c     config_plugin_instances.obj
 0002:0000509c       ??_R2QPopupMenu@@8         1001609c     config_plugin_instances.obj
 0002:000050bc       ??_R1A@?0A@EA@QPopupMenu@@8 100160bc     config_plugin_instances.obj
 0002:000050d8       ??_R1IM@?0A@EA@QMenuData@@8 100160d8     config_plugin_instances.obj
 0002:000050f4       ??_R3QMenuData@@8          100160f4     config_plugin_instances.obj
 0002:00005104       ??_R2QMenuData@@8          10016104     config_plugin_instances.obj
 0002:0000510c       ??_R1A@?0A@EA@QMenuData@@8 1001610c     config_plugin_instances.obj
 0002:00005128       ??_R4QPopupMenu@@6BQPaintDevice@@@ 10016128     config_plugin_instances.obj
 0002:0000513c       ??_R4QPopupMenu@@6B@       1001613c     config_plugin_instances.obj
 0002:00005150       ??_R4QAction@@6B@          10016150     config_plugin_instances.obj
 0002:00005164       ??_R3QAction@@8            10016164     config_plugin_instances.obj
 0002:00005174       ??_R2QAction@@8            10016174     config_plugin_instances.obj
 0002:00005184       ??_R1A@?0A@EA@QAction@@8   10016184     config_plugin_instances.obj
 0002:000051a0       ??_R4QGuardedPtrPrivate@@6B@ 100161a0     config_plugin_instances.obj
 0002:000051b4       ??_R3QGuardedPtrPrivate@@8 100161b4     config_plugin_instances.obj
 0002:000051c4       ??_R2QGuardedPtrPrivate@@8 100161c4     config_plugin_instances.obj
 0002:000051d8       ??_R1A@?0A@EA@QGuardedPtrPrivate@@8 100161d8     config_plugin_instances.obj
 0002:000051f4       ??_R1CI@?0A@EA@QShared@@8  100161f4     config_plugin_instances.obj
 0002:00005210       ??_R1A@?0A@EA@QGDict@@8    10016210     config_plugin_instances.obj
 0002:0000522c       ??_R3QGDict@@8             1001622c     config_plugin_instances.obj
 0002:0000523c       ??_R2QGDict@@8             1001623c     config_plugin_instances.obj
 0002:00005248       ??_R4QDockWindowList@@6B@  10016248     config_plugin_instances.obj
 0002:0000525c       ??_R3QDockWindowList@@8    1001625c     config_plugin_instances.obj
 0002:0000526c       ??_R2QDockWindowList@@8    1001626c     config_plugin_instances.obj
 0002:00005280       ??_R1A@?0A@EA@QDockWindowList@@8 10016280     config_plugin_instances.obj
 0002:0000529c       ??_R1A@?0A@EA@?$QPtrList@VQDockWindow@@@@8 1001629c     config_plugin_instances.obj
 0002:000052b8       ??_R3?$QPtrList@VQDockWindow@@@@8 100162b8     config_plugin_instances.obj
 0002:000052c8       ??_R2?$QPtrList@VQDockWindow@@@@8 100162c8     config_plugin_instances.obj
 0002:000052d8       ??_R4QPopupMenuList@@6B@   100162d8     config_plugin_instances.obj
 0002:000052ec       ??_R3QPopupMenuList@@8     100162ec     config_plugin_instances.obj
 0002:000052fc       ??_R2QPopupMenuList@@8     100162fc     config_plugin_instances.obj
 0002:00005310       ??_R1A@?0A@EA@QPopupMenuList@@8 10016310     config_plugin_instances.obj
 0002:0000532c       ??_R1A@?0A@EA@?$QPtrList@VQPopupMenu@@@@8 1001632c     config_plugin_instances.obj
 0002:00005348       ??_R3?$QPtrList@VQPopupMenu@@@@8 10016348     config_plugin_instances.obj
 0002:00005358       ??_R2?$QPtrList@VQPopupMenu@@@@8 10016358     config_plugin_instances.obj
 0002:00005368       ??_R4?$QPtrList@VQPopupMenu@@@@6B@ 10016368     config_plugin_instances.obj
 0002:0000537c       ??_R4config_plugin_base@@6BQObject@@@ 1001637c     config_plugin_instances.obj
 0002:00005390       ??_R3config_plugin_base@@8 10016390     config_plugin_instances.obj
 0002:000053a0       ??_R2config_plugin_base@@8 100163a0     config_plugin_instances.obj
 0002:000053b8       ??_R1A@?0A@EA@config_plugin_base@@8 100163b8     config_plugin_instances.obj
 0002:000053d4       ??_R4config_plugin_base@@6BQPaintDevice@@@ 100163d4     config_plugin_instances.obj
 0002:000053e8       ??_R4config_plugin_instances@@6BQObject@@@ 100163e8     config_plugin_instances.obj
 0002:000053fc       ??_R3config_plugin_instances@@8 100163fc     config_plugin_instances.obj
 0002:0000540c       ??_R2config_plugin_instances@@8 1001640c     config_plugin_instances.obj
 0002:00005428       ??_R1A@?0A@EA@config_plugin_instances@@8 10016428     config_plugin_instances.obj
 0002:00005444       ??_R4config_plugin_instances@@6BQPaintDevice@@@ 10016444     config_plugin_instances.obj
 0002:00005458       ??_R4?$QDict@VQAction@@@@6B@ 10016458     config_plugin_instances.obj
 0002:0000546c       ??_R3?$QDict@VQAction@@@@8 1001646c     config_plugin_instances.obj
 0002:0000547c       ??_R2?$QDict@VQAction@@@@8 1001647c     config_plugin_instances.obj
 0002:0000548c       ??_R1A@?0A@EA@?$QDict@VQAction@@@@8 1001648c     config_plugin_instances.obj
 0002:000054a8       ??_R4QDomElement@@6B@      100164a8     config_plugin_instancesdlgimpl.obj
 0002:000054bc       ??_R3QDomElement@@8        100164bc     config_plugin_instancesdlgimpl.obj
 0002:000054cc       ??_R2QDomElement@@8        100164cc     config_plugin_instancesdlgimpl.obj
 0002:000054d8       ??_R1A@?0A@EA@QDomElement@@8 100164d8     config_plugin_instancesdlgimpl.obj
 0002:000054f4       ??_R1A@?0A@EA@QDomNode@@8  100164f4     config_plugin_instancesdlgimpl.obj
 0002:00005510       ??_R3QDomNode@@8           10016510     config_plugin_instancesdlgimpl.obj
 0002:00005520       ??_R2QDomNode@@8           10016520     config_plugin_instancesdlgimpl.obj
 0002:00005528       ??_R4QDomDocument@@6B@     10016528     config_plugin_instancesdlgimpl.obj
 0002:0000553c       ??_R3QDomDocument@@8       1001653c     config_plugin_instancesdlgimpl.obj
 0002:0000554c       ??_R2QDomDocument@@8       1001654c     config_plugin_instancesdlgimpl.obj
 0002:00005558       ??_R1A@?0A@EA@QDomDocument@@8 10016558     config_plugin_instancesdlgimpl.obj
 0002:00005574       ??_R4config_plugin_instancesDlg@@6BQObject@@@ 10016574     config_plugin_instancesdlgimpl.obj
 0002:00005588       ??_R3config_plugin_instancesDlg@@8 10016588     config_plugin_instancesdlgimpl.obj
 0002:00005598       ??_R2config_plugin_instancesDlg@@8 10016598     config_plugin_instancesdlgimpl.obj
 0002:000055b4       ??_R1A@?0A@EA@config_plugin_instancesDlg@@8 100165b4     config_plugin_instancesdlgimpl.obj
 0002:000055d0       ??_R1A@?0A@EA@config_plugin_instancesDlgBase@@8 100165d0     config_plugin_instancesdlgimpl.obj
 0002:000055ec       ??_R3config_plugin_instancesDlgBase@@8 100165ec     config_plugin_instancesdlgimpl.obj
 0002:000055fc       ??_R2config_plugin_instancesDlgBase@@8 100165fc     config_plugin_instancesdlgimpl.obj
 0002:00005614       ??_R4config_plugin_instancesDlg@@6BQPaintDevice@@@ 10016614     config_plugin_instancesdlgimpl.obj
 0002:00005628       ??_R4?$QPtrList@VdeviceRow@@@@6B@ 10016628     config_plugin_instancesdlgimpl.obj
 0002:0000563c       ??_R3?$QPtrList@VdeviceRow@@@@8 1001663c     config_plugin_instancesdlgimpl.obj
 0002:0000564c       ??_R2?$QPtrList@VdeviceRow@@@@8 1001664c     config_plugin_instancesdlgimpl.obj
 0002:0000565c       ??_R1A@?0A@EA@?$QPtrList@VdeviceRow@@@@8 1001665c     config_plugin_instancesdlgimpl.obj
 0002:00005678       ??_R4?$QPtrList@VviewRow@@@@6B@ 10016678     config_plugin_instancesdlgimpl.obj
 0002:0000568c       ??_R3?$QPtrList@VviewRow@@@@8 1001668c     config_plugin_instancesdlgimpl.obj
 0002:0000569c       ??_R2?$QPtrList@VviewRow@@@@8 1001669c     config_plugin_instancesdlgimpl.obj
 0002:000056ac       ??_R1A@?0A@EA@?$QPtrList@VviewRow@@@@8 100166ac     config_plugin_instancesdlgimpl.obj
 0002:000056c8       ??_R4?$QPtrList@VgroupRow@@@@6B@ 100166c8     config_plugin_instancesdlgimpl.obj
 0002:000056dc       ??_R3?$QPtrList@VgroupRow@@@@8 100166dc     config_plugin_instancesdlgimpl.obj
 0002:000056ec       ??_R2?$QPtrList@VgroupRow@@@@8 100166ec     config_plugin_instancesdlgimpl.obj
 0002:000056fc       ??_R1A@?0A@EA@?$QPtrList@VgroupRow@@@@8 100166fc     config_plugin_instancesdlgimpl.obj
 0002:00005718       ??_R4deviceRow@@6B@        10016718     deviceRow.obj
 0002:0000572c       ??_R3deviceRow@@8          1001672c     deviceRow.obj
 0002:0000573c       ??_R2deviceRow@@8          1001673c     deviceRow.obj
 0002:00005744       ??_R1A@?0A@EA@deviceRow@@8 10016744     deviceRow.obj
 0002:00005760       ??_R4QPushButton@@6BQObject@@@ 10016760     devicetypes.obj
 0002:00005774       ??_R3QPushButton@@8        10016774     devicetypes.obj
 0002:00005784       ??_R2QPushButton@@8        10016784     devicetypes.obj
 0002:000057a0       ??_R1A@?0A@EA@QPushButton@@8 100167a0     devicetypes.obj
 0002:000057bc       ??_R1A@?0A@EA@QButton@@8   100167bc     devicetypes.obj
 0002:000057d8       ??_R3QButton@@8            100167d8     devicetypes.obj
 0002:000057e8       ??_R2QButton@@8            100167e8     devicetypes.obj
 0002:00005800       ??_R4QPushButton@@6BQPaintDevice@@@ 10016800     devicetypes.obj
 0002:00005814       ??_R4QVBoxLayout@@6BQObject@@@ 10016814     devicetypes.obj
 0002:00005828       ??_R3QVBoxLayout@@8        10016828     devicetypes.obj
 0002:00005838       ??_R2QVBoxLayout@@8        10016838     devicetypes.obj
 0002:00005854       ??_R1A@?0A@EA@QVBoxLayout@@8 10016854     devicetypes.obj
 0002:00005870       ??_R1A@?0A@EA@QBoxLayout@@8 10016870     devicetypes.obj
 0002:0000588c       ??_R3QBoxLayout@@8         1001688c     devicetypes.obj
 0002:0000589c       ??_R2QBoxLayout@@8         1001689c     devicetypes.obj
 0002:000058b4       ??_R1A@?0A@EA@QLayout@@8   100168b4     devicetypes.obj
 0002:000058d0       ??_R3QLayout@@8            100168d0     devicetypes.obj
 0002:000058e0       ??_R2QLayout@@8            100168e0     devicetypes.obj
 0002:000058f4       ??_R1CI@?0A@EA@QLayoutItem@@8 100168f4     devicetypes.obj
 0002:00005910       ??_R3QLayoutItem@@8        10016910     devicetypes.obj
 0002:00005920       ??_R2QLayoutItem@@8        10016920     devicetypes.obj
 0002:00005928       ??_R1A@?0A@EA@QLayoutItem@@8 10016928     devicetypes.obj
 0002:00005944       ??_R4QVBoxLayout@@6BQLayoutItem@@@ 10016944     devicetypes.obj
 0002:00005958       ??_R4QHBoxLayout@@6BQObject@@@ 10016958     devicetypes.obj
 0002:0000596c       ??_R3QHBoxLayout@@8        1001696c     devicetypes.obj
 0002:0000597c       ??_R2QHBoxLayout@@8        1001697c     devicetypes.obj
 0002:00005998       ??_R1A@?0A@EA@QHBoxLayout@@8 10016998     devicetypes.obj
 0002:000059b4       ??_R4QHBoxLayout@@6BQLayoutItem@@@ 100169b4     devicetypes.obj
 0002:000059c8       ??_R4QLabel@@6BQObject@@@  100169c8     devicetypes.obj
 0002:000059dc       ??_R3QLabel@@8             100169dc     devicetypes.obj
 0002:000059ec       ??_R2QLabel@@8             100169ec     devicetypes.obj
 0002:00005a08       ??_R1A@?0A@EA@QLabel@@8    10016a08     devicetypes.obj
 0002:00005a24       ??_R4QLabel@@6BQPaintDevice@@@ 10016a24     devicetypes.obj
 0002:00005a38       ??_R4QListBox@@6BQObject@@@ 10016a38     devicetypes.obj
 0002:00005a4c       ??_R3QListBox@@8           10016a4c     devicetypes.obj
 0002:00005a5c       ??_R2QListBox@@8           10016a5c     devicetypes.obj
 0002:00005a7c       ??_R1A@?0A@EA@QListBox@@8  10016a7c     devicetypes.obj
 0002:00005a98       ??_R1A@?0A@EA@QScrollView@@8 10016a98     devicetypes.obj
 0002:00005ab4       ??_R3QScrollView@@8        10016ab4     devicetypes.obj
 0002:00005ac4       ??_R2QScrollView@@8        10016ac4     devicetypes.obj
 0002:00005ae0       ??_R4QListBox@@6BQPaintDevice@@@ 10016ae0     devicetypes.obj
 0002:00005af4       ??_R4devicetypesBase@@6BQObject@@@ 10016af4     devicetypes.obj
 0002:00005b08       ??_R3devicetypesBase@@8    10016b08     devicetypes.obj
 0002:00005b18       ??_R2devicetypesBase@@8    10016b18     devicetypes.obj
 0002:00005b34       ??_R1A@?0A@EA@devicetypesBase@@8 10016b34     devicetypes.obj
 0002:00005b50       ??_R1A@?0A@EA@QDialog@@8   10016b50     devicetypes.obj
 0002:00005b6c       ??_R3QDialog@@8            10016b6c     devicetypes.obj
 0002:00005b7c       ??_R2QDialog@@8            10016b7c     devicetypes.obj
 0002:00005b94       ??_R4devicetypesBase@@6BQPaintDevice@@@ 10016b94     devicetypes.obj
 0002:00005ba8       ??_R4QSpacerItem@@6B@      10016ba8     devicetypes.obj
 0002:00005bbc       ??_R3QSpacerItem@@8        10016bbc     devicetypes.obj
 0002:00005bcc       ??_R2QSpacerItem@@8        10016bcc     devicetypes.obj
 0002:00005bd8       ??_R1A@?0A@EA@QSpacerItem@@8 10016bd8     devicetypes.obj
 0002:00005bf4       ??_R4devicetypes@@6BQObject@@@ 10016bf4     devicetypesimpl.obj
 0002:00005c08       ??_R3devicetypes@@8        10016c08     devicetypesimpl.obj
 0002:00005c18       ??_R2devicetypes@@8        10016c18     devicetypesimpl.obj
 0002:00005c38       ??_R1A@?0A@EA@devicetypes@@8 10016c38     devicetypesimpl.obj
 0002:00005c54       ??_R4devicetypes@@6BQPaintDevice@@@ 10016c54     devicetypesimpl.obj
 0002:00005c68       ??_R4groupRow@@6B@         10016c68     groupRow.obj
 0002:00005c7c       ??_R3groupRow@@8           10016c7c     groupRow.obj
 0002:00005c8c       ??_R2groupRow@@8           10016c8c     groupRow.obj
 0002:00005c94       ??_R1A@?0A@EA@groupRow@@8  10016c94     groupRow.obj
 0002:00005cb0       ??_R4instancesCustomTable@@6BQObject@@@ 10016cb0     instancesCustomTable.obj
 0002:00005cc4       ??_R3instancesCustomTable@@8 10016cc4     instancesCustomTable.obj
 0002:00005cd4       ??_R2instancesCustomTable@@8 10016cd4     instancesCustomTable.obj
 0002:00005cfc       ??_R1A@?0A@EA@instancesCustomTable@@8 10016cfc     instancesCustomTable.obj
 0002:00005d18       ??_R1A@?0A@EA@cfg_Table@@8 10016d18     instancesCustomTable.obj
 0002:00005d34       ??_R3cfg_Table@@8          10016d34     instancesCustomTable.obj
 0002:00005d44       ??_R2cfg_Table@@8          10016d44     instancesCustomTable.obj
 0002:00005d68       ??_R1A@?0A@EA@QTable@@8    10016d68     instancesCustomTable.obj
 0002:00005d84       ??_R3QTable@@8             10016d84     instancesCustomTable.obj
 0002:00005d94       ??_R2QTable@@8             10016d94     instancesCustomTable.obj
 0002:00005db4       ??_R4instancesCustomTable@@6BQPaintDevice@@@ 10016db4     instancesCustomTable.obj
 0002:00005dc8       ??_R4config_plugin_desc_base@@6B@ 10016dc8     plugindesc.obj
 0002:00005ddc       ??_R3config_plugin_desc_base@@8 10016ddc     plugindesc.obj
 0002:00005dec       ??_R2config_plugin_desc_base@@8 10016dec     plugindesc.obj
 0002:00005df4       ??_R1A@?0A@EA@config_plugin_desc_base@@8 10016df4     plugindesc.obj
 0002:00005e10       ??_R4plugindesc@@6B@       10016e10     plugindesc.obj
 0002:00005e24       ??_R3plugindesc@@8         10016e24     plugindesc.obj
 0002:00005e34       ??_R2plugindesc@@8         10016e34     plugindesc.obj
 0002:00005e40       ??_R1A@?0A@EA@plugindesc@@8 10016e40     plugindesc.obj
 0002:00005e5c       ??_R4viewRow@@6B@          10016e5c     viewRow.obj
 0002:00005e70       ??_R3viewRow@@8            10016e70     viewRow.obj
 0002:00005e80       ??_R2viewRow@@8            10016e80     viewRow.obj
 0002:00005e88       ??_R1A@?0A@EA@viewRow@@8   10016e88     viewRow.obj
 0002:00005ea4       ??_R4QWidget@@6BQObject@@@ 10016ea4     config_plugin_instancesdlg.obj
 0002:00005eb8       ??_R4QWidget@@6BQPaintDevice@@@ 10016eb8     config_plugin_instancesdlg.obj
 0002:00005ecc       ??_R4QTabWidget@@6BQObject@@@ 10016ecc     config_plugin_instancesdlg.obj
 0002:00005ee0       ??_R3QTabWidget@@8         10016ee0     config_plugin_instancesdlg.obj
 0002:00005ef0       ??_R2QTabWidget@@8         10016ef0     config_plugin_instancesdlg.obj
 0002:00005f08       ??_R1A@?0A@EA@QTabWidget@@8 10016f08     config_plugin_instancesdlg.obj
 0002:00005f24       ??_R4QTabWidget@@6BQPaintDevice@@@ 10016f24     config_plugin_instancesdlg.obj
 0002:00005f38       ??_R4config_plugin_instancesDlgBase@@6BQObject@@@ 10016f38     config_plugin_instancesdlg.obj
 0002:00005f4c       ??_R4config_plugin_instancesDlgBase@@6BQPaintDevice@@@ 10016f4c     config_plugin_instancesdlg.obj
 0002:00005f60       ??_R4cfg_Table@@6BQObject@@@ 10016f60     cfg_widgets001:cfg_Table.obj
 0002:00005f74       ??_R4cfg_Table@@6BQPaintDevice@@@ 10016f74     cfg_widgets001:cfg_Table.obj
 0002:00005f88       ??_R4type_info@@6B@        10016f88     MSVCRT:ti_inst.obj
 0002:00005f9c       ??_R3type_info@@8          10016f9c     MSVCRT:ti_inst.obj
 0002:00005fac       ??_R2type_info@@8          10016fac     MSVCRT:ti_inst.obj
 0002:00005fb4       ??_R1A@?0A@EA@type_info@@8 10016fb4     MSVCRT:ti_inst.obj
 0002:00005fd0       ___safe_se_handler_table   10016fd0     <linker-defined>
 0002:000060e0       ___rtc_iaa                 100170e0     MSVCRT:initsect.obj
 0002:000060e4       ___rtc_izz                 100170e4     MSVCRT:initsect.obj
 0002:000060e8       ___rtc_taa                 100170e8     MSVCRT:initsect.obj
 0002:000060ec       ___rtc_tzz                 100170ec     MSVCRT:initsect.obj
 0002:000087d8       __IMPORT_DESCRIPTOR_config_icons 100197d8     config_icons:config_icons.dll
 0002:000087ec       __IMPORT_DESCRIPTOR_qt-mt323 100197ec     qt-mt323:qt-mt323.dll
 0002:00008800       __IMPORT_DESCRIPTOR_MSVCR120 10019800     MSVCRT:MSVCR120.dll
 0002:00008814       __IMPORT_DESCRIPTOR_KERNEL32 10019814     kernel32:KERNEL32.dll
 0002:00008828       __NULL_IMPORT_DESCRIPTOR   10019828     config_icons:config_icons.dll
 0003:000001e8       ___security_cookie         100231e8     MSVCRT:gs_cookie.obj
 0003:000001ec       ___security_cookie_complement 100231ec     MSVCRT:gs_cookie.obj
 0003:000001f0       ___native_dllmain_reason   100231f0     MSVCRT:natstart.obj
 0003:000001f4       ??_R0?AUQShared@@@8        100231f4     config_plugin_instances.obj
 0003:0000020c       ??_R0?AVQGList@@@8         1002320c     config_plugin_instances.obj
 0003:00000224       ??_R0?AVQPtrCollection@@@8 10023224     config_plugin_instances.obj
 0003:00000244       ??_R0?AVQToolBar@@@8       10023244     config_plugin_instances.obj
 0003:0000025c       ??_R0?AVQDockWindow@@@8    1002325c     config_plugin_instances.obj
 0003:00000278       ??_R0?AVQFrame@@@8         10023278     config_plugin_instances.obj
 0003:00000290       ??_R0?AVQWidget@@@8        10023290     config_plugin_instances.obj
 0003:000002a8       ??_R0?AVQObject@@@8        100232a8     config_plugin_instances.obj
 0003:000002c0       ??_R0?AVQt@@@8             100232c0     config_plugin_instances.obj
 0003:000002d4       ??_R0?AVQPaintDevice@@@8   100232d4     config_plugin_instances.obj
 0003:000002f0       ??_R0?AVQPopupMenu@@@8     100232f0     config_plugin_instances.obj
 0003:0000030c       ??_R0?AVQMenuData@@@8      1002330c     config_plugin_instances.obj
 0003:00000324       ??_R0?AVQAction@@@8        10023324     config_plugin_instances.obj
 0003:0000033c       ??_R0?AVQGuardedPtrPrivate@@@8 1002333c     config_plugin_instances.obj
 0003:00000360       ??_R0?AVQGDict@@@8         10023360     config_plugin_instances.obj
 0003:00000378       ??_R0?AVQDockWindowList@@@8 10023378     config_plugin_instances.obj
 0003:00000398       ??_R0?AV?$QPtrList@VQDockWindow@@@@@8 10023398     config_plugin_instances.obj
 0003:000003c0       ??_R0?AVQPopupMenuList@@@8 100233c0     config_plugin_instances.obj
 0003:000003e0       ??_R0?AV?$QPtrList@VQPopupMenu@@@@@8 100233e0     config_plugin_instances.obj
 0003:00000408       ??_R0?AVconfig_plugin_base@@@8 10023408     config_plugin_instances.obj
 0003:0000042c       ??_R0?AVconfig_plugin_instances@@@8 1002342c     config_plugin_instances.obj
 0003:00000454       ??_R0?AV?$QDict@VQAction@@@@@8 10023454     config_plugin_instances.obj
 0003:00000478       ??_R0?AVQDomElement@@@8    10023478     config_plugin_instancesdlgimpl.obj
 0003:00000494       ??_R0?AVQDomNode@@@8       10023494     config_plugin_instancesdlgimpl.obj
 0003:000004ac       ??_R0?AVQDomDocument@@@8   100234ac     config_plugin_instancesdlgimpl.obj
 0003:000004c8       ??_R0?AVconfig_plugin_instancesDlg@@@8 100234c8     config_plugin_instancesdlgimpl.obj
 0003:000004f4       ??_R0?AVconfig_plugin_instancesDlgBase@@@8 100234f4     config_plugin_instancesdlgimpl.obj
 0003:00000524       ??_R0?AV?$QPtrList@VdeviceRow@@@@@8 10023524     config_plugin_instancesdlgimpl.obj
 0003:0000054c       ??_R0?AV?$QPtrList@VviewRow@@@@@8 1002354c     config_plugin_instancesdlgimpl.obj
 0003:00000570       ??_R0?AV?$QPtrList@VgroupRow@@@@@8 10023570     config_plugin_instancesdlgimpl.obj
 0003:00000598       ??_R0?AVdeviceRow@@@8      10023598     deviceRow.obj
 0003:000005b0       ??_R0?AVQPushButton@@@8    100235b0     devicetypes.obj
 0003:000005cc       ??_R0?AVQButton@@@8        100235cc     devicetypes.obj
 0003:000005e4       ??_R0?AVQVBoxLayout@@@8    100235e4     devicetypes.obj
 0003:00000600       ??_R0?AVQBoxLayout@@@8     10023600     devicetypes.obj
 0003:0000061c       ??_R0?AVQLayout@@@8        1002361c     devicetypes.obj
 0003:00000634       ??_R0?AVQLayoutItem@@@8    10023634     devicetypes.obj
 0003:00000650       ??_R0?AVQHBoxLayout@@@8    10023650     devicetypes.obj
 0003:0000066c       ??_R0?AVQLabel@@@8         1002366c     devicetypes.obj
 0003:00000684       ??_R0?AVQListBox@@@8       10023684     devicetypes.obj
 0003:0000069c       ??_R0?AVQScrollView@@@8    1002369c     devicetypes.obj
 0003:000006b8       ??_R0?AVdevicetypesBase@@@8 100236b8     devicetypes.obj
 0003:000006d8       ??_R0?AVQDialog@@@8        100236d8     devicetypes.obj
 0003:000006f0       ??_R0?AVQSpacerItem@@@8    100236f0     devicetypes.obj
 0003:0000070c       ??_R0?AVdevicetypes@@@8    1002370c     devicetypesimpl.obj
 0003:00000728       ??_R0?AVgroupRow@@@8       10023728     groupRow.obj
 0003:00000740       ??_R0?AVinstancesCustomTable@@@8 10023740     instancesCustomTable.obj
 0003:00000764       ??_R0?AVcfg_Table@@@8      10023764     instancesCustomTable.obj
 0003:0000077c       ??_R0?AVQTable@@@8         1002377c     instancesCustomTable.obj
 0003:00000794       ??_R0?AVconfig_plugin_desc_base@@@8 10023794     plugindesc.obj
 0003:000007bc       ??_R0?AVplugindesc@@@8     100237bc     plugindesc.obj
 0003:000007d8       ??_R0?AVviewRow@@@8        100237d8     viewRow.obj
 0003:000007f0       ??_R0?AVQTabWidget@@@8     100237f0     config_plugin_instancesdlg.obj
 0003:0000080c       ??_R0?AVtype_info@@@8      1002380c     MSVCRT:ti_inst.obj
 0003:00000828       ?metaObj@devicetypesBase@@0PAVQMetaObject@@A 10023828     moc_devicetypes.obj
 0003:00000830       ?metaObj@devicetypes@@0PAVQMetaObject@@A 10023830     moc_devicetypesimpl.obj
 0003:00000838       ?metaObj@config_plugin_instances@@0PAVQMetaObject@@A 10023838     moc_config_plugin_instances.obj
 0003:00000864       ?metaObj@config_plugin_instancesDlgBase@@0PAVQMetaObject@@A 10023864     moc_config_plugin_instancesdlg.obj
 0003:0000086c       ?metaObj@config_plugin_instancesDlg@@0PAVQMetaObject@@A 1002386c     moc_config_plugin_instancesdlgimpl.obj
 0003:000009e8       ?metaObj@instancesCustomTable@@0PAVQMetaObject@@A 100239e8     moc_instancesCustomTable.obj
 0003:000009f4       ?metaObj@toolWindowBase@@0PAVQMetaObject@@A 100239f4     moc_toolwindow.obj
 0003:000009fc       ?metaObj@toolWindow@@0PAVQMetaObject@@A 100239fc     moc_toolwindowimpl.obj
 0003:00000a28       ?metaObj@cfg_Table@@0PAVQMetaObject@@A 10023a28     cfg_widgets001:moc_cfg_Table.obj
 0003:00000d68       ?__type_info_root_node@@3U__type_info_node@@A 10023d68     MSVCRT:tncleanup.obj
 0003:00000d70       ___native_startup_lock     10023d70     <common>
 0003:00000d74       ___native_startup_state    10023d74     <common>
 0003:00000d78       ___dyn_tls_init_callback   10023d78     <common>
 0003:00000d7c       ___onexitend               10023d7c     <common>
 0003:00000d80       ___onexitbegin             10023d80     <common>

 entry point at        0001:0000d3ca

 Static symbols

 0001:00000000       ??__EcleanUp_devicetypesBase@@YAXXZ 10001000 f   moc_devicetypes.obj
 0001:00000021       ??__EcleanUp_devicetypes@@YAXXZ 10001021 f   moc_devicetypesimpl.obj
 0001:00000042       ??__EcleanUp_config_plugin_instances@@YAXXZ 10001042 f   moc_config_plugin_instances.obj
 0001:00000063       ??__EcleanUp_config_plugin_instancesDlgBase@@YAXXZ 10001063 f   moc_config_plugin_instancesdlg.obj
 0001:00000084       ??__EcleanUp_config_plugin_instancesDlg@@YAXXZ 10001084 f   moc_config_plugin_instancesdlgimpl.obj
 0001:000000a5       ??__EcleanUp_instancesCustomTable@@YAXXZ 100010a5 f   moc_instancesCustomTable.obj
 0001:000000c6       ??__EcleanUp_toolWindowBase@@YAXXZ 100010c6 f   moc_toolwindow.obj
 0001:000000e7       ??__EcleanUp_toolWindow@@YAXXZ 100010e7 f   moc_toolwindowimpl.obj
 0001:00000108       ??__EcleanUp_cfg_Table@@YAXXZ 10001108 f   cfg_widgets001:moc_cfg_Table.obj
 0001:0000ac84       $LN85                      1000bc84     moc_config_plugin_instancesdlgimpl.obj
 0001:0000d187       _pre_c_init                1000e187 f   MSVCRT:crtdll.obj
 0001:0000d3ed       ___DllMainCRTStartup       1000e3ed f   MSVCRT:crtdll.obj
 0001:0000d670       $$000000                   1000e670     MSVCRT:sehprolg4.obj
 0001:0000d97c       __unwindfunclet$??0config_plugin_base@@QAE@ABVQString@@00@Z$0 1000e97c f   config_plugin_instances.obj
 0001:0000d985       __unwindfunclet$??0config_plugin_base@@QAE@ABVQString@@00@Z$1 1000e985 f   config_plugin_instances.obj
 0001:0000d991       __unwindfunclet$??0config_plugin_base@@QAE@ABVQString@@00@Z$2 1000e991 f   config_plugin_instances.obj
 0001:0000d99d       __unwindfunclet$??0config_plugin_base@@QAE@ABVQString@@00@Z$3 1000e99d f   config_plugin_instances.obj
 0001:0000d9a9       __ehhandler$??0config_plugin_base@@QAE@ABVQString@@00@Z 1000e9a9 f   config_plugin_instances.obj
 0001:0000d9c4       __unwindfunclet$??0config_plugin_instances@@QAE@ABVQString@@00@Z$0 1000e9c4 f   config_plugin_instances.obj
 0001:0000d9cc       __unwindfunclet$??0config_plugin_instances@@QAE@ABVQString@@00@Z$1 1000e9cc f   config_plugin_instances.obj
 0001:0000d9d7       __unwindfunclet$??0config_plugin_instances@@QAE@ABVQString@@00@Z$2 1000e9d7 f   config_plugin_instances.obj
 0001:0000d9e2       __unwindfunclet$??0config_plugin_instances@@QAE@ABVQString@@00@Z$3 1000e9e2 f   config_plugin_instances.obj
 0001:0000d9f0       __unwindfunclet$??0config_plugin_instances@@QAE@ABVQString@@00@Z$4 1000e9f0 f   config_plugin_instances.obj
 0001:0000d9fe       __unwindfunclet$??0config_plugin_instances@@QAE@ABVQString@@00@Z$5 1000e9fe f   config_plugin_instances.obj
 0001:0000da0d       __unwindfunclet$??0config_plugin_instances@@QAE@ABVQString@@00@Z$6 1000ea0d f   config_plugin_instances.obj
 0001:0000da17       __unwindfunclet$??0config_plugin_instances@@QAE@ABVQString@@00@Z$7 1000ea17 f   config_plugin_instances.obj
 0001:0000da21       __unwindfunclet$??0config_plugin_instances@@QAE@ABVQString@@00@Z$8 1000ea21 f   config_plugin_instances.obj
 0001:0000da3b       __unwindfunclet$??0config_plugin_instances@@QAE@ABVQString@@00@Z$9 1000ea3b f   config_plugin_instances.obj
 0001:0000da45       __unwindfunclet$??0config_plugin_instances@@QAE@ABVQString@@00@Z$10 1000ea45 f   config_plugin_instances.obj
 0001:0000da4f       __unwindfunclet$??0config_plugin_instances@@QAE@ABVQString@@00@Z$11 1000ea4f f   config_plugin_instances.obj
 0001:0000da69       __unwindfunclet$??0config_plugin_instances@@QAE@ABVQString@@00@Z$12 1000ea69 f   config_plugin_instances.obj
 0001:0000da83       __unwindfunclet$??0config_plugin_instances@@QAE@ABVQString@@00@Z$13 1000ea83 f   config_plugin_instances.obj
 0001:0000da9d       __unwindfunclet$??0config_plugin_instances@@QAE@ABVQString@@00@Z$14 1000ea9d f   config_plugin_instances.obj
 0001:0000dab7       __unwindfunclet$??0config_plugin_instances@@QAE@ABVQString@@00@Z$16 1000eab7 f   config_plugin_instances.obj
 0001:0000dac1       __unwindfunclet$??0config_plugin_instances@@QAE@ABVQString@@00@Z$17 1000eac1 f   config_plugin_instances.obj
 0001:0000dadb       __unwindfunclet$??0config_plugin_instances@@QAE@ABVQString@@00@Z$18 1000eadb f   config_plugin_instances.obj
 0001:0000daf5       __unwindfunclet$??0config_plugin_instances@@QAE@ABVQString@@00@Z$19 1000eaf5 f   config_plugin_instances.obj
 0001:0000db14       __unwindfunclet$??0config_plugin_instances@@QAE@ABVQString@@00@Z$20 1000eb14 f   config_plugin_instances.obj
 0001:0000db33       __unwindfunclet$??0config_plugin_instances@@QAE@ABVQString@@00@Z$22 1000eb33 f   config_plugin_instances.obj
 0001:0000db3d       __unwindfunclet$??0config_plugin_instances@@QAE@ABVQString@@00@Z$23 1000eb3d f   config_plugin_instances.obj
 0001:0000db5c       __unwindfunclet$??0config_plugin_instances@@QAE@ABVQString@@00@Z$24 1000eb5c f   config_plugin_instances.obj
 0001:0000db7b       __unwindfunclet$??0config_plugin_instances@@QAE@ABVQString@@00@Z$25 1000eb7b f   config_plugin_instances.obj
 0001:0000db9a       __unwindfunclet$??0config_plugin_instances@@QAE@ABVQString@@00@Z$26 1000eb9a f   config_plugin_instances.obj
 0001:0000dbb9       __ehhandler$??0config_plugin_instances@@QAE@ABVQString@@00@Z 1000ebb9 f   config_plugin_instances.obj
 0001:0000dbd4       __unwindfunclet$??1?$QDict@VQAction@@@@UAE@XZ$0 1000ebd4 f   config_plugin_instances.obj
 0001:0000dbdd       __ehhandler$??1?$QDict@VQAction@@@@UAE@XZ 1000ebdd f   config_plugin_instances.obj
 0001:0000dbf8       __unwindfunclet$??1?$QPtrList@VviewRow@@@@UAE@XZ$0 1000ebf8 f   config_plugin_instances.obj
 0001:0000dbf8       __unwindfunclet$??1?$QPtrList@VgroupRow@@@@UAE@XZ$0 1000ebf8 f   config_plugin_instances.obj
 0001:0000dbf8       __unwindfunclet$??1?$QPtrList@VQPopupMenu@@@@UAE@XZ$0 1000ebf8 f   config_plugin_instances.obj
 0001:0000dbf8       __unwindfunclet$??1?$QPtrList@VdeviceRow@@@@UAE@XZ$0 1000ebf8 f   config_plugin_instances.obj
 0001:0000dc01       __ehhandler$??1?$QPtrList@VviewRow@@@@UAE@XZ 1000ec01 f   config_plugin_instances.obj
 0001:0000dc01       __ehhandler$??1?$QPtrList@VgroupRow@@@@UAE@XZ 1000ec01 f   config_plugin_instances.obj
 0001:0000dc01       __ehhandler$??1?$QPtrList@VQPopupMenu@@@@UAE@XZ 1000ec01 f   config_plugin_instances.obj
 0001:0000dc01       __ehhandler$??1?$QPtrList@VdeviceRow@@@@UAE@XZ 1000ec01 f   config_plugin_instances.obj
 0001:0000dc1c       __unwindfunclet$??1QDockWindowList@@UAE@XZ$0 1000ec1c f   config_plugin_instances.obj
 0001:0000dc25       __unwindfunclet$??1QDockWindowList@@UAE@XZ$1 1000ec25 f   config_plugin_instances.obj
 0001:0000dc2e       __ehhandler$??1QDockWindowList@@UAE@XZ 1000ec2e f   config_plugin_instances.obj
 0001:0000dc49       __unwindfunclet$??1QPopupMenuList@@UAE@XZ$0 1000ec49 f   config_plugin_instances.obj
 0001:0000dc51       __ehhandler$??1QPopupMenuList@@UAE@XZ 1000ec51 f   config_plugin_instances.obj
 0001:0000dc6c       __unwindfunclet$??1config_plugin_base@@UAE@XZ$0 1000ec6c f   config_plugin_instances.obj
 0001:0000dc75       __unwindfunclet$??1config_plugin_base@@UAE@XZ$1 1000ec75 f   config_plugin_instances.obj
 0001:0000dc81       __unwindfunclet$??1config_plugin_base@@UAE@XZ$2 1000ec81 f   config_plugin_instances.obj
 0001:0000dc8d       __ehhandler$??1config_plugin_base@@UAE@XZ 1000ec8d f   config_plugin_instances.obj
 0001:0000dca8       __unwindfunclet$??1config_plugin_instances@@UAE@XZ$0 1000eca8 f   config_plugin_instances.obj
 0001:0000dcb0       __unwindfunclet$??1config_plugin_instances@@UAE@XZ$1 1000ecb0 f   config_plugin_instances.obj
 0001:0000dcbb       __unwindfunclet$??1config_plugin_instances@@UAE@XZ$2 1000ecbb f   config_plugin_instances.obj
 0001:0000dcc6       __unwindfunclet$??1config_plugin_instances@@UAE@XZ$3 1000ecc6 f   config_plugin_instances.obj
 0001:0000dcd4       __unwindfunclet$??1config_plugin_instances@@UAE@XZ$4 1000ecd4 f   config_plugin_instances.obj
 0001:0000dce2       __unwindfunclet$??1config_plugin_instances@@UAE@XZ$5 1000ece2 f   config_plugin_instances.obj
 0001:0000dcf1       __ehhandler$??1config_plugin_instances@@UAE@XZ 1000ecf1 f   config_plugin_instances.obj
 0001:0000dd0c       __unwindfunclet$?about@config_plugin_base@@UAE?AVQString@@XZ$0 1000ed0c f   config_plugin_instances.obj
 0001:0000dd15       __unwindfunclet$?about@config_plugin_base@@UAE?AVQString@@XZ$1 1000ed15 f   config_plugin_instances.obj
 0001:0000dd2f       __ehhandler$?about@config_plugin_base@@UAE?AVQString@@XZ 1000ed2f f   config_plugin_instances.obj
 0001:0000dd4a       __unwindfunclet$?about@config_plugin_instances@@UAE?AVQString@@XZ$0 1000ed4a f   config_plugin_instances.obj
 0001:0000dd53       __unwindfunclet$?about@config_plugin_instances@@UAE?AVQString@@XZ$1 1000ed53 f   config_plugin_instances.obj
 0001:0000dd5c       __unwindfunclet$?about@config_plugin_instances@@UAE?AVQString@@XZ$2 1000ed5c f   config_plugin_instances.obj
 0001:0000dd65       __unwindfunclet$?about@config_plugin_instances@@UAE?AVQString@@XZ$3 1000ed65 f   config_plugin_instances.obj
 0001:0000dd6e       __unwindfunclet$?about@config_plugin_instances@@UAE?AVQString@@XZ$4 1000ed6e f   config_plugin_instances.obj
 0001:0000dd88       __ehhandler$?about@config_plugin_instances@@UAE?AVQString@@XZ 1000ed88 f   config_plugin_instances.obj
 0001:0000dda3       __unwindfunclet$?activate@config_plugin_instances@@UAEX_N@Z$0 1000eda3 f   config_plugin_instances.obj
 0001:0000ddac       __unwindfunclet$?activate@config_plugin_instances@@UAEX_N@Z$2 1000edac f   config_plugin_instances.obj
 0001:0000ddb5       __unwindfunclet$?activate@config_plugin_instances@@UAEX_N@Z$4 1000edb5 f   config_plugin_instances.obj
 0001:0000ddbe       __unwindfunclet$?activate@config_plugin_instances@@UAEX_N@Z$5 1000edbe f   config_plugin_instances.obj
 0001:0000ddc7       __unwindfunclet$?activate@config_plugin_instances@@UAEX_N@Z$6 1000edc7 f   config_plugin_instances.obj
 0001:0000ddd0       __unwindfunclet$?activate@config_plugin_instances@@UAEX_N@Z$7 1000edd0 f   config_plugin_instances.obj
 0001:0000ddd9       __unwindfunclet$?activate@config_plugin_instances@@UAEX_N@Z$8 1000edd9 f   config_plugin_instances.obj
 0001:0000dde2       __unwindfunclet$?activate@config_plugin_instances@@UAEX_N@Z$9 1000ede2 f   config_plugin_instances.obj
 0001:0000ddeb       __unwindfunclet$?activate@config_plugin_instances@@UAEX_N@Z$10 1000edeb f   config_plugin_instances.obj
 0001:0000ddf4       __unwindfunclet$?activate@config_plugin_instances@@UAEX_N@Z$11 1000edf4 f   config_plugin_instances.obj
 0001:0000ddfd       __unwindfunclet$?activate@config_plugin_instances@@UAEX_N@Z$12 1000edfd f   config_plugin_instances.obj
 0001:0000de06       __unwindfunclet$?activate@config_plugin_instances@@UAEX_N@Z$13 1000ee06 f   config_plugin_instances.obj
 0001:0000de0f       __ehhandler$?activate@config_plugin_instances@@UAEX_N@Z 1000ee0f f   config_plugin_instances.obj
 0001:0000de2a       __unwindfunclet$?apply@config_plugin_instances@@UAEXXZ$0 1000ee2a f   config_plugin_instances.obj
 0001:0000de33       __unwindfunclet$?apply@config_plugin_instances@@UAEXXZ$1 1000ee33 f   config_plugin_instances.obj
 0001:0000de3c       __unwindfunclet$?apply@config_plugin_instances@@UAEXXZ$2 1000ee3c f   config_plugin_instances.obj
 0001:0000de45       __ehhandler$?apply@config_plugin_instances@@UAEXXZ 1000ee45 f   config_plugin_instances.obj
 0001:0000de60       __unwindfunclet$?setDirty@config_plugin_instancesDlg@@QAEXXZ$0 1000ee60 f   config_plugin_instances.obj
 0001:0000de60       __unwindfunclet$?closeEvent@config_plugin_instances@@UAEXPAVQCloseEvent@@@Z$0 1000ee60 f   config_plugin_instances.obj
 0001:0000de69       __ehhandler$?setDirty@config_plugin_instancesDlg@@QAEXXZ 1000ee69 f   config_plugin_instances.obj
 0001:0000de69       __ehhandler$?closeEvent@config_plugin_instances@@UAEXPAVQCloseEvent@@@Z 1000ee69 f   config_plugin_instances.obj
 0001:0000de84       __unwindfunclet$?menus@config_plugin_instances@@UAE?AVQPopupMenuList@@XZ$0 1000ee84 f   config_plugin_instances.obj
 0001:0000de9d       __ehhandler$?menus@config_plugin_instances@@UAE?AVQPopupMenuList@@XZ 1000ee9d f   config_plugin_instances.obj
 0001:0000deb8       __unwindfunclet$?navigate@config_plugin_instances@@UAEXABVQString@@0@Z$0 1000eeb8 f   config_plugin_instances.obj
 0001:0000dec1       __unwindfunclet$?navigate@config_plugin_instances@@UAEXABVQString@@0@Z$1 1000eec1 f   config_plugin_instances.obj
 0001:0000deca       __unwindfunclet$?navigate@config_plugin_instances@@UAEXABVQString@@0@Z$2 1000eeca f   config_plugin_instances.obj
 0001:0000ded3       __ehhandler$?navigate@config_plugin_instances@@UAEXABVQString@@0@Z 1000eed3 f   config_plugin_instances.obj
 0001:0000deee       __unwindfunclet$?reply@config_plugin_instances@@UAEXPAVresponse@@@Z$0 1000eeee f   config_plugin_instances.obj
 0001:0000def7       __unwindfunclet$?reply@config_plugin_instances@@UAEXPAVresponse@@@Z$1 1000eef7 f   config_plugin_instances.obj
 0001:0000df00       __unwindfunclet$?reply@config_plugin_instances@@UAEXPAVresponse@@@Z$2 1000ef00 f   config_plugin_instances.obj
 0001:0000df09       __unwindfunclet$?reply@config_plugin_instances@@UAEXPAVresponse@@@Z$3 1000ef09 f   config_plugin_instances.obj
 0001:0000df12       __unwindfunclet$?reply@config_plugin_instances@@UAEXPAVresponse@@@Z$4 1000ef12 f   config_plugin_instances.obj
 0001:0000df1b       __unwindfunclet$?reply@config_plugin_instances@@UAEXPAVresponse@@@Z$5 1000ef1b f   config_plugin_instances.obj
 0001:0000df24       __unwindfunclet$?reply@config_plugin_instances@@UAEXPAVresponse@@@Z$6 1000ef24 f   config_plugin_instances.obj
 0001:0000df2d       __unwindfunclet$?reply@config_plugin_instances@@UAEXPAVresponse@@@Z$7 1000ef2d f   config_plugin_instances.obj
 0001:0000df36       __unwindfunclet$?reply@config_plugin_instances@@UAEXPAVresponse@@@Z$8 1000ef36 f   config_plugin_instances.obj
 0001:0000df3f       __unwindfunclet$?reply@config_plugin_instances@@UAEXPAVresponse@@@Z$9 1000ef3f f   config_plugin_instances.obj
 0001:0000df48       __unwindfunclet$?reply@config_plugin_instances@@UAEXPAVresponse@@@Z$10 1000ef48 f   config_plugin_instances.obj
 0001:0000df51       __unwindfunclet$?reply@config_plugin_instances@@UAEXPAVresponse@@@Z$11 1000ef51 f   config_plugin_instances.obj
 0001:0000df5a       __unwindfunclet$?reply@config_plugin_instances@@UAEXPAVresponse@@@Z$12 1000ef5a f   config_plugin_instances.obj
 0001:0000df63       __unwindfunclet$?reply@config_plugin_instances@@UAEXPAVresponse@@@Z$13 1000ef63 f   config_plugin_instances.obj
 0001:0000df6c       __unwindfunclet$?reply@config_plugin_instances@@UAEXPAVresponse@@@Z$14 1000ef6c f   config_plugin_instances.obj
 0001:0000df75       __unwindfunclet$?reply@config_plugin_instances@@UAEXPAVresponse@@@Z$15 1000ef75 f   config_plugin_instances.obj
 0001:0000df7e       __unwindfunclet$?reply@config_plugin_instances@@UAEXPAVresponse@@@Z$16 1000ef7e f   config_plugin_instances.obj
 0001:0000df87       __unwindfunclet$?reply@config_plugin_instances@@UAEXPAVresponse@@@Z$17 1000ef87 f   config_plugin_instances.obj
 0001:0000df90       __unwindfunclet$?reply@config_plugin_instances@@UAEXPAVresponse@@@Z$18 1000ef90 f   config_plugin_instances.obj
 0001:0000df99       __unwindfunclet$?reply@config_plugin_instances@@UAEXPAVresponse@@@Z$19 1000ef99 f   config_plugin_instances.obj
 0001:0000dfa2       __unwindfunclet$?reply@config_plugin_instances@@UAEXPAVresponse@@@Z$20 1000efa2 f   config_plugin_instances.obj
 0001:0000dfab       __unwindfunclet$?reply@config_plugin_instances@@UAEXPAVresponse@@@Z$22 1000efab f   config_plugin_instances.obj
 0001:0000dfb4       __ehhandler$?reply@config_plugin_instances@@UAEXPAVresponse@@@Z 1000efb4 f   config_plugin_instances.obj
 0001:0000dfcf       __unwindfunclet$?toolbars@config_plugin_instances@@UAE?AVQDockWindowList@@XZ$0 1000efcf f   config_plugin_instances.obj
 0001:0000dfe8       __ehhandler$?toolbars@config_plugin_instances@@UAE?AVQDockWindowList@@XZ 1000efe8 f   config_plugin_instances.obj
 0001:0000e003       __unwindfunclet$??0config_plugin_instancesDlg@@QAE@ABVQString@@PAVQWidget@@PBDI@Z$0 1000f003 f   config_plugin_instancesdlgimpl.obj
 0001:0000e00b       __unwindfunclet$??0config_plugin_instancesDlg@@QAE@ABVQString@@PAVQWidget@@PBDI@Z$1 1000f00b f   config_plugin_instancesdlgimpl.obj
 0001:0000e01a       __unwindfunclet$??0config_plugin_instancesDlg@@QAE@ABVQString@@PAVQWidget@@PBDI@Z$2 1000f01a f   config_plugin_instancesdlgimpl.obj
 0001:0000e029       __unwindfunclet$??0config_plugin_instancesDlg@@QAE@ABVQString@@PAVQWidget@@PBDI@Z$3 1000f029 f   config_plugin_instancesdlgimpl.obj
 0001:0000e038       __unwindfunclet$??0config_plugin_instancesDlg@@QAE@ABVQString@@PAVQWidget@@PBDI@Z$4 1000f038 f   config_plugin_instancesdlgimpl.obj
 0001:0000e047       __unwindfunclet$??0config_plugin_instancesDlg@@QAE@ABVQString@@PAVQWidget@@PBDI@Z$5 1000f047 f   config_plugin_instancesdlgimpl.obj
 0001:0000e056       __unwindfunclet$??0config_plugin_instancesDlg@@QAE@ABVQString@@PAVQWidget@@PBDI@Z$6 1000f056 f   config_plugin_instancesdlgimpl.obj
 0001:0000e065       __unwindfunclet$??0config_plugin_instancesDlg@@QAE@ABVQString@@PAVQWidget@@PBDI@Z$7 1000f065 f   config_plugin_instancesdlgimpl.obj
 0001:0000e074       __unwindfunclet$??0config_plugin_instancesDlg@@QAE@ABVQString@@PAVQWidget@@PBDI@Z$8 1000f074 f   config_plugin_instancesdlgimpl.obj
 0001:0000e083       __unwindfunclet$??0config_plugin_instancesDlg@@QAE@ABVQString@@PAVQWidget@@PBDI@Z$9 1000f083 f   config_plugin_instancesdlgimpl.obj
 0001:0000e092       __unwindfunclet$??0config_plugin_instancesDlg@@QAE@ABVQString@@PAVQWidget@@PBDI@Z$10 1000f092 f   config_plugin_instancesdlgimpl.obj
 0001:0000e09b       __unwindfunclet$??0config_plugin_instancesDlg@@QAE@ABVQString@@PAVQWidget@@PBDI@Z$11 1000f09b f   config_plugin_instancesdlgimpl.obj
 0001:0000e0a4       __unwindfunclet$??0config_plugin_instancesDlg@@QAE@ABVQString@@PAVQWidget@@PBDI@Z$12 1000f0a4 f   config_plugin_instancesdlgimpl.obj
 0001:0000e0ad       __unwindfunclet$??0config_plugin_instancesDlg@@QAE@ABVQString@@PAVQWidget@@PBDI@Z$13 1000f0ad f   config_plugin_instancesdlgimpl.obj
 0001:0000e0b6       __unwindfunclet$??0config_plugin_instancesDlg@@QAE@ABVQString@@PAVQWidget@@PBDI@Z$14 1000f0b6 f   config_plugin_instancesdlgimpl.obj
 0001:0000e0bf       __unwindfunclet$??0config_plugin_instancesDlg@@QAE@ABVQString@@PAVQWidget@@PBDI@Z$15 1000f0bf f   config_plugin_instancesdlgimpl.obj
 0001:0000e0c8       __unwindfunclet$??0config_plugin_instancesDlg@@QAE@ABVQString@@PAVQWidget@@PBDI@Z$16 1000f0c8 f   config_plugin_instancesdlgimpl.obj
 0001:0000e0d1       __unwindfunclet$??0config_plugin_instancesDlg@@QAE@ABVQString@@PAVQWidget@@PBDI@Z$17 1000f0d1 f   config_plugin_instancesdlgimpl.obj
 0001:0000e0da       __unwindfunclet$??0config_plugin_instancesDlg@@QAE@ABVQString@@PAVQWidget@@PBDI@Z$18 1000f0da f   config_plugin_instancesdlgimpl.obj
 0001:0000e0e3       __unwindfunclet$??0config_plugin_instancesDlg@@QAE@ABVQString@@PAVQWidget@@PBDI@Z$19 1000f0e3 f   config_plugin_instancesdlgimpl.obj
 0001:0000e0ec       __unwindfunclet$??0config_plugin_instancesDlg@@QAE@ABVQString@@PAVQWidget@@PBDI@Z$20 1000f0ec f   config_plugin_instancesdlgimpl.obj
 0001:0000e0f5       __unwindfunclet$??0config_plugin_instancesDlg@@QAE@ABVQString@@PAVQWidget@@PBDI@Z$21 1000f0f5 f   config_plugin_instancesdlgimpl.obj
 0001:0000e0fe       __unwindfunclet$??0config_plugin_instancesDlg@@QAE@ABVQString@@PAVQWidget@@PBDI@Z$22 1000f0fe f   config_plugin_instancesdlgimpl.obj
 0001:0000e107       __unwindfunclet$??0config_plugin_instancesDlg@@QAE@ABVQString@@PAVQWidget@@PBDI@Z$23 1000f107 f   config_plugin_instancesdlgimpl.obj
 0001:0000e110       __unwindfunclet$??0config_plugin_instancesDlg@@QAE@ABVQString@@PAVQWidget@@PBDI@Z$24 1000f110 f   config_plugin_instancesdlgimpl.obj
 0001:0000e119       __unwindfunclet$??0config_plugin_instancesDlg@@QAE@ABVQString@@PAVQWidget@@PBDI@Z$25 1000f119 f   config_plugin_instancesdlgimpl.obj
 0001:0000e122       __unwindfunclet$??0config_plugin_instancesDlg@@QAE@ABVQString@@PAVQWidget@@PBDI@Z$26 1000f122 f   config_plugin_instancesdlgimpl.obj
 0001:0000e12b       __unwindfunclet$??0config_plugin_instancesDlg@@QAE@ABVQString@@PAVQWidget@@PBDI@Z$27 1000f12b f   config_plugin_instancesdlgimpl.obj
 0001:0000e134       __unwindfunclet$??0config_plugin_instancesDlg@@QAE@ABVQString@@PAVQWidget@@PBDI@Z$28 1000f134 f   config_plugin_instancesdlgimpl.obj
 0001:0000e13d       __unwindfunclet$??0config_plugin_instancesDlg@@QAE@ABVQString@@PAVQWidget@@PBDI@Z$29 1000f13d f   config_plugin_instancesdlgimpl.obj
 0001:0000e146       __unwindfunclet$??0config_plugin_instancesDlg@@QAE@ABVQString@@PAVQWidget@@PBDI@Z$30 1000f146 f   config_plugin_instancesdlgimpl.obj
 0001:0000e14f       __unwindfunclet$??0config_plugin_instancesDlg@@QAE@ABVQString@@PAVQWidget@@PBDI@Z$31 1000f14f f   config_plugin_instancesdlgimpl.obj
 0001:0000e158       __unwindfunclet$??0config_plugin_instancesDlg@@QAE@ABVQString@@PAVQWidget@@PBDI@Z$32 1000f158 f   config_plugin_instancesdlgimpl.obj
 0001:0000e161       __unwindfunclet$??0config_plugin_instancesDlg@@QAE@ABVQString@@PAVQWidget@@PBDI@Z$33 1000f161 f   config_plugin_instancesdlgimpl.obj
 0001:0000e16a       __unwindfunclet$??0config_plugin_instancesDlg@@QAE@ABVQString@@PAVQWidget@@PBDI@Z$34 1000f16a f   config_plugin_instancesdlgimpl.obj
 0001:0000e173       __unwindfunclet$??0config_plugin_instancesDlg@@QAE@ABVQString@@PAVQWidget@@PBDI@Z$35 1000f173 f   config_plugin_instancesdlgimpl.obj
 0001:0000e17c       __unwindfunclet$??0config_plugin_instancesDlg@@QAE@ABVQString@@PAVQWidget@@PBDI@Z$36 1000f17c f   config_plugin_instancesdlgimpl.obj
 0001:0000e185       __unwindfunclet$??0config_plugin_instancesDlg@@QAE@ABVQString@@PAVQWidget@@PBDI@Z$37 1000f185 f   config_plugin_instancesdlgimpl.obj
 0001:0000e18e       __ehhandler$??0config_plugin_instancesDlg@@QAE@ABVQString@@PAVQWidget@@PBDI@Z 1000f18e f   config_plugin_instancesdlgimpl.obj
 0001:0000e1a9       __unwindfunclet$??1config_plugin_instancesDlg@@UAE@XZ$0 1000f1a9 f   config_plugin_instancesdlgimpl.obj
 0001:0000e1b1       __unwindfunclet$??1config_plugin_instancesDlg@@UAE@XZ$1 1000f1b1 f   config_plugin_instancesdlgimpl.obj
 0001:0000e1c0       __unwindfunclet$??1config_plugin_instancesDlg@@UAE@XZ$2 1000f1c0 f   config_plugin_instancesdlgimpl.obj
 0001:0000e1cf       __unwindfunclet$??1config_plugin_instancesDlg@@UAE@XZ$3 1000f1cf f   config_plugin_instancesdlgimpl.obj
 0001:0000e1de       __unwindfunclet$??1config_plugin_instancesDlg@@UAE@XZ$4 1000f1de f   config_plugin_instancesdlgimpl.obj
 0001:0000e1ed       __unwindfunclet$??1config_plugin_instancesDlg@@UAE@XZ$5 1000f1ed f   config_plugin_instancesdlgimpl.obj
 0001:0000e1fc       __unwindfunclet$??1config_plugin_instancesDlg@@UAE@XZ$6 1000f1fc f   config_plugin_instancesdlgimpl.obj
 0001:0000e20b       __unwindfunclet$??1config_plugin_instancesDlg@@UAE@XZ$7 1000f20b f   config_plugin_instancesdlgimpl.obj
 0001:0000e21a       __unwindfunclet$??1config_plugin_instancesDlg@@UAE@XZ$8 1000f21a f   config_plugin_instancesdlgimpl.obj
 0001:0000e229       __ehhandler$??1config_plugin_instancesDlg@@UAE@XZ 1000f229 f   config_plugin_instancesdlgimpl.obj
 0001:0000e244       __unwindfunclet$?addDeviceNodeFromRow@config_plugin_instancesDlg@@QAE_NH@Z$0 1000f244 f   config_plugin_instancesdlgimpl.obj
 0001:0000e24e       __unwindfunclet$?addDeviceNodeFromRow@config_plugin_instancesDlg@@QAE_NH@Z$1 1000f24e f   config_plugin_instancesdlgimpl.obj
 0001:0000e257       __unwindfunclet$?addDeviceNodeFromRow@config_plugin_instancesDlg@@QAE_NH@Z$2 1000f257 f   config_plugin_instancesdlgimpl.obj
 0001:0000e260       __unwindfunclet$?addDeviceNodeFromRow@config_plugin_instancesDlg@@QAE_NH@Z$3 1000f260 f   config_plugin_instancesdlgimpl.obj
 0001:0000e269       __unwindfunclet$?addDeviceNodeFromRow@config_plugin_instancesDlg@@QAE_NH@Z$4 1000f269 f   config_plugin_instancesdlgimpl.obj
 0001:0000e272       __unwindfunclet$?addDeviceNodeFromRow@config_plugin_instancesDlg@@QAE_NH@Z$5 1000f272 f   config_plugin_instancesdlgimpl.obj
 0001:0000e27b       __unwindfunclet$?addDeviceNodeFromRow@config_plugin_instancesDlg@@QAE_NH@Z$6 1000f27b f   config_plugin_instancesdlgimpl.obj
 0001:0000e284       __unwindfunclet$?addDeviceNodeFromRow@config_plugin_instancesDlg@@QAE_NH@Z$7 1000f284 f   config_plugin_instancesdlgimpl.obj
 0001:0000e28d       __unwindfunclet$?addDeviceNodeFromRow@config_plugin_instancesDlg@@QAE_NH@Z$8 1000f28d f   config_plugin_instancesdlgimpl.obj
 0001:0000e296       __unwindfunclet$?addDeviceNodeFromRow@config_plugin_instancesDlg@@QAE_NH@Z$9 1000f296 f   config_plugin_instancesdlgimpl.obj
 0001:0000e29f       __unwindfunclet$?addDeviceNodeFromRow@config_plugin_instancesDlg@@QAE_NH@Z$10 1000f29f f   config_plugin_instancesdlgimpl.obj
 0001:0000e2a8       __unwindfunclet$?addDeviceNodeFromRow@config_plugin_instancesDlg@@QAE_NH@Z$11 1000f2a8 f   config_plugin_instancesdlgimpl.obj
 0001:0000e2b1       __unwindfunclet$?addDeviceNodeFromRow@config_plugin_instancesDlg@@QAE_NH@Z$12 1000f2b1 f   config_plugin_instancesdlgimpl.obj
 0001:0000e2ba       __unwindfunclet$?addDeviceNodeFromRow@config_plugin_instancesDlg@@QAE_NH@Z$13 1000f2ba f   config_plugin_instancesdlgimpl.obj
 0001:0000e2c3       __unwindfunclet$?addDeviceNodeFromRow@config_plugin_instancesDlg@@QAE_NH@Z$15 1000f2c3 f   config_plugin_instancesdlgimpl.obj
 0001:0000e2cc       __unwindfunclet$?addDeviceNodeFromRow@config_plugin_instancesDlg@@QAE_NH@Z$16 1000f2cc f   config_plugin_instancesdlgimpl.obj
 0001:0000e2d5       __unwindfunclet$?addDeviceNodeFromRow@config_plugin_instancesDlg@@QAE_NH@Z$17 1000f2d5 f   config_plugin_instancesdlgimpl.obj
 0001:0000e2de       __unwindfunclet$?addDeviceNodeFromRow@config_plugin_instancesDlg@@QAE_NH@Z$19 1000f2de f   config_plugin_instancesdlgimpl.obj
 0001:0000e2e7       __unwindfunclet$?addDeviceNodeFromRow@config_plugin_instancesDlg@@QAE_NH@Z$20 1000f2e7 f   config_plugin_instancesdlgimpl.obj
 0001:0000e2f0       __unwindfunclet$?addDeviceNodeFromRow@config_plugin_instancesDlg@@QAE_NH@Z$21 1000f2f0 f   config_plugin_instancesdlgimpl.obj
 0001:0000e2f9       __unwindfunclet$?addDeviceNodeFromRow@config_plugin_instancesDlg@@QAE_NH@Z$22 1000f2f9 f   config_plugin_instancesdlgimpl.obj
 0001:0000e302       __unwindfunclet$?addDeviceNodeFromRow@config_plugin_instancesDlg@@QAE_NH@Z$23 1000f302 f   config_plugin_instancesdlgimpl.obj
 0001:0000e30b       __unwindfunclet$?addDeviceNodeFromRow@config_plugin_instancesDlg@@QAE_NH@Z$24 1000f30b f   config_plugin_instancesdlgimpl.obj
 0001:0000e314       __unwindfunclet$?addDeviceNodeFromRow@config_plugin_instancesDlg@@QAE_NH@Z$25 1000f314 f   config_plugin_instancesdlgimpl.obj
 0001:0000e31d       __unwindfunclet$?addDeviceNodeFromRow@config_plugin_instancesDlg@@QAE_NH@Z$26 1000f31d f   config_plugin_instancesdlgimpl.obj
 0001:0000e326       __ehhandler$?addDeviceNodeFromRow@config_plugin_instancesDlg@@QAE_NH@Z 1000f326 f   config_plugin_instancesdlgimpl.obj
 0001:0000e341       __unwindfunclet$?addGroupToInstanceNodeFromRow@config_plugin_instancesDlg@@QAE_NHVQString@@@Z$0 1000f341 f   config_plugin_instancesdlgimpl.obj
 0001:0000e34a       __unwindfunclet$?addGroupToInstanceNodeFromRow@config_plugin_instancesDlg@@QAE_NHVQString@@@Z$1 1000f34a f   config_plugin_instancesdlgimpl.obj
 0001:0000e354       __unwindfunclet$?addGroupToInstanceNodeFromRow@config_plugin_instancesDlg@@QAE_NHVQString@@@Z$2 1000f354 f   config_plugin_instancesdlgimpl.obj
 0001:0000e35d       __unwindfunclet$?addGroupToInstanceNodeFromRow@config_plugin_instancesDlg@@QAE_NHVQString@@@Z$3 1000f35d f   config_plugin_instancesdlgimpl.obj
 0001:0000e366       __unwindfunclet$?addGroupToInstanceNodeFromRow@config_plugin_instancesDlg@@QAE_NHVQString@@@Z$4 1000f366 f   config_plugin_instancesdlgimpl.obj
 0001:0000e36f       __unwindfunclet$?addGroupToInstanceNodeFromRow@config_plugin_instancesDlg@@QAE_NHVQString@@@Z$5 1000f36f f   config_plugin_instancesdlgimpl.obj
 0001:0000e378       __unwindfunclet$?addGroupToInstanceNodeFromRow@config_plugin_instancesDlg@@QAE_NHVQString@@@Z$6 1000f378 f   config_plugin_instancesdlgimpl.obj
 0001:0000e381       __unwindfunclet$?addGroupToInstanceNodeFromRow@config_plugin_instancesDlg@@QAE_NHVQString@@@Z$14 1000f381 f   config_plugin_instancesdlgimpl.obj
 0001:0000e38a       __unwindfunclet$?addGroupToInstanceNodeFromRow@config_plugin_instancesDlg@@QAE_NHVQString@@@Z$7 1000f38a f   config_plugin_instancesdlgimpl.obj
 0001:0000e393       __unwindfunclet$?addGroupToInstanceNodeFromRow@config_plugin_instancesDlg@@QAE_NHVQString@@@Z$8 1000f393 f   config_plugin_instancesdlgimpl.obj
 0001:0000e39c       __unwindfunclet$?addGroupToInstanceNodeFromRow@config_plugin_instancesDlg@@QAE_NHVQString@@@Z$9 1000f39c f   config_plugin_instancesdlgimpl.obj
 0001:0000e3a5       __unwindfunclet$?addGroupToInstanceNodeFromRow@config_plugin_instancesDlg@@QAE_NHVQString@@@Z$10 1000f3a5 f   config_plugin_instancesdlgimpl.obj
 0001:0000e3ae       __unwindfunclet$?addGroupToInstanceNodeFromRow@config_plugin_instancesDlg@@QAE_NHVQString@@@Z$11 1000f3ae f   config_plugin_instancesdlgimpl.obj
 0001:0000e3b7       __unwindfunclet$?addGroupToInstanceNodeFromRow@config_plugin_instancesDlg@@QAE_NHVQString@@@Z$12 1000f3b7 f   config_plugin_instancesdlgimpl.obj
 0001:0000e3c0       __ehhandler$?addGroupToInstanceNodeFromRow@config_plugin_instancesDlg@@QAE_NHVQString@@@Z 1000f3c0 f   config_plugin_instancesdlgimpl.obj
 0001:0000e3db       __unwindfunclet$?addViewNodeFromRow@config_plugin_instancesDlg@@QAE_NH@Z$0 1000f3db f   config_plugin_instancesdlgimpl.obj
 0001:0000e3e5       __unwindfunclet$?addViewNodeFromRow@config_plugin_instancesDlg@@QAE_NH@Z$1 1000f3e5 f   config_plugin_instancesdlgimpl.obj
 0001:0000e3ee       __unwindfunclet$?addViewNodeFromRow@config_plugin_instancesDlg@@QAE_NH@Z$2 1000f3ee f   config_plugin_instancesdlgimpl.obj
 0001:0000e3f7       __unwindfunclet$?addViewNodeFromRow@config_plugin_instancesDlg@@QAE_NH@Z$3 1000f3f7 f   config_plugin_instancesdlgimpl.obj
 0001:0000e400       __unwindfunclet$?addViewNodeFromRow@config_plugin_instancesDlg@@QAE_NH@Z$4 1000f400 f   config_plugin_instancesdlgimpl.obj
 0001:0000e409       __unwindfunclet$?addViewNodeFromRow@config_plugin_instancesDlg@@QAE_NH@Z$5 1000f409 f   config_plugin_instancesdlgimpl.obj
 0001:0000e412       __unwindfunclet$?addViewNodeFromRow@config_plugin_instancesDlg@@QAE_NH@Z$6 1000f412 f   config_plugin_instancesdlgimpl.obj
 0001:0000e41b       __unwindfunclet$?addViewNodeFromRow@config_plugin_instancesDlg@@QAE_NH@Z$7 1000f41b f   config_plugin_instancesdlgimpl.obj
 0001:0000e424       __unwindfunclet$?addViewNodeFromRow@config_plugin_instancesDlg@@QAE_NH@Z$8 1000f424 f   config_plugin_instancesdlgimpl.obj
 0001:0000e42d       __unwindfunclet$?addViewNodeFromRow@config_plugin_instancesDlg@@QAE_NH@Z$9 1000f42d f   config_plugin_instancesdlgimpl.obj
 0001:0000e436       __unwindfunclet$?addViewNodeFromRow@config_plugin_instancesDlg@@QAE_NH@Z$10 1000f436 f   config_plugin_instancesdlgimpl.obj
 0001:0000e43f       __unwindfunclet$?addViewNodeFromRow@config_plugin_instancesDlg@@QAE_NH@Z$11 1000f43f f   config_plugin_instancesdlgimpl.obj
 0001:0000e448       __unwindfunclet$?addViewNodeFromRow@config_plugin_instancesDlg@@QAE_NH@Z$12 1000f448 f   config_plugin_instancesdlgimpl.obj
 0001:0000e451       __ehhandler$?addViewNodeFromRow@config_plugin_instancesDlg@@QAE_NH@Z 1000f451 f   config_plugin_instancesdlgimpl.obj
 0001:0000e46c       __unwindfunclet$?clipboardDataChange@config_plugin_instancesDlg@@QAEXXZ$0 1000f46c f   config_plugin_instancesdlgimpl.obj
 0001:0000e475       __unwindfunclet$?clipboardDataChange@config_plugin_instancesDlg@@QAEXXZ$1 1000f475 f   config_plugin_instancesdlgimpl.obj
 0001:0000e47e       __unwindfunclet$?clipboardDataChange@config_plugin_instancesDlg@@QAEXXZ$2 1000f47e f   config_plugin_instancesdlgimpl.obj
 0001:0000e487       __unwindfunclet$?clipboardDataChange@config_plugin_instancesDlg@@QAEXXZ$3 1000f487 f   config_plugin_instancesdlgimpl.obj
 0001:0000e490       __unwindfunclet$?clipboardDataChange@config_plugin_instancesDlg@@QAEXXZ$4 1000f490 f   config_plugin_instancesdlgimpl.obj
 0001:0000e499       __unwindfunclet$?clipboardDataChange@config_plugin_instancesDlg@@QAEXXZ$5 1000f499 f   config_plugin_instancesdlgimpl.obj
 0001:0000e4a2       __unwindfunclet$?clipboardDataChange@config_plugin_instancesDlg@@QAEXXZ$6 1000f4a2 f   config_plugin_instancesdlgimpl.obj
 0001:0000e4ab       __unwindfunclet$?clipboardDataChange@config_plugin_instancesDlg@@QAEXXZ$7 1000f4ab f   config_plugin_instancesdlgimpl.obj
 0001:0000e4b4       __unwindfunclet$?clipboardDataChange@config_plugin_instancesDlg@@QAEXXZ$8 1000f4b4 f   config_plugin_instancesdlgimpl.obj
 0001:0000e4bd       __unwindfunclet$?clipboardDataChange@config_plugin_instancesDlg@@QAEXXZ$9 1000f4bd f   config_plugin_instancesdlgimpl.obj
 0001:0000e4c6       __ehhandler$?clipboardDataChange@config_plugin_instancesDlg@@QAEXXZ 1000f4c6 f   config_plugin_instancesdlgimpl.obj
 0001:0000e4e1       __unwindfunclet$?copySelectedToClipboard@config_plugin_instancesDlg@@QAEXXZ$0 1000f4e1 f   config_plugin_instancesdlgimpl.obj
 0001:0000e4ea       __unwindfunclet$?copySelectedToClipboard@config_plugin_instancesDlg@@QAEXXZ$1 1000f4ea f   config_plugin_instancesdlgimpl.obj
 0001:0000e4f3       __unwindfunclet$?copySelectedToClipboard@config_plugin_instancesDlg@@QAEXXZ$2 1000f4f3 f   config_plugin_instancesdlgimpl.obj
 0001:0000e4fc       __unwindfunclet$?copySelectedToClipboard@config_plugin_instancesDlg@@QAEXXZ$3 1000f4fc f   config_plugin_instancesdlgimpl.obj
 0001:0000e505       __unwindfunclet$?copySelectedToClipboard@config_plugin_instancesDlg@@QAEXXZ$4 1000f505 f   config_plugin_instancesdlgimpl.obj
 0001:0000e50e       __unwindfunclet$?copySelectedToClipboard@config_plugin_instancesDlg@@QAEXXZ$6 1000f50e f   config_plugin_instancesdlgimpl.obj
 0001:0000e517       __unwindfunclet$?copySelectedToClipboard@config_plugin_instancesDlg@@QAEXXZ$7 1000f517 f   config_plugin_instancesdlgimpl.obj
 0001:0000e520       __unwindfunclet$?copySelectedToClipboard@config_plugin_instancesDlg@@QAEXXZ$8 1000f520 f   config_plugin_instancesdlgimpl.obj
 0001:0000e529       __unwindfunclet$?copySelectedToClipboard@config_plugin_instancesDlg@@QAEXXZ$9 1000f529 f   config_plugin_instancesdlgimpl.obj
 0001:0000e532       __unwindfunclet$?copySelectedToClipboard@config_plugin_instancesDlg@@QAEXXZ$10 1000f532 f   config_plugin_instancesdlgimpl.obj
 0001:0000e53b       __unwindfunclet$?copySelectedToClipboard@config_plugin_instancesDlg@@QAEXXZ$11 1000f53b f   config_plugin_instancesdlgimpl.obj
 0001:0000e544       __unwindfunclet$?copySelectedToClipboard@config_plugin_instancesDlg@@QAEXXZ$12 1000f544 f   config_plugin_instancesdlgimpl.obj
 0001:0000e54d       __unwindfunclet$?copySelectedToClipboard@config_plugin_instancesDlg@@QAEXXZ$13 1000f54d f   config_plugin_instancesdlgimpl.obj
 0001:0000e556       __unwindfunclet$?copySelectedToClipboard@config_plugin_instancesDlg@@QAEXXZ$15 1000f556 f   config_plugin_instancesdlgimpl.obj
 0001:0000e55f       __unwindfunclet$?copySelectedToClipboard@config_plugin_instancesDlg@@QAEXXZ$16 1000f55f f   config_plugin_instancesdlgimpl.obj
 0001:0000e568       __ehhandler$?copySelectedToClipboard@config_plugin_instancesDlg@@QAEXXZ 1000f568 f   config_plugin_instancesdlgimpl.obj
 0001:0000e583       __unwindfunclet$?deviceInstanceChanged@config_plugin_instancesDlg@@QAEXHH@Z$0 1000f583 f   config_plugin_instancesdlgimpl.obj
 0001:0000e58c       __unwindfunclet$?deviceInstanceChanged@config_plugin_instancesDlg@@QAEXHH@Z$1 1000f58c f   config_plugin_instancesdlgimpl.obj
 0001:0000e595       __ehhandler$?deviceInstanceChanged@config_plugin_instancesDlg@@QAEXHH@Z 1000f595 f   config_plugin_instancesdlgimpl.obj
 0001:0000e5b0       __unwindfunclet$?doCreateNewInstance@config_plugin_instancesDlg@@QAEXXZ$0 1000f5b0 f   config_plugin_instancesdlgimpl.obj
 0001:0000e5b9       __unwindfunclet$?doCreateNewInstance@config_plugin_instancesDlg@@QAEXXZ$1 1000f5b9 f   config_plugin_instancesdlgimpl.obj
 0001:0000e5c2       __unwindfunclet$?doCreateNewInstance@config_plugin_instancesDlg@@QAEXXZ$4 1000f5c2 f   config_plugin_instancesdlgimpl.obj
 0001:0000e5cb       __unwindfunclet$?doCreateNewInstance@config_plugin_instancesDlg@@QAEXXZ$10 1000f5cb f   config_plugin_instancesdlgimpl.obj
 0001:0000e5d4       __unwindfunclet$?doCreateNewInstance@config_plugin_instancesDlg@@QAEXXZ$6 1000f5d4 f   config_plugin_instancesdlgimpl.obj
 0001:0000e5dd       __unwindfunclet$?doCreateNewInstance@config_plugin_instancesDlg@@QAEXXZ$11 1000f5dd f   config_plugin_instancesdlgimpl.obj
 0001:0000e5e6       __unwindfunclet$?doCreateNewInstance@config_plugin_instancesDlg@@QAEXXZ$8 1000f5e6 f   config_plugin_instancesdlgimpl.obj
 0001:0000e5ef       __unwindfunclet$?doCreateNewInstance@config_plugin_instancesDlg@@QAEXXZ$2 1000f5ef f   config_plugin_instancesdlgimpl.obj
 0001:0000e5f8       __unwindfunclet$?doCreateNewInstance@config_plugin_instancesDlg@@QAEXXZ$9 1000f5f8 f   config_plugin_instancesdlgimpl.obj
 0001:0000e601       __ehhandler$?doCreateNewInstance@config_plugin_instancesDlg@@QAEXXZ 1000f601 f   config_plugin_instancesdlgimpl.obj
 0001:0000e61c       __unwindfunclet$?doDeleteInstance@config_plugin_instancesDlg@@QAEXXZ$0 1000f61c f   config_plugin_instancesdlgimpl.obj
 0001:0000e625       __unwindfunclet$?doDeleteInstance@config_plugin_instancesDlg@@QAEXXZ$1 1000f625 f   config_plugin_instancesdlgimpl.obj
 0001:0000e62e       __unwindfunclet$?doDeleteInstance@config_plugin_instancesDlg@@QAEXXZ$2 1000f62e f   config_plugin_instancesdlgimpl.obj
 0001:0000e637       __unwindfunclet$?doDeleteInstance@config_plugin_instancesDlg@@QAEXXZ$3 1000f637 f   config_plugin_instancesdlgimpl.obj
 0001:0000e640       __unwindfunclet$?doDeleteInstance@config_plugin_instancesDlg@@QAEXXZ$4 1000f640 f   config_plugin_instancesdlgimpl.obj
 0001:0000e649       __unwindfunclet$?doDeleteInstance@config_plugin_instancesDlg@@QAEXXZ$14 1000f649 f   config_plugin_instancesdlgimpl.obj
 0001:0000e655       __unwindfunclet$?doDeleteInstance@config_plugin_instancesDlg@@QAEXXZ$15 1000f655 f   config_plugin_instancesdlgimpl.obj
 0001:0000e65f       __unwindfunclet$?doDeleteInstance@config_plugin_instancesDlg@@QAEXXZ$16 1000f65f f   config_plugin_instancesdlgimpl.obj
 0001:0000e668       __unwindfunclet$?doDeleteInstance@config_plugin_instancesDlg@@QAEXXZ$17 1000f668 f   config_plugin_instancesdlgimpl.obj
 0001:0000e671       __unwindfunclet$?doDeleteInstance@config_plugin_instancesDlg@@QAEXXZ$18 1000f671 f   config_plugin_instancesdlgimpl.obj
 0001:0000e67a       __unwindfunclet$?doDeleteInstance@config_plugin_instancesDlg@@QAEXXZ$19 1000f67a f   config_plugin_instancesdlgimpl.obj
 0001:0000e683       __unwindfunclet$?doDeleteInstance@config_plugin_instancesDlg@@QAEXXZ$20 1000f683 f   config_plugin_instancesdlgimpl.obj
 0001:0000e68f       __unwindfunclet$?doDeleteInstance@config_plugin_instancesDlg@@QAEXXZ$22 1000f68f f   config_plugin_instancesdlgimpl.obj
 0001:0000e69b       __unwindfunclet$?doDeleteInstance@config_plugin_instancesDlg@@QAEXXZ$23 1000f69b f   config_plugin_instancesdlgimpl.obj
 0001:0000e6a7       __unwindfunclet$?doDeleteInstance@config_plugin_instancesDlg@@QAEXXZ$24 1000f6a7 f   config_plugin_instancesdlgimpl.obj
 0001:0000e6b3       __unwindfunclet$?doDeleteInstance@config_plugin_instancesDlg@@QAEXXZ$25 1000f6b3 f   config_plugin_instancesdlgimpl.obj
 0001:0000e6bd       __unwindfunclet$?doDeleteInstance@config_plugin_instancesDlg@@QAEXXZ$26 1000f6bd f   config_plugin_instancesdlgimpl.obj
 0001:0000e6c6       __unwindfunclet$?doDeleteInstance@config_plugin_instancesDlg@@QAEXXZ$27 1000f6c6 f   config_plugin_instancesdlgimpl.obj
 0001:0000e6cf       __unwindfunclet$?doDeleteInstance@config_plugin_instancesDlg@@QAEXXZ$28 1000f6cf f   config_plugin_instancesdlgimpl.obj
 0001:0000e6d8       __unwindfunclet$?doDeleteInstance@config_plugin_instancesDlg@@QAEXXZ$29 1000f6d8 f   config_plugin_instancesdlgimpl.obj
 0001:0000e6e1       __unwindfunclet$?doDeleteInstance@config_plugin_instancesDlg@@QAEXXZ$30 1000f6e1 f   config_plugin_instancesdlgimpl.obj
 0001:0000e6ea       __unwindfunclet$?doDeleteInstance@config_plugin_instancesDlg@@QAEXXZ$31 1000f6ea f   config_plugin_instancesdlgimpl.obj
 0001:0000e6f3       __unwindfunclet$?doDeleteInstance@config_plugin_instancesDlg@@QAEXXZ$32 1000f6f3 f   config_plugin_instancesdlgimpl.obj
 0001:0000e6fc       __unwindfunclet$?doDeleteInstance@config_plugin_instancesDlg@@QAEXXZ$33 1000f6fc f   config_plugin_instancesdlgimpl.obj
 0001:0000e705       __unwindfunclet$?doDeleteInstance@config_plugin_instancesDlg@@QAEXXZ$34 1000f705 f   config_plugin_instancesdlgimpl.obj
 0001:0000e70e       __unwindfunclet$?doDeleteInstance@config_plugin_instancesDlg@@QAEXXZ$36 1000f70e f   config_plugin_instancesdlgimpl.obj
 0001:0000e71a       __unwindfunclet$?doDeleteInstance@config_plugin_instancesDlg@@QAEXXZ$37 1000f71a f   config_plugin_instancesdlgimpl.obj
 0001:0000e726       __unwindfunclet$?doDeleteInstance@config_plugin_instancesDlg@@QAEXXZ$5 1000f726 f   config_plugin_instancesdlgimpl.obj
 0001:0000e72f       __unwindfunclet$?doDeleteInstance@config_plugin_instancesDlg@@QAEXXZ$6 1000f72f f   config_plugin_instancesdlgimpl.obj
 0001:0000e739       __unwindfunclet$?doDeleteInstance@config_plugin_instancesDlg@@QAEXXZ$7 1000f739 f   config_plugin_instancesdlgimpl.obj
 0001:0000e742       __unwindfunclet$?doDeleteInstance@config_plugin_instancesDlg@@QAEXXZ$8 1000f742 f   config_plugin_instancesdlgimpl.obj
 0001:0000e74b       __unwindfunclet$?doDeleteInstance@config_plugin_instancesDlg@@QAEXXZ$9 1000f74b f   config_plugin_instancesdlgimpl.obj
 0001:0000e754       __unwindfunclet$?doDeleteInstance@config_plugin_instancesDlg@@QAEXXZ$10 1000f754 f   config_plugin_instancesdlgimpl.obj
 0001:0000e75d       __unwindfunclet$?doDeleteInstance@config_plugin_instancesDlg@@QAEXXZ$11 1000f75d f   config_plugin_instancesdlgimpl.obj
 0001:0000e769       __unwindfunclet$?doDeleteInstance@config_plugin_instancesDlg@@QAEXXZ$13 1000f769 f   config_plugin_instancesdlgimpl.obj
 0001:0000e775       __ehhandler$?doDeleteInstance@config_plugin_instancesDlg@@QAEXXZ 1000f775 f   config_plugin_instancesdlgimpl.obj
 0001:0000e793       __unwindfunclet$?doDuplicateInstance@config_plugin_instancesDlg@@QAEXXZ$0 1000f793 f   config_plugin_instancesdlgimpl.obj
 0001:0000e79e       __unwindfunclet$?doDuplicateInstance@config_plugin_instancesDlg@@QAEXXZ$1 1000f79e f   config_plugin_instancesdlgimpl.obj
 0001:0000e7a9       __unwindfunclet$?doDuplicateInstance@config_plugin_instancesDlg@@QAEXXZ$2 1000f7a9 f   config_plugin_instancesdlgimpl.obj
 0001:0000e7b4       __unwindfunclet$?doDuplicateInstance@config_plugin_instancesDlg@@QAEXXZ$3 1000f7b4 f   config_plugin_instancesdlgimpl.obj
 0001:0000e7bd       __unwindfunclet$?doDuplicateInstance@config_plugin_instancesDlg@@QAEXXZ$4 1000f7bd f   config_plugin_instancesdlgimpl.obj
 0001:0000e7c6       __unwindfunclet$?doDuplicateInstance@config_plugin_instancesDlg@@QAEXXZ$5 1000f7c6 f   config_plugin_instancesdlgimpl.obj
 0001:0000e7cf       __unwindfunclet$?doDuplicateInstance@config_plugin_instancesDlg@@QAEXXZ$6 1000f7cf f   config_plugin_instancesdlgimpl.obj
 0001:0000e7d8       __unwindfunclet$?doDuplicateInstance@config_plugin_instancesDlg@@QAEXXZ$34 1000f7d8 f   config_plugin_instancesdlgimpl.obj
 0001:0000e7e4       __unwindfunclet$?doDuplicateInstance@config_plugin_instancesDlg@@QAEXXZ$35 1000f7e4 f   config_plugin_instancesdlgimpl.obj
 0001:0000e7ed       __unwindfunclet$?doDuplicateInstance@config_plugin_instancesDlg@@QAEXXZ$77 1000f7ed f   config_plugin_instancesdlgimpl.obj
 0001:0000e7f6       __unwindfunclet$?doDuplicateInstance@config_plugin_instancesDlg@@QAEXXZ$36 1000f7f6 f   config_plugin_instancesdlgimpl.obj
 0001:0000e800       __unwindfunclet$?doDuplicateInstance@config_plugin_instancesDlg@@QAEXXZ$37 1000f800 f   config_plugin_instancesdlgimpl.obj
 0001:0000e822       __unwindfunclet$?doDuplicateInstance@config_plugin_instancesDlg@@QAEXXZ$38 1000f822 f   config_plugin_instancesdlgimpl.obj
 0001:0000e844       __unwindfunclet$?doDuplicateInstance@config_plugin_instancesDlg@@QAEXXZ$39 1000f844 f   config_plugin_instancesdlgimpl.obj
 0001:0000e866       __unwindfunclet$?doDuplicateInstance@config_plugin_instancesDlg@@QAEXXZ$41 1000f866 f   config_plugin_instancesdlgimpl.obj
 0001:0000e870       __unwindfunclet$?doDuplicateInstance@config_plugin_instancesDlg@@QAEXXZ$42 1000f870 f   config_plugin_instancesdlgimpl.obj
 0001:0000e879       __unwindfunclet$?doDuplicateInstance@config_plugin_instancesDlg@@QAEXXZ$43 1000f879 f   config_plugin_instancesdlgimpl.obj
 0001:0000e882       __unwindfunclet$?doDuplicateInstance@config_plugin_instancesDlg@@QAEXXZ$44 1000f882 f   config_plugin_instancesdlgimpl.obj
 0001:0000e88e       __unwindfunclet$?doDuplicateInstance@config_plugin_instancesDlg@@QAEXXZ$45 1000f88e f   config_plugin_instancesdlgimpl.obj
 0001:0000e897       __unwindfunclet$?doDuplicateInstance@config_plugin_instancesDlg@@QAEXXZ$46 1000f897 f   config_plugin_instancesdlgimpl.obj
 0001:0000e8a3       __unwindfunclet$?doDuplicateInstance@config_plugin_instancesDlg@@QAEXXZ$50 1000f8a3 f   config_plugin_instancesdlgimpl.obj
 0001:0000e8af       __unwindfunclet$?doDuplicateInstance@config_plugin_instancesDlg@@QAEXXZ$47 1000f8af f   config_plugin_instancesdlgimpl.obj
 0001:0000e8b8       __unwindfunclet$?doDuplicateInstance@config_plugin_instancesDlg@@QAEXXZ$49 1000f8b8 f   config_plugin_instancesdlgimpl.obj
 0001:0000e8c1       __unwindfunclet$?doDuplicateInstance@config_plugin_instancesDlg@@QAEXXZ$51 1000f8c1 f   config_plugin_instancesdlgimpl.obj
 0001:0000e8ca       __unwindfunclet$?doDuplicateInstance@config_plugin_instancesDlg@@QAEXXZ$52 1000f8ca f   config_plugin_instancesdlgimpl.obj
 0001:0000e8d6       __unwindfunclet$?doDuplicateInstance@config_plugin_instancesDlg@@QAEXXZ$53 1000f8d6 f   config_plugin_instancesdlgimpl.obj
 0001:0000e8e2       __unwindfunclet$?doDuplicateInstance@config_plugin_instancesDlg@@QAEXXZ$54 1000f8e2 f   config_plugin_instancesdlgimpl.obj
 0001:0000e8eb       __unwindfunclet$?doDuplicateInstance@config_plugin_instancesDlg@@QAEXXZ$78 1000f8eb f   config_plugin_instancesdlgimpl.obj
 0001:0000e8f4       __unwindfunclet$?doDuplicateInstance@config_plugin_instancesDlg@@QAEXXZ$55 1000f8f4 f   config_plugin_instancesdlgimpl.obj
 0001:0000e8fe       __unwindfunclet$?doDuplicateInstance@config_plugin_instancesDlg@@QAEXXZ$56 1000f8fe f   config_plugin_instancesdlgimpl.obj
 0001:0000e920       __unwindfunclet$?doDuplicateInstance@config_plugin_instancesDlg@@QAEXXZ$58 1000f920 f   config_plugin_instancesdlgimpl.obj
 0001:0000e92a       __unwindfunclet$?doDuplicateInstance@config_plugin_instancesDlg@@QAEXXZ$59 1000f92a f   config_plugin_instancesdlgimpl.obj
 0001:0000e933       __unwindfunclet$?doDuplicateInstance@config_plugin_instancesDlg@@QAEXXZ$60 1000f933 f   config_plugin_instancesdlgimpl.obj
 0001:0000e93c       __unwindfunclet$?doDuplicateInstance@config_plugin_instancesDlg@@QAEXXZ$61 1000f93c f   config_plugin_instancesdlgimpl.obj
 0001:0000e948       __unwindfunclet$?doDuplicateInstance@config_plugin_instancesDlg@@QAEXXZ$62 1000f948 f   config_plugin_instancesdlgimpl.obj
 0001:0000e951       __unwindfunclet$?doDuplicateInstance@config_plugin_instancesDlg@@QAEXXZ$63 1000f951 f   config_plugin_instancesdlgimpl.obj
 0001:0000e95d       __unwindfunclet$?doDuplicateInstance@config_plugin_instancesDlg@@QAEXXZ$64 1000f95d f   config_plugin_instancesdlgimpl.obj
 0001:0000e966       __unwindfunclet$?doDuplicateInstance@config_plugin_instancesDlg@@QAEXXZ$65 1000f966 f   config_plugin_instancesdlgimpl.obj
 0001:0000e96f       __unwindfunclet$?doDuplicateInstance@config_plugin_instancesDlg@@QAEXXZ$66 1000f96f f   config_plugin_instancesdlgimpl.obj
 0001:0000e978       __unwindfunclet$?doDuplicateInstance@config_plugin_instancesDlg@@QAEXXZ$67 1000f978 f   config_plugin_instancesdlgimpl.obj
 0001:0000e984       __unwindfunclet$?doDuplicateInstance@config_plugin_instancesDlg@@QAEXXZ$71 1000f984 f   config_plugin_instancesdlgimpl.obj
 0001:0000e990       __unwindfunclet$?doDuplicateInstance@config_plugin_instancesDlg@@QAEXXZ$68 1000f990 f   config_plugin_instancesdlgimpl.obj
 0001:0000e99c       __unwindfunclet$?doDuplicateInstance@config_plugin_instancesDlg@@QAEXXZ$70 1000f99c f   config_plugin_instancesdlgimpl.obj
 0001:0000e9a8       __unwindfunclet$?doDuplicateInstance@config_plugin_instancesDlg@@QAEXXZ$72 1000f9a8 f   config_plugin_instancesdlgimpl.obj
 0001:0000e9b4       __unwindfunclet$?doDuplicateInstance@config_plugin_instancesDlg@@QAEXXZ$7 1000f9b4 f   config_plugin_instancesdlgimpl.obj
 0001:0000e9c0       __unwindfunclet$?doDuplicateInstance@config_plugin_instancesDlg@@QAEXXZ$8 1000f9c0 f   config_plugin_instancesdlgimpl.obj
 0001:0000e9c9       __unwindfunclet$?doDuplicateInstance@config_plugin_instancesDlg@@QAEXXZ$76 1000f9c9 f   config_plugin_instancesdlgimpl.obj
 0001:0000e9d2       __unwindfunclet$?doDuplicateInstance@config_plugin_instancesDlg@@QAEXXZ$10 1000f9d2 f   config_plugin_instancesdlgimpl.obj
 0001:0000e9dc       __unwindfunclet$?doDuplicateInstance@config_plugin_instancesDlg@@QAEXXZ$11 1000f9dc f   config_plugin_instancesdlgimpl.obj
 0001:0000e9f9       __unwindfunclet$?doDuplicateInstance@config_plugin_instancesDlg@@QAEXXZ$12 1000f9f9 f   config_plugin_instancesdlgimpl.obj
 0001:0000ea16       __unwindfunclet$?doDuplicateInstance@config_plugin_instancesDlg@@QAEXXZ$13 1000fa16 f   config_plugin_instancesdlgimpl.obj
 0001:0000ea33       __unwindfunclet$?doDuplicateInstance@config_plugin_instancesDlg@@QAEXXZ$14 1000fa33 f   config_plugin_instancesdlgimpl.obj
 0001:0000ea50       __unwindfunclet$?doDuplicateInstance@config_plugin_instancesDlg@@QAEXXZ$15 1000fa50 f   config_plugin_instancesdlgimpl.obj
 0001:0000ea6d       __unwindfunclet$?doDuplicateInstance@config_plugin_instancesDlg@@QAEXXZ$16 1000fa6d f   config_plugin_instancesdlgimpl.obj
 0001:0000ea8a       __unwindfunclet$?doDuplicateInstance@config_plugin_instancesDlg@@QAEXXZ$17 1000fa8a f   config_plugin_instancesdlgimpl.obj
 0001:0000eaa7       __unwindfunclet$?doDuplicateInstance@config_plugin_instancesDlg@@QAEXXZ$18 1000faa7 f   config_plugin_instancesdlgimpl.obj
 0001:0000eab1       __unwindfunclet$?doDuplicateInstance@config_plugin_instancesDlg@@QAEXXZ$19 1000fab1 f   config_plugin_instancesdlgimpl.obj
 0001:0000eaba       __unwindfunclet$?doDuplicateInstance@config_plugin_instancesDlg@@QAEXXZ$20 1000faba f   config_plugin_instancesdlgimpl.obj
 0001:0000eac3       __unwindfunclet$?doDuplicateInstance@config_plugin_instancesDlg@@QAEXXZ$21 1000fac3 f   config_plugin_instancesdlgimpl.obj
 0001:0000eacf       __unwindfunclet$?doDuplicateInstance@config_plugin_instancesDlg@@QAEXXZ$22 1000facf f   config_plugin_instancesdlgimpl.obj
 0001:0000ead8       __unwindfunclet$?doDuplicateInstance@config_plugin_instancesDlg@@QAEXXZ$23 1000fad8 f   config_plugin_instancesdlgimpl.obj
 0001:0000eae4       __unwindfunclet$?doDuplicateInstance@config_plugin_instancesDlg@@QAEXXZ$27 1000fae4 f   config_plugin_instancesdlgimpl.obj
 0001:0000eaf0       __unwindfunclet$?doDuplicateInstance@config_plugin_instancesDlg@@QAEXXZ$24 1000faf0 f   config_plugin_instancesdlgimpl.obj
 0001:0000eafc       __unwindfunclet$?doDuplicateInstance@config_plugin_instancesDlg@@QAEXXZ$26 1000fafc f   config_plugin_instancesdlgimpl.obj
 0001:0000eb08       __unwindfunclet$?doDuplicateInstance@config_plugin_instancesDlg@@QAEXXZ$28 1000fb08 f   config_plugin_instancesdlgimpl.obj
 0001:0000eb11       __unwindfunclet$?doDuplicateInstance@config_plugin_instancesDlg@@QAEXXZ$30 1000fb11 f   config_plugin_instancesdlgimpl.obj
 0001:0000eb1d       __unwindfunclet$?doDuplicateInstance@config_plugin_instancesDlg@@QAEXXZ$31 1000fb1d f   config_plugin_instancesdlgimpl.obj
 0001:0000eb29       __unwindfunclet$?doDuplicateInstance@config_plugin_instancesDlg@@QAEXXZ$32 1000fb29 f   config_plugin_instancesdlgimpl.obj
 0001:0000eb35       __unwindfunclet$?doDuplicateInstance@config_plugin_instancesDlg@@QAEXXZ$33 1000fb35 f   config_plugin_instancesdlgimpl.obj
 0001:0000eb41       __ehhandler$?doDuplicateInstance@config_plugin_instancesDlg@@QAEXXZ 1000fb41 f   config_plugin_instancesdlgimpl.obj
 0001:0000eb5f       __unwindfunclet$?groupNameIsUnique@config_plugin_instancesDlg@@QAE_NVQString@@@Z$0 1000fb5f f   config_plugin_instancesdlgimpl.obj
 0001:0000eb68       __unwindfunclet$?groupNameIsUnique@config_plugin_instancesDlg@@QAE_NVQString@@@Z$1 1000fb68 f   config_plugin_instancesdlgimpl.obj
 0001:0000eb71       __ehhandler$?groupNameIsUnique@config_plugin_instancesDlg@@QAE_NVQString@@@Z 1000fb71 f   config_plugin_instancesdlgimpl.obj
 0001:0000eb8c       __unwindfunclet$?instanceNameIsUnique@config_plugin_instancesDlg@@QAE_NVQString@@@Z$0 1000fb8c f   config_plugin_instancesdlgimpl.obj
 0001:0000eb95       __unwindfunclet$?instanceNameIsUnique@config_plugin_instancesDlg@@QAE_NVQString@@@Z$1 1000fb95 f   config_plugin_instancesdlgimpl.obj
 0001:0000eb9f       __unwindfunclet$?instanceNameIsUnique@config_plugin_instancesDlg@@QAE_NVQString@@@Z$2 1000fb9f f   config_plugin_instancesdlgimpl.obj
 0001:0000eba8       __unwindfunclet$?instanceNameIsUnique@config_plugin_instancesDlg@@QAE_NVQString@@@Z$3 1000fba8 f   config_plugin_instancesdlgimpl.obj
 0001:0000ebb1       __unwindfunclet$?instanceNameIsUnique@config_plugin_instancesDlg@@QAE_NVQString@@@Z$4 1000fbb1 f   config_plugin_instancesdlgimpl.obj
 0001:0000ebba       __unwindfunclet$?instanceNameIsUnique@config_plugin_instancesDlg@@QAE_NVQString@@@Z$5 1000fbba f   config_plugin_instancesdlgimpl.obj
 0001:0000ebc3       __unwindfunclet$?instanceNameIsUnique@config_plugin_instancesDlg@@QAE_NVQString@@@Z$6 1000fbc3 f   config_plugin_instancesdlgimpl.obj
 0001:0000ebcc       __unwindfunclet$?instanceNameIsUnique@config_plugin_instancesDlg@@QAE_NVQString@@@Z$7 1000fbcc f   config_plugin_instancesdlgimpl.obj
 0001:0000ebd5       __unwindfunclet$?instanceNameIsUnique@config_plugin_instancesDlg@@QAE_NVQString@@@Z$8 1000fbd5 f   config_plugin_instancesdlgimpl.obj
 0001:0000ebde       __ehhandler$?instanceNameIsUnique@config_plugin_instancesDlg@@QAE_NVQString@@@Z 1000fbde f   config_plugin_instancesdlgimpl.obj
 0001:0000ebf9       __unwindfunclet$?load@config_plugin_instancesDlg@@QAE_NABVQString@@@Z$0 1000fbf9 f   config_plugin_instancesdlgimpl.obj
 0001:0000ec02       __unwindfunclet$?load@config_plugin_instancesDlg@@QAE_NABVQString@@@Z$1 1000fc02 f   config_plugin_instancesdlgimpl.obj
 0001:0000ec0b       __unwindfunclet$?load@config_plugin_instancesDlg@@QAE_NABVQString@@@Z$2 1000fc0b f   config_plugin_instancesdlgimpl.obj
 0001:0000ec15       __unwindfunclet$?load@config_plugin_instancesDlg@@QAE_NABVQString@@@Z$3 1000fc15 f   config_plugin_instancesdlgimpl.obj
 0001:0000ec21       __unwindfunclet$?load@config_plugin_instancesDlg@@QAE_NABVQString@@@Z$4 1000fc21 f   config_plugin_instancesdlgimpl.obj
 0001:0000ec2b       __unwindfunclet$?load@config_plugin_instancesDlg@@QAE_NABVQString@@@Z$5 1000fc2b f   config_plugin_instancesdlgimpl.obj
 0001:0000ec34       __unwindfunclet$?load@config_plugin_instancesDlg@@QAE_NABVQString@@@Z$6 1000fc34 f   config_plugin_instancesdlgimpl.obj
 0001:0000ec3d       __unwindfunclet$?load@config_plugin_instancesDlg@@QAE_NABVQString@@@Z$7 1000fc3d f   config_plugin_instancesdlgimpl.obj
 0001:0000ec46       __unwindfunclet$?load@config_plugin_instancesDlg@@QAE_NABVQString@@@Z$8 1000fc46 f   config_plugin_instancesdlgimpl.obj
 0001:0000ec4f       __unwindfunclet$?load@config_plugin_instancesDlg@@QAE_NABVQString@@@Z$9 1000fc4f f   config_plugin_instancesdlgimpl.obj
 0001:0000ec58       __unwindfunclet$?load@config_plugin_instancesDlg@@QAE_NABVQString@@@Z$10 1000fc58 f   config_plugin_instancesdlgimpl.obj
 0001:0000ec61       __unwindfunclet$?load@config_plugin_instancesDlg@@QAE_NABVQString@@@Z$11 1000fc61 f   config_plugin_instancesdlgimpl.obj
 0001:0000ec6a       __unwindfunclet$?load@config_plugin_instancesDlg@@QAE_NABVQString@@@Z$12 1000fc6a f   config_plugin_instancesdlgimpl.obj
 0001:0000ec73       __unwindfunclet$?load@config_plugin_instancesDlg@@QAE_NABVQString@@@Z$13 1000fc73 f   config_plugin_instancesdlgimpl.obj
 0001:0000ec7c       __unwindfunclet$?load@config_plugin_instancesDlg@@QAE_NABVQString@@@Z$14 1000fc7c f   config_plugin_instancesdlgimpl.obj
 0001:0000ec85       __unwindfunclet$?load@config_plugin_instancesDlg@@QAE_NABVQString@@@Z$15 1000fc85 f   config_plugin_instancesdlgimpl.obj
 0001:0000ec8e       __unwindfunclet$?load@config_plugin_instancesDlg@@QAE_NABVQString@@@Z$16 1000fc8e f   config_plugin_instancesdlgimpl.obj
 0001:0000ec97       __unwindfunclet$?load@config_plugin_instancesDlg@@QAE_NABVQString@@@Z$17 1000fc97 f   config_plugin_instancesdlgimpl.obj
 0001:0000eca0       __unwindfunclet$?load@config_plugin_instancesDlg@@QAE_NABVQString@@@Z$18 1000fca0 f   config_plugin_instancesdlgimpl.obj
 0001:0000eca9       __unwindfunclet$?load@config_plugin_instancesDlg@@QAE_NABVQString@@@Z$19 1000fca9 f   config_plugin_instancesdlgimpl.obj
 0001:0000ecb2       __unwindfunclet$?load@config_plugin_instancesDlg@@QAE_NABVQString@@@Z$20 1000fcb2 f   config_plugin_instancesdlgimpl.obj
 0001:0000ecbb       __unwindfunclet$?load@config_plugin_instancesDlg@@QAE_NABVQString@@@Z$21 1000fcbb f   config_plugin_instancesdlgimpl.obj
 0001:0000ecc7       __unwindfunclet$?load@config_plugin_instancesDlg@@QAE_NABVQString@@@Z$22 1000fcc7 f   config_plugin_instancesdlgimpl.obj
 0001:0000ecd3       __unwindfunclet$?load@config_plugin_instancesDlg@@QAE_NABVQString@@@Z$23 1000fcd3 f   config_plugin_instancesdlgimpl.obj
 0001:0000ecdc       __unwindfunclet$?load@config_plugin_instancesDlg@@QAE_NABVQString@@@Z$24 1000fcdc f   config_plugin_instancesdlgimpl.obj
 0001:0000ece8       __unwindfunclet$?load@config_plugin_instancesDlg@@QAE_NABVQString@@@Z$25 1000fce8 f   config_plugin_instancesdlgimpl.obj
 0001:0000ecf4       __unwindfunclet$?load@config_plugin_instancesDlg@@QAE_NABVQString@@@Z$26 1000fcf4 f   config_plugin_instancesdlgimpl.obj
 0001:0000ed00       __unwindfunclet$?load@config_plugin_instancesDlg@@QAE_NABVQString@@@Z$27 1000fd00 f   config_plugin_instancesdlgimpl.obj
 0001:0000ed0c       __unwindfunclet$?load@config_plugin_instancesDlg@@QAE_NABVQString@@@Z$28 1000fd0c f   config_plugin_instancesdlgimpl.obj
 0001:0000ed18       __unwindfunclet$?load@config_plugin_instancesDlg@@QAE_NABVQString@@@Z$29 1000fd18 f   config_plugin_instancesdlgimpl.obj
 0001:0000ed24       __unwindfunclet$?load@config_plugin_instancesDlg@@QAE_NABVQString@@@Z$30 1000fd24 f   config_plugin_instancesdlgimpl.obj
 0001:0000ed2d       __unwindfunclet$?load@config_plugin_instancesDlg@@QAE_NABVQString@@@Z$31 1000fd2d f   config_plugin_instancesdlgimpl.obj
 0001:0000ed39       __unwindfunclet$?load@config_plugin_instancesDlg@@QAE_NABVQString@@@Z$32 1000fd39 f   config_plugin_instancesdlgimpl.obj
 0001:0000ed42       __unwindfunclet$?load@config_plugin_instancesDlg@@QAE_NABVQString@@@Z$33 1000fd42 f   config_plugin_instancesdlgimpl.obj
 0001:0000ed4e       __unwindfunclet$?load@config_plugin_instancesDlg@@QAE_NABVQString@@@Z$34 1000fd4e f   config_plugin_instancesdlgimpl.obj
 0001:0000ed5a       __unwindfunclet$?load@config_plugin_instancesDlg@@QAE_NABVQString@@@Z$35 1000fd5a f   config_plugin_instancesdlgimpl.obj
 0001:0000ed66       __unwindfunclet$?load@config_plugin_instancesDlg@@QAE_NABVQString@@@Z$36 1000fd66 f   config_plugin_instancesdlgimpl.obj
 0001:0000ed72       __unwindfunclet$?load@config_plugin_instancesDlg@@QAE_NABVQString@@@Z$37 1000fd72 f   config_plugin_instancesdlgimpl.obj
 0001:0000ed7e       __unwindfunclet$?load@config_plugin_instancesDlg@@QAE_NABVQString@@@Z$38 1000fd7e f   config_plugin_instancesdlgimpl.obj
 0001:0000ed8a       __unwindfunclet$?load@config_plugin_instancesDlg@@QAE_NABVQString@@@Z$39 1000fd8a f   config_plugin_instancesdlgimpl.obj
 0001:0000ed96       __unwindfunclet$?load@config_plugin_instancesDlg@@QAE_NABVQString@@@Z$40 1000fd96 f   config_plugin_instancesdlgimpl.obj
 0001:0000eda2       __unwindfunclet$?load@config_plugin_instancesDlg@@QAE_NABVQString@@@Z$41 1000fda2 f   config_plugin_instancesdlgimpl.obj
 0001:0000edae       __unwindfunclet$?load@config_plugin_instancesDlg@@QAE_NABVQString@@@Z$42 1000fdae f   config_plugin_instancesdlgimpl.obj
 0001:0000edba       __unwindfunclet$?load@config_plugin_instancesDlg@@QAE_NABVQString@@@Z$43 1000fdba f   config_plugin_instancesdlgimpl.obj
 0001:0000edc3       __unwindfunclet$?load@config_plugin_instancesDlg@@QAE_NABVQString@@@Z$44 1000fdc3 f   config_plugin_instancesdlgimpl.obj
 0001:0000edcf       __unwindfunclet$?load@config_plugin_instancesDlg@@QAE_NABVQString@@@Z$45 1000fdcf f   config_plugin_instancesdlgimpl.obj
 0001:0000eddb       __unwindfunclet$?load@config_plugin_instancesDlg@@QAE_NABVQString@@@Z$46 1000fddb f   config_plugin_instancesdlgimpl.obj
 0001:0000ede4       __unwindfunclet$?load@config_plugin_instancesDlg@@QAE_NABVQString@@@Z$47 1000fde4 f   config_plugin_instancesdlgimpl.obj
 0001:0000eded       __unwindfunclet$?load@config_plugin_instancesDlg@@QAE_NABVQString@@@Z$48 1000fded f   config_plugin_instancesdlgimpl.obj
 0001:0000edf6       __unwindfunclet$?load@config_plugin_instancesDlg@@QAE_NABVQString@@@Z$50 1000fdf6 f   config_plugin_instancesdlgimpl.obj
 0001:0000ee02       __unwindfunclet$?load@config_plugin_instancesDlg@@QAE_NABVQString@@@Z$51 1000fe02 f   config_plugin_instancesdlgimpl.obj
 0001:0000ee0e       __unwindfunclet$?load@config_plugin_instancesDlg@@QAE_NABVQString@@@Z$52 1000fe0e f   config_plugin_instancesdlgimpl.obj
 0001:0000ee1a       __unwindfunclet$?load@config_plugin_instancesDlg@@QAE_NABVQString@@@Z$53 1000fe1a f   config_plugin_instancesdlgimpl.obj
 0001:0000ee23       __unwindfunclet$?load@config_plugin_instancesDlg@@QAE_NABVQString@@@Z$54 1000fe23 f   config_plugin_instancesdlgimpl.obj
 0001:0000ee2c       __unwindfunclet$?load@config_plugin_instancesDlg@@QAE_NABVQString@@@Z$55 1000fe2c f   config_plugin_instancesdlgimpl.obj
 0001:0000ee35       __unwindfunclet$?load@config_plugin_instancesDlg@@QAE_NABVQString@@@Z$56 1000fe35 f   config_plugin_instancesdlgimpl.obj
 0001:0000ee3e       __unwindfunclet$?load@config_plugin_instancesDlg@@QAE_NABVQString@@@Z$57 1000fe3e f   config_plugin_instancesdlgimpl.obj
 0001:0000ee47       __unwindfunclet$?load@config_plugin_instancesDlg@@QAE_NABVQString@@@Z$58 1000fe47 f   config_plugin_instancesdlgimpl.obj
 0001:0000ee53       __unwindfunclet$?load@config_plugin_instancesDlg@@QAE_NABVQString@@@Z$59 1000fe53 f   config_plugin_instancesdlgimpl.obj
 0001:0000ee5d       __unwindfunclet$?load@config_plugin_instancesDlg@@QAE_NABVQString@@@Z$60 1000fe5d f   config_plugin_instancesdlgimpl.obj
 0001:0000ee66       __unwindfunclet$?load@config_plugin_instancesDlg@@QAE_NABVQString@@@Z$61 1000fe66 f   config_plugin_instancesdlgimpl.obj
 0001:0000ee6f       __unwindfunclet$?load@config_plugin_instancesDlg@@QAE_NABVQString@@@Z$62 1000fe6f f   config_plugin_instancesdlgimpl.obj
 0001:0000ee78       __unwindfunclet$?load@config_plugin_instancesDlg@@QAE_NABVQString@@@Z$63 1000fe78 f   config_plugin_instancesdlgimpl.obj
 0001:0000ee81       __unwindfunclet$?load@config_plugin_instancesDlg@@QAE_NABVQString@@@Z$64 1000fe81 f   config_plugin_instancesdlgimpl.obj
 0001:0000ee8a       __unwindfunclet$?load@config_plugin_instancesDlg@@QAE_NABVQString@@@Z$65 1000fe8a f   config_plugin_instancesdlgimpl.obj
 0001:0000ee93       __unwindfunclet$?load@config_plugin_instancesDlg@@QAE_NABVQString@@@Z$66 1000fe93 f   config_plugin_instancesdlgimpl.obj
 0001:0000ee9f       __ehhandler$?load@config_plugin_instancesDlg@@QAE_NABVQString@@@Z 1000fe9f f   config_plugin_instancesdlgimpl.obj
 0001:0000eebd       __unwindfunclet$?pasteCompositesXMLFragment@config_plugin_instancesDlg@@QAEXXZ$0 1000febd f   config_plugin_instancesdlgimpl.obj
 0001:0000eec6       __unwindfunclet$?pasteCompositesXMLFragment@config_plugin_instancesDlg@@QAEXXZ$1 1000fec6 f   config_plugin_instancesdlgimpl.obj
 0001:0000eed2       __unwindfunclet$?pasteCompositesXMLFragment@config_plugin_instancesDlg@@QAEXXZ$2 1000fed2 f   config_plugin_instancesdlgimpl.obj
 0001:0000eedb       __unwindfunclet$?pasteCompositesXMLFragment@config_plugin_instancesDlg@@QAEXXZ$3 1000fedb f   config_plugin_instancesdlgimpl.obj
 0001:0000eee4       __unwindfunclet$?pasteCompositesXMLFragment@config_plugin_instancesDlg@@QAEXXZ$4 1000fee4 f   config_plugin_instancesdlgimpl.obj
 0001:0000eeed       __unwindfunclet$?pasteCompositesXMLFragment@config_plugin_instancesDlg@@QAEXXZ$5 1000feed f   config_plugin_instancesdlgimpl.obj
 0001:0000eef6       __unwindfunclet$?pasteCompositesXMLFragment@config_plugin_instancesDlg@@QAEXXZ$6 1000fef6 f   config_plugin_instancesdlgimpl.obj
 0001:0000eeff       __unwindfunclet$?pasteCompositesXMLFragment@config_plugin_instancesDlg@@QAEXXZ$7 1000feff f   config_plugin_instancesdlgimpl.obj
 0001:0000ef08       __unwindfunclet$?pasteCompositesXMLFragment@config_plugin_instancesDlg@@QAEXXZ$8 1000ff08 f   config_plugin_instancesdlgimpl.obj
 0001:0000ef11       __unwindfunclet$?pasteCompositesXMLFragment@config_plugin_instancesDlg@@QAEXXZ$9 1000ff11 f   config_plugin_instancesdlgimpl.obj
 0001:0000ef1a       __unwindfunclet$?pasteCompositesXMLFragment@config_plugin_instancesDlg@@QAEXXZ$11 1000ff1a f   config_plugin_instancesdlgimpl.obj
 0001:0000ef23       __unwindfunclet$?pasteCompositesXMLFragment@config_plugin_instancesDlg@@QAEXXZ$12 1000ff23 f   config_plugin_instancesdlgimpl.obj
 0001:0000ef2c       __unwindfunclet$?pasteCompositesXMLFragment@config_plugin_instancesDlg@@QAEXXZ$13 1000ff2c f   config_plugin_instancesdlgimpl.obj
 0001:0000ef38       __unwindfunclet$?pasteCompositesXMLFragment@config_plugin_instancesDlg@@QAEXXZ$14 1000ff38 f   config_plugin_instancesdlgimpl.obj
 0001:0000ef41       __unwindfunclet$?pasteCompositesXMLFragment@config_plugin_instancesDlg@@QAEXXZ$15 1000ff41 f   config_plugin_instancesdlgimpl.obj
 0001:0000ef4d       __unwindfunclet$?pasteCompositesXMLFragment@config_plugin_instancesDlg@@QAEXXZ$25 1000ff4d f   config_plugin_instancesdlgimpl.obj
 0001:0000ef59       __unwindfunclet$?pasteCompositesXMLFragment@config_plugin_instancesDlg@@QAEXXZ$16 1000ff59 f   config_plugin_instancesdlgimpl.obj
 0001:0000ef65       __unwindfunclet$?pasteCompositesXMLFragment@config_plugin_instancesDlg@@QAEXXZ$18 1000ff65 f   config_plugin_instancesdlgimpl.obj
 0001:0000ef71       __unwindfunclet$?pasteCompositesXMLFragment@config_plugin_instancesDlg@@QAEXXZ$19 1000ff71 f   config_plugin_instancesdlgimpl.obj
 0001:0000ef7a       __unwindfunclet$?pasteCompositesXMLFragment@config_plugin_instancesDlg@@QAEXXZ$20 1000ff7a f   config_plugin_instancesdlgimpl.obj
 0001:0000ef83       __unwindfunclet$?pasteCompositesXMLFragment@config_plugin_instancesDlg@@QAEXXZ$21 1000ff83 f   config_plugin_instancesdlgimpl.obj
 0001:0000ef8c       __unwindfunclet$?pasteCompositesXMLFragment@config_plugin_instancesDlg@@QAEXXZ$22 1000ff8c f   config_plugin_instancesdlgimpl.obj
 0001:0000ef95       __unwindfunclet$?pasteCompositesXMLFragment@config_plugin_instancesDlg@@QAEXXZ$23 1000ff95 f   config_plugin_instancesdlgimpl.obj
 0001:0000ef9e       __unwindfunclet$?pasteCompositesXMLFragment@config_plugin_instancesDlg@@QAEXXZ$24 1000ff9e f   config_plugin_instancesdlgimpl.obj
 0001:0000efa7       __unwindfunclet$?pasteCompositesXMLFragment@config_plugin_instancesDlg@@QAEXXZ$26 1000ffa7 f   config_plugin_instancesdlgimpl.obj
 0001:0000efb3       __unwindfunclet$?pasteCompositesXMLFragment@config_plugin_instancesDlg@@QAEXXZ$28 1000ffb3 f   config_plugin_instancesdlgimpl.obj
 0001:0000efbc       __unwindfunclet$?pasteCompositesXMLFragment@config_plugin_instancesDlg@@QAEXXZ$29 1000ffbc f   config_plugin_instancesdlgimpl.obj
 0001:0000efc8       __unwindfunclet$?pasteCompositesXMLFragment@config_plugin_instancesDlg@@QAEXXZ$30 1000ffc8 f   config_plugin_instancesdlgimpl.obj
 0001:0000efd1       __unwindfunclet$?pasteCompositesXMLFragment@config_plugin_instancesDlg@@QAEXXZ$31 1000ffd1 f   config_plugin_instancesdlgimpl.obj
 0001:0000efda       __unwindfunclet$?pasteCompositesXMLFragment@config_plugin_instancesDlg@@QAEXXZ$32 1000ffda f   config_plugin_instancesdlgimpl.obj
 0001:0000efe3       __unwindfunclet$?pasteCompositesXMLFragment@config_plugin_instancesDlg@@QAEXXZ$33 1000ffe3 f   config_plugin_instancesdlgimpl.obj
 0001:0000efef       __unwindfunclet$?pasteCompositesXMLFragment@config_plugin_instancesDlg@@QAEXXZ$34 1000ffef f   config_plugin_instancesdlgimpl.obj
 0001:0000eff8       __unwindfunclet$?pasteCompositesXMLFragment@config_plugin_instancesDlg@@QAEXXZ$35 1000fff8 f   config_plugin_instancesdlgimpl.obj
 0001:0000f004       __unwindfunclet$?pasteCompositesXMLFragment@config_plugin_instancesDlg@@QAEXXZ$36 10010004 f   config_plugin_instancesdlgimpl.obj
 0001:0000f00d       __unwindfunclet$?pasteCompositesXMLFragment@config_plugin_instancesDlg@@QAEXXZ$37 1001000d f   config_plugin_instancesdlgimpl.obj
 0001:0000f019       __ehhandler$?pasteCompositesXMLFragment@config_plugin_instancesDlg@@QAEXXZ 10010019 f   config_plugin_instancesdlgimpl.obj
 0001:0000f037       __unwindfunclet$?pasteDeviceData@config_plugin_instancesDlg@@QAEXXZ$0 10010037 f   config_plugin_instancesdlgimpl.obj
 0001:0000f040       __unwindfunclet$?pasteDeviceData@config_plugin_instancesDlg@@QAEXXZ$1 10010040 f   config_plugin_instancesdlgimpl.obj
 0001:0000f049       __unwindfunclet$?pasteDeviceData@config_plugin_instancesDlg@@QAEXXZ$2 10010049 f   config_plugin_instancesdlgimpl.obj
 0001:0000f052       __unwindfunclet$?pasteDeviceData@config_plugin_instancesDlg@@QAEXXZ$3 10010052 f   config_plugin_instancesdlgimpl.obj
 0001:0000f05d       __unwindfunclet$?pasteDeviceData@config_plugin_instancesDlg@@QAEXXZ$4 1001005d f   config_plugin_instancesdlgimpl.obj
 0001:0000f066       __unwindfunclet$?pasteDeviceData@config_plugin_instancesDlg@@QAEXXZ$5 10010066 f   config_plugin_instancesdlgimpl.obj
 0001:0000f06f       __unwindfunclet$?pasteDeviceData@config_plugin_instancesDlg@@QAEXXZ$6 1001006f f   config_plugin_instancesdlgimpl.obj
 0001:0000f078       __unwindfunclet$?pasteDeviceData@config_plugin_instancesDlg@@QAEXXZ$7 10010078 f   config_plugin_instancesdlgimpl.obj
 0001:0000f081       __unwindfunclet$?pasteDeviceData@config_plugin_instancesDlg@@QAEXXZ$8 10010081 f   config_plugin_instancesdlgimpl.obj
 0001:0000f08a       __unwindfunclet$?pasteDeviceData@config_plugin_instancesDlg@@QAEXXZ$9 1001008a f   config_plugin_instancesdlgimpl.obj
 0001:0000f093       __unwindfunclet$?pasteDeviceData@config_plugin_instancesDlg@@QAEXXZ$10 10010093 f   config_plugin_instancesdlgimpl.obj
 0001:0000f09c       __unwindfunclet$?pasteDeviceData@config_plugin_instancesDlg@@QAEXXZ$12 1001009c f   config_plugin_instancesdlgimpl.obj
 0001:0000f0a8       __unwindfunclet$?pasteDeviceData@config_plugin_instancesDlg@@QAEXXZ$13 100100a8 f   config_plugin_instancesdlgimpl.obj
 0001:0000f0b2       __unwindfunclet$?pasteDeviceData@config_plugin_instancesDlg@@QAEXXZ$14 100100b2 f   config_plugin_instancesdlgimpl.obj
 0001:0000f0bb       __unwindfunclet$?pasteDeviceData@config_plugin_instancesDlg@@QAEXXZ$15 100100bb f   config_plugin_instancesdlgimpl.obj
 0001:0000f0c4       __unwindfunclet$?pasteDeviceData@config_plugin_instancesDlg@@QAEXXZ$16 100100c4 f   config_plugin_instancesdlgimpl.obj
 0001:0000f0d0       __unwindfunclet$?pasteDeviceData@config_plugin_instancesDlg@@QAEXXZ$17 100100d0 f   config_plugin_instancesdlgimpl.obj
 0001:0000f0d9       __unwindfunclet$?pasteDeviceData@config_plugin_instancesDlg@@QAEXXZ$18 100100d9 f   config_plugin_instancesdlgimpl.obj
 0001:0000f0e5       __unwindfunclet$?pasteDeviceData@config_plugin_instancesDlg@@QAEXXZ$20 100100e5 f   config_plugin_instancesdlgimpl.obj
 0001:0000f0ee       __unwindfunclet$?pasteDeviceData@config_plugin_instancesDlg@@QAEXXZ$21 100100ee f   config_plugin_instancesdlgimpl.obj
 0001:0000f0f7       __unwindfunclet$?pasteDeviceData@config_plugin_instancesDlg@@QAEXXZ$22 100100f7 f   config_plugin_instancesdlgimpl.obj
 0001:0000f100       __unwindfunclet$?pasteDeviceData@config_plugin_instancesDlg@@QAEXXZ$23 10010100 f   config_plugin_instancesdlgimpl.obj
 0001:0000f109       __unwindfunclet$?pasteDeviceData@config_plugin_instancesDlg@@QAEXXZ$24 10010109 f   config_plugin_instancesdlgimpl.obj
 0001:0000f112       __unwindfunclet$?pasteDeviceData@config_plugin_instancesDlg@@QAEXXZ$26 10010112 f   config_plugin_instancesdlgimpl.obj
 0001:0000f11e       __unwindfunclet$?pasteDeviceData@config_plugin_instancesDlg@@QAEXXZ$27 1001011e f   config_plugin_instancesdlgimpl.obj
 0001:0000f127       __unwindfunclet$?pasteDeviceData@config_plugin_instancesDlg@@QAEXXZ$28 10010127 f   config_plugin_instancesdlgimpl.obj
 0001:0000f133       __unwindfunclet$?pasteDeviceData@config_plugin_instancesDlg@@QAEXXZ$30 10010133 f   config_plugin_instancesdlgimpl.obj
 0001:0000f13c       __unwindfunclet$?pasteDeviceData@config_plugin_instancesDlg@@QAEXXZ$31 1001013c f   config_plugin_instancesdlgimpl.obj
 0001:0000f145       __unwindfunclet$?pasteDeviceData@config_plugin_instancesDlg@@QAEXXZ$32 10010145 f   config_plugin_instancesdlgimpl.obj
 0001:0000f151       __unwindfunclet$?pasteDeviceData@config_plugin_instancesDlg@@QAEXXZ$33 10010151 f   config_plugin_instancesdlgimpl.obj
 0001:0000f15a       __unwindfunclet$?pasteDeviceData@config_plugin_instancesDlg@@QAEXXZ$19 1001015a f   config_plugin_instancesdlgimpl.obj
 0001:0000f163       __unwindfunclet$?pasteDeviceData@config_plugin_instancesDlg@@QAEXXZ$35 10010163 f   config_plugin_instancesdlgimpl.obj
 0001:0000f16f       __unwindfunclet$?pasteDeviceData@config_plugin_instancesDlg@@QAEXXZ$36 1001016f f   config_plugin_instancesdlgimpl.obj
 0001:0000f17b       __unwindfunclet$?pasteDeviceData@config_plugin_instancesDlg@@QAEXXZ$37 1001017b f   config_plugin_instancesdlgimpl.obj
 0001:0000f187       __unwindfunclet$?pasteDeviceData@config_plugin_instancesDlg@@QAEXXZ$39 10010187 f   config_plugin_instancesdlgimpl.obj
 0001:0000f193       __unwindfunclet$?pasteDeviceData@config_plugin_instancesDlg@@QAEXXZ$40 10010193 f   config_plugin_instancesdlgimpl.obj
 0001:0000f19f       __ehhandler$?pasteDeviceData@config_plugin_instancesDlg@@QAEXXZ 1001019f f   config_plugin_instancesdlgimpl.obj
 0001:0000f1bd       __unwindfunclet$?pasteGroupData@config_plugin_instancesDlg@@QAEXXZ$0 100101bd f   config_plugin_instancesdlgimpl.obj
 0001:0000f1c6       __unwindfunclet$?pasteGroupData@config_plugin_instancesDlg@@QAEXXZ$1 100101c6 f   config_plugin_instancesdlgimpl.obj
 0001:0000f1cf       __unwindfunclet$?pasteGroupData@config_plugin_instancesDlg@@QAEXXZ$2 100101cf f   config_plugin_instancesdlgimpl.obj
 0001:0000f1da       __unwindfunclet$?pasteGroupData@config_plugin_instancesDlg@@QAEXXZ$3 100101da f   config_plugin_instancesdlgimpl.obj
 0001:0000f1e3       __unwindfunclet$?pasteGroupData@config_plugin_instancesDlg@@QAEXXZ$4 100101e3 f   config_plugin_instancesdlgimpl.obj
 0001:0000f1ec       __unwindfunclet$?pasteGroupData@config_plugin_instancesDlg@@QAEXXZ$5 100101ec f   config_plugin_instancesdlgimpl.obj
 0001:0000f1f5       __unwindfunclet$?pasteGroupData@config_plugin_instancesDlg@@QAEXXZ$6 100101f5 f   config_plugin_instancesdlgimpl.obj
 0001:0000f1fe       __unwindfunclet$?pasteGroupData@config_plugin_instancesDlg@@QAEXXZ$7 100101fe f   config_plugin_instancesdlgimpl.obj
 0001:0000f207       __unwindfunclet$?pasteGroupData@config_plugin_instancesDlg@@QAEXXZ$8 10010207 f   config_plugin_instancesdlgimpl.obj
 0001:0000f210       __unwindfunclet$?pasteGroupData@config_plugin_instancesDlg@@QAEXXZ$9 10010210 f   config_plugin_instancesdlgimpl.obj
 0001:0000f219       __unwindfunclet$?pasteGroupData@config_plugin_instancesDlg@@QAEXXZ$11 10010219 f   config_plugin_instancesdlgimpl.obj
 0001:0000f222       __unwindfunclet$?pasteGroupData@config_plugin_instancesDlg@@QAEXXZ$12 10010222 f   config_plugin_instancesdlgimpl.obj
 0001:0000f22c       __unwindfunclet$?pasteGroupData@config_plugin_instancesDlg@@QAEXXZ$13 1001022c f   config_plugin_instancesdlgimpl.obj
 0001:0000f235       __unwindfunclet$?pasteGroupData@config_plugin_instancesDlg@@QAEXXZ$14 10010235 f   config_plugin_instancesdlgimpl.obj
 0001:0000f23e       __unwindfunclet$?pasteGroupData@config_plugin_instancesDlg@@QAEXXZ$15 1001023e f   config_plugin_instancesdlgimpl.obj
 0001:0000f247       __unwindfunclet$?pasteGroupData@config_plugin_instancesDlg@@QAEXXZ$16 10010247 f   config_plugin_instancesdlgimpl.obj
 0001:0000f250       __unwindfunclet$?pasteGroupData@config_plugin_instancesDlg@@QAEXXZ$17 10010250 f   config_plugin_instancesdlgimpl.obj
 0001:0000f259       __unwindfunclet$?pasteGroupData@config_plugin_instancesDlg@@QAEXXZ$18 10010259 f   config_plugin_instancesdlgimpl.obj
 0001:0000f262       __unwindfunclet$?pasteGroupData@config_plugin_instancesDlg@@QAEXXZ$19 10010262 f   config_plugin_instancesdlgimpl.obj
 0001:0000f26b       __unwindfunclet$?pasteGroupData@config_plugin_instancesDlg@@QAEXXZ$20 1001026b f   config_plugin_instancesdlgimpl.obj
 0001:0000f274       __unwindfunclet$?pasteGroupData@config_plugin_instancesDlg@@QAEXXZ$21 10010274 f   config_plugin_instancesdlgimpl.obj
 0001:0000f27d       __unwindfunclet$?pasteGroupData@config_plugin_instancesDlg@@QAEXXZ$22 1001027d f   config_plugin_instancesdlgimpl.obj
 0001:0000f286       __unwindfunclet$?pasteGroupData@config_plugin_instancesDlg@@QAEXXZ$23 10010286 f   config_plugin_instancesdlgimpl.obj
 0001:0000f28f       __unwindfunclet$?pasteGroupData@config_plugin_instancesDlg@@QAEXXZ$24 1001028f f   config_plugin_instancesdlgimpl.obj
 0001:0000f29b       __unwindfunclet$?pasteGroupData@config_plugin_instancesDlg@@QAEXXZ$25 1001029b f   config_plugin_instancesdlgimpl.obj
 0001:0000f2a7       __unwindfunclet$?pasteGroupData@config_plugin_instancesDlg@@QAEXXZ$26 100102a7 f   config_plugin_instancesdlgimpl.obj
 0001:0000f2b0       __ehhandler$?pasteGroupData@config_plugin_instancesDlg@@QAEXXZ 100102b0 f   config_plugin_instancesdlgimpl.obj
 0001:0000f2ce       __unwindfunclet$?db@@YAXABVQString@@@Z$0 100102ce f   config_plugin_instancesdlgimpl.obj
 0001:0000f2ce       __unwindfunclet$?pasteOptions@config_plugin_instancesDlg@@QAEXXZ$0 100102ce f   config_plugin_instancesdlgimpl.obj
 0001:0000f2d7       __ehhandler$?db@@YAXABVQString@@@Z 100102d7 f   config_plugin_instancesdlgimpl.obj
 0001:0000f2d7       __ehhandler$?pasteOptions@config_plugin_instancesDlg@@QAEXXZ 100102d7 f   config_plugin_instancesdlgimpl.obj
 0001:0000f2f2       __unwindfunclet$?save@config_plugin_instancesDlg@@QAE_NABVQString@@@Z$0 100102f2 f   config_plugin_instancesdlgimpl.obj
 0001:0000f2fb       __unwindfunclet$?save@config_plugin_instancesDlg@@QAE_NABVQString@@@Z$1 100102fb f   config_plugin_instancesdlgimpl.obj
 0001:0000f304       __unwindfunclet$?save@config_plugin_instancesDlg@@QAE_NABVQString@@@Z$2 10010304 f   config_plugin_instancesdlgimpl.obj
 0001:0000f30d       __ehhandler$?save@config_plugin_instancesDlg@@QAE_NABVQString@@@Z 1001030d f   config_plugin_instancesdlgimpl.obj
 0001:0000f328       __unwindfunclet$?selectDevicetypes@config_plugin_instancesDlg@@QAEXHHHABVQPoint@@@Z$0 10010328 f   config_plugin_instancesdlgimpl.obj
 0001:0000f331       __unwindfunclet$?selectDevicetypes@config_plugin_instancesDlg@@QAEXHHHABVQPoint@@@Z$1 10010331 f   config_plugin_instancesdlgimpl.obj
 0001:0000f33a       __unwindfunclet$?selectDevicetypes@config_plugin_instancesDlg@@QAEXHHHABVQPoint@@@Z$2 1001033a f   config_plugin_instancesdlgimpl.obj
 0001:0000f344       __unwindfunclet$?selectDevicetypes@config_plugin_instancesDlg@@QAEXHHHABVQPoint@@@Z$4 10010344 f   config_plugin_instancesdlgimpl.obj
 0001:0000f34d       __unwindfunclet$?selectDevicetypes@config_plugin_instancesDlg@@QAEXHHHABVQPoint@@@Z$5 1001034d f   config_plugin_instancesdlgimpl.obj
 0001:0000f356       __unwindfunclet$?selectDevicetypes@config_plugin_instancesDlg@@QAEXHHHABVQPoint@@@Z$6 10010356 f   config_plugin_instancesdlgimpl.obj
 0001:0000f35f       __ehhandler$?selectDevicetypes@config_plugin_instancesDlg@@QAEXHHHABVQPoint@@@Z 1001035f f   config_plugin_instancesdlgimpl.obj
 0001:0000f37a       __unwindfunclet$?typeIsValid@config_plugin_instancesDlg@@QAE_NVQString@@@Z$0 1001037a f   config_plugin_instancesdlgimpl.obj
 0001:0000f383       __ehhandler$?typeIsValid@config_plugin_instancesDlg@@QAE_NVQString@@@Z 10010383 f   config_plugin_instancesdlgimpl.obj
 0001:0000f39e       __unwindfunclet$?valueCompositeGroupChanged@config_plugin_instancesDlg@@QAEXHH@Z$0 1001039e f   config_plugin_instancesdlgimpl.obj
 0001:0000f3a7       __unwindfunclet$?valueCompositeGroupChanged@config_plugin_instancesDlg@@QAEXHH@Z$1 100103a7 f   config_plugin_instancesdlgimpl.obj
 0001:0000f3b1       __unwindfunclet$?valueCompositeGroupChanged@config_plugin_instancesDlg@@QAEXHH@Z$2 100103b1 f   config_plugin_instancesdlgimpl.obj
 0001:0000f3ba       __unwindfunclet$?valueCompositeGroupChanged@config_plugin_instancesDlg@@QAEXHH@Z$3 100103ba f   config_plugin_instancesdlgimpl.obj
 0001:0000f3c3       __unwindfunclet$?valueCompositeGroupChanged@config_plugin_instancesDlg@@QAEXHH@Z$4 100103c3 f   config_plugin_instancesdlgimpl.obj
 0001:0000f3cc       __unwindfunclet$?valueCompositeGroupChanged@config_plugin_instancesDlg@@QAEXHH@Z$5 100103cc f   config_plugin_instancesdlgimpl.obj
 0001:0000f3d5       __unwindfunclet$?valueCompositeGroupChanged@config_plugin_instancesDlg@@QAEXHH@Z$6 100103d5 f   config_plugin_instancesdlgimpl.obj
 0001:0000f3de       __unwindfunclet$?valueCompositeGroupChanged@config_plugin_instancesDlg@@QAEXHH@Z$7 100103de f   config_plugin_instancesdlgimpl.obj
 0001:0000f3e7       __unwindfunclet$?valueCompositeGroupChanged@config_plugin_instancesDlg@@QAEXHH@Z$8 100103e7 f   config_plugin_instancesdlgimpl.obj
 0001:0000f3f0       __unwindfunclet$?valueCompositeGroupChanged@config_plugin_instancesDlg@@QAEXHH@Z$9 100103f0 f   config_plugin_instancesdlgimpl.obj
 0001:0000f3f9       __unwindfunclet$?valueCompositeGroupChanged@config_plugin_instancesDlg@@QAEXHH@Z$10 100103f9 f   config_plugin_instancesdlgimpl.obj
 0001:0000f402       __unwindfunclet$?valueCompositeGroupChanged@config_plugin_instancesDlg@@QAEXHH@Z$11 10010402 f   config_plugin_instancesdlgimpl.obj
 0001:0000f40b       __unwindfunclet$?valueCompositeGroupChanged@config_plugin_instancesDlg@@QAEXHH@Z$12 1001040b f   config_plugin_instancesdlgimpl.obj
 0001:0000f414       __unwindfunclet$?valueCompositeGroupChanged@config_plugin_instancesDlg@@QAEXHH@Z$13 10010414 f   config_plugin_instancesdlgimpl.obj
 0001:0000f41d       __unwindfunclet$?valueCompositeGroupChanged@config_plugin_instancesDlg@@QAEXHH@Z$14 1001041d f   config_plugin_instancesdlgimpl.obj
 0001:0000f426       __unwindfunclet$?valueCompositeGroupChanged@config_plugin_instancesDlg@@QAEXHH@Z$15 10010426 f   config_plugin_instancesdlgimpl.obj
 0001:0000f42f       __ehhandler$?valueCompositeGroupChanged@config_plugin_instancesDlg@@QAEXHH@Z 1001042f f   config_plugin_instancesdlgimpl.obj
 0001:0000f44a       __unwindfunclet$?valueCompositeTopChanged@config_plugin_instancesDlg@@QAEXHH@Z$0 1001044a f   config_plugin_instancesdlgimpl.obj
 0001:0000f453       __unwindfunclet$?valueCompositeTopChanged@config_plugin_instancesDlg@@QAEXHH@Z$1 10010453 f   config_plugin_instancesdlgimpl.obj
 0001:0000f45d       __unwindfunclet$?valueCompositeTopChanged@config_plugin_instancesDlg@@QAEXHH@Z$2 1001045d f   config_plugin_instancesdlgimpl.obj
 0001:0000f466       __unwindfunclet$?valueCompositeTopChanged@config_plugin_instancesDlg@@QAEXHH@Z$3 10010466 f   config_plugin_instancesdlgimpl.obj
 0001:0000f46f       __unwindfunclet$?valueCompositeTopChanged@config_plugin_instancesDlg@@QAEXHH@Z$4 1001046f f   config_plugin_instancesdlgimpl.obj
 0001:0000f478       __unwindfunclet$?valueCompositeTopChanged@config_plugin_instancesDlg@@QAEXHH@Z$5 10010478 f   config_plugin_instancesdlgimpl.obj
 0001:0000f481       __unwindfunclet$?valueCompositeTopChanged@config_plugin_instancesDlg@@QAEXHH@Z$6 10010481 f   config_plugin_instancesdlgimpl.obj
 0001:0000f48a       __unwindfunclet$?valueCompositeTopChanged@config_plugin_instancesDlg@@QAEXHH@Z$7 1001048a f   config_plugin_instancesdlgimpl.obj
 0001:0000f493       __unwindfunclet$?valueCompositeTopChanged@config_plugin_instancesDlg@@QAEXHH@Z$9 10010493 f   config_plugin_instancesdlgimpl.obj
 0001:0000f49c       __unwindfunclet$?valueCompositeTopChanged@config_plugin_instancesDlg@@QAEXHH@Z$8 1001049c f   config_plugin_instancesdlgimpl.obj
 0001:0000f4a5       __ehhandler$?valueCompositeTopChanged@config_plugin_instancesDlg@@QAEXHH@Z 100104a5 f   config_plugin_instancesdlgimpl.obj
 0001:0000f4c0       __unwindfunclet$?valueDevicesChanged@config_plugin_instancesDlg@@QAEXHH@Z$0 100104c0 f   config_plugin_instancesdlgimpl.obj
 0001:0000f4c9       __unwindfunclet$?valueDevicesChanged@config_plugin_instancesDlg@@QAEXHH@Z$5 100104c9 f   config_plugin_instancesdlgimpl.obj
 0001:0000f4d3       __unwindfunclet$?valueDevicesChanged@config_plugin_instancesDlg@@QAEXHH@Z$3 100104d3 f   config_plugin_instancesdlgimpl.obj
 0001:0000f4dc       __unwindfunclet$?valueDevicesChanged@config_plugin_instancesDlg@@QAEXHH@Z$4 100104dc f   config_plugin_instancesdlgimpl.obj
 0001:0000f4e5       __unwindfunclet$?valueDevicesChanged@config_plugin_instancesDlg@@QAEXHH@Z$6 100104e5 f   config_plugin_instancesdlgimpl.obj
 0001:0000f4ee       __unwindfunclet$?valueDevicesChanged@config_plugin_instancesDlg@@QAEXHH@Z$7 100104ee f   config_plugin_instancesdlgimpl.obj
 0001:0000f4f7       __unwindfunclet$?valueDevicesChanged@config_plugin_instancesDlg@@QAEXHH@Z$8 100104f7 f   config_plugin_instancesdlgimpl.obj
 0001:0000f500       __unwindfunclet$?valueDevicesChanged@config_plugin_instancesDlg@@QAEXHH@Z$9 10010500 f   config_plugin_instancesdlgimpl.obj
 0001:0000f509       __unwindfunclet$?valueDevicesChanged@config_plugin_instancesDlg@@QAEXHH@Z$10 10010509 f   config_plugin_instancesdlgimpl.obj
 0001:0000f512       __unwindfunclet$?valueDevicesChanged@config_plugin_instancesDlg@@QAEXHH@Z$11 10010512 f   config_plugin_instancesdlgimpl.obj
 0001:0000f51b       __unwindfunclet$?valueDevicesChanged@config_plugin_instancesDlg@@QAEXHH@Z$27 1001051b f   config_plugin_instancesdlgimpl.obj
 0001:0000f524       __unwindfunclet$?valueDevicesChanged@config_plugin_instancesDlg@@QAEXHH@Z$13 10010524 f   config_plugin_instancesdlgimpl.obj
 0001:0000f52d       __unwindfunclet$?valueDevicesChanged@config_plugin_instancesDlg@@QAEXHH@Z$14 1001052d f   config_plugin_instancesdlgimpl.obj
 0001:0000f536       __unwindfunclet$?valueDevicesChanged@config_plugin_instancesDlg@@QAEXHH@Z$15 10010536 f   config_plugin_instancesdlgimpl.obj
 0001:0000f53f       __unwindfunclet$?valueDevicesChanged@config_plugin_instancesDlg@@QAEXHH@Z$16 1001053f f   config_plugin_instancesdlgimpl.obj
 0001:0000f548       __unwindfunclet$?valueDevicesChanged@config_plugin_instancesDlg@@QAEXHH@Z$17 10010548 f   config_plugin_instancesdlgimpl.obj
 0001:0000f551       __unwindfunclet$?valueDevicesChanged@config_plugin_instancesDlg@@QAEXHH@Z$19 10010551 f   config_plugin_instancesdlgimpl.obj
 0001:0000f55a       __unwindfunclet$?valueDevicesChanged@config_plugin_instancesDlg@@QAEXHH@Z$20 1001055a f   config_plugin_instancesdlgimpl.obj
 0001:0000f563       __unwindfunclet$?valueDevicesChanged@config_plugin_instancesDlg@@QAEXHH@Z$21 10010563 f   config_plugin_instancesdlgimpl.obj
 0001:0000f56c       __unwindfunclet$?valueDevicesChanged@config_plugin_instancesDlg@@QAEXHH@Z$23 1001056c f   config_plugin_instancesdlgimpl.obj
 0001:0000f575       __unwindfunclet$?valueDevicesChanged@config_plugin_instancesDlg@@QAEXHH@Z$24 10010575 f   config_plugin_instancesdlgimpl.obj
 0001:0000f57e       __unwindfunclet$?valueDevicesChanged@config_plugin_instancesDlg@@QAEXHH@Z$25 1001057e f   config_plugin_instancesdlgimpl.obj
 0001:0000f587       __unwindfunclet$?valueDevicesChanged@config_plugin_instancesDlg@@QAEXHH@Z$26 10010587 f   config_plugin_instancesdlgimpl.obj
 0001:0000f590       __unwindfunclet$?valueDevicesChanged@config_plugin_instancesDlg@@QAEXHH@Z$12 10010590 f   config_plugin_instancesdlgimpl.obj
 0001:0000f599       __ehhandler$?valueDevicesChanged@config_plugin_instancesDlg@@QAEXHH@Z 10010599 f   config_plugin_instancesdlgimpl.obj
 0001:0000f5b4       __unwindfunclet$?viewGroupChanged@config_plugin_instancesDlg@@QAEXHH@Z$0 100105b4 f   config_plugin_instancesdlgimpl.obj
 0001:0000f5bd       __unwindfunclet$?viewGroupChanged@config_plugin_instancesDlg@@QAEXHH@Z$1 100105bd f   config_plugin_instancesdlgimpl.obj
 0001:0000f5c6       __ehhandler$?viewGroupChanged@config_plugin_instancesDlg@@QAEXHH@Z 100105c6 f   config_plugin_instancesdlgimpl.obj
 0001:0000f5e1       __unwindfunclet$?viewInstanceChanged@config_plugin_instancesDlg@@QAEXHH@Z$0 100105e1 f   config_plugin_instancesdlgimpl.obj
 0001:0000f5ea       __unwindfunclet$?viewInstanceChanged@config_plugin_instancesDlg@@QAEXHH@Z$1 100105ea f   config_plugin_instancesdlgimpl.obj
 0001:0000f5f4       __unwindfunclet$?viewInstanceChanged@config_plugin_instancesDlg@@QAEXHH@Z$2 100105f4 f   config_plugin_instancesdlgimpl.obj
 0001:0000f5fd       __unwindfunclet$?viewInstanceChanged@config_plugin_instancesDlg@@QAEXHH@Z$3 100105fd f   config_plugin_instancesdlgimpl.obj
 0001:0000f606       __unwindfunclet$?viewInstanceChanged@config_plugin_instancesDlg@@QAEXHH@Z$4 10010606 f   config_plugin_instancesdlgimpl.obj
 0001:0000f60f       __unwindfunclet$?viewInstanceChanged@config_plugin_instancesDlg@@QAEXHH@Z$5 1001060f f   config_plugin_instancesdlgimpl.obj
 0001:0000f618       __unwindfunclet$?viewInstanceChanged@config_plugin_instancesDlg@@QAEXHH@Z$6 10010618 f   config_plugin_instancesdlgimpl.obj
 0001:0000f621       __unwindfunclet$?viewInstanceChanged@config_plugin_instancesDlg@@QAEXHH@Z$7 10010621 f   config_plugin_instancesdlgimpl.obj
 0001:0000f62a       __unwindfunclet$?viewInstanceChanged@config_plugin_instancesDlg@@QAEXHH@Z$8 1001062a f   config_plugin_instancesdlgimpl.obj
 0001:0000f633       __unwindfunclet$?viewInstanceChanged@config_plugin_instancesDlg@@QAEXHH@Z$9 10010633 f   config_plugin_instancesdlgimpl.obj
 0001:0000f63c       __unwindfunclet$?viewInstanceChanged@config_plugin_instancesDlg@@QAEXHH@Z$10 1001063c f   config_plugin_instancesdlgimpl.obj
 0001:0000f645       __unwindfunclet$?viewInstanceChanged@config_plugin_instancesDlg@@QAEXHH@Z$11 10010645 f   config_plugin_instancesdlgimpl.obj
 0001:0000f64e       __unwindfunclet$?viewInstanceChanged@config_plugin_instancesDlg@@QAEXHH@Z$12 1001064e f   config_plugin_instancesdlgimpl.obj
 0001:0000f657       __unwindfunclet$?viewInstanceChanged@config_plugin_instancesDlg@@QAEXHH@Z$13 10010657 f   config_plugin_instancesdlgimpl.obj
 0001:0000f660       __unwindfunclet$?viewInstanceChanged@config_plugin_instancesDlg@@QAEXHH@Z$14 10010660 f   config_plugin_instancesdlgimpl.obj
 0001:0000f669       __unwindfunclet$?viewInstanceChanged@config_plugin_instancesDlg@@QAEXHH@Z$15 10010669 f   config_plugin_instancesdlgimpl.obj
 0001:0000f672       __unwindfunclet$?viewInstanceChanged@config_plugin_instancesDlg@@QAEXHH@Z$16 10010672 f   config_plugin_instancesdlgimpl.obj
 0001:0000f67b       __unwindfunclet$?viewInstanceChanged@config_plugin_instancesDlg@@QAEXHH@Z$17 1001067b f   config_plugin_instancesdlgimpl.obj
 0001:0000f684       __unwindfunclet$?viewInstanceChanged@config_plugin_instancesDlg@@QAEXHH@Z$18 10010684 f   config_plugin_instancesdlgimpl.obj
 0001:0000f68d       __unwindfunclet$?viewInstanceChanged@config_plugin_instancesDlg@@QAEXHH@Z$19 1001068d f   config_plugin_instancesdlgimpl.obj
 0001:0000f696       __unwindfunclet$?viewInstanceChanged@config_plugin_instancesDlg@@QAEXHH@Z$20 10010696 f   config_plugin_instancesdlgimpl.obj
 0001:0000f69f       __unwindfunclet$?viewInstanceChanged@config_plugin_instancesDlg@@QAEXHH@Z$21 1001069f f   config_plugin_instancesdlgimpl.obj
 0001:0000f6a8       __unwindfunclet$?viewInstanceChanged@config_plugin_instancesDlg@@QAEXHH@Z$22 100106a8 f   config_plugin_instancesdlgimpl.obj
 0001:0000f6b1       __unwindfunclet$?viewInstanceChanged@config_plugin_instancesDlg@@QAEXHH@Z$23 100106b1 f   config_plugin_instancesdlgimpl.obj
 0001:0000f6ba       __ehhandler$?viewInstanceChanged@config_plugin_instancesDlg@@QAEXHH@Z 100106ba f   config_plugin_instancesdlgimpl.obj
 0001:0000f6d5       __unwindfunclet$??0deviceRow@@QAE@ABVQString@@0000000@Z$0 100106d5 f   deviceRow.obj
 0001:0000f6e1       __unwindfunclet$??0deviceRow@@QAE@ABVQString@@0000000@Z$1 100106e1 f   deviceRow.obj
 0001:0000f6ed       __unwindfunclet$??0deviceRow@@QAE@ABVQString@@0000000@Z$2 100106ed f   deviceRow.obj
 0001:0000f6f9       __unwindfunclet$??0deviceRow@@QAE@ABVQString@@0000000@Z$3 100106f9 f   deviceRow.obj
 0001:0000f705       __unwindfunclet$??0deviceRow@@QAE@ABVQString@@0000000@Z$4 10010705 f   deviceRow.obj
 0001:0000f711       __unwindfunclet$??0deviceRow@@QAE@ABVQString@@0000000@Z$5 10010711 f   deviceRow.obj
 0001:0000f71d       __unwindfunclet$??0deviceRow@@QAE@ABVQString@@0000000@Z$6 1001071d f   deviceRow.obj
 0001:0000f729       __unwindfunclet$??0deviceRow@@QAE@ABVQString@@0000000@Z$7 10010729 f   deviceRow.obj
 0001:0000f735       __ehhandler$??0deviceRow@@QAE@ABVQString@@0000000@Z 10010735 f   deviceRow.obj
 0001:0000f750       __unwindfunclet$??1deviceRow@@UAE@XZ$0 10010750 f   deviceRow.obj
 0001:0000f75c       __unwindfunclet$??1deviceRow@@UAE@XZ$1 1001075c f   deviceRow.obj
 0001:0000f768       __unwindfunclet$??1deviceRow@@UAE@XZ$2 10010768 f   deviceRow.obj
 0001:0000f774       __unwindfunclet$??1deviceRow@@UAE@XZ$3 10010774 f   deviceRow.obj
 0001:0000f780       __unwindfunclet$??1deviceRow@@UAE@XZ$4 10010780 f   deviceRow.obj
 0001:0000f78c       __unwindfunclet$??1deviceRow@@UAE@XZ$5 1001078c f   deviceRow.obj
 0001:0000f798       __unwindfunclet$??1deviceRow@@UAE@XZ$6 10010798 f   deviceRow.obj
 0001:0000f7a4       __ehhandler$??1deviceRow@@UAE@XZ 100107a4 f   deviceRow.obj
 0001:0000f7bf       __unwindfunclet$??0devicetypesBase@@QAE@PAVQWidget@@PBD_NI@Z$0 100107bf f   devicetypes.obj
 0001:0000f7c8       __unwindfunclet$??0devicetypesBase@@QAE@PAVQWidget@@PBD_NI@Z$1 100107c8 f   devicetypes.obj
 0001:0000f7d2       __unwindfunclet$??0devicetypesBase@@QAE@PAVQWidget@@PBD_NI@Z$2 100107d2 f   devicetypes.obj
 0001:0000f7dc       __unwindfunclet$??0devicetypesBase@@QAE@PAVQWidget@@PBD_NI@Z$3 100107dc f   devicetypes.obj
 0001:0000f7e6       __unwindfunclet$??0devicetypesBase@@QAE@PAVQWidget@@PBD_NI@Z$4 100107e6 f   devicetypes.obj
 0001:0000f7f0       __unwindfunclet$??0devicetypesBase@@QAE@PAVQWidget@@PBD_NI@Z$5 100107f0 f   devicetypes.obj
 0001:0000f7fa       __unwindfunclet$??0devicetypesBase@@QAE@PAVQWidget@@PBD_NI@Z$6 100107fa f   devicetypes.obj
 0001:0000f804       __unwindfunclet$??0devicetypesBase@@QAE@PAVQWidget@@PBD_NI@Z$7 10010804 f   devicetypes.obj
 0001:0000f80e       __ehhandler$??0devicetypesBase@@QAE@PAVQWidget@@PBD_NI@Z 1001080e f   devicetypes.obj
 0001:0000f829       __unwindfunclet$?languageChange@devicetypesBase@@MAEXXZ$0 10010829 f   devicetypes.obj
 0001:0000f832       __unwindfunclet$?languageChange@devicetypesBase@@MAEXXZ$1 10010832 f   devicetypes.obj
 0001:0000f83b       __unwindfunclet$?languageChange@devicetypesBase@@MAEXXZ$2 1001083b f   devicetypes.obj
 0001:0000f844       __unwindfunclet$?languageChange@devicetypesBase@@MAEXXZ$3 10010844 f   devicetypes.obj
 0001:0000f84d       __ehhandler$?languageChange@devicetypesBase@@MAEXXZ 1001084d f   devicetypes.obj
 0001:0000f868       __unwindfunclet$??0groupRow@@QAE@ABVQString@@0@Z$0 10010868 f   groupRow.obj
 0001:0000f874       __unwindfunclet$??0groupRow@@QAE@ABVQString@@0@Z$1 10010874 f   groupRow.obj
 0001:0000f880       __ehhandler$??0groupRow@@QAE@ABVQString@@0@Z 10010880 f   groupRow.obj
 0001:0000f89b       __unwindfunclet$??1groupRow@@UAE@XZ$0 1001089b f   groupRow.obj
 0001:0000f8a7       __ehhandler$??1groupRow@@UAE@XZ 100108a7 f   groupRow.obj
 0001:0000f8c2       __unwindfunclet$??0instancesCustomTable@@QAE@PAVQWidget@@PBD@Z$0 100108c2 f   instancesCustomTable.obj
 0001:0000f8ca       __unwindfunclet$??0instancesCustomTable@@QAE@PAVQWidget@@PBD@Z$1 100108ca f   instancesCustomTable.obj
 0001:0000f8d9       __ehhandler$??0instancesCustomTable@@QAE@PAVQWidget@@PBD@Z 100108d9 f   instancesCustomTable.obj
 0001:0000f8f4       __unwindfunclet$??1instancesCustomTable@@UAE@XZ$0 100108f4 f   instancesCustomTable.obj
 0001:0000f8fc       __ehhandler$??1instancesCustomTable@@UAE@XZ 100108fc f   instancesCustomTable.obj
 0001:0000f917       __unwindfunclet$?create@plugindesc@@UAEPAVconfig_plugin_base@@ABVQString@@00@Z$0 10010917 f   plugindesc.obj
 0001:0000f917       __unwindfunclet$??0?$QGuardedPtr@VQPopupMenu@@@@QAE@XZ$0 10010917 f   plugindesc.obj
 0001:0000f917       __unwindfunclet$??0?$QGuardedPtr@VQDockWindow@@@@QAE@XZ$0 10010917 f   plugindesc.obj
 0001:0000f917       __unwindfunclet$??4?$QGuardedPtr@VQDockWindow@@@@QAEAAV0@PAVQDockWindow@@@Z$0 10010917 f   plugindesc.obj
 0001:0000f917       __unwindfunclet$??4?$QGuardedPtr@VQPopupMenu@@@@QAEAAV0@PAVQPopupMenu@@@Z$0 10010917 f   plugindesc.obj
 0001:0000f921       __ehhandler$??4?$QGuardedPtr@VQPopupMenu@@@@QAEAAV0@PAVQPopupMenu@@@Z 10010921 f   plugindesc.obj
 0001:0000f921       __ehhandler$?create@plugindesc@@UAEPAVconfig_plugin_base@@ABVQString@@00@Z 10010921 f   plugindesc.obj
 0001:0000f921       __ehhandler$??0?$QGuardedPtr@VQPopupMenu@@@@QAE@XZ 10010921 f   plugindesc.obj
 0001:0000f921       __ehhandler$??4?$QGuardedPtr@VQDockWindow@@@@QAEAAV0@PAVQDockWindow@@@Z 10010921 f   plugindesc.obj
 0001:0000f921       __ehhandler$??0?$QGuardedPtr@VQDockWindow@@@@QAE@XZ 10010921 f   plugindesc.obj
 0001:0000f93c       __unwindfunclet$?keys@plugindesc@@UAE?AVQStringList@@ABVQString@@0@Z$0 1001093c f   plugindesc.obj
 0001:0000f956       __unwindfunclet$?keys@plugindesc@@UAE?AVQStringList@@ABVQString@@0@Z$1 10010956 f   plugindesc.obj
 0001:0000f95f       __ehhandler$?keys@plugindesc@@UAE?AVQStringList@@ABVQString@@0@Z 1001095f f   plugindesc.obj
 0001:0000f97a       __unwindfunclet$??0viewRow@@QAE@ABVQString@@000@Z$0 1001097a f   viewRow.obj
 0001:0000f986       __unwindfunclet$??0viewRow@@QAE@ABVQString@@000@Z$1 10010986 f   viewRow.obj
 0001:0000f992       __unwindfunclet$??0viewRow@@QAE@ABVQString@@000@Z$2 10010992 f   viewRow.obj
 0001:0000f99e       __unwindfunclet$??0viewRow@@QAE@ABVQString@@000@Z$3 1001099e f   viewRow.obj
 0001:0000f9aa       __ehhandler$??0viewRow@@QAE@ABVQString@@000@Z 100109aa f   viewRow.obj
 0001:0000f9c5       __unwindfunclet$??1viewRow@@UAE@XZ$0 100109c5 f   viewRow.obj
 0001:0000f9d1       __unwindfunclet$??1viewRow@@UAE@XZ$1 100109d1 f   viewRow.obj
 0001:0000f9dd       __unwindfunclet$??1viewRow@@UAE@XZ$2 100109dd f   viewRow.obj
 0001:0000f9e9       __ehhandler$??1viewRow@@UAE@XZ 100109e9 f   viewRow.obj
 0001:0000fa04       __unwindfunclet$??0config_plugin_instancesDlgBase@@QAE@PAVQWidget@@PBDI@Z$0 10010a04 f   config_plugin_instancesdlg.obj
 0001:0000fa0d       __unwindfunclet$??0config_plugin_instancesDlgBase@@QAE@PAVQWidget@@PBDI@Z$1 10010a0d f   config_plugin_instancesdlg.obj
 0001:0000fa1c       __unwindfunclet$??0config_plugin_instancesDlgBase@@QAE@PAVQWidget@@PBDI@Z$2 10010a1c f   config_plugin_instancesdlg.obj
 0001:0000fa26       __unwindfunclet$??0config_plugin_instancesDlgBase@@QAE@PAVQWidget@@PBDI@Z$3 10010a26 f   config_plugin_instancesdlg.obj
 0001:0000fa30       __unwindfunclet$??0config_plugin_instancesDlgBase@@QAE@PAVQWidget@@PBDI@Z$4 10010a30 f   config_plugin_instancesdlg.obj
 0001:0000fa3a       __unwindfunclet$??0config_plugin_instancesDlgBase@@QAE@PAVQWidget@@PBDI@Z$5 10010a3a f   config_plugin_instancesdlg.obj
 0001:0000fa44       __unwindfunclet$??0config_plugin_instancesDlgBase@@QAE@PAVQWidget@@PBDI@Z$6 10010a44 f   config_plugin_instancesdlg.obj
 0001:0000fa4e       __unwindfunclet$??0config_plugin_instancesDlgBase@@QAE@PAVQWidget@@PBDI@Z$7 10010a4e f   config_plugin_instancesdlg.obj
 0001:0000fa58       __unwindfunclet$??0config_plugin_instancesDlgBase@@QAE@PAVQWidget@@PBDI@Z$8 10010a58 f   config_plugin_instancesdlg.obj
 0001:0000fa62       __unwindfunclet$??0config_plugin_instancesDlgBase@@QAE@PAVQWidget@@PBDI@Z$9 10010a62 f   config_plugin_instancesdlg.obj
 0001:0000fa6c       __unwindfunclet$??0config_plugin_instancesDlgBase@@QAE@PAVQWidget@@PBDI@Z$10 10010a6c f   config_plugin_instancesdlg.obj
 0001:0000fa75       __unwindfunclet$??0config_plugin_instancesDlgBase@@QAE@PAVQWidget@@PBDI@Z$11 10010a75 f   config_plugin_instancesdlg.obj
 0001:0000fa7f       __unwindfunclet$??0config_plugin_instancesDlgBase@@QAE@PAVQWidget@@PBDI@Z$12 10010a7f f   config_plugin_instancesdlg.obj
 0001:0000fa89       __unwindfunclet$??0config_plugin_instancesDlgBase@@QAE@PAVQWidget@@PBDI@Z$13 10010a89 f   config_plugin_instancesdlg.obj
 0001:0000fa93       __unwindfunclet$??0config_plugin_instancesDlgBase@@QAE@PAVQWidget@@PBDI@Z$14 10010a93 f   config_plugin_instancesdlg.obj
 0001:0000fa9d       __unwindfunclet$??0config_plugin_instancesDlgBase@@QAE@PAVQWidget@@PBDI@Z$15 10010a9d f   config_plugin_instancesdlg.obj
 0001:0000faa7       __unwindfunclet$??0config_plugin_instancesDlgBase@@QAE@PAVQWidget@@PBDI@Z$16 10010aa7 f   config_plugin_instancesdlg.obj
 0001:0000fab1       __unwindfunclet$??0config_plugin_instancesDlgBase@@QAE@PAVQWidget@@PBDI@Z$17 10010ab1 f   config_plugin_instancesdlg.obj
 0001:0000faba       __unwindfunclet$??0config_plugin_instancesDlgBase@@QAE@PAVQWidget@@PBDI@Z$18 10010aba f   config_plugin_instancesdlg.obj
 0001:0000fac4       __unwindfunclet$??0config_plugin_instancesDlgBase@@QAE@PAVQWidget@@PBDI@Z$19 10010ac4 f   config_plugin_instancesdlg.obj
 0001:0000face       __unwindfunclet$??0config_plugin_instancesDlgBase@@QAE@PAVQWidget@@PBDI@Z$20 10010ace f   config_plugin_instancesdlg.obj
 0001:0000fad8       __unwindfunclet$??0config_plugin_instancesDlgBase@@QAE@PAVQWidget@@PBDI@Z$21 10010ad8 f   config_plugin_instancesdlg.obj
 0001:0000fae2       __unwindfunclet$??0config_plugin_instancesDlgBase@@QAE@PAVQWidget@@PBDI@Z$22 10010ae2 f   config_plugin_instancesdlg.obj
 0001:0000faec       __ehhandler$??0config_plugin_instancesDlgBase@@QAE@PAVQWidget@@PBDI@Z 10010aec f   config_plugin_instancesdlg.obj
 0001:0000fb07       __unwindfunclet$??1config_plugin_instancesDlgBase@@UAE@XZ$0 10010b07 f   config_plugin_instancesdlg.obj
 0001:0000fb10       __ehhandler$??1config_plugin_instancesDlgBase@@UAE@XZ 10010b10 f   config_plugin_instancesdlg.obj
 0001:0000fb2b       __unwindfunclet$?languageChange@config_plugin_instancesDlgBase@@MAEXXZ$0 10010b2b f   config_plugin_instancesdlg.obj
 0001:0000fb34       __unwindfunclet$?languageChange@config_plugin_instancesDlgBase@@MAEXXZ$1 10010b34 f   config_plugin_instancesdlg.obj
 0001:0000fb3d       __unwindfunclet$?languageChange@config_plugin_instancesDlgBase@@MAEXXZ$2 10010b3d f   config_plugin_instancesdlg.obj
 0001:0000fb46       __unwindfunclet$?languageChange@config_plugin_instancesDlgBase@@MAEXXZ$3 10010b46 f   config_plugin_instancesdlg.obj
 0001:0000fb4f       __unwindfunclet$?languageChange@config_plugin_instancesDlgBase@@MAEXXZ$4 10010b4f f   config_plugin_instancesdlg.obj
 0001:0000fb58       __unwindfunclet$?languageChange@config_plugin_instancesDlgBase@@MAEXXZ$5 10010b58 f   config_plugin_instancesdlg.obj
 0001:0000fb61       __unwindfunclet$?languageChange@config_plugin_instancesDlgBase@@MAEXXZ$6 10010b61 f   config_plugin_instancesdlg.obj
 0001:0000fb6a       __ehhandler$?languageChange@config_plugin_instancesDlgBase@@MAEXXZ 10010b6a f   config_plugin_instancesdlg.obj
 0001:0000fb85       __unwindfunclet$?qt_emit@config_plugin_instancesDlg@@UAE_NHPAUQUObject@@@Z$0 10010b85 f   moc_config_plugin_instances.obj
 0001:0000fb85       __unwindfunclet$?qt_emit@config_plugin_instances@@UAE_NHPAUQUObject@@@Z$0 10010b85 f   moc_config_plugin_instances.obj
 0001:0000fb8e       __ehhandler$?qt_emit@config_plugin_instancesDlg@@UAE_NHPAUQUObject@@@Z 10010b8e f   moc_config_plugin_instances.obj
 0001:0000fb8e       __ehhandler$?qt_emit@config_plugin_instances@@UAE_NHPAUQUObject@@@Z 10010b8e f   moc_config_plugin_instances.obj
 0001:0000fba9       __unwindfunclet$?command@config_plugin_instances@@IAEXVQString@@0@Z$0 10010ba9 f   moc_config_plugin_instancesdlgimpl.obj
 0001:0000fba9       __unwindfunclet$?command@config_plugin_instancesDlg@@IAEXVQString@@0@Z$0 10010ba9 f   moc_config_plugin_instancesdlgimpl.obj
 0001:0000fbb2       __unwindfunclet$?command@config_plugin_instances@@IAEXVQString@@0@Z$1 10010bb2 f   moc_config_plugin_instancesdlgimpl.obj
 0001:0000fbb2       __unwindfunclet$?command@config_plugin_instancesDlg@@IAEXVQString@@0@Z$1 10010bb2 f   moc_config_plugin_instancesdlgimpl.obj
 0001:0000fbbb       __unwindfunclet$?command@config_plugin_instancesDlg@@IAEXVQString@@0@Z$2 10010bbb f   moc_config_plugin_instancesdlgimpl.obj
 0001:0000fbbb       __unwindfunclet$?command@config_plugin_instances@@IAEXVQString@@0@Z$2 10010bbb f   moc_config_plugin_instancesdlgimpl.obj
 0001:0000fbcf       __ehhandler$?command@config_plugin_instances@@IAEXVQString@@0@Z 10010bcf f   moc_config_plugin_instancesdlgimpl.obj
 0001:0000fbcf       __ehhandler$?command@config_plugin_instancesDlg@@IAEXVQString@@0@Z 10010bcf f   moc_config_plugin_instancesdlgimpl.obj
 0001:0000fbf4       __unwindfunclet$??0cfg_Table@@QAE@PAVQWidget@@PBD@Z$0 10010bf4 f   cfg_widgets001:cfg_Table.obj
 0001:0000fbfd       __ehhandler$??0cfg_Table@@QAE@PAVQWidget@@PBD@Z 10010bfd f   cfg_widgets001:cfg_Table.obj
 0001:0000fc18       __unwindfunclet$?clipBoardDataChanged@cfg_Table@@IAEXXZ$0 10010c18 f   cfg_widgets001:cfg_Table.obj
 0001:0000fc21       __ehhandler$?clipBoardDataChanged@cfg_Table@@IAEXXZ 10010c21 f   cfg_widgets001:cfg_Table.obj
 0001:0000fc3c       __unwindfunclet$?copyToClipboard@cfg_Table@@QAEXXZ$0 10010c3c f   cfg_widgets001:cfg_Table.obj
 0001:0000fc45       __unwindfunclet$?copyToClipboard@cfg_Table@@QAEXXZ$1 10010c45 f   cfg_widgets001:cfg_Table.obj
 0001:0000fc4e       __unwindfunclet$?copyToClipboard@cfg_Table@@QAEXXZ$2 10010c4e f   cfg_widgets001:cfg_Table.obj
 0001:0000fc57       __ehhandler$?copyToClipboard@cfg_Table@@QAEXXZ 10010c57 f   cfg_widgets001:cfg_Table.obj
 0001:0000fc72       __unwindfunclet$?deleteItems@cfg_Table@@QAEXXZ$0 10010c72 f   cfg_widgets001:cfg_Table.obj
 0001:0000fc7b       __ehhandler$?deleteItems@cfg_Table@@QAEXXZ 10010c7b f   cfg_widgets001:cfg_Table.obj
 0001:0000fc96       __unwindfunclet$?fillUndoBuffer@cfg_Table@@AAEXXZ$0 10010c96 f   cfg_widgets001:cfg_Table.obj
 0001:0000fca0       __unwindfunclet$?fillUndoBuffer@cfg_Table@@AAEXXZ$1 10010ca0 f   cfg_widgets001:cfg_Table.obj
 0001:0000fca9       __unwindfunclet$?fillUndoBuffer@cfg_Table@@AAEXXZ$2 10010ca9 f   cfg_widgets001:cfg_Table.obj
 0001:0000fcb2       __unwindfunclet$?fillUndoBuffer@cfg_Table@@AAEXXZ$3 10010cb2 f   cfg_widgets001:cfg_Table.obj
 0001:0000fcbb       __ehhandler$?fillUndoBuffer@cfg_Table@@AAEXXZ 10010cbb f   cfg_widgets001:cfg_Table.obj
 0001:0000fcd6       __unwindfunclet$?pasteClipboard@cfg_Table@@QAEXXZ$0 10010cd6 f   cfg_widgets001:cfg_Table.obj
 0001:0000fcdf       __unwindfunclet$?pasteClipboard@cfg_Table@@QAEXXZ$1 10010cdf f   cfg_widgets001:cfg_Table.obj
 0001:0000fce8       __unwindfunclet$?pasteClipboard@cfg_Table@@QAEXXZ$2 10010ce8 f   cfg_widgets001:cfg_Table.obj
 0001:0000fcf1       __unwindfunclet$?pasteClipboard@cfg_Table@@QAEXXZ$3 10010cf1 f   cfg_widgets001:cfg_Table.obj
 0001:0000fcfa       __unwindfunclet$?pasteClipboard@cfg_Table@@QAEXXZ$4 10010cfa f   cfg_widgets001:cfg_Table.obj
 0001:0000fd03       __unwindfunclet$?pasteClipboard@cfg_Table@@QAEXXZ$5 10010d03 f   cfg_widgets001:cfg_Table.obj
 0001:0000fd0c       __unwindfunclet$?pasteClipboard@cfg_Table@@QAEXXZ$6 10010d0c f   cfg_widgets001:cfg_Table.obj
 0001:0000fd15       __unwindfunclet$?pasteClipboard@cfg_Table@@QAEXXZ$7 10010d15 f   cfg_widgets001:cfg_Table.obj
 0001:0000fd1e       __unwindfunclet$?pasteClipboard@cfg_Table@@QAEXXZ$8 10010d1e f   cfg_widgets001:cfg_Table.obj
 0001:0000fd27       __unwindfunclet$?pasteClipboard@cfg_Table@@QAEXXZ$9 10010d27 f   cfg_widgets001:cfg_Table.obj
 0001:0000fd30       __unwindfunclet$?pasteClipboard@cfg_Table@@QAEXXZ$10 10010d30 f   cfg_widgets001:cfg_Table.obj
 0001:0000fd39       __unwindfunclet$?pasteClipboard@cfg_Table@@QAEXXZ$11 10010d39 f   cfg_widgets001:cfg_Table.obj
 0001:0000fd42       __unwindfunclet$?pasteClipboard@cfg_Table@@QAEXXZ$12 10010d42 f   cfg_widgets001:cfg_Table.obj
 0001:0000fd4b       __unwindfunclet$?pasteClipboard@cfg_Table@@QAEXXZ$13 10010d4b f   cfg_widgets001:cfg_Table.obj
 0001:0000fd54       __ehhandler$?pasteClipboard@cfg_Table@@QAEXXZ 10010d54 f   cfg_widgets001:cfg_Table.obj
 0001:0000fd6f       __unwindfunclet$?undoPaste@cfg_Table@@QAEXXZ$0 10010d6f f   cfg_widgets001:cfg_Table.obj
 0001:0000fd78       __unwindfunclet$?undoPaste@cfg_Table@@QAEXXZ$1 10010d78 f   cfg_widgets001:cfg_Table.obj
 0001:0000fd81       __unwindfunclet$?undoPaste@cfg_Table@@QAEXXZ$2 10010d81 f   cfg_widgets001:cfg_Table.obj
 0001:0000fd8a       __ehhandler$?undoPaste@cfg_Table@@QAEXXZ 10010d8a f   cfg_widgets001:cfg_Table.obj
 0001:0000fda5       ??__FcleanUp_devicetypesBase@@YAXXZ 10010da5 f   moc_devicetypes.obj
 0001:0000fdb0       ??__FcleanUp_devicetypes@@YAXXZ 10010db0 f   moc_devicetypesimpl.obj
 0001:0000fdbb       ??__FcleanUp_config_plugin_instances@@YAXXZ 10010dbb f   moc_config_plugin_instances.obj
 0001:0000fdc6       ??__FcleanUp_config_plugin_instancesDlgBase@@YAXXZ 10010dc6 f   moc_config_plugin_instancesdlg.obj
 0001:0000fdd1       ??__FcleanUp_config_plugin_instancesDlg@@YAXXZ 10010dd1 f   moc_config_plugin_instancesdlgimpl.obj
 0001:0000fddc       ??__FcleanUp_instancesCustomTable@@YAXXZ 10010ddc f   moc_instancesCustomTable.obj
 0001:0000fde7       ??__FcleanUp_toolWindowBase@@YAXXZ 10010de7 f   moc_toolwindow.obj
 0001:0000fdf2       ??__FcleanUp_toolWindow@@YAXXZ 10010df2 f   moc_toolwindowimpl.obj
 0001:0000fdfd       ??__FcleanUp_cfg_Table@@YAXXZ 10010dfd f   cfg_widgets001:moc_cfg_Table.obj
 0002:00000d4c       _cleanUp_devicetypesBase$initializer$ 10011d4c     moc_devicetypes.obj
 0002:00000d50       _cleanUp_devicetypes$initializer$ 10011d50     moc_devicetypesimpl.obj
 0002:00000d54       _cleanUp_config_plugin_instances$initializer$ 10011d54     moc_config_plugin_instances.obj
 0002:00000d58       _cleanUp_config_plugin_instancesDlgBase$initializer$ 10011d58     moc_config_plugin_instancesdlg.obj
 0002:00000d5c       _cleanUp_config_plugin_instancesDlg$initializer$ 10011d5c     moc_config_plugin_instancesdlgimpl.obj
 0002:00000d60       _cleanUp_instancesCustomTable$initializer$ 10011d60     moc_instancesCustomTable.obj
 0002:00000d64       _cleanUp_toolWindowBase$initializer$ 10011d64     moc_toolwindow.obj
 0002:00000d68       _cleanUp_toolWindow$initializer$ 10011d68     moc_toolwindowimpl.obj
 0002:00000d6c       _cleanUp_cfg_Table$initializer$ 10011d6c     cfg_widgets001:moc_cfg_Table.obj
 0002:00000d78       _pcinit                    10011d78     MSVCRT:crtdll.obj
 0002:00000d7c       _pinit                     10011d7c     MSVCRT:atonexit.obj
 0002:00003554       ?slot_0@?3??staticMetaObject@devicetypesBase@@SAPAVQMetaObject@@XZ@4UQUMethod@@B 10014554     moc_devicetypes.obj
 0002:00003570       ?slot_tbl@?3??staticMetaObject@devicetypesBase@@SAPAVQMetaObject@@XZ@4QBUQMetaData@@B 10014570     moc_devicetypes.obj
 0002:00003d90       ?slot_0@?3??staticMetaObject@config_plugin_instances@@SAPAVQMetaObject@@XZ@4UQUMethod@@B 10014d90     moc_config_plugin_instances.obj
 0002:00003db0       ?slot_tbl@?3??staticMetaObject@config_plugin_instances@@SAPAVQMetaObject@@XZ@4QBUQMetaData@@B 10014db0     moc_config_plugin_instances.obj
 0002:00003de8       ?signal_0@?3??staticMetaObject@config_plugin_instances@@SAPAVQMetaObject@@XZ@4UQUMethod@@B 10014de8     moc_config_plugin_instances.obj
 0002:00003dfc       ?signal_tbl@?3??staticMetaObject@config_plugin_instances@@SAPAVQMetaObject@@XZ@4QBUQMetaData@@B 10014dfc     moc_config_plugin_instances.obj
 0002:00003e24       ?slot_0@?3??staticMetaObject@config_plugin_instancesDlgBase@@SAPAVQMetaObject@@XZ@4UQUMethod@@B 10014e24     moc_config_plugin_instancesdlg.obj
 0002:00003e30       ?slot_tbl@?3??staticMetaObject@config_plugin_instancesDlgBase@@SAPAVQMetaObject@@XZ@4QBUQMetaData@@B 10014e30     moc_config_plugin_instancesdlg.obj
 0002:00003e3c       ?slot_0@?3??staticMetaObject@config_plugin_instancesDlg@@SAPAVQMetaObject@@XZ@4UQUMethod@@B 10014e3c     moc_config_plugin_instancesdlgimpl.obj
 0002:00003e68       ?slot_1@?3??staticMetaObject@config_plugin_instancesDlg@@SAPAVQMetaObject@@XZ@4UQUMethod@@B 10014e68     moc_config_plugin_instancesdlgimpl.obj
 0002:00003e88       ?slot_2@?3??staticMetaObject@config_plugin_instancesDlg@@SAPAVQMetaObject@@XZ@4UQUMethod@@B 10014e88     moc_config_plugin_instancesdlgimpl.obj
 0002:00003e94       ?slot_3@?3??staticMetaObject@config_plugin_instancesDlg@@SAPAVQMetaObject@@XZ@4UQUMethod@@B 10014e94     moc_config_plugin_instancesdlgimpl.obj
 0002:00003ebc       ?slot_4@?3??staticMetaObject@config_plugin_instancesDlg@@SAPAVQMetaObject@@XZ@4UQUMethod@@B 10014ebc     moc_config_plugin_instancesdlgimpl.obj
 0002:00003ee4       ?slot_5@?3??staticMetaObject@config_plugin_instancesDlg@@SAPAVQMetaObject@@XZ@4UQUMethod@@B 10014ee4     moc_config_plugin_instancesdlgimpl.obj
 0002:00003f10       ?slot_6@?3??staticMetaObject@config_plugin_instancesDlg@@SAPAVQMetaObject@@XZ@4UQUMethod@@B 10014f10     moc_config_plugin_instancesdlgimpl.obj
 0002:00003f30       ?slot_7@?3??staticMetaObject@config_plugin_instancesDlg@@SAPAVQMetaObject@@XZ@4UQUMethod@@B 10014f30     moc_config_plugin_instancesdlgimpl.obj
 0002:00003f54       ?slot_8@?3??staticMetaObject@config_plugin_instancesDlg@@SAPAVQMetaObject@@XZ@4UQUMethod@@B 10014f54     moc_config_plugin_instancesdlgimpl.obj
 0002:00003f70       ?slot_9@?3??staticMetaObject@config_plugin_instancesDlg@@SAPAVQMetaObject@@XZ@4UQUMethod@@B 10014f70     moc_config_plugin_instancesdlgimpl.obj
 0002:00003f8c       ?slot_10@?3??staticMetaObject@config_plugin_instancesDlg@@SAPAVQMetaObject@@XZ@4UQUMethod@@B 10014f8c     moc_config_plugin_instancesdlgimpl.obj
 0002:00003fb0       ?slot_11@?3??staticMetaObject@config_plugin_instancesDlg@@SAPAVQMetaObject@@XZ@4UQUMethod@@B 10014fb0     moc_config_plugin_instancesdlgimpl.obj
 0002:00003fd8       ?slot_12@?3??staticMetaObject@config_plugin_instancesDlg@@SAPAVQMetaObject@@XZ@4UQUMethod@@B 10014fd8     moc_config_plugin_instancesdlgimpl.obj
 0002:00003ff8       ?slot_13@?3??staticMetaObject@config_plugin_instancesDlg@@SAPAVQMetaObject@@XZ@4UQUMethod@@B 10014ff8     moc_config_plugin_instancesdlgimpl.obj
 0002:00004018       ?slot_14@?3??staticMetaObject@config_plugin_instancesDlg@@SAPAVQMetaObject@@XZ@4UQUMethod@@B 10015018     moc_config_plugin_instancesdlgimpl.obj
 0002:0000403c       ?slot_15@?3??staticMetaObject@config_plugin_instancesDlg@@SAPAVQMetaObject@@XZ@4UQUMethod@@B 1001503c     moc_config_plugin_instancesdlgimpl.obj
 0002:00004064       ?slot_16@?3??staticMetaObject@config_plugin_instancesDlg@@SAPAVQMetaObject@@XZ@4UQUMethod@@B 10015064     moc_config_plugin_instancesdlgimpl.obj
 0002:00004084       ?slot_17@?3??staticMetaObject@config_plugin_instancesDlg@@SAPAVQMetaObject@@XZ@4UQUMethod@@B 10015084     moc_config_plugin_instancesdlgimpl.obj
 0002:000040ac       ?slot_18@?3??staticMetaObject@config_plugin_instancesDlg@@SAPAVQMetaObject@@XZ@4UQUMethod@@B 100150ac     moc_config_plugin_instancesdlgimpl.obj
 0002:000040cc       ?slot_19@?3??staticMetaObject@config_plugin_instancesDlg@@SAPAVQMetaObject@@XZ@4UQUMethod@@B 100150cc     moc_config_plugin_instancesdlgimpl.obj
 0002:000040ec       ?slot_20@?3??staticMetaObject@config_plugin_instancesDlg@@SAPAVQMetaObject@@XZ@4UQUMethod@@B 100150ec     moc_config_plugin_instancesdlgimpl.obj
 0002:0000410c       ?slot_21@?3??staticMetaObject@config_plugin_instancesDlg@@SAPAVQMetaObject@@XZ@4UQUMethod@@B 1001510c     moc_config_plugin_instancesdlgimpl.obj
 0002:0000412c       ?slot_22@?3??staticMetaObject@config_plugin_instancesDlg@@SAPAVQMetaObject@@XZ@4UQUMethod@@B 1001512c     moc_config_plugin_instancesdlgimpl.obj
 0002:00004154       ?slot_23@?3??staticMetaObject@config_plugin_instancesDlg@@SAPAVQMetaObject@@XZ@4UQUMethod@@B 10015154     moc_config_plugin_instancesdlgimpl.obj
 0002:00004178       ?slot_tbl@?3??staticMetaObject@config_plugin_instancesDlg@@SAPAVQMetaObject@@XZ@4QBUQMetaData@@B 10015178     moc_config_plugin_instancesdlgimpl.obj
 0002:00004528       ?signal_0@?3??staticMetaObject@config_plugin_instancesDlg@@SAPAVQMetaObject@@XZ@4UQUMethod@@B 10015528     moc_config_plugin_instancesdlgimpl.obj
 0002:00004534       ?signal_tbl@?3??staticMetaObject@config_plugin_instancesDlg@@SAPAVQMetaObject@@XZ@4QBUQMetaData@@B 10015534     moc_config_plugin_instancesdlgimpl.obj
 0002:00004558       ?slot_0@?3??staticMetaObject@instancesCustomTable@@SAPAVQMetaObject@@XZ@4UQUMethod@@B 10015558     moc_instancesCustomTable.obj
 0002:00004574       ?slot_1@?3??staticMetaObject@instancesCustomTable@@SAPAVQMetaObject@@XZ@4UQUMethod@@B 10015574     moc_instancesCustomTable.obj
 0002:00004588       ?slot_2@?3??staticMetaObject@instancesCustomTable@@SAPAVQMetaObject@@XZ@4UQUMethod@@B 10015588     moc_instancesCustomTable.obj
 0002:00004594       ?slot_tbl@?3??staticMetaObject@instancesCustomTable@@SAPAVQMetaObject@@XZ@4QBUQMetaData@@B 10015594     moc_instancesCustomTable.obj
 0002:00004604       ?slot_0@?3??staticMetaObject@toolWindowBase@@SAPAVQMetaObject@@XZ@4UQUMethod@@B 10015604     moc_toolwindow.obj
 0002:00004610       ?slot_tbl@?3??staticMetaObject@toolWindowBase@@SAPAVQMetaObject@@XZ@4QBUQMetaData@@B 10015610     moc_toolwindow.obj
 0002:00004638       ?slot_0@?3??staticMetaObject@toolWindow@@SAPAVQMetaObject@@XZ@4UQUMethod@@B 10015638     moc_toolwindowimpl.obj
 0002:00004658       ?slot_tbl@?3??staticMetaObject@toolWindow@@SAPAVQMetaObject@@XZ@4QBUQMetaData@@B 10015658     moc_toolwindowimpl.obj
 0002:00004688       ?signal_0@?3??staticMetaObject@toolWindow@@SAPAVQMetaObject@@XZ@4UQUMethod@@B 10015688     moc_toolwindowimpl.obj
 0002:000046a4       ?signal_tbl@?3??staticMetaObject@toolWindow@@SAPAVQMetaObject@@XZ@4QBUQMetaData@@B 100156a4     moc_toolwindowimpl.obj
 0002:00004bc0       ?slot_0@?3??staticMetaObject@cfg_Table@@SAPAVQMetaObject@@XZ@4UQUMethod@@B 10015bc0     cfg_widgets001:moc_cfg_Table.obj
 0002:00004bd8       ?slot_1@?3??staticMetaObject@cfg_Table@@SAPAVQMetaObject@@XZ@4UQUMethod@@B 10015bd8     cfg_widgets001:moc_cfg_Table.obj
 0002:00004bf4       ?slot_2@?3??staticMetaObject@cfg_Table@@SAPAVQMetaObject@@XZ@4UQUMethod@@B 10015bf4     cfg_widgets001:moc_cfg_Table.obj
 0002:00004c0c       ?slot_3@?3??staticMetaObject@cfg_Table@@SAPAVQMetaObject@@XZ@4UQUMethod@@B 10015c0c     cfg_widgets001:moc_cfg_Table.obj
 0002:00004c28       ?slot_4@?3??staticMetaObject@cfg_Table@@SAPAVQMetaObject@@XZ@4UQUMethod@@B 10015c28     cfg_widgets001:moc_cfg_Table.obj
 0002:00004c4c       ?slot_tbl@?3??staticMetaObject@cfg_Table@@SAPAVQMetaObject@@XZ@4QBUQMetaData@@B 10015c4c     cfg_widgets001:moc_cfg_Table.obj
 0002:00004ce4       ?signal_0@?3??staticMetaObject@cfg_Table@@SAPAVQMetaObject@@XZ@4UQUMethod@@B 10015ce4     cfg_widgets001:moc_cfg_Table.obj
 0002:00004cfc       ?signal_1@?3??staticMetaObject@cfg_Table@@SAPAVQMetaObject@@XZ@4UQUMethod@@B 10015cfc     cfg_widgets001:moc_cfg_Table.obj
 0002:00004d1c       ?signal_tbl@?3??staticMetaObject@cfg_Table@@SAPAVQMetaObject@@XZ@4QBUQMetaData@@B 10015d1c     cfg_widgets001:moc_cfg_Table.obj
 0002:00004d6c       _GS_ExceptionPointers      10015d6c     MSVCRT:gs_report.obj
 0002:000060f0       __unwindtable$??1QDockWindowList@@UAE@XZ 100170f0     config_plugin_instances.obj
 0002:00006100       __ehfuncinfo$??1QDockWindowList@@UAE@XZ 10017100     config_plugin_instances.obj
 0002:00006124       __unwindtable$??1?$QPtrList@VdeviceRow@@@@UAE@XZ 10017124     config_plugin_instances.obj
 0002:00006124       __unwindtable$??1?$QPtrList@VQPopupMenu@@@@UAE@XZ 10017124     config_plugin_instances.obj
 0002:00006124       __unwindtable$??1?$QPtrList@VviewRow@@@@UAE@XZ 10017124     config_plugin_instances.obj
 0002:00006124       __unwindtable$??1?$QPtrList@VgroupRow@@@@UAE@XZ 10017124     config_plugin_instances.obj
 0002:0000612c       __ehfuncinfo$??1?$QPtrList@VviewRow@@@@UAE@XZ 1001712c     config_plugin_instances.obj
 0002:0000612c       __ehfuncinfo$??1?$QPtrList@VQPopupMenu@@@@UAE@XZ 1001712c     config_plugin_instances.obj
 0002:0000612c       __ehfuncinfo$??1?$QPtrList@VgroupRow@@@@UAE@XZ 1001712c     config_plugin_instances.obj
 0002:0000612c       __ehfuncinfo$??1?$QPtrList@VdeviceRow@@@@UAE@XZ 1001712c     config_plugin_instances.obj
 0002:00006150       __unwindtable$??1QPopupMenuList@@UAE@XZ 10017150     config_plugin_instances.obj
 0002:00006158       __ehfuncinfo$??1QPopupMenuList@@UAE@XZ 10017158     config_plugin_instances.obj
 0002:0000617c       __unwindtable$??0config_plugin_base@@QAE@ABVQString@@00@Z 1001717c     config_plugin_instances.obj
 0002:0000619c       __ehfuncinfo$??0config_plugin_base@@QAE@ABVQString@@00@Z 1001719c     config_plugin_instances.obj
 0002:000061c0       __unwindtable$??1config_plugin_base@@UAE@XZ 100171c0     config_plugin_instances.obj
 0002:000061d8       __ehfuncinfo$??1config_plugin_base@@UAE@XZ 100171d8     config_plugin_instances.obj
 0002:000061fc       __unwindtable$?about@config_plugin_base@@UAE?AVQString@@XZ 100171fc     config_plugin_instances.obj
 0002:0000620c       __ehfuncinfo$?about@config_plugin_base@@UAE?AVQString@@XZ 1001720c     config_plugin_instances.obj
 0002:00006230       __ehfuncinfo$??0config_plugin_instances@@QAE@ABVQString@@00@Z 10017230     config_plugin_instances.obj
 0002:00006254       __unwindtable$??0config_plugin_instances@@QAE@ABVQString@@00@Z 10017254     config_plugin_instances.obj
 0002:00006384       __ehfuncinfo$??1config_plugin_instances@@UAE@XZ 10017384     config_plugin_instances.obj
 0002:000063a8       __unwindtable$??1config_plugin_instances@@UAE@XZ 100173a8     config_plugin_instances.obj
 0002:000063d8       __unwindtable$?toolbars@config_plugin_instances@@UAE?AVQDockWindowList@@XZ 100173d8     config_plugin_instances.obj
 0002:000063e0       __ehfuncinfo$?toolbars@config_plugin_instances@@UAE?AVQDockWindowList@@XZ 100173e0     config_plugin_instances.obj
 0002:00006404       __unwindtable$?menus@config_plugin_instances@@UAE?AVQPopupMenuList@@XZ 10017404     config_plugin_instances.obj
 0002:0000640c       __ehfuncinfo$?menus@config_plugin_instances@@UAE?AVQPopupMenuList@@XZ 1001740c     config_plugin_instances.obj
 0002:00006430       __ehfuncinfo$?reply@config_plugin_instances@@UAEXPAVresponse@@@Z 10017430     config_plugin_instances.obj
 0002:00006454       __unwindtable$?reply@config_plugin_instances@@UAEXPAVresponse@@@Z 10017454     config_plugin_instances.obj
 0002:00006504       __unwindtable$?navigate@config_plugin_instances@@UAEXABVQString@@0@Z 10017504     config_plugin_instances.obj
 0002:0000651c       __ehfuncinfo$?navigate@config_plugin_instances@@UAEXABVQString@@0@Z 1001751c     config_plugin_instances.obj
 0002:00006540       __ehfuncinfo$?activate@config_plugin_instances@@UAEX_N@Z 10017540     config_plugin_instances.obj
 0002:00006564       __unwindtable$?activate@config_plugin_instances@@UAEX_N@Z 10017564     config_plugin_instances.obj
 0002:000065c4       __unwindtable$?setDirty@config_plugin_instancesDlg@@QAEXXZ 100175c4     config_plugin_instances.obj
 0002:000065c4       __unwindtable$?closeEvent@config_plugin_instances@@UAEXPAVQCloseEvent@@@Z 100175c4     config_plugin_instances.obj
 0002:000065cc       __ehfuncinfo$?closeEvent@config_plugin_instances@@UAEXPAVQCloseEvent@@@Z 100175cc     config_plugin_instances.obj
 0002:000065cc       __ehfuncinfo$?setDirty@config_plugin_instancesDlg@@QAEXXZ 100175cc     config_plugin_instances.obj
 0002:000065f0       __unwindtable$?apply@config_plugin_instances@@UAEXXZ 100175f0     config_plugin_instances.obj
 0002:00006608       __ehfuncinfo$?apply@config_plugin_instances@@UAEXXZ 10017608     config_plugin_instances.obj
 0002:0000662c       __ehfuncinfo$?about@config_plugin_instances@@UAE?AVQString@@XZ 1001762c     config_plugin_instances.obj
 0002:00006650       __unwindtable$?about@config_plugin_instances@@UAE?AVQString@@XZ 10017650     config_plugin_instances.obj
 0002:00006678       __unwindtable$??1?$QDict@VQAction@@@@UAE@XZ 10017678     config_plugin_instances.obj
 0002:00006680       __ehfuncinfo$??1?$QDict@VQAction@@@@UAE@XZ 10017680     config_plugin_instances.obj
 0002:000066a4       __ehfuncinfo$??0config_plugin_instancesDlg@@QAE@ABVQString@@PAVQWidget@@PBDI@Z 100176a4     config_plugin_instancesdlgimpl.obj
 0002:000066c8       __unwindtable$??0config_plugin_instancesDlg@@QAE@ABVQString@@PAVQWidget@@PBDI@Z 100176c8     config_plugin_instancesdlgimpl.obj
 0002:000067f8       __ehfuncinfo$??1config_plugin_instancesDlg@@UAE@XZ 100177f8     config_plugin_instancesdlgimpl.obj
 0002:0000681c       __unwindtable$??1config_plugin_instancesDlg@@UAE@XZ 1001781c     config_plugin_instancesdlgimpl.obj
 0002:00006864       __ehfuncinfo$?load@config_plugin_instancesDlg@@QAE_NABVQString@@@Z 10017864     config_plugin_instancesdlgimpl.obj
 0002:00006888       __unwindtable$?load@config_plugin_instancesDlg@@QAE_NABVQString@@@Z 10017888     config_plugin_instancesdlgimpl.obj
 0002:00006a98       __unwindtable$?save@config_plugin_instancesDlg@@QAE_NABVQString@@@Z 10017a98     config_plugin_instancesdlgimpl.obj
 0002:00006ab0       __ehfuncinfo$?save@config_plugin_instancesDlg@@QAE_NABVQString@@@Z 10017ab0     config_plugin_instancesdlgimpl.obj
 0002:00006ad4       __ehfuncinfo$?selectDevicetypes@config_plugin_instancesDlg@@QAEXHHHABVQPoint@@@Z 10017ad4     config_plugin_instancesdlgimpl.obj
 0002:00006af8       __unwindtable$?selectDevicetypes@config_plugin_instancesDlg@@QAEXHHHABVQPoint@@@Z 10017af8     config_plugin_instancesdlgimpl.obj
 0002:00006b28       __ehfuncinfo$?pasteCompositesXMLFragment@config_plugin_instancesDlg@@QAEXXZ 10017b28     config_plugin_instancesdlgimpl.obj
 0002:00006b4c       __unwindtable$?pasteCompositesXMLFragment@config_plugin_instancesDlg@@QAEXXZ 10017b4c     config_plugin_instancesdlgimpl.obj
 0002:00006c6c       __ehfuncinfo$?pasteGroupData@config_plugin_instancesDlg@@QAEXXZ 10017c6c     config_plugin_instancesdlgimpl.obj
 0002:00006c90       __unwindtable$?pasteGroupData@config_plugin_instancesDlg@@QAEXXZ 10017c90     config_plugin_instancesdlgimpl.obj
 0002:00006d68       __ehfuncinfo$?addGroupToInstanceNodeFromRow@config_plugin_instancesDlg@@QAE_NHVQString@@@Z 10017d68     config_plugin_instancesdlgimpl.obj
 0002:00006d8c       __unwindtable$?addGroupToInstanceNodeFromRow@config_plugin_instancesDlg@@QAE_NHVQString@@@Z 10017d8c     config_plugin_instancesdlgimpl.obj
 0002:00006e04       __ehfuncinfo$?addViewNodeFromRow@config_plugin_instancesDlg@@QAE_NH@Z 10017e04     config_plugin_instancesdlgimpl.obj
 0002:00006e28       __unwindtable$?addViewNodeFromRow@config_plugin_instancesDlg@@QAE_NH@Z 10017e28     config_plugin_instancesdlgimpl.obj
 0002:00006e98       __ehfuncinfo$?addDeviceNodeFromRow@config_plugin_instancesDlg@@QAE_NH@Z 10017e98     config_plugin_instancesdlgimpl.obj
 0002:00006ebc       __unwindtable$?addDeviceNodeFromRow@config_plugin_instancesDlg@@QAE_NH@Z 10017ebc     config_plugin_instancesdlgimpl.obj
 0002:00006fac       __ehfuncinfo$?pasteDeviceData@config_plugin_instancesDlg@@QAEXXZ 10017fac     config_plugin_instancesdlgimpl.obj
 0002:00006fd0       __unwindtable$?pasteDeviceData@config_plugin_instancesDlg@@QAEXXZ 10017fd0     config_plugin_instancesdlgimpl.obj
 0002:00007118       __unwindtable$?pasteOptions@config_plugin_instancesDlg@@QAEXXZ 10018118     config_plugin_instancesdlgimpl.obj
 0002:00007118       __unwindtable$?db@@YAXABVQString@@@Z 10018118     config_plugin_instancesdlgimpl.obj
 0002:00007120       __ehfuncinfo$?pasteOptions@config_plugin_instancesDlg@@QAEXXZ 10018120     config_plugin_instancesdlgimpl.obj
 0002:00007120       __ehfuncinfo$?db@@YAXABVQString@@@Z 10018120     config_plugin_instancesdlgimpl.obj
 0002:00007144       __ehfuncinfo$?copySelectedToClipboard@config_plugin_instancesDlg@@QAEXXZ 10018144     config_plugin_instancesdlgimpl.obj
 0002:00007168       __unwindtable$?copySelectedToClipboard@config_plugin_instancesDlg@@QAEXXZ 10018168     config_plugin_instancesdlgimpl.obj
 0002:000071f0       __ehfuncinfo$?clipboardDataChange@config_plugin_instancesDlg@@QAEXXZ 100181f0     config_plugin_instancesdlgimpl.obj
 0002:00007214       __unwindtable$?clipboardDataChange@config_plugin_instancesDlg@@QAEXXZ 10018214     config_plugin_instancesdlgimpl.obj
 0002:00007264       __unwindtable$?groupNameIsUnique@config_plugin_instancesDlg@@QAE_NVQString@@@Z 10018264     config_plugin_instancesdlgimpl.obj
 0002:00007274       __ehfuncinfo$?groupNameIsUnique@config_plugin_instancesDlg@@QAE_NVQString@@@Z 10018274     config_plugin_instancesdlgimpl.obj
 0002:00007298       __unwindtable$?typeIsValid@config_plugin_instancesDlg@@QAE_NVQString@@@Z 10018298     config_plugin_instancesdlgimpl.obj
 0002:000072a0       __ehfuncinfo$?typeIsValid@config_plugin_instancesDlg@@QAE_NVQString@@@Z 100182a0     config_plugin_instancesdlgimpl.obj
 0002:000072c4       __ehfuncinfo$?instanceNameIsUnique@config_plugin_instancesDlg@@QAE_NVQString@@@Z 100182c4     config_plugin_instancesdlgimpl.obj
 0002:000072e8       __unwindtable$?instanceNameIsUnique@config_plugin_instancesDlg@@QAE_NVQString@@@Z 100182e8     config_plugin_instancesdlgimpl.obj
 0002:00007330       __ehfuncinfo$?valueCompositeGroupChanged@config_plugin_instancesDlg@@QAEXHH@Z 10018330     config_plugin_instancesdlgimpl.obj
 0002:00007354       __unwindtable$?valueCompositeGroupChanged@config_plugin_instancesDlg@@QAEXHH@Z 10018354     config_plugin_instancesdlgimpl.obj
 0002:000073d4       __unwindtable$?viewGroupChanged@config_plugin_instancesDlg@@QAEXHH@Z 100183d4     config_plugin_instancesdlgimpl.obj
 0002:000073e4       __ehfuncinfo$?viewGroupChanged@config_plugin_instancesDlg@@QAEXHH@Z 100183e4     config_plugin_instancesdlgimpl.obj
 0002:00007408       __ehfuncinfo$?valueCompositeTopChanged@config_plugin_instancesDlg@@QAEXHH@Z 10018408     config_plugin_instancesdlgimpl.obj
 0002:0000742c       __unwindtable$?valueCompositeTopChanged@config_plugin_instancesDlg@@QAEXHH@Z 1001842c     config_plugin_instancesdlgimpl.obj
 0002:0000747c       __ehfuncinfo$?doDuplicateInstance@config_plugin_instancesDlg@@QAEXXZ 1001847c     config_plugin_instancesdlgimpl.obj
 0002:000074a0       __unwindtable$?doDuplicateInstance@config_plugin_instancesDlg@@QAEXXZ 100184a0     config_plugin_instancesdlgimpl.obj
 0002:00007720       __ehfuncinfo$?doDeleteInstance@config_plugin_instancesDlg@@QAEXXZ 10018720     config_plugin_instancesdlgimpl.obj
 0002:00007744       __unwindtable$?doDeleteInstance@config_plugin_instancesDlg@@QAEXXZ 10018744     config_plugin_instancesdlgimpl.obj
 0002:0000785c       __ehfuncinfo$?doCreateNewInstance@config_plugin_instancesDlg@@QAEXXZ 1001885c     config_plugin_instancesdlgimpl.obj
 0002:00007880       __unwindtable$?doCreateNewInstance@config_plugin_instancesDlg@@QAEXXZ 10018880     config_plugin_instancesdlgimpl.obj
 0002:000078c8       __ehfuncinfo$?valueDevicesChanged@config_plugin_instancesDlg@@QAEXHH@Z 100188c8     config_plugin_instancesdlgimpl.obj
 0002:000078ec       __unwindtable$?valueDevicesChanged@config_plugin_instancesDlg@@QAEXHH@Z 100188ec     config_plugin_instancesdlgimpl.obj
 0002:000079cc       __ehfuncinfo$?viewInstanceChanged@config_plugin_instancesDlg@@QAEXHH@Z 100189cc     config_plugin_instancesdlgimpl.obj
 0002:000079f0       __unwindtable$?viewInstanceChanged@config_plugin_instancesDlg@@QAEXHH@Z 100189f0     config_plugin_instancesdlgimpl.obj
 0002:00007ab0       __unwindtable$?deviceInstanceChanged@config_plugin_instancesDlg@@QAEXHH@Z 10018ab0     config_plugin_instancesdlgimpl.obj
 0002:00007ac0       __ehfuncinfo$?deviceInstanceChanged@config_plugin_instancesDlg@@QAEXHH@Z 10018ac0     config_plugin_instancesdlgimpl.obj
 0002:00007ae4       __ehfuncinfo$??0deviceRow@@QAE@ABVQString@@0000000@Z 10018ae4     deviceRow.obj
 0002:00007b08       __unwindtable$??0deviceRow@@QAE@ABVQString@@0000000@Z 10018b08     deviceRow.obj
 0002:00007b48       __ehfuncinfo$??1deviceRow@@UAE@XZ 10018b48     deviceRow.obj
 0002:00007b6c       __unwindtable$??1deviceRow@@UAE@XZ 10018b6c     deviceRow.obj
 0002:00007ba4       __ehfuncinfo$??0devicetypesBase@@QAE@PAVQWidget@@PBD_NI@Z 10018ba4     devicetypes.obj
 0002:00007bc8       __unwindtable$??0devicetypesBase@@QAE@PAVQWidget@@PBD_NI@Z 10018bc8     devicetypes.obj
 0002:00007c08       __unwindtable$?languageChange@devicetypesBase@@MAEXXZ 10018c08     devicetypes.obj
 0002:00007c28       __ehfuncinfo$?languageChange@devicetypesBase@@MAEXXZ 10018c28     devicetypes.obj
 0002:00007c4c       __unwindtable$??0groupRow@@QAE@ABVQString@@0@Z 10018c4c     groupRow.obj
 0002:00007c5c       __ehfuncinfo$??0groupRow@@QAE@ABVQString@@0@Z 10018c5c     groupRow.obj
 0002:00007c80       __unwindtable$??1groupRow@@UAE@XZ 10018c80     groupRow.obj
 0002:00007c88       __ehfuncinfo$??1groupRow@@UAE@XZ 10018c88     groupRow.obj
 0002:00007cac       __unwindtable$??0instancesCustomTable@@QAE@PAVQWidget@@PBD@Z 10018cac     instancesCustomTable.obj
 0002:00007cbc       __ehfuncinfo$??0instancesCustomTable@@QAE@PAVQWidget@@PBD@Z 10018cbc     instancesCustomTable.obj
 0002:00007ce0       __unwindtable$??1instancesCustomTable@@UAE@XZ 10018ce0     instancesCustomTable.obj
 0002:00007ce8       __ehfuncinfo$??1instancesCustomTable@@UAE@XZ 10018ce8     instancesCustomTable.obj
 0002:00007d0c       __unwindtable$?keys@plugindesc@@UAE?AVQStringList@@ABVQString@@0@Z 10018d0c     plugindesc.obj
 0002:00007d1c       __ehfuncinfo$?keys@plugindesc@@UAE?AVQStringList@@ABVQString@@0@Z 10018d1c     plugindesc.obj
 0002:00007d40       __unwindtable$??4?$QGuardedPtr@VQPopupMenu@@@@QAEAAV0@PAVQPopupMenu@@@Z 10018d40     plugindesc.obj
 0002:00007d40       __unwindtable$??4?$QGuardedPtr@VQDockWindow@@@@QAEAAV0@PAVQDockWindow@@@Z 10018d40     plugindesc.obj
 0002:00007d40       __unwindtable$??0?$QGuardedPtr@VQPopupMenu@@@@QAE@XZ 10018d40     plugindesc.obj
 0002:00007d40       __unwindtable$?create@plugindesc@@UAEPAVconfig_plugin_base@@ABVQString@@00@Z 10018d40     plugindesc.obj
 0002:00007d40       __unwindtable$??0?$QGuardedPtr@VQDockWindow@@@@QAE@XZ 10018d40     plugindesc.obj
 0002:00007d48       __ehfuncinfo$??0?$QGuardedPtr@VQPopupMenu@@@@QAE@XZ 10018d48     plugindesc.obj
 0002:00007d48       __ehfuncinfo$??4?$QGuardedPtr@VQDockWindow@@@@QAEAAV0@PAVQDockWindow@@@Z 10018d48     plugindesc.obj
 0002:00007d48       __ehfuncinfo$?create@plugindesc@@UAEPAVconfig_plugin_base@@ABVQString@@00@Z 10018d48     plugindesc.obj
 0002:00007d48       __ehfuncinfo$??4?$QGuardedPtr@VQPopupMenu@@@@QAEAAV0@PAVQPopupMenu@@@Z 10018d48     plugindesc.obj
 0002:00007d48       __ehfuncinfo$??0?$QGuardedPtr@VQDockWindow@@@@QAE@XZ 10018d48     plugindesc.obj
 0002:00007d6c       __unwindtable$??0viewRow@@QAE@ABVQString@@000@Z 10018d6c     viewRow.obj
 0002:00007d8c       __ehfuncinfo$??0viewRow@@QAE@ABVQString@@000@Z 10018d8c     viewRow.obj
 0002:00007db0       __unwindtable$??1viewRow@@UAE@XZ 10018db0     viewRow.obj
 0002:00007dc8       __ehfuncinfo$??1viewRow@@UAE@XZ 10018dc8     viewRow.obj
 0002:00007dec       __ehfuncinfo$??0config_plugin_instancesDlgBase@@QAE@PAVQWidget@@PBDI@Z 10018dec     config_plugin_instancesdlg.obj
 0002:00007e10       __unwindtable$??0config_plugin_instancesDlgBase@@QAE@PAVQWidget@@PBDI@Z 10018e10     config_plugin_instancesdlg.obj
 0002:00007ec8       __unwindtable$??1config_plugin_instancesDlgBase@@UAE@XZ 10018ec8     config_plugin_instancesdlg.obj
 0002:00007ed0       __ehfuncinfo$??1config_plugin_instancesDlgBase@@UAE@XZ 10018ed0     config_plugin_instancesdlg.obj
 0002:00007ef4       __ehfuncinfo$?languageChange@config_plugin_instancesDlgBase@@MAEXXZ 10018ef4     config_plugin_instancesdlg.obj
 0002:00007f18       __unwindtable$?languageChange@config_plugin_instancesDlgBase@@MAEXXZ 10018f18     config_plugin_instancesdlg.obj
 0002:00007f50       __unwindtable$?qt_emit@config_plugin_instancesDlg@@UAE_NHPAUQUObject@@@Z 10018f50     moc_config_plugin_instances.obj
 0002:00007f50       __unwindtable$?qt_emit@config_plugin_instances@@UAE_NHPAUQUObject@@@Z 10018f50     moc_config_plugin_instances.obj
 0002:00007f58       __ehfuncinfo$?qt_emit@config_plugin_instancesDlg@@UAE_NHPAUQUObject@@@Z 10018f58     moc_config_plugin_instances.obj
 0002:00007f58       __ehfuncinfo$?qt_emit@config_plugin_instances@@UAE_NHPAUQUObject@@@Z 10018f58     moc_config_plugin_instances.obj
 0002:00007f7c       __unwindtable$?command@config_plugin_instancesDlg@@IAEXVQString@@0@Z 10018f7c     moc_config_plugin_instancesdlgimpl.obj
 0002:00007f7c       __unwindtable$?command@config_plugin_instances@@IAEXVQString@@0@Z 10018f7c     moc_config_plugin_instancesdlgimpl.obj
 0002:00007f94       __ehfuncinfo$?command@config_plugin_instances@@IAEXVQString@@0@Z 10018f94     moc_config_plugin_instancesdlgimpl.obj
 0002:00007f94       __ehfuncinfo$?command@config_plugin_instancesDlg@@IAEXVQString@@0@Z 10018f94     moc_config_plugin_instancesdlgimpl.obj
 0002:00007fb8       __unwindtable$??0cfg_Table@@QAE@PAVQWidget@@PBD@Z 10018fb8     cfg_widgets001:cfg_Table.obj
 0002:00007fc0       __ehfuncinfo$??0cfg_Table@@QAE@PAVQWidget@@PBD@Z 10018fc0     cfg_widgets001:cfg_Table.obj
 0002:00007fe4       __unwindtable$?deleteItems@cfg_Table@@QAEXXZ 10018fe4     cfg_widgets001:cfg_Table.obj
 0002:00007fec       __ehfuncinfo$?deleteItems@cfg_Table@@QAEXXZ 10018fec     cfg_widgets001:cfg_Table.obj
 0002:00008010       __unwindtable$?copyToClipboard@cfg_Table@@QAEXXZ 10019010     cfg_widgets001:cfg_Table.obj
 0002:00008028       __ehfuncinfo$?copyToClipboard@cfg_Table@@QAEXXZ 10019028     cfg_widgets001:cfg_Table.obj
 0002:0000804c       __unwindtable$?undoPaste@cfg_Table@@QAEXXZ 1001904c     cfg_widgets001:cfg_Table.obj
 0002:00008064       __ehfuncinfo$?undoPaste@cfg_Table@@QAEXXZ 10019064     cfg_widgets001:cfg_Table.obj
 0002:00008088       __ehfuncinfo$?pasteClipboard@cfg_Table@@QAEXXZ 10019088     cfg_widgets001:cfg_Table.obj
 0002:000080ac       __unwindtable$?pasteClipboard@cfg_Table@@QAEXXZ 100190ac     cfg_widgets001:cfg_Table.obj
 0002:0000811c       __unwindtable$?clipBoardDataChanged@cfg_Table@@IAEXXZ 1001911c     cfg_widgets001:cfg_Table.obj
 0002:00008124       __ehfuncinfo$?clipBoardDataChanged@cfg_Table@@IAEXXZ 10019124     cfg_widgets001:cfg_Table.obj
 0002:00008148       __unwindtable$?fillUndoBuffer@cfg_Table@@AAEXXZ 10019148     cfg_widgets001:cfg_Table.obj
 0002:00008168       __ehfuncinfo$?fillUndoBuffer@cfg_Table@@AAEXXZ 10019168     cfg_widgets001:cfg_Table.obj
 0002:00008190       __sehtable$__onexit        10019190     MSVCRT:atonexit.obj
 0002:000081b0       __sehtable$??_L@YGXPAXIHP6EX0@Z1@Z 100191b0     MSVCRT:ehvecctr.obj
 0002:000081d0       __sehtable$??_M@YGXPAXIHP6EX0@Z@Z 100191d0     MSVCRT:ehvecdtr.obj
 0002:000081f0       __sehtable$?__ArrayUnwind@@YGXPAXIHP6EX0@Z@Z 100191f0     MSVCRT:ehvecdtr.obj
 0002:00008210       __sehtable$___DllMainCRTStartup 10019210     MSVCRT:crtdll.obj
 0002:00008238       __sehtable$__IsNonwritableInCurrentImage 10019238     MSVCRT:pesect.obj
 0002:00008260       .edata                     10019260     config_plugin_instances.exp
 0002:00008288       rgpv                       10019288     config_plugin_instances.exp
 0002:000082fc       rgszName                   100192fc     config_plugin_instances.exp
 0002:00008370       rgwOrd                     10019370     config_plugin_instances.exp
 0002:000083aa       szName                     100193aa     config_plugin_instances.exp
 0002:000083c6       $N00001                    100193c6     config_plugin_instances.exp
 0002:000083e0       $N00002                    100193e0     config_plugin_instances.exp
 0002:00008404       $N00003                    10019404     config_plugin_instances.exp
 0002:00008419       $N00004                    10019419     config_plugin_instances.exp
 0002:00008437       $N00005                    10019437     config_plugin_instances.exp
 0002:00008453       $N00006                    10019453     config_plugin_instances.exp
 0002:00008474       $N00007                    10019474     config_plugin_instances.exp
 0002:0000848a       $N00008                    1001948a     config_plugin_instances.exp
 0002:000084a9       $N00009                    100194a9     config_plugin_instances.exp
 0002:000084d1       $N00010                    100194d1     config_plugin_instances.exp
 0002:000084f9       $N00011                    100194f9     config_plugin_instances.exp
 0002:0000851c       $N00012                    1001951c     config_plugin_instances.exp
 0002:0000853a       $N00013                    1001953a     config_plugin_instances.exp
 0002:00008559       $N00014                    10019559     config_plugin_instances.exp
 0002:0000857b       $N00015                    1001957b     config_plugin_instances.exp
 0002:000085a2       $N00016                    100195a2     config_plugin_instances.exp
 0002:000085cf       $N00017                    100195cf     config_plugin_instances.exp
 0002:000085f1       $N00018                    100195f1     config_plugin_instances.exp
 0002:00008617       $N00019                    10019617     config_plugin_instances.exp
 0002:00008637       $N00020                    10019637     config_plugin_instances.exp
 0002:00008661       $N00021                    10019661     config_plugin_instances.exp
 0002:0000868d       $N00022                    1001968d     config_plugin_instances.exp
 0002:000086bc       $N00023                    100196bc     config_plugin_instances.exp
 0002:000086fd       $N00024                    100196fd     config_plugin_instances.exp
 0002:0000872f       $N00025                    1001972f     config_plugin_instances.exp
 0002:00008753       $N00026                    10019753     config_plugin_instances.exp
 0002:0000877b       $N00027                    1001977b     config_plugin_instances.exp
 0002:00008798       $N00028                    10019798     config_plugin_instances.exp
 0002:000087b8       $N00029                    100197b8     config_plugin_instances.exp
 0002:000095a4       .idata$6                   1001a5a4     config_icons:config_icons.dll
 0002:00011826       .idata$6                   10022826     qt-mt323:qt-mt323.dll
 0002:00011876       .idata$6                   10022876     MSVCRT:MSVCR120.dll
 0002:00011cd2       .idata$6                   10022cd2     kernel32:KERNEL32.dll
 0003:00000000       _GREENTIK                  10023000     config_plugin_instancesdlgimpl.obj
 0003:00000048       _CROSS                     10023048     config_plugin_instancesdlgimpl.obj
 0003:00000090       _config_plugin_instances_XPM 10023090     plugindesc.obj
 0003:000000d4       ?param_slot_0@?3??staticMetaObject@config_plugin_instances@@SAPAVQMetaObject@@XZ@4QBUQUParameter@@B 100230d4     moc_config_plugin_instances.obj
 0003:00000108       ?param_slot_1@?3??staticMetaObject@config_plugin_instancesDlg@@SAPAVQMetaObject@@XZ@4QBUQUParameter@@B 10023108     moc_config_plugin_instancesdlgimpl.obj
 0003:00000148       ?param_slot_21@?3??staticMetaObject@config_plugin_instancesDlg@@SAPAVQMetaObject@@XZ@4QBUQUParameter@@B 10023148     moc_config_plugin_instancesdlgimpl.obj
 0003:00000168       ?param_slot_23@?3??staticMetaObject@config_plugin_instancesDlg@@SAPAVQMetaObject@@XZ@4QBUQUParameter@@B 10023168     moc_config_plugin_instancesdlgimpl.obj
 0003:00000188       ?param_slot_0@?3??staticMetaObject@instancesCustomTable@@SAPAVQMetaObject@@XZ@4QBUQUParameter@@B 10023188     moc_instancesCustomTable.obj
 0003:00000198       ?param_slot_1@?3??staticMetaObject@instancesCustomTable@@SAPAVQMetaObject@@XZ@4QBUQUParameter@@B 10023198     moc_instancesCustomTable.obj
 0003:000001b8       ?param_slot_2@?3??staticMetaObject@instancesCustomTable@@SAPAVQMetaObject@@XZ@4QBUQUParameter@@B 100231b8     moc_instancesCustomTable.obj
 0003:0000082c       _cleanUp_devicetypesBase   1002382c     moc_devicetypes.obj
 0003:00000834       _cleanUp_devicetypes       10023834     moc_devicetypesimpl.obj
 0003:0000083c       _cleanUp_config_plugin_instances 1002383c     moc_config_plugin_instances.obj
 0003:00000840       ?$S1@?3??staticMetaObject@config_plugin_instances@@SAPAVQMetaObject@@XZ@4IA 10023840     moc_config_plugin_instances.obj
 0003:00000844       ?param_signal_0@?3??staticMetaObject@config_plugin_instances@@SAPAVQMetaObject@@XZ@4QBUQUParameter@@B 10023844     moc_config_plugin_instances.obj
 0003:00000868       _cleanUp_config_plugin_instancesDlgBase 10023868     moc_config_plugin_instancesdlg.obj
 0003:00000870       _cleanUp_config_plugin_instancesDlg 10023870     moc_config_plugin_instancesdlgimpl.obj
 0003:00000874       ?$S1@?3??staticMetaObject@config_plugin_instancesDlg@@SAPAVQMetaObject@@XZ@4IA 10023874     moc_config_plugin_instancesdlgimpl.obj
 0003:00000878       ?param_slot_5@?3??staticMetaObject@config_plugin_instancesDlg@@SAPAVQMetaObject@@XZ@4QBUQUParameter@@B 10023878     moc_config_plugin_instancesdlgimpl.obj
 0003:000008a8       ?param_slot_6@?3??staticMetaObject@config_plugin_instancesDlg@@SAPAVQMetaObject@@XZ@4QBUQUParameter@@B 100238a8     moc_config_plugin_instancesdlgimpl.obj
 0003:000008c8       ?param_slot_7@?3??staticMetaObject@config_plugin_instancesDlg@@SAPAVQMetaObject@@XZ@4QBUQUParameter@@B 100238c8     moc_config_plugin_instancesdlgimpl.obj
 0003:000008e8       ?param_slot_12@?3??staticMetaObject@config_plugin_instancesDlg@@SAPAVQMetaObject@@XZ@4QBUQUParameter@@B 100238e8     moc_config_plugin_instancesdlgimpl.obj
 0003:00000908       ?param_slot_13@?3??staticMetaObject@config_plugin_instancesDlg@@SAPAVQMetaObject@@XZ@4QBUQUParameter@@B 10023908     moc_config_plugin_instancesdlgimpl.obj
 0003:00000928       ?param_slot_14@?3??staticMetaObject@config_plugin_instancesDlg@@SAPAVQMetaObject@@XZ@4QBUQUParameter@@B 10023928     moc_config_plugin_instancesdlgimpl.obj
 0003:00000948       ?param_slot_15@?3??staticMetaObject@config_plugin_instancesDlg@@SAPAVQMetaObject@@XZ@4QBUQUParameter@@B 10023948     moc_config_plugin_instancesdlgimpl.obj
 0003:00000968       ?param_slot_16@?3??staticMetaObject@config_plugin_instancesDlg@@SAPAVQMetaObject@@XZ@4QBUQUParameter@@B 10023968     moc_config_plugin_instancesdlgimpl.obj
 0003:00000988       ?param_slot_17@?3??staticMetaObject@config_plugin_instancesDlg@@SAPAVQMetaObject@@XZ@4QBUQUParameter@@B 10023988     moc_config_plugin_instancesdlgimpl.obj
 0003:000009a8       ?param_slot_22@?3??staticMetaObject@config_plugin_instancesDlg@@SAPAVQMetaObject@@XZ@4QBUQUParameter@@B 100239a8     moc_config_plugin_instancesdlgimpl.obj
 0003:000009c8       ?param_signal_0@?3??staticMetaObject@config_plugin_instancesDlg@@SAPAVQMetaObject@@XZ@4QBUQUParameter@@B 100239c8     moc_config_plugin_instancesdlgimpl.obj
 0003:000009ec       _cleanUp_instancesCustomTable 100239ec     moc_instancesCustomTable.obj
 0003:000009f0       ?$S1@?3??staticMetaObject@instancesCustomTable@@SAPAVQMetaObject@@XZ@4IA 100239f0     moc_instancesCustomTable.obj
 0003:000009f8       _cleanUp_toolWindowBase    100239f8     moc_toolwindow.obj
 0003:00000a00       _cleanUp_toolWindow        10023a00     moc_toolwindowimpl.obj
 0003:00000a04       ?param_slot_0@?3??staticMetaObject@toolWindow@@SAPAVQMetaObject@@XZ@4QBUQUParameter@@B 10023a04     moc_toolwindowimpl.obj
 0003:00000a14       ?$S1@?3??staticMetaObject@toolWindow@@SAPAVQMetaObject@@XZ@4IA 10023a14     moc_toolwindowimpl.obj
 0003:00000a18       ?param_signal_0@?3??staticMetaObject@toolWindow@@SAPAVQMetaObject@@XZ@4QBUQUParameter@@B 10023a18     moc_toolwindowimpl.obj
 0003:00000a2c       _cleanUp_cfg_Table         10023a2c     cfg_widgets001:moc_cfg_Table.obj
 0003:00000a30       ?param_signal_1@?3??staticMetaObject@cfg_Table@@SAPAVQMetaObject@@XZ@4QBUQUParameter@@B 10023a30     cfg_widgets001:moc_cfg_Table.obj
 0003:00000a40       ?$S1@?3??staticMetaObject@cfg_Table@@SAPAVQMetaObject@@XZ@4IA 10023a40     cfg_widgets001:moc_cfg_Table.obj
 0003:00000a44       ___proc_attached           10023a44     MSVCRT:crtdll.obj
 0003:00000a48       _GS_ExceptionRecord        10023a48     MSVCRT:gs_report.obj
 0003:00000a98       _GS_ContextRecord          10023a98     MSVCRT:gs_report.obj
 0003:00000d64       _DebuggerWasPresent        10023d64     MSVCRT:gs_report.obj
 0004:000000f0       $R000000                   100240f0     Script1.res
 0004:000005a8       $R0004B8                   100245a8     Script1.res
 0004:00000a90       $R0009A0                   10024a90     Script1.res
